 ProcList

 Timestamp is 64827016 (Fri Jun  9 01:19:34 2023)

 Preferred load address is 10000000

 Start         Length     Name                   Class
 0001:00000000 00000080H .text$di                CODE
 0001:00000080 00039b70H .text$mn                CODE
 0001:00039bf0 00001eb0H .text$x                 CODE
 0001:0003baa0 0000016fH .text$yd                CODE
 0002:00000000 00000240H .idata$5                DATA
 0002:00000240 00000004H .00cfg                  DATA
 0002:00000244 00000004H .CRT$XCA                DATA
 0002:00000248 0000000cH .CRT$XCC                DATA
 0002:00000254 00000008H .CRT$XCL                DATA
 0002:0000025c 0000000cH .CRT$XCU                DATA
 0002:00000268 00000004H .CRT$XCZ                DATA
 0002:0000026c 00000004H .CRT$XIA                DATA
 0002:00000270 00000014H .CRT$XIC                DATA
 0002:00000284 00000004H .CRT$XIZ                DATA
 0002:00000288 00000004H .CRT$XPA                DATA
 0002:0000028c 00000008H .CRT$XPX                DATA
 0002:00000294 00000004H .CRT$XPXA               DATA
 0002:00000298 00000004H .CRT$XPZ                DATA
 0002:0000029c 00000004H .CRT$XTA                DATA
 0002:000002a0 00000010H .CRT$XTZ                DATA
 0002:000002a4 00000000H .gfids$y                DATA
 0002:000002b0 0000d310H .rdata                  DATA
 0002:0000d5c0 00000000H .rdata$CastGuardVftablesA DATA
 0002:0000d5c0 00000000H .rdata$CastGuardVftablesC DATA
 0002:0000d5c0 00000978H .rdata$r                DATA
 0002:0000df38 000001acH .rdata$sxdata           DATA
 0002:0000e0e4 00000070H .rdata$voltmd           DATA
 0002:0000e154 00000364H .rdata$zzzdbg           DATA
 0002:0000e4b8 00000004H .rtc$IAA                DATA
 0002:0000e4bc 00000004H .rtc$IZZ                DATA
 0002:0000e4c0 00000004H .rtc$TAA                DATA
 0002:0000e4c4 00000004H .rtc$TZZ                DATA
 0002:0000e4c8 00002548H .xdata$x                DATA
 0002:00010a10 000001a0H .edata                  DATA
 0002:00010bb0 000000a0H .idata$2                DATA
 0002:00010c50 00000014H .idata$3                DATA
 0002:00010c64 00000240H .idata$4                DATA
 0002:00010ea4 00000a10H .idata$6                DATA
 0003:00000000 000009d0H .data                   DATA
 0003:000009d0 00000318H .data$r                 DATA
 0003:00000ce8 000005e8H .data$rs                DATA
 0003:000012d0 00001a2cH .bss                    DATA
 0004:00000000 00000060H .rsrc$01                DATA
 0004:00000060 00000340H .rsrc$02                DATA

  Address         Publics by Value              Rva+Base       Lib:Object

 0000:00000000       __except_list              00000000     <absolute>
 0000:00000000       ___x64_code_ranges_to_entry_points_count 00000000     <absolute>
 0000:00000000       ___guard_eh_cont_table     00000000     <absolute>
 0000:00000000       ___guard_fids_count        00000000     <absolute>
 0000:00000000       ___arm64x_native_entrypoint 00000000     <absolute>
 0000:00000000       ___guard_iat_table         00000000     <absolute>
 0000:00000000       ___guard_longjmp_table     00000000     <absolute>
 0000:00000000       ___arm64x_extra_rfe_table  00000000     <absolute>
 0000:00000000       ___arm64x_redirection_metadata 00000000     <absolute>
 0000:00000000       ___guard_eh_cont_count     00000000     <absolute>
 0000:00000000       ___hybrid_code_map_count   00000000     <absolute>
 0000:00000000       ___guard_iat_count         00000000     <absolute>
 0000:00000000       ___x64_code_ranges_to_entry_points 00000000     <absolute>
 0000:00000000       ___guard_longjmp_count     00000000     <absolute>
 0000:00000000       ___hybrid_code_map         00000000     <absolute>
 0000:00000000       ___guard_check_icall_a64n_fptr 00000000     <absolute>
 0000:00000000       ___arm64x_redirection_metadata_count 00000000     <absolute>
 0000:00000000       ___arm64x_extra_rfe_table_size 00000000     <absolute>
 0000:00000000       ___hybrid_auxiliary_iat    00000000     <absolute>
 0000:00000000       ___dynamic_value_reloc_table 00000000     <absolute>
 0000:00000000       ___enclave_config          00000000     <absolute>
 0000:00000000       ___guard_fids_table        00000000     <absolute>
 0000:00000000       ___AbsoluteZero            00000000     <absolute>
 0000:00000000       ___hybrid_auxiliary_iat_copy 00000000     <absolute>
 0000:0000006b       ___safe_se_handler_count   0000006b     <absolute>
 0000:00000100       ___guard_flags             00000100     <absolute>
 0000:00000000       ___ImageBase               10000000     <linker-defined>
 0001:00000080       ?WriteToFile@@YAIPAXABV?$basic_string_view@_WU?$char_traits@_W@std@@@std@@@Z 10001080 f   fileio.obj
 0001:000000b0       ??1?$vector@Umode@@V?$allocator@Umode@@@std@@@std@@QAE@XZ 100010b0 f i fileio.obj
 0001:00000140       ??1?$basic_string@_WU?$char_traits@_W@std@@V?$allocator@_W@2@@std@@QAE@XZ 10001140 f i fileio.obj
 0001:00000140       ?_Tidy_deallocate@?$basic_string@_WU?$char_traits@_W@std@@V?$allocator@_W@2@@std@@AAEXXZ 10001140 f i fileio.obj
 0001:00000140       ??1PerfLib@@QAE@XZ         10001140 f i perfthread.obj
 0001:000001a0       ?deallocate@?$allocator@_W@std@@QAEXQA_WI@Z 100011a0 f i fileio.obj
 0001:000001e0       ??1mode@@QAE@XZ            100011e0 f i fileio.obj
 0001:00000200       ??1columns@@QAE@XZ         10001200 f i fileio.obj
 0001:000002f0       ___local_stdio_printf_options 100012f0 f i format.obj
 0001:00000300       ??0exception@std@@QAE@QBD@Z 10001300 f i format.obj
 0001:00000340       ??0exception@std@@QAE@ABV01@@Z 10001340 f i format.obj
 0001:00000370       ?what@exception@std@@UBEPBDXZ 10001370 f i format.obj
 0001:00000380       ??_Eexception@std@@UAEPAXI@Z 10001380 f i * CIL library *:* CIL module *
 0001:00000380       ??_Gexception@std@@UAEPAXI@Z 10001380 f i format.obj
 0001:00000380       ??_Gbad_alloc@std@@UAEPAXI@Z 10001380 f i format.obj
 0001:00000380       ??_Gruntime_error@std@@UAEPAXI@Z 10001380 f i format.obj
 0001:00000380       ??_Gformat_error@v10@fmt@@UAEPAXI@Z 10001380 f i format.obj
 0001:00000380       ??_Eformat_error@v10@fmt@@UAEPAXI@Z 10001380 f i * CIL library *:* CIL module *
 0001:00000380       ??_Ebad_array_new_length@std@@UAEPAXI@Z 10001380 f i * CIL library *:* CIL module *
 0001:00000380       ??_Ebad_alloc@std@@UAEPAXI@Z 10001380 f i * CIL library *:* CIL module *
 0001:00000380       ??_Gbad_array_new_length@std@@UAEPAXI@Z 10001380 f i format.obj
 0001:00000380       ??_Eruntime_error@std@@UAEPAXI@Z 10001380 f i * CIL library *:* CIL module *
 0001:000003b0       ??1bad_array_new_length@std@@UAE@XZ 100013b0 f i format.obj
 0001:000003b0       ??1format_error@v10@fmt@@UAE@XZ 100013b0 f i format.obj
 0001:000003b0       ??1bad_function_call@std@@UAE@XZ 100013b0 f i libcpmt:xthrow.obj
 0001:000003b0       ??1bad_exception@std@@UAE@XZ 100013b0 f i libvcruntime:frame.obj
 0001:000003b0       ??1runtime_error@std@@UAE@XZ 100013b0 f i format.obj
 0001:000003b0       ??1bad_alloc@std@@UAE@XZ   100013b0 f i format.obj
 0001:000003b0       ??1length_error@std@@UAE@XZ 100013b0 f i libcpmt:xthrow.obj
 0001:000003b0       ??1out_of_range@std@@UAE@XZ 100013b0 f i libcpmt:xthrow.obj
 0001:000003d0       ??0bad_array_new_length@std@@QAE@XZ 100013d0 f i format.obj
 0001:000003f0       ?__scrt_throw_std_bad_array_new_length@@YAXXZ 100013f0 f i LIBCMT:throw_bad_alloc.obj
 0001:000003f0       ?_Throw_bad_array_new_length@std@@YAXXZ 100013f0 f i format.obj
 0001:00000410       ??0bad_array_new_length@std@@QAE@ABV01@@Z 10001410 f i format.obj
 0001:00000450       ??0bad_alloc@std@@QAE@ABV01@@Z 10001450 f i format.obj
 0001:00000490       ?_Xlen_string@std@@YAXXZ   10001490 f i format.obj
 0001:000004a0       ??0runtime_error@std@@QAE@PBD@Z 100014a0 f i format.obj
 0001:000004e0       ??0runtime_error@std@@QAE@ABV01@@Z 100014e0 f i format.obj
 0001:00000520       ?count_digits@detail@v10@fmt@@YAH_K@Z 10001520 f i format.obj
 0001:00000580       ??1?$basic_string@DU?$char_traits@D@std@@V?$allocator@D@2@@std@@QAE@XZ 10001580 f i format.obj
 0001:00000580       ??1?$thousands_sep_result@_W@detail@v10@fmt@@QAE@XZ 10001580 f i format.obj
 0001:000005d0       ?umul128_upper64@dragonbox@detail@v10@fmt@@YA_K_K0@Z 100015d0 f i format.obj
 0001:00000640       ?umul192_upper128@dragonbox@detail@v10@fmt@@YA?AVuint128_fallback@234@_KV5234@@Z 10001640 f i format.obj
 0001:00000760       ?needs_escape@detail@v10@fmt@@YA_NI@Z 10001760 f i format.obj
 0001:00000880       ?prefix_append@detail@v10@fmt@@YAXAAII@Z 10001880 f i format.obj
 0001:000008b0       ?adjust_precision@detail@v10@fmt@@YAXAAHH@Z 100018b0 f i format.obj
 0001:00000970       ??_3bigint@detail@v10@fmt@@QAEAAV0123@H@Z 10001970 f i format.obj
 0001:00000a20       ?compare@detail@v10@fmt@@YAHABVbigint@123@0@Z 10001a20 f i format.obj
 0001:00000ad0       ?add_compare@detail@v10@fmt@@YAHABVbigint@123@00@Z 10001ad0 f i format.obj
 0001:00000c50       ?assign_pow10@bigint@detail@v10@fmt@@QAEXH@Z 10001c50 f i format.obj
 0001:00000d30       ?square@bigint@detail@v10@fmt@@QAEXXZ 10001d30 f i format.obj
 0001:000010e0       ?divmod_assign@bigint@detail@v10@fmt@@QAEHABV1234@@Z 100020e0 f i format.obj
 0001:000012a0       ?format_dragon@detail@v10@fmt@@YAXU?$basic_fp@Vuint128_fallback@detail@v10@fmt@@@123@IHAAV?$buffer@D@123@AAH@Z 100022a0 f i format.obj
 0001:00001d20       ??1?$basic_memory_buffer@I$0CA@V?$allocator@I@std@@@v10@fmt@@QAE@XZ 10002d20 f i format.obj
 0001:00001d20       ??1bigint@detail@v10@fmt@@QAE@XZ 10002d20 f i format.obj
 0001:00001d70       ??_E_Facet_base@std@@UAEPAXI@Z 10002d70 f i * CIL library *:* CIL module *
 0001:00001d70       ??_G_Facet_base@std@@UAEPAXI@Z 10002d70 f i format.obj
 0001:00001da0       ??0_Locinfo@std@@QAE@PBD@Z 10002da0 f i format.obj
 0001:00001e50       ??1_Locinfo@std@@QAE@XZ    10002e50 f i format.obj
 0001:00001f30       ?_Incref@facet@locale@std@@UAEXXZ 10002f30 f i format.obj
 0001:00001f40       ?_Decref@facet@locale@std@@UAEPAV_Facet_base@3@XZ 10002f40 f i format.obj
 0001:00001f60       ??1facet@locale@std@@MAE@XZ 10002f60 f i format.obj
 0001:00001f70       ??1locale@std@@QAE@XZ      10002f70 f i format.obj
 0001:00001f90       ??$_Maklocstr@_W@std@@YAPA_WPBDPA_WABU_Cvtvec@@@Z 10002f90 f i format.obj
 0001:00002060       ?throw_format_error@detail@v10@fmt@@YAXPBD@Z 10003060 f   format.obj
 0001:00002100       ?compute_mul_parity@?$cache_accessor@M@dragonbox@detail@v10@fmt@@SA?AUcompute_mul_parity_result@12345@IAB_KH@Z 10003100 f i format.obj
 0001:00002160       ?get_cached_power@?$cache_accessor@N@dragonbox@detail@v10@fmt@@SA?AVuint128_fallback@345@H@Z 10003160 f i format.obj
 0001:000023a0       ?compute_mul_parity@?$cache_accessor@N@dragonbox@detail@v10@fmt@@SA?AUcompute_mul_parity_result@12345@_KABVuint128_fallback@345@H@Z 100033a0 f i format.obj
 0001:000024b0       ?remove_trailing_zeros@dragonbox@detail@v10@fmt@@YAHAAI@Z 100034b0 f i format.obj
 0001:00002500       ?remove_trailing_zeros@dragonbox@detail@v10@fmt@@YAHAA_K@Z 10003500 f i format.obj
 0001:00002700       ?is_printable@detail@v10@fmt@@YA_NGPBUsingleton@123@IPBE1I@Z 10003700 f i format.obj
 0001:000027c0       ?do_truename@?$numpunct@_W@std@@MBE?AV?$basic_string@_WU?$char_traits@_W@std@@V?$allocator@_W@2@@2@XZ 100037c0 f i format.obj
 0001:00002850       ?do_falsename@?$numpunct@_W@std@@MBE?AV?$basic_string@_WU?$char_traits@_W@std@@V?$allocator@_W@2@@2@XZ 10003850 f i format.obj
 0001:000028e0       ?do_grouping@?$numpunct@_W@std@@MBE?AV?$basic_string@DU?$char_traits@D@std@@V?$allocator@D@2@@2@XZ 100038e0 f i format.obj
 0001:00002960       ?do_thousands_sep@?$numpunct@_W@std@@MBE_WXZ 10003960 f i format.obj
 0001:00002970       ?do_decimal_point@?$numpunct@_W@std@@MBE_WXZ 10003970 f i format.obj
 0001:00002980       ??1?$_Yarn@D@std@@QAE@XZ   10003980 f i format.obj
 0001:00002980       ??1?$_Yarn@_W@std@@QAE@XZ  10003980 f i format.obj
 0001:000029a0       ?grow@?$basic_memory_buffer@H$0BPE@V?$allocator@H@std@@@v10@fmt@@MAEXI@Z 100039a0 f i format.obj
 0001:000029a0       ?grow@?$basic_memory_buffer@I$0CA@V?$allocator@I@std@@@v10@fmt@@MAEXI@Z 100039a0 f i format.obj
 0001:00002ab0       ??1?$basic_memory_buffer@D$0BPE@V?$allocator@D@std@@@v10@fmt@@QAE@XZ 10003ab0 f i format.obj
 0001:00002af0       ?grow@?$basic_memory_buffer@D$0BPE@V?$allocator@D@std@@@v10@fmt@@MAEXI@Z 10003af0 f i format.obj
 0001:00002bc0       ??1?$basic_memory_buffer@_W$0BPE@V?$allocator@_W@std@@@v10@fmt@@QAE@XZ 10003bc0 f i format.obj
 0001:00002c10       ?grow@?$basic_memory_buffer@_W$0BPE@V?$allocator@_W@std@@@v10@fmt@@MAEXI@Z 10003c10 f i format.obj
 0001:00002d10       ?try_resize@?$buffer@D@detail@v10@fmt@@QAEXI@Z 10003d10 f i format.obj
 0001:00002d40       ??0?$basic_string@DU?$char_traits@D@std@@V?$allocator@D@2@@std@@QAE@ABV01@@Z 10003d40 f i format.obj
 0001:00002de0       ??_G?$numpunct@_W@std@@MAEPAXI@Z 10003de0 f i format.obj
 0001:00002de0       ??_E?$numpunct@_W@std@@MAEPAXI@Z 10003de0 f i * CIL library *:* CIL module *
 0001:00002e30       ?deallocate@?$allocator@I@std@@QAEXQAII@Z 10003e30 f i format.obj
 0001:00002e70       ?assign@?$basic_string@_WU?$char_traits@_W@std@@V?$allocator@_W@2@@std@@QAEAAV12@QB_WI@Z 10003e70 f i format.obj
 0001:00002f80       ??0?$basic_string@_WU?$char_traits@_W@std@@V?$allocator@_W@2@@std@@QAE@QB_W@Z 10003f80 f i format.obj
 0001:00003010       ?assign@?$basic_string@DU?$char_traits@D@std@@V?$allocator@D@2@@std@@QAEAAV12@QBDI@Z 10004010 f i format.obj
 0001:00003110       ?allocate@?$allocator@I@std@@QAEPAII@Z 10004110 f i format.obj
 0001:00003110       ?allocate@?$allocator@PAUHINSTANCE__@@@std@@QAEPAPAUHINSTANCE__@@I@Z 10004110 f i Plist.obj
 0001:00003170       ?allocate@?$allocator@_W@std@@QAEPA_WI@Z 10004170 f i format.obj
 0001:000031d0       ?allocate@?$allocator@E@std@@QAEPAEI@Z 100041d0 f i perfthread.obj
 0001:000031d0       ?allocate@?$allocator@D@std@@QAEPADI@Z 100041d0 f i format.obj
 0001:00003230       ??$assign@_K$0A@@bigint@detail@v10@fmt@@AAEX_K@Z 10004230 f i format.obj
 0001:00003290       ??$?XH@bigint@detail@v10@fmt@@QAEAAV0123@H@Z 10004290 f i format.obj
 0001:00003310       ??$?4Vuint128_fallback@detail@v10@fmt@@@bigint@detail@v10@fmt@@QAEXVuint128_fallback@123@@Z 10004310 f i format.obj
 0001:000033a0       ??$use_facet@V?$numpunct@_W@std@@@std@@YAABV?$numpunct@_W@0@ABVlocale@0@@Z 100043a0 f i format.obj
 0001:00003630       ??$to_decimal@M@dragonbox@detail@v10@fmt@@YA?AU?$decimal_fp@M@0123@M@Z 10004630 f i format.obj
 0001:000038e0       ??$to_decimal@N@dragonbox@detail@v10@fmt@@YA?AU?$decimal_fp@N@0123@N@Z 100048e0 f i format.obj
 0001:00003d30       ??$append@D@?$buffer@D@detail@v10@fmt@@QAEXPBD0@Z 10004d30 f i format.obj
 0001:00003da0       ??0format_error@v10@fmt@@QAE@ABV012@@Z 10004da0 f i format.obj
 0001:00003de0       ??1?$unique_ptr@V_Facet_base@std@@U?$default_delete@V_Facet_base@std@@@2@@std@@QAE@XZ 10004de0 f i format.obj
 0001:00003df0       ??1?$_Tidy_guard@V?$numpunct@_W@std@@@std@@QAE@XZ 10004df0 f i format.obj
 0001:00003e20       ??$multiply@Vuint128_fallback@detail@v10@fmt@@$0A@@bigint@detail@v10@fmt@@AAEXVuint128_fallback@123@@Z 10004e20 f i format.obj
 0001:00004040       ??$format_decimal@DI@detail@v10@fmt@@YA?AU?$format_decimal_result@PAD@012@PADIH@Z 10005040 f i format.obj
 0001:000040b0       ??$format_decimal@D_K@detail@v10@fmt@@YA?AU?$format_decimal_result@PAD@012@PAD_KH@Z 100050b0 f i format.obj
 0001:000041e0       ??$write@DVappender@v10@fmt@@I$0A@@detail@v10@fmt@@YA?AVappender@12@V312@I@Z 100051e0 f i format.obj
 0001:00004290       ??$write@DVappender@v10@fmt@@_K$0A@@detail@v10@fmt@@YA?AVappender@12@V312@_K@Z 10005290 f i format.obj
 0001:00004370       ??$make_write_int_arg@_J@detail@v10@fmt@@YA?AU?$write_int_arg@_K@012@_JW4type@sign@12@@Z 10005370 f i format.obj
 0001:000043e0       ??1?$basic_memory_buffer@H$0BPE@V?$allocator@H@std@@@v10@fmt@@QAE@XZ 100053e0 f i format.obj
 0001:00004430       ??$format_hexfloat@N$0A@@detail@v10@fmt@@YAXNHUfloat_specs@012@AAV?$buffer@D@012@@Z 10005430 f i format.obj
 0001:00004700       ??$format_float@N@detail@v10@fmt@@YAHNHUfloat_specs@012@AAV?$buffer@D@012@@Z 10005700 f i format.obj
 0001:00004d50       ??R<lambda_1>@?DN@???$format_float@N@detail@v10@fmt@@YAHNHUfloat_specs@123@AAV?$buffer@D@123@@Z@QBE@IPAD@Z 10005d50 f i format.obj
 0001:00004e00       ??$fill_n@Vappender@v10@fmt@@HD@detail@v10@fmt@@YA?AVappender@12@V312@HABD@Z 10005e00 f i format.obj
 0001:00004e70       ??$format_uint@$03D_K@detail@v10@fmt@@YAPADPAD_KH_N@Z 10005e70 f i format.obj
 0001:00004ec0       ??$count_digits@$02_K@detail@v10@fmt@@YAH_K@Z 10005ec0 f i format.obj
 0001:00004ef0       ??__Ks@string_literals@literals@std@@YA?AV?$basic_string@_WU?$char_traits@_W@std@@V?$allocator@_W@2@@3@PB_WI@Z 10005ef0 f i handles.obj
 0001:00004f60       ??$decimal_point@_W@detail@v10@fmt@@YA_WVlocale_ref@012@@Z 10005f60 f i handles.obj
 0001:00005030       ?write_loc@detail@v10@fmt@@YA_NV?$back_insert_iterator@V?$buffer@_W@detail@v10@fmt@@@std@@Vloc_value@23@ABU?$format_specs@_W@23@Vlocale_ref@123@@Z 10006030 f i handles.obj
 0001:00005320       ??1?$loc_writer@_W@detail@v10@fmt@@QAE@XZ 10006320 f i handles.obj
 0001:00005410       ??$parse_format_specs@_W@detail@v10@fmt@@YAPB_WPB_W0AAU?$dynamic_format_specs@_W@012@AAV?$basic_format_parse_context@_W@12@W4type@012@@Z 10006410 f i handles.obj
 0001:00005ae0       ??$parse_dynamic_spec@_W@detail@v10@fmt@@YAPB_WPB_W0AAHAAU?$arg_ref@_W@012@AAV?$basic_format_parse_context@_W@12@@Z 10006ae0 f i handles.obj
 0001:00005b90       ??$parse_arg_id@_WAAU?$dynamic_spec_id_handler@_W@detail@v10@fmt@@@detail@v10@fmt@@YAPB_WPB_W0AAU?$dynamic_spec_id_handler@_W@012@@Z 10006b90 f i handles.obj
 0001:00005d10       ??1DebugToken@@QAE@XZ      10006d10 f i handles.obj
 0001:00006030       ??$format@K@far@@YA?A_PV?$basic_format_string@_WK@v10@fmt@@ABK@Z 10007030 f i handles.obj
 0001:00006030       ??$format@I@far@@YA?A_PV?$basic_format_string@_WI@v10@fmt@@ABI@Z 10007030 f i Pclass.obj
 0001:00006880       ??$format@V?$basic_string_view@_WU?$char_traits@_W@std@@@std@@K@far@@YA?A_PV?$basic_format_string@_WV?$basic_string_view@_WU?$char_traits@_W@std@@@std@@K@v10@fmt@@ABV?$basic_string_view@_WU?$char_traits@_W@std@@@std@@ABK@Z 10007880 f i handles.obj
 0001:00006ac0       ?PrintHandleInfo@@YA_NKPAX_NPAVPerfThread@@@Z 10007ac0 f   handles.obj
 0001:00006f90       ??$format@PB_WPB_WPB_WPB_WPB_W@far@@YA?A_PV?$basic_format_string@_WPB_WPB_WPB_WPB_WPB_W@v10@fmt@@ABQB_W1111@Z 10007f90 f i handles.obj
 0001:00007060       ??$parse_nonnegative_int@_W@detail@v10@fmt@@YAHAAPB_WPB_WH@Z 10008060 f i handles.obj
 0001:00007100       ?c_str@?$basic_string@_WU?$char_traits@_W@std@@V?$allocator@_W@2@@std@@QBEPB_WXZ 10008100 f i handles.obj
 0001:00007110       ??$format@GKV?$basic_string@_WU?$char_traits@_W@std@@V?$allocator@_W@2@@std@@V12@@far@@YA?A_PV?$basic_format_string@_WGKV?$basic_string@_WU?$char_traits@_W@std@@V?$allocator@_W@2@@std@@V12@@v10@fmt@@ABGABKABV?$basic_string@_WU?$char_traits@_W@std@@V?$allocator@_W@2@@std@@3@Z 10008110 f i handles.obj
 0001:000071f0       ??1?$unique_ptr@UPROCLIST_SYSTEM_HANDLE_INFORMATION@@Uvirtual_deleter@@@std@@QAE@XZ 100081f0 f i handles.obj
 0001:00007210       ??1?$scoped_lock@VPerfThread@@@std@@QAE@XZ 10008210 f i handles.obj
 0001:00007220       ??1?$unique_ptr@_WUlocal_deleter@@@std@@QAE@XZ 10008220 f i handles.obj
 0001:00007230       ??1?$unique_ptr@$$BY0A@_WU?$default_delete@$$BY0A@_W@std@@@std@@QAE@XZ 10008230 f i handles.obj
 0001:00007230       ??1?$unique_ptr@$$BY0A@DU?$default_delete@$$BY0A@D@std@@@std@@QAE@XZ 10008230 f i handles.obj
 0001:00007240       ??1?$unique_ptr@XUfree_deleter@@@std@@QAE@XZ 10008240 f i handles.obj
 0001:00007240       ??1?$unique_ptr@UPluginPanelItem@@Ufree_deleter@@@std@@QAE@XZ 10008240 f i Pclass.obj
 0001:00007250       ??1?$unique_ptr@XUhandle_closer@@@std@@QAE@XZ 10008250 f i handles.obj
 0001:00007260       ??4?$basic_string@_WU?$char_traits@_W@std@@V?$allocator@_W@2@@std@@QAEAAV01@$$QAV01@@Z 10008260 f i handles.obj
 0001:00007330       ??0?$basic_string@_WU?$char_traits@_W@std@@V?$allocator@_W@2@@std@@QAE@$$QAV01@@Z 10008330 f i handles.obj
 0001:000073c0       ??0?$basic_string@_WU?$char_traits@_W@std@@V?$allocator@_W@2@@std@@QAE@XZ 100083c0 f i handles.obj
 0001:00007410       ??0?$basic_string@_WU?$char_traits@_W@std@@V?$allocator@_W@2@@std@@QAE@ABV01@@Z 10008410 f i handles.obj
 0001:000074c0       ?starts_with@?$basic_string_view@_WU?$char_traits@_W@std@@@std@@QBE_NV12@@Z 100084c0 f i handles.obj
 0001:000074f0       ?assign@?$basic_string@_WU?$char_traits@_W@std@@V?$allocator@_W@2@@std@@QAEAAV12@I_W@Z 100084f0 f i handles.obj
 0001:00007620       ?compare@?$_WChar_traits@_W@std@@SAHQB_W0I@Z 10008620 f i handles.obj
 0001:00007680       ?on_replacement_field@format_handler@?1???$vformat_to@_W@detail@v10@fmt@@YAXAAV?$buffer@_W@234@V?$basic_string_view@_W@34@V?$basic_format_args@V?$basic_format_context@V?$back_insert_iterator@V?$buffer@_W@detail@v10@fmt@@@std@@_W@v10@fmt@@@34@Vlocale_ref@234@@Z@QAEXHPB_W@Z 10008680 f i handles.obj
 0001:000076f0       ?on_format_specs@format_handler@?1???$vformat_to@_W@detail@v10@fmt@@YAXAAV?$buffer@_W@234@V?$basic_string_view@_W@34@V?$basic_format_args@V?$basic_format_context@V?$back_insert_iterator@V?$buffer@_W@detail@v10@fmt@@@std@@_W@v10@fmt@@@34@Vlocale_ref@234@@Z@QAEPB_WHPB_W4@Z 100086f0 f i handles.obj
 0001:00007930       ??$vformat@_W$0A@@v10@fmt@@YA?AV?$basic_string@_WU?$char_traits@_W@std@@V?$allocator@_W@2@@std@@V?$basic_string_view@_W@01@V?$basic_format_args@V?$basic_format_context@V?$back_insert_iterator@V?$buffer@_W@detail@v10@fmt@@@std@@_W@v10@fmt@@@01@@Z 10008930 f i handles.obj
 0001:00007b90       ??$?0V?$basic_string_view@_WU?$char_traits@_W@std@@@std@@$0A@@?$basic_string@_WU?$char_traits@_W@std@@V?$allocator@_W@2@@std@@QAE@ABV?$basic_string_view@_WU?$char_traits@_W@std@@@1@ABV?$allocator@_W@1@@Z 10008b90 f i handles.obj
 0001:00007c00       ?get@?$basic_format_args@V?$basic_format_context@V?$back_insert_iterator@V?$buffer@_W@detail@v10@fmt@@@std@@_W@v10@fmt@@@v10@fmt@@QBE?AV?$basic_format_arg@V?$basic_format_context@V?$back_insert_iterator@V?$buffer@_W@detail@v10@fmt@@@std@@_W@v10@fmt@@@23@H@Z 10008c00 f i handles.obj
 0001:00007c90       ??$visit_format_arg@AAU?$loc_writer@_W@detail@v10@fmt@@V?$basic_format_context@Vappender@v10@fmt@@D@34@@v10@fmt@@YA_NAAU?$loc_writer@_W@detail@01@ABV?$basic_format_arg@V?$basic_format_context@Vappender@v10@fmt@@D@v10@fmt@@@01@@Z 10008c90 f i handles.obj
 0001:00008100       ??$visit_format_arg@U?$default_arg_formatter@_W@detail@v10@fmt@@V?$basic_format_context@V?$back_insert_iterator@V?$buffer@_W@detail@v10@fmt@@@std@@_W@34@@v10@fmt@@YA?AV?$back_insert_iterator@V?$buffer@_W@detail@v10@fmt@@@std@@$$QAU?$default_arg_formatter@_W@detail@01@ABV?$basic_format_arg@V?$basic_format_context@V?$back_insert_iterator@V?$buffer@_W@detail@v10@fmt@@@std@@_W@v10@fmt@@@01@@Z 10009100 f i handles.obj
 0001:00008820       ??$visit_format_arg@AAU?$arg_formatter@_W@detail@v10@fmt@@V?$basic_format_context@V?$back_insert_iterator@V?$buffer@_W@detail@v10@fmt@@@std@@_W@34@@v10@fmt@@YA?AV?$back_insert_iterator@V?$buffer@_W@detail@v10@fmt@@@std@@AAU?$arg_formatter@_W@detail@01@ABV?$basic_format_arg@V?$basic_format_context@V?$back_insert_iterator@V?$buffer@_W@detail@v10@fmt@@@std@@_W@v10@fmt@@@01@@Z 10009820 f i handles.obj
 0001:00008c30       ??$parse_format_string@$0A@_WUformat_handler@?1???$vformat_to@_W@detail@v10@fmt@@YAXAAV?$buffer@_W@234@V?$basic_string_view@_W@34@V?$basic_format_args@V?$basic_format_context@V?$back_insert_iterator@V?$buffer@_W@detail@v10@fmt@@@std@@_W@v10@fmt@@@34@Vlocale_ref@234@@Z@@detail@v10@fmt@@YAXV?$basic_string_view@_W@12@$$QAUformat_handler@?1???$vformat_to@_W@012@YAXAAV?$buffer@_W@012@0V?$basic_format_args@V?$basic_format_context@V?$back_insert_iterator@V?$buffer@_W@detail@v10@fmt@@@std@@_W@v10@fmt@@@12@Vlocale_ref@012@@Z@@Z 10009c30 f i handles.obj
 0001:000090f0       ??Rwriter@?1???$parse_format_string@$0A@_WUformat_handler@?1???$vformat_to@_W@detail@v10@fmt@@YAXAAV?$buffer@_W@234@V?$basic_string_view@_W@34@V?$basic_format_args@V?$basic_format_context@V?$back_insert_iterator@V?$buffer@_W@detail@v10@fmt@@@std@@_W@v10@fmt@@@34@Vlocale_ref@234@@Z@@detail@v10@fmt@@YAXV?$basic_string_view@_W@23@$$QAUformat_handler@?1???$vformat_to@_W@123@YAXAAV?$buffer@_W@123@0V?$basic_format_args@V?$basic_format_context@V?$back_insert_iterator@V?$buffer@_W@detail@v10@fmt@@@std@@_W@v10@fmt@@@23@Vlocale_ref@123@@Z@@Z@QAEXPB_W5@Z 1000a0f0 f i handles.obj
 0001:000091a0       ??$get_id@_W@?$basic_format_args@V?$basic_format_context@V?$back_insert_iterator@V?$buffer@_W@detail@v10@fmt@@@std@@_W@v10@fmt@@@v10@fmt@@QBEHV?$basic_string_view@_W@12@@Z 1000a1a0 f i handles.obj
 0001:00009250       ??$_Reallocate_grow_by@V<lambda_1>@?1??append@?$basic_string@_WU?$char_traits@_W@std@@V?$allocator@_W@2@@std@@QAEAAV34@QB_WI@Z@PB_WI@?$basic_string@_WU?$char_traits@_W@std@@V?$allocator@_W@2@@std@@AAEAAV01@IV<lambda_1>@?1??append@01@QAEAAV01@QB_WI@Z@PB_WI@Z 1000a250 f i handles.obj
 0001:00009380       ??$get_dynamic_spec@Vwidth_checker@detail@v10@fmt@@V?$basic_format_arg@V?$basic_format_context@V?$back_insert_iterator@V?$buffer@_W@detail@v10@fmt@@@std@@_W@v10@fmt@@@34@Uerror_handler@234@@detail@v10@fmt@@YAHV?$basic_format_arg@V?$basic_format_context@V?$back_insert_iterator@V?$buffer@_W@detail@v10@fmt@@@std@@_W@v10@fmt@@@12@Uerror_handler@012@@Z 1000a380 f i handles.obj
 0001:00009450       ??$get_arg@V?$basic_format_context@V?$back_insert_iterator@V?$buffer@_W@detail@v10@fmt@@@std@@_W@v10@fmt@@V?$basic_string_view@_W@23@@detail@v10@fmt@@YA?AV?$basic_format_arg@V?$basic_format_context@V?$back_insert_iterator@V?$buffer@_W@detail@v10@fmt@@@std@@_W@v10@fmt@@@12@AAV?$basic_format_context@V?$back_insert_iterator@V?$buffer@_W@detail@v10@fmt@@@std@@_W@12@V?$basic_string_view@_W@12@@Z 1000a450 f i handles.obj
 0001:000094c0       ??$get_dynamic_spec@Vprecision_checker@detail@v10@fmt@@V?$basic_format_arg@V?$basic_format_context@V?$back_insert_iterator@V?$buffer@_W@detail@v10@fmt@@@std@@_W@v10@fmt@@@34@Uerror_handler@234@@detail@v10@fmt@@YAHV?$basic_format_arg@V?$basic_format_context@V?$back_insert_iterator@V?$buffer@_W@detail@v10@fmt@@@std@@_W@v10@fmt@@@12@Uerror_handler@012@@Z 1000a4c0 f i handles.obj
 0001:00009590       ??1?$digit_grouping@_W@detail@v10@fmt@@QAE@XZ 1000a590 f i handles.obj
 0001:00009630       ??0?$digit_grouping@_W@detail@v10@fmt@@QAE@V?$basic_string@DU?$char_traits@D@std@@V?$allocator@D@2@@std@@V?$basic_string@_WU?$char_traits@_W@std@@V?$allocator@_W@2@@5@@Z 1000a630 f i handles.obj
 0001:000096d0       ??$write_int@V?$back_insert_iterator@V?$buffer@_W@detail@v10@fmt@@@std@@_K_W@detail@v10@fmt@@YA?AV?$back_insert_iterator@V?$buffer@_W@detail@v10@fmt@@@std@@V34@_KIABU?$format_specs@_W@12@ABV?$digit_grouping@_W@012@@Z 1000a6d0 f i handles.obj
 0001:00009840       ??$write@_WV?$back_insert_iterator@V?$buffer@_W@detail@v10@fmt@@@std@@H$0A@@detail@v10@fmt@@YA?AV?$back_insert_iterator@V?$buffer@_W@detail@v10@fmt@@@std@@V34@HABU?$format_specs@_W@12@Vlocale_ref@012@@Z 1000a840 f i handles.obj
 0001:00009900       ??$write@_WV?$back_insert_iterator@V?$buffer@_W@detail@v10@fmt@@@std@@_J$0A@@detail@v10@fmt@@YA?AV?$back_insert_iterator@V?$buffer@_W@detail@v10@fmt@@@std@@V34@_J@Z 1000a900 f i handles.obj
 0001:00009a90       ??$write@_WV?$back_insert_iterator@V?$buffer@_W@detail@v10@fmt@@@std@@_N$0A@@detail@v10@fmt@@YA?AV?$back_insert_iterator@V?$buffer@_W@detail@v10@fmt@@@std@@V34@_NABU?$format_specs@_W@12@Vlocale_ref@012@@Z 1000aa90 f i handles.obj
 0001:00009b70       ??$copy_str@_WPB_WV?$back_insert_iterator@V?$buffer@_W@detail@v10@fmt@@@std@@@detail@v10@fmt@@YA?AV?$back_insert_iterator@V?$buffer@_W@detail@v10@fmt@@@std@@PB_W0V34@@Z 1000ab70 f i handles.obj
 0001:00009b70       ??$copy_str@_WPA_WV?$back_insert_iterator@V?$buffer@_W@detail@v10@fmt@@@std@@@detail@v10@fmt@@YA?AV?$back_insert_iterator@V?$buffer@_W@detail@v10@fmt@@@std@@PA_W0V34@@Z 1000ab70 f i handles.obj
 0001:00009bd0       ??$write@_WV?$back_insert_iterator@V?$buffer@_W@detail@v10@fmt@@@std@@I$0A@@detail@v10@fmt@@YA?AV?$back_insert_iterator@V?$buffer@_W@detail@v10@fmt@@@std@@V34@IABU?$format_specs@_W@12@Vlocale_ref@012@@Z 1000abd0 f i handles.obj
 0001:00009c80       ??$write@_WV?$back_insert_iterator@V?$buffer@_W@detail@v10@fmt@@@std@@M$0A@@detail@v10@fmt@@YA?AV?$back_insert_iterator@V?$buffer@_W@detail@v10@fmt@@@std@@V34@MU?$format_specs@_W@12@Vlocale_ref@012@@Z 1000ac80 f i handles.obj
 0001:00009d30       ??$write@_WV?$back_insert_iterator@V?$buffer@_W@detail@v10@fmt@@@std@@N$0A@@detail@v10@fmt@@YA?AV?$back_insert_iterator@V?$buffer@_W@detail@v10@fmt@@@std@@V34@NU?$format_specs@_W@12@Vlocale_ref@012@@Z 1000ad30 f i handles.obj
 0001:00009dd0       ??$write@_WV?$back_insert_iterator@V?$buffer@_W@detail@v10@fmt@@@std@@O$0A@@detail@v10@fmt@@YA?AV?$back_insert_iterator@V?$buffer@_W@detail@v10@fmt@@@std@@V34@OU?$format_specs@_W@12@Vlocale_ref@012@@Z 1000add0 f i handles.obj
 0001:00009e70       ??$parse_arg_id@_WAAUid_adapter@?1???$parse_replacement_field@_WAAUformat_handler@?1???$vformat_to@_W@detail@v10@fmt@@YAXAAV?$buffer@_W@234@V?$basic_string_view@_W@34@V?$basic_format_args@V?$basic_format_context@V?$back_insert_iterator@V?$buffer@_W@detail@v10@fmt@@@std@@_W@v10@fmt@@@34@Vlocale_ref@234@@Z@@detail@v10@fmt@@YAPB_WPB_W0AAUformat_handler@?1???$vformat_to@_W@234@YAXAAV?$buffer@_W@234@V?$basic_string_view@_W@34@V?$basic_format_args@V?$basic_format_context@V?$back_insert_iterator@V?$buffer@_W@detail@v10@fmt@@@std@@_W@v10@fmt@@@34@Vlocale_ref@234@@Z@@Z@@detail@v10@fmt@@YAPB_WPB_W0AAUid_adapter@?1???$parse_replacement_field@_WAAUformat_handler@?1???$vformat_to@_W@detail@v10@fmt@@YAXAAV?$buffer@_W@234@V?$basic_string_view@_W@34@V?$basic_format_args@V?$basic_format_context@V?$back_insert_iterator@V?$buffer@_W@detail@v10@fmt@@@std@@_W@v10@fmt@@@34@Vlocale_ref@234@@Z@@012@YAPB_W00AAUformat_handler@?1???$vformat_to@_W@012@YAXAAV?$buffer@_W@012@V?$basic_string_view@_W@12@V?$basic_format_args@V?$basic_format_context@V?$back_insert_iterator@V?$buffer@_W@detail@v10@fmt@@@std@@_W@v10@fmt@@@12@Vlocale_ref@012@@Z@@Z@@Z 1000ae70 f i handles.obj
 0001:00009ff0       ?count_separators@?$digit_grouping@_W@detail@v10@fmt@@QBEHH@Z 1000aff0 f i handles.obj
 0001:0000a070       ??4?$back_insert_iterator@V?$buffer@_W@detail@v10@fmt@@@std@@QAEAAV01@$$QA_W@Z 1000b070 f i handles.obj
 0001:0000a0b0       ??$apply@V?$back_insert_iterator@V?$buffer@_W@detail@v10@fmt@@@std@@D@?$digit_grouping@_W@detail@v10@fmt@@QBE?AV?$back_insert_iterator@V?$buffer@_W@detail@v10@fmt@@@std@@V45@V?$basic_string_view@D@23@@Z 1000b0b0 f i handles.obj
 0001:0000a3a0       ??$format_decimal@_WI@detail@v10@fmt@@YA?AU?$format_decimal_result@PA_W@012@PA_WIH@Z 1000b3a0 f i handles.obj
 0001:0000a430       ??$write@_WV?$back_insert_iterator@V?$buffer@_W@detail@v10@fmt@@@std@@@detail@v10@fmt@@YA?AV?$back_insert_iterator@V?$buffer@_W@detail@v10@fmt@@@std@@V34@V?$basic_string_view@_W@12@ABU?$format_specs@_W@12@@Z 1000b430 f i handles.obj
 0001:0000a600       ??$format_decimal@_W_K@detail@v10@fmt@@YA?AU?$format_decimal_result@PA_W@012@PA_W_KH@Z 1000b600 f i handles.obj
 0001:0000a740       ??$write_nonfinite@_WV?$back_insert_iterator@V?$buffer@_W@detail@v10@fmt@@@std@@@detail@v10@fmt@@YA?AV?$back_insert_iterator@V?$buffer@_W@detail@v10@fmt@@@std@@V34@_NU?$format_specs@_W@12@ABUfloat_specs@012@@Z 1000b740 f i handles.obj
 0001:0000a850       ??$write_ptr@_WV?$back_insert_iterator@V?$buffer@_W@detail@v10@fmt@@@std@@I@detail@v10@fmt@@YA?AV?$back_insert_iterator@V?$buffer@_W@detail@v10@fmt@@@std@@V34@IPBU?$format_specs@_W@12@@Z 1000b850 f i handles.obj
 0001:0000a910       ??R<lambda_1>@?1???$write_ptr@_WV?$back_insert_iterator@V?$buffer@_W@detail@v10@fmt@@@std@@I@detail@v10@fmt@@YA?AV?$back_insert_iterator@V?$buffer@_W@detail@v10@fmt@@@std@@V45@IPBU?$format_specs@_W@23@@Z@QBE@0@Z 1000b910 f i handles.obj
 0001:0000a980       ??$write_char@_WV?$back_insert_iterator@V?$buffer@_W@detail@v10@fmt@@@std@@@detail@v10@fmt@@YA?AV?$back_insert_iterator@V?$buffer@_W@detail@v10@fmt@@@std@@V34@_WABU?$format_specs@_W@12@@Z 1000b980 f i handles.obj
 0001:0000aa10       ??R<lambda_1>@?1???$write_char@_WV?$back_insert_iterator@V?$buffer@_W@detail@v10@fmt@@@std@@@detail@v10@fmt@@YA?AV?$back_insert_iterator@V?$buffer@_W@detail@v10@fmt@@@std@@V45@_WABU?$format_specs@_W@23@@Z@QBE@0@Z 1000ba10 f i handles.obj
 0001:0000ab20       ??$write_float@_WV?$back_insert_iterator@V?$buffer@_W@detail@v10@fmt@@@std@@M@detail@v10@fmt@@YA?AV?$back_insert_iterator@V?$buffer@_W@detail@v10@fmt@@@std@@V34@MU?$format_specs@_W@12@Vlocale_ref@012@@Z 1000bb20 f i handles.obj
 0001:0000aec0       ??$write_float@_WV?$back_insert_iterator@V?$buffer@_W@detail@v10@fmt@@@std@@N@detail@v10@fmt@@YA?AV?$back_insert_iterator@V?$buffer@_W@detail@v10@fmt@@@std@@V34@NU?$format_specs@_W@12@Vlocale_ref@012@@Z 1000bec0 f i handles.obj
 0001:0000b250       ??$write_float@_WV?$back_insert_iterator@V?$buffer@_W@detail@v10@fmt@@@std@@O@detail@v10@fmt@@YA?AV?$back_insert_iterator@V?$buffer@_W@detail@v10@fmt@@@std@@V34@OU?$format_specs@_W@12@Vlocale_ref@012@@Z 1000c250 f i handles.obj
 0001:0000b5e0       ??$fill@V?$back_insert_iterator@V?$buffer@_W@detail@v10@fmt@@@std@@_W@detail@v10@fmt@@YA?AV?$back_insert_iterator@V?$buffer@_W@detail@v10@fmt@@@std@@V34@IABU?$fill_t@_W@012@@Z 1000c5e0 f i handles.obj
 0001:0000b690       ??$write_padded@$00V?$back_insert_iterator@V?$buffer@_W@detail@v10@fmt@@@std@@_WV<lambda_1>@?1???$write@_WV?$back_insert_iterator@V?$buffer@_W@detail@v10@fmt@@@std@@@detail@v10@fmt@@YA?AV12@V12@V?$basic_string_view@_W@56@ABU?$format_specs@_W@56@@Z@@detail@v10@fmt@@YA?AV?$back_insert_iterator@V?$buffer@_W@detail@v10@fmt@@@std@@V34@ABU?$format_specs@_W@12@II$$QAV<lambda_1>@?1???$write@_WV?$back_insert_iterator@V?$buffer@_W@detail@v10@fmt@@@std@@@012@YA?AV34@0V?$basic_string_view@_W@12@1@Z@@Z 1000c690 f i handles.obj
 0001:0000b810       ??$write_int@_WV?$back_insert_iterator@V?$buffer@_W@detail@v10@fmt@@@std@@I@detail@v10@fmt@@YA?AV?$back_insert_iterator@V?$buffer@_W@detail@v10@fmt@@@std@@V34@U?$write_int_arg@I@012@ABU?$format_specs@_W@12@Vlocale_ref@012@@Z 1000c810 f i handles.obj
 0001:0000ba40       ??R<lambda_3>@?8???$write_int@_WV?$back_insert_iterator@V?$buffer@_W@detail@v10@fmt@@@std@@I@detail@v10@fmt@@YA?AV?$back_insert_iterator@V?$buffer@_W@detail@v10@fmt@@@std@@V45@U?$write_int_arg@I@123@ABU?$format_specs@_W@23@Vlocale_ref@123@@Z@QBE@0@Z 1000ca40 f i handles.obj
 0001:0000bae0       ??R<lambda_4>@?M@???$write_int@_WV?$back_insert_iterator@V?$buffer@_W@detail@v10@fmt@@@std@@I@detail@v10@fmt@@YA?AV?$back_insert_iterator@V?$buffer@_W@detail@v10@fmt@@@std@@V45@U?$write_int_arg@I@123@ABU?$format_specs@_W@23@Vlocale_ref@123@@Z@QBE@0@Z 1000cae0 f i handles.obj
 0001:0000bb80       ??$copy_str@_WPBDV?$back_insert_iterator@V?$buffer@_W@detail@v10@fmt@@@std@@@detail@v10@fmt@@YA?AV?$back_insert_iterator@V?$buffer@_W@detail@v10@fmt@@@std@@PBD0V34@@Z 1000cb80 f i handles.obj
 0001:0000bbe0       ??$do_write_float@V?$back_insert_iterator@V?$buffer@_W@detail@v10@fmt@@@std@@U?$decimal_fp@M@dragonbox@detail@v10@fmt@@_WV?$digit_grouping@_W@567@@detail@v10@fmt@@YA?AV?$back_insert_iterator@V?$buffer@_W@detail@v10@fmt@@@std@@V34@ABU?$decimal_fp@M@dragonbox@012@ABU?$format_specs@_W@12@Ufloat_specs@012@Vlocale_ref@012@@Z 1000cbe0 f i handles.obj
 0001:0000c170       ??R<lambda_2>@?4???$do_write_float@V?$back_insert_iterator@V?$buffer@_W@detail@v10@fmt@@@std@@U?$decimal_fp@M@dragonbox@detail@v10@fmt@@_WV?$digit_grouping@_W@567@@detail@v10@fmt@@YA?AV?$back_insert_iterator@V?$buffer@_W@detail@v10@fmt@@@std@@V45@ABU?$decimal_fp@M@dragonbox@123@ABU?$format_specs@_W@23@Ufloat_specs@123@Vlocale_ref@123@@Z@QBE@0@Z 1000d170 f i handles.obj
 0001:0000c230       ??R<lambda_3>@?BD@???$do_write_float@V?$back_insert_iterator@V?$buffer@_W@detail@v10@fmt@@@std@@U?$decimal_fp@M@dragonbox@detail@v10@fmt@@_WV?$digit_grouping@_W@567@@detail@v10@fmt@@YA?AV?$back_insert_iterator@V?$buffer@_W@detail@v10@fmt@@@std@@V45@ABU?$decimal_fp@M@dragonbox@123@ABU?$format_specs@_W@23@Ufloat_specs@123@Vlocale_ref@123@@Z@QBE@0@Z 1000d230 f i handles.obj
 0001:0000c4a0       ??R<lambda_4>@?BO@???$do_write_float@V?$back_insert_iterator@V?$buffer@_W@detail@v10@fmt@@@std@@U?$decimal_fp@M@dragonbox@detail@v10@fmt@@_WV?$digit_grouping@_W@567@@detail@v10@fmt@@YA?AV?$back_insert_iterator@V?$buffer@_W@detail@v10@fmt@@@std@@V45@ABU?$decimal_fp@M@dragonbox@123@ABU?$format_specs@_W@23@Ufloat_specs@123@Vlocale_ref@123@@Z@QBE@0@Z 1000d4a0 f i handles.obj
 0001:0000c6a0       ??R<lambda_5>@?1???$do_write_float@V?$back_insert_iterator@V?$buffer@_W@detail@v10@fmt@@@std@@U?$decimal_fp@M@dragonbox@detail@v10@fmt@@_WV?$digit_grouping@_W@567@@detail@v10@fmt@@YA?AV?$back_insert_iterator@V?$buffer@_W@detail@v10@fmt@@@std@@V45@ABU?$decimal_fp@M@dragonbox@123@ABU?$format_specs@_W@23@Ufloat_specs@123@Vlocale_ref@123@@Z@QBE@0@Z 1000d6a0 f i handles.obj
 0001:0000c7d0       ??$do_write_float@V?$back_insert_iterator@V?$buffer@_W@detail@v10@fmt@@@std@@U?$decimal_fp@N@dragonbox@detail@v10@fmt@@_WV?$digit_grouping@_W@567@@detail@v10@fmt@@YA?AV?$back_insert_iterator@V?$buffer@_W@detail@v10@fmt@@@std@@V34@ABU?$decimal_fp@N@dragonbox@012@ABU?$format_specs@_W@12@Ufloat_specs@012@Vlocale_ref@012@@Z 1000d7d0 f i handles.obj
 0001:0000ce80       ??R<lambda_2>@?4???$do_write_float@V?$back_insert_iterator@V?$buffer@_W@detail@v10@fmt@@@std@@U?$decimal_fp@N@dragonbox@detail@v10@fmt@@_WV?$digit_grouping@_W@567@@detail@v10@fmt@@YA?AV?$back_insert_iterator@V?$buffer@_W@detail@v10@fmt@@@std@@V45@ABU?$decimal_fp@N@dragonbox@123@ABU?$format_specs@_W@23@Ufloat_specs@123@Vlocale_ref@123@@Z@QBE@0@Z 1000de80 f i handles.obj
 0001:0000cf40       ??R<lambda_3>@?BD@???$do_write_float@V?$back_insert_iterator@V?$buffer@_W@detail@v10@fmt@@@std@@U?$decimal_fp@N@dragonbox@detail@v10@fmt@@_WV?$digit_grouping@_W@567@@detail@v10@fmt@@YA?AV?$back_insert_iterator@V?$buffer@_W@detail@v10@fmt@@@std@@V45@ABU?$decimal_fp@N@dragonbox@123@ABU?$format_specs@_W@23@Ufloat_specs@123@Vlocale_ref@123@@Z@QBE@0@Z 1000df40 f i handles.obj
 0001:0000d1e0       ??R<lambda_4>@?BO@???$do_write_float@V?$back_insert_iterator@V?$buffer@_W@detail@v10@fmt@@@std@@U?$decimal_fp@N@dragonbox@detail@v10@fmt@@_WV?$digit_grouping@_W@567@@detail@v10@fmt@@YA?AV?$back_insert_iterator@V?$buffer@_W@detail@v10@fmt@@@std@@V45@ABU?$decimal_fp@N@dragonbox@123@ABU?$format_specs@_W@23@Ufloat_specs@123@Vlocale_ref@123@@Z@QBE@0@Z 1000e1e0 f i handles.obj
 0001:0000d400       ??R<lambda_5>@?1???$do_write_float@V?$back_insert_iterator@V?$buffer@_W@detail@v10@fmt@@@std@@U?$decimal_fp@N@dragonbox@detail@v10@fmt@@_WV?$digit_grouping@_W@567@@detail@v10@fmt@@YA?AV?$back_insert_iterator@V?$buffer@_W@detail@v10@fmt@@@std@@V45@ABU?$decimal_fp@N@dragonbox@123@ABU?$format_specs@_W@23@Ufloat_specs@123@Vlocale_ref@123@@Z@QBE@0@Z 1000e400 f i handles.obj
 0001:0000d540       ??$format_uint@$03_WV?$back_insert_iterator@V?$buffer@_W@detail@v10@fmt@@@std@@I@detail@v10@fmt@@YA?AV?$back_insert_iterator@V?$buffer@_W@detail@v10@fmt@@@std@@V34@IH_N@Z 1000e540 f i handles.obj
 0001:0000d620       ??$write_int@_WV?$back_insert_iterator@V?$buffer@_W@detail@v10@fmt@@@std@@_K@detail@v10@fmt@@YA?AV?$back_insert_iterator@V?$buffer@_W@detail@v10@fmt@@@std@@V34@U?$write_int_arg@_K@012@ABU?$format_specs@_W@12@Vlocale_ref@012@@Z 1000e620 f i handles.obj
 0001:0000d890       ??R<lambda_2>@?5???$write_int@_WV?$back_insert_iterator@V?$buffer@_W@detail@v10@fmt@@@std@@_K@detail@v10@fmt@@YA?AV?$back_insert_iterator@V?$buffer@_W@detail@v10@fmt@@@std@@V45@U?$write_int_arg@_K@123@ABU?$format_specs@_W@23@Vlocale_ref@123@@Z@QBE@0@Z 1000e890 f i handles.obj
 0001:0000d980       ??R<lambda_3>@?8???$write_int@_WV?$back_insert_iterator@V?$buffer@_W@detail@v10@fmt@@@std@@_K@detail@v10@fmt@@YA?AV?$back_insert_iterator@V?$buffer@_W@detail@v10@fmt@@@std@@V45@U?$write_int_arg@_K@123@ABU?$format_specs@_W@23@Vlocale_ref@123@@Z@QBE@0@Z 1000e980 f i handles.obj
 0001:0000da40       ??R<lambda_4>@?M@???$write_int@_WV?$back_insert_iterator@V?$buffer@_W@detail@v10@fmt@@@std@@_K@detail@v10@fmt@@YA?AV?$back_insert_iterator@V?$buffer@_W@detail@v10@fmt@@@std@@V45@U?$write_int_arg@_K@123@ABU?$format_specs@_W@23@Vlocale_ref@123@@Z@QBE@0@Z 1000ea40 f i handles.obj
 0001:0000db00       ??$parse_float_type_spec@Uerror_handler@detail@v10@fmt@@_W@detail@v10@fmt@@YA?AUfloat_specs@012@ABU?$format_specs@_W@12@$$QAUerror_handler@012@@Z 1000eb00 f i handles.obj
 0001:0000dc00       ??$write_bytes@$01_WV?$back_insert_iterator@V?$buffer@_W@detail@v10@fmt@@@std@@@detail@v10@fmt@@YA?AV?$back_insert_iterator@V?$buffer@_W@detail@v10@fmt@@@std@@V34@V?$basic_string_view@D@12@ABU?$format_specs@_W@12@@Z 1000ec00 f i handles.obj
 0001:0000dca0       ??0?$digit_grouping@_W@detail@v10@fmt@@QAE@Vlocale_ref@123@_N@Z 1000eca0 f i handles.obj
 0001:0000dfc0       ??$fill_n@V?$back_insert_iterator@V?$buffer@_W@detail@v10@fmt@@@std@@I_W@detail@v10@fmt@@YA?AV?$back_insert_iterator@V?$buffer@_W@detail@v10@fmt@@@std@@V34@IAB_W@Z 1000efc0 f i handles.obj
 0001:0000e030       ??$find_escape@_W@detail@v10@fmt@@YA?AU?$find_escape_result@_W@012@PB_W0@Z 1000f030 f i handles.obj
 0001:0000e0b0       ??$write_escaped_cp@V?$back_insert_iterator@V?$buffer@_W@detail@v10@fmt@@@std@@_W@detail@v10@fmt@@YA?AV?$back_insert_iterator@V?$buffer@_W@detail@v10@fmt@@@std@@V34@ABU?$find_escape_result@_W@012@@Z 1000f0b0 f i handles.obj
 0001:0000e3d0       ??$write_int@V?$back_insert_iterator@V?$buffer@_W@detail@v10@fmt@@@std@@_WV<lambda_1>@?4???$write_int@_WV?$back_insert_iterator@V?$buffer@_W@detail@v10@fmt@@@std@@I@detail@v10@fmt@@YA?AV12@V12@U?$write_int_arg@I@456@ABU?$format_specs@_W@56@Vlocale_ref@456@@Z@@detail@v10@fmt@@YA?AV?$back_insert_iterator@V?$buffer@_W@detail@v10@fmt@@@std@@V34@HIABU?$format_specs@_W@12@V<lambda_1>@?4???$write_int@_WV?$back_insert_iterator@V?$buffer@_W@detail@v10@fmt@@@std@@I@012@YA?AV34@0U?$write_int_arg@I@012@1Vlocale_ref@012@@Z@@Z 1000f3d0 f i handles.obj
 0001:0000e5e0       ??$write_int@V?$back_insert_iterator@V?$buffer@_W@detail@v10@fmt@@@std@@_WV<lambda_2>@?5???$write_int@_WV?$back_insert_iterator@V?$buffer@_W@detail@v10@fmt@@@std@@I@detail@v10@fmt@@YA?AV12@V12@U?$write_int_arg@I@456@ABU?$format_specs@_W@56@Vlocale_ref@456@@Z@@detail@v10@fmt@@YA?AV?$back_insert_iterator@V?$buffer@_W@detail@v10@fmt@@@std@@V34@HIABU?$format_specs@_W@12@V<lambda_2>@?5???$write_int@_WV?$back_insert_iterator@V?$buffer@_W@detail@v10@fmt@@@std@@I@012@YA?AV34@0U?$write_int_arg@I@012@1Vlocale_ref@012@@Z@@Z 1000f5e0 f i handles.obj
 0001:0000e780       ??$write_int@V?$back_insert_iterator@V?$buffer@_W@detail@v10@fmt@@@std@@_WV<lambda_3>@?8???$write_int@_WV?$back_insert_iterator@V?$buffer@_W@detail@v10@fmt@@@std@@I@detail@v10@fmt@@YA?AV12@V12@U?$write_int_arg@I@456@ABU?$format_specs@_W@56@Vlocale_ref@456@@Z@@detail@v10@fmt@@YA?AV?$back_insert_iterator@V?$buffer@_W@detail@v10@fmt@@@std@@V34@HIABU?$format_specs@_W@12@V<lambda_3>@?8???$write_int@_WV?$back_insert_iterator@V?$buffer@_W@detail@v10@fmt@@@std@@I@012@YA?AV34@0U?$write_int_arg@I@012@1Vlocale_ref@012@@Z@@Z 1000f780 f i handles.obj
 0001:0000e920       ??$write_int@V?$back_insert_iterator@V?$buffer@_W@detail@v10@fmt@@@std@@_WV<lambda_4>@?M@???$write_int@_WV?$back_insert_iterator@V?$buffer@_W@detail@v10@fmt@@@std@@I@detail@v10@fmt@@YA?AV12@V12@U?$write_int_arg@I@456@ABU?$format_specs@_W@56@Vlocale_ref@456@@Z@@detail@v10@fmt@@YA?AV?$back_insert_iterator@V?$buffer@_W@detail@v10@fmt@@@std@@V34@HIABU?$format_specs@_W@12@V<lambda_4>@?M@???$write_int@_WV?$back_insert_iterator@V?$buffer@_W@detail@v10@fmt@@@std@@I@012@YA?AV34@0U?$write_int_arg@I@012@1Vlocale_ref@012@@Z@@Z 1000f920 f i handles.obj
 0001:0000eac0       ??$write_significand@V?$back_insert_iterator@V?$buffer@_W@detail@v10@fmt@@@std@@I_W$0A@@detail@v10@fmt@@YA?AV?$back_insert_iterator@V?$buffer@_W@detail@v10@fmt@@@std@@V34@IHH_W@Z 1000fac0 f i handles.obj
 0001:0000ebb0       ??$fill_n@V?$back_insert_iterator@V?$buffer@_W@detail@v10@fmt@@@std@@H_W@detail@v10@fmt@@YA?AV?$back_insert_iterator@V?$buffer@_W@detail@v10@fmt@@@std@@V34@HAB_W@Z 1000fbb0 f i handles.obj
 0001:0000ec20       ??$write_exponent@_WV?$back_insert_iterator@V?$buffer@_W@detail@v10@fmt@@@std@@@detail@v10@fmt@@YA?AV?$back_insert_iterator@V?$buffer@_W@detail@v10@fmt@@@std@@HV34@@Z 1000fc20 f i handles.obj
 0001:0000ed60       ??$write_significand@V?$back_insert_iterator@V?$buffer@_W@detail@v10@fmt@@@std@@_K_W$0A@@detail@v10@fmt@@YA?AV?$back_insert_iterator@V?$buffer@_W@detail@v10@fmt@@@std@@V34@_KHH_W@Z 1000fd60 f i handles.obj
 0001:0000ef40       ??$copy_str_noinline@_WPADV?$back_insert_iterator@V?$buffer@_W@detail@v10@fmt@@@std@@@detail@v10@fmt@@YA?AV?$back_insert_iterator@V?$buffer@_W@detail@v10@fmt@@@std@@PAD0V34@@Z 1000ff40 f i handles.obj
 0001:0000ef90       ??$write_int@V?$back_insert_iterator@V?$buffer@_W@detail@v10@fmt@@@std@@_WV<lambda_1>@?4???$write_int@_WV?$back_insert_iterator@V?$buffer@_W@detail@v10@fmt@@@std@@_K@detail@v10@fmt@@YA?AV12@V12@U?$write_int_arg@_K@456@ABU?$format_specs@_W@56@Vlocale_ref@456@@Z@@detail@v10@fmt@@YA?AV?$back_insert_iterator@V?$buffer@_W@detail@v10@fmt@@@std@@V34@HIABU?$format_specs@_W@12@V<lambda_1>@?4???$write_int@_WV?$back_insert_iterator@V?$buffer@_W@detail@v10@fmt@@@std@@_K@012@YA?AV34@0U?$write_int_arg@_K@012@1Vlocale_ref@012@@Z@@Z 1000ff90 f i handles.obj
 0001:0000f1c0       ??$write_int@V?$back_insert_iterator@V?$buffer@_W@detail@v10@fmt@@@std@@_WV<lambda_2>@?5???$write_int@_WV?$back_insert_iterator@V?$buffer@_W@detail@v10@fmt@@@std@@_K@detail@v10@fmt@@YA?AV12@V12@U?$write_int_arg@_K@456@ABU?$format_specs@_W@56@Vlocale_ref@456@@Z@@detail@v10@fmt@@YA?AV?$back_insert_iterator@V?$buffer@_W@detail@v10@fmt@@@std@@V34@HIABU?$format_specs@_W@12@V<lambda_2>@?5???$write_int@_WV?$back_insert_iterator@V?$buffer@_W@detail@v10@fmt@@@std@@_K@012@YA?AV34@0U?$write_int_arg@_K@012@1Vlocale_ref@012@@Z@@Z 100101c0 f i handles.obj
 0001:0000f370       ??$write_int@V?$back_insert_iterator@V?$buffer@_W@detail@v10@fmt@@@std@@_WV<lambda_3>@?8???$write_int@_WV?$back_insert_iterator@V?$buffer@_W@detail@v10@fmt@@@std@@_K@detail@v10@fmt@@YA?AV12@V12@U?$write_int_arg@_K@456@ABU?$format_specs@_W@56@Vlocale_ref@456@@Z@@detail@v10@fmt@@YA?AV?$back_insert_iterator@V?$buffer@_W@detail@v10@fmt@@@std@@V34@HIABU?$format_specs@_W@12@V<lambda_3>@?8???$write_int@_WV?$back_insert_iterator@V?$buffer@_W@detail@v10@fmt@@@std@@_K@012@YA?AV34@0U?$write_int_arg@_K@012@1Vlocale_ref@012@@Z@@Z 10010370 f i handles.obj
 0001:0000f520       ??$write_int@V?$back_insert_iterator@V?$buffer@_W@detail@v10@fmt@@@std@@_WV<lambda_4>@?M@???$write_int@_WV?$back_insert_iterator@V?$buffer@_W@detail@v10@fmt@@@std@@_K@detail@v10@fmt@@YA?AV12@V12@U?$write_int_arg@_K@456@ABU?$format_specs@_W@56@Vlocale_ref@456@@Z@@detail@v10@fmt@@YA?AV?$back_insert_iterator@V?$buffer@_W@detail@v10@fmt@@@std@@V34@HIABU?$format_specs@_W@12@V<lambda_4>@?M@???$write_int@_WV?$back_insert_iterator@V?$buffer@_W@detail@v10@fmt@@@std@@_K@012@YA?AV34@0U?$write_int_arg@_K@012@1Vlocale_ref@012@@Z@@Z 10010520 f i handles.obj
 0001:0000f6d0       ??$do_write_float@V?$back_insert_iterator@V?$buffer@_W@detail@v10@fmt@@@std@@Ubig_decimal_fp@detail@v10@fmt@@_WV?$digit_grouping@_W@456@@detail@v10@fmt@@YA?AV?$back_insert_iterator@V?$buffer@_W@detail@v10@fmt@@@std@@V34@ABUbig_decimal_fp@012@ABU?$format_specs@_W@12@Ufloat_specs@012@Vlocale_ref@012@@Z 100106d0 f i handles.obj
 0001:0000fbe0       ??R<lambda_2>@?4???$do_write_float@V?$back_insert_iterator@V?$buffer@_W@detail@v10@fmt@@@std@@Ubig_decimal_fp@detail@v10@fmt@@_WV?$digit_grouping@_W@456@@detail@v10@fmt@@YA?AV?$back_insert_iterator@V?$buffer@_W@detail@v10@fmt@@@std@@V45@ABUbig_decimal_fp@123@ABU?$format_specs@_W@23@Ufloat_specs@123@Vlocale_ref@123@@Z@QBE@0@Z 10010be0 f i handles.obj
 0001:0000fca0       ??R<lambda_3>@?BD@???$do_write_float@V?$back_insert_iterator@V?$buffer@_W@detail@v10@fmt@@@std@@Ubig_decimal_fp@detail@v10@fmt@@_WV?$digit_grouping@_W@456@@detail@v10@fmt@@YA?AV?$back_insert_iterator@V?$buffer@_W@detail@v10@fmt@@@std@@V45@ABUbig_decimal_fp@123@ABU?$format_specs@_W@23@Ufloat_specs@123@Vlocale_ref@123@@Z@QBE@0@Z 10010ca0 f i handles.obj
 0001:0000fed0       ??R<lambda_4>@?BO@???$do_write_float@V?$back_insert_iterator@V?$buffer@_W@detail@v10@fmt@@@std@@Ubig_decimal_fp@detail@v10@fmt@@_WV?$digit_grouping@_W@456@@detail@v10@fmt@@YA?AV?$back_insert_iterator@V?$buffer@_W@detail@v10@fmt@@@std@@V45@ABUbig_decimal_fp@123@ABU?$format_specs@_W@23@Ufloat_specs@123@Vlocale_ref@123@@Z@QBE@0@Z 10010ed0 f i handles.obj
 0001:000100d0       ??$write_codepoint@$01_WV?$back_insert_iterator@V?$buffer@_W@detail@v10@fmt@@@std@@@detail@v10@fmt@@YA?AV?$back_insert_iterator@V?$buffer@_W@detail@v10@fmt@@@std@@V34@DI@Z 100110d0 f i handles.obj
 0001:00010170       ??$apply@V?$back_insert_iterator@V?$buffer@_W@detail@v10@fmt@@@std@@_W@?$digit_grouping@_W@detail@v10@fmt@@QBE?AV?$back_insert_iterator@V?$buffer@_W@detail@v10@fmt@@@std@@V45@V?$basic_string_view@_W@23@@Z 10011170 f i handles.obj
 0001:00010460       ??$write_significand@V?$back_insert_iterator@V?$buffer@_W@detail@v10@fmt@@@std@@_W@detail@v10@fmt@@YA?AV?$back_insert_iterator@V?$buffer@_W@detail@v10@fmt@@@std@@V34@PBDHH_W@Z 10011460 f i handles.obj
 0001:000104e0       ??$write_padded@$01V?$back_insert_iterator@V?$buffer@_W@detail@v10@fmt@@@std@@_WAAV<lambda_5>@?1???$do_write_float@V?$back_insert_iterator@V?$buffer@_W@detail@v10@fmt@@@std@@Ubig_decimal_fp@detail@v10@fmt@@_WV?$digit_grouping@_W@456@@detail@v10@fmt@@YA?AV12@V12@ABUbig_decimal_fp@456@ABU?$format_specs@_W@56@Ufloat_specs@456@Vlocale_ref@456@@Z@@detail@v10@fmt@@YA?AV?$back_insert_iterator@V?$buffer@_W@detail@v10@fmt@@@std@@V34@ABU?$format_specs@_W@12@IIAAV<lambda_5>@?1???$do_write_float@V?$back_insert_iterator@V?$buffer@_W@detail@v10@fmt@@@std@@Ubig_decimal_fp@detail@v10@fmt@@_WV?$digit_grouping@_W@456@@012@YA?AV34@0ABUbig_decimal_fp@012@1Ufloat_specs@012@Vlocale_ref@012@@Z@@Z 100114e0 f i handles.obj
 0001:00010630       ??0PluginSettings@@QAE@ABU_GUID@@P6GHPAXW4FAR_SETTINGS_CONTROL_COMMANDS@@H1@Z@Z 10011630 f i Pcfg.obj
 0001:000106b0       ??1PluginSettings@@QAE@XZ  100116b0 f i Pcfg.obj
 0001:00010700       ?Set@PluginSettings@@QAE_NIPB_WH@Z 10011700 f i Pcfg.obj
 0001:00010750       ?SaveValue@PluginCheckBoxBinding@@UAEXPBUFarDialogItem@@H@Z 10011750 f i Pcfg.obj
 0001:000107a0       ??_GPluginCheckBoxBinding@@UAEPAXI@Z 100117a0 f i Pcfg.obj
 0001:000107a0       ??_GPluginEditFieldBinding@@UAEPAXI@Z 100117a0 f i Pclass.obj
 0001:000107a0       ??_EPluginEditFieldBinding@@UAEPAXI@Z 100117a0 f i * CIL library *:* CIL module *
 0001:000107a0       ??_EPluginCheckBoxBinding@@UAEPAXI@Z 100117a0 f i * CIL library *:* CIL module *
 0001:000107c0       ??0PluginDialogBuilder@@QAE@ABUPluginStartupInfo@@ABU_GUID@@1HPB_WP6GHPAXHH3@Z3_K@Z 100117c0 f i Pcfg.obj
 0001:000108c0       ??1PluginDialogBuilder@@QAE@XZ 100118c0 f i Pcfg.obj
 0001:00010940       ?AddText@PluginDialogBuilder@@QAEPAUFarDialogItem@@H@Z 10011940 f i Pcfg.obj
 0001:00010980       ?AddCheckbox@PluginDialogBuilder@@QAEPAUFarDialogItem@@HPAHH_N@Z 10011980 f i Pcfg.obj
 0001:00010a90       ?AddSeparator@PluginDialogBuilder@@QAEXH@Z 10011a90 f i Pcfg.obj
 0001:00010ad0       ?AddOKCancel@PluginDialogBuilder@@QAEXHHH_N@Z 10011ad0 f i Pcfg.obj
 0001:00010b50       ?AddButtons@PluginDialogBuilder@@QAEXHPBHHH@Z 10011b50 f i Pcfg.obj
 0001:00010d70       ?ShowDialogEx@PluginDialogBuilder@@QAEHXZ 10011d70 f i Pcfg.obj
 0001:00010fd0       ?ShowDialog@PluginDialogBuilder@@QAE_NXZ 10011fd0 f i Pcfg.obj
 0001:00011000       ?AddDialogItem@PluginDialogBuilder@@AAEPAUFarDialogItem@@W4FARDIALOGITEMTYPES@@PB_W@Z 10012000 f i Pcfg.obj
 0001:00011120       ?Config@@YAHXZ             10012120 f   Pcfg.obj
 0001:000114c0       ?Read@options@@QAEXXZ      100124c0 f   Pcfg.obj
 0001:000117f0       _ceilf                     100127f0 f i Pclass.obj
 0001:00011820       ?SmartReread@PerfThread@@QAEXXZ 10012820 f i Pclass.obj
 0001:00011860       ?SaveValue@PluginEditFieldBinding@@UAEXPBUFarDialogItem@@H@Z 10012860 f i Pclass.obj
 0001:000118c0       ?AddEditField@PluginDialogBuilder@@QAEPAUFarDialogItem@@PA_WHHPB_W_N@Z 100128c0 f i Pclass.obj
 0001:00011970       ?OpenSubKey@PluginSettings@@QAEHIPB_W@Z 10012970 f i Pclass.obj
 0001:000119a0       ?Get@PluginSettings@@QAEPB_WIPB_W0@Z 100129a0 f i Pclass.obj
 0001:000119f0       ?Get@PluginSettings@@QAE_NIPB_W_N@Z 100129f0 f i Pclass.obj
 0001:00011a70       ?Set@PluginSettings@@QAE_NIPB_W_N@Z 10012a70 f i Pclass.obj
 0001:00012160       ??$format@V?$basic_string_view@_WU?$char_traits@_W@std@@@std@@@far@@YA?A_PV?$basic_format_string@_WV?$basic_string_view@_WU?$char_traits@_W@std@@@std@@@v10@fmt@@ABV?$basic_string_view@_WU?$char_traits@_W@std@@@std@@@Z 10013160 f i Pclass.obj
 0001:000121e0       ??$format@V?$basic_string@_WU?$char_traits@_W@std@@V?$allocator@_W@2@@std@@@far@@YA?A_PV?$basic_format_string@_WV?$basic_string@_WU?$char_traits@_W@std@@V?$allocator@_W@2@@std@@@v10@fmt@@ABV?$basic_string@_WU?$char_traits@_W@std@@V?$allocator@_W@2@@std@@@Z 100131e0 f i Pclass.obj
 0001:000122c0       ??0Plist@@QAE@XZ           100132c0 f   Pclass.obj
 0001:00012cc0       ?InitializePanelModes@Plist@@SAXXZ 10013cc0 f   Pclass.obj
 0001:00013c00       ?SavePanelModes@Plist@@SAXXZ 10014c00 f   Pclass.obj
 0001:00014110       ??1StrTok@@QAE@XZ          10015110 f i Pclass.obj
 0001:000141c0       ?GetOpenPanelInfo@Plist@@QAEXPAUOpenPanelInfo@@@Z 100151c0 f   Pclass.obj
 0001:00014530       ??$format@PB_W@far@@YA?A_PV?$basic_format_string@_WPB_W@v10@fmt@@ABQB_W@Z 10015530 f i Pclass.obj
 0001:00014530       ??$format@PA_W@far@@YA?A_PV?$basic_format_string@_WPA_W@v10@fmt@@ABQA_W@Z 10015530 f i Plist.obj
 0001:000145b0       ??$format@V?$basic_string@_WU?$char_traits@_W@std@@V?$allocator@_W@2@@std@@PB_W@far@@YA?A_PV?$basic_format_string@_WV?$basic_string@_WU?$char_traits@_W@std@@V?$allocator@_W@2@@std@@PB_W@v10@fmt@@ABV?$basic_string@_WU?$char_traits@_W@std@@V?$allocator@_W@2@@std@@ABQB_W@Z 100155b0 f i Pclass.obj
 0001:00014710       ?GetFindData@Plist@@QAEHAAPAUPluginPanelItem@@AAI_K@Z 10015710 f   Pclass.obj
 0001:00015680       ??$emplace_back@V?$basic_string@_WU?$char_traits@_W@std@@V?$allocator@_W@2@@std@@@?$vector@V?$basic_string@_WU?$char_traits@_W@std@@V?$allocator@_W@2@@std@@V?$allocator@V?$basic_string@_WU?$char_traits@_W@std@@V?$allocator@_W@2@@std@@@2@@std@@QAE?A_T$$QAV?$basic_string@_WU?$char_traits@_W@std@@V?$allocator@_W@2@@1@@Z 10016680 f i Pclass.obj
 0001:00015740       ??1?$unordered_map@KPAUHWND__@@U?$hash@K@std@@U?$equal_to@K@3@V?$allocator@U?$pair@$$CBKPAUHWND__@@@std@@@3@@std@@QAE@XZ 10016740 f i Pclass.obj
 0001:00015750       ??1?$_Hash@V?$_Umap_traits@KPAUHWND__@@V?$_Uhash_compare@KU?$hash@K@std@@U?$equal_to@K@2@@std@@V?$allocator@U?$pair@$$CBKPAUHWND__@@@std@@@3@$0A@@std@@@std@@QAE@XZ 10016750 f i Pclass.obj
 0001:00015a50       ??1?$pair@KV?$basic_string@_WU?$char_traits@_W@std@@V?$allocator@_W@2@@std@@@std@@QAE@XZ 10016a50 f i Pclass.obj
 0001:00015a50       ??1?$pair@JV?$basic_string@_WU?$char_traits@_W@std@@V?$allocator@_W@2@@std@@@std@@QAE@XZ 10016a50 f i Pclass.obj
 0001:00016080       ??$format@_J@far@@YA?A_PV?$basic_format_string@_W_J@v10@fmt@@AB_J@Z 10017080 f i Pclass.obj
 0001:00016100       ??$format@V?$basic_string@_WU?$char_traits@_W@std@@V?$allocator@_W@2@@std@@_J@far@@YA?A_PV?$basic_format_string@_WV?$basic_string@_WU?$char_traits@_W@std@@V?$allocator@_W@2@@std@@_J@v10@fmt@@ABV?$basic_string@_WU?$char_traits@_W@std@@V?$allocator@_W@2@@std@@AB_J@Z 10017100 f i Pclass.obj
 0001:000161a0       ??$format@_J_JPB_W@far@@YA?A_PV?$basic_format_string@_W_J_JPB_W@v10@fmt@@AB_J1ABQB_W@Z 100171a0 f i Pclass.obj
 0001:00016250       ?GetFiles@Plist@@QAEHPAUPluginPanelItem@@IHPAPB_W_KAAUoptions@@@Z 10017250 f   Pclass.obj
 0001:00017850       ??0ProcessData@@QAE@XZ     10018850 f i Pclass.obj
 0001:000178f0       ??$format@V?$basic_string@_WU?$char_traits@_W@std@@V?$allocator@_W@2@@std@@PB_WHPB_W@far@@YA?A_PV?$basic_format_string@_WV?$basic_string@_WU?$char_traits@_W@std@@V?$allocator@_W@2@@std@@PB_WHPB_W@v10@fmt@@ABV?$basic_string@_WU?$char_traits@_W@std@@V?$allocator@_W@2@@std@@ABQB_WABH2@Z 100188f0 f i Pclass.obj
 0001:000179c0       ??$format@V?$basic_string@_WU?$char_traits@_W@std@@V?$allocator@_W@2@@std@@V12@@far@@YA?A_PV?$basic_format_string@_WV?$basic_string@_WU?$char_traits@_W@std@@V?$allocator@_W@2@@std@@V12@@v10@fmt@@ABV?$basic_string@_WU?$char_traits@_W@std@@V?$allocator@_W@2@@std@@1@Z 100189c0 f i Pclass.obj
 0001:00017a60       ??$format@V?$basic_string@_WU?$char_traits@_W@std@@V?$allocator@_W@2@@std@@K@far@@YA?A_PV?$basic_format_string@_WV?$basic_string@_WU?$char_traits@_W@std@@V?$allocator@_W@2@@std@@K@v10@fmt@@ABV?$basic_string@_WU?$char_traits@_W@std@@V?$allocator@_W@2@@std@@ABK@Z 10018a60 f i Pclass.obj
 0001:00017a60       ??$format@V?$basic_string@_WU?$char_traits@_W@std@@V?$allocator@_W@2@@std@@I@far@@YA?A_PV?$basic_format_string@_WV?$basic_string@_WU?$char_traits@_W@std@@V?$allocator@_W@2@@std@@I@v10@fmt@@ABV?$basic_string@_WU?$char_traits@_W@std@@V?$allocator@_W@2@@std@@ABI@Z 10018a60 f i Pclass.obj
 0001:00017b00       ??$format@KPB_W@far@@YA?A_PV?$basic_format_string@_WKPB_W@v10@fmt@@ABKABQB_W@Z 10018b00 f i Pclass.obj
 0001:00017b90       ??$format@V?$basic_string@_WU?$char_traits@_W@std@@V?$allocator@_W@2@@std@@$$BY0DC@_W$$BY0DC@_W@far@@YA?A_PV?$basic_format_string@_WV?$basic_string@_WU?$char_traits@_W@std@@V?$allocator@_W@2@@std@@$$BY0DC@_W$$BY0DC@_W@v10@fmt@@ABV?$basic_string@_WU?$char_traits@_W@std@@V?$allocator@_W@2@@std@@AAY0DC@$$CB_W2@Z 10018b90 f i Pclass.obj
 0001:00017c30       ??$format@V?$basic_string@_WU?$char_traits@_W@std@@V?$allocator@_W@2@@std@@$$BY0BAE@_W@far@@YA?A_PV?$basic_format_string@_WV?$basic_string@_WU?$char_traits@_W@std@@V?$allocator@_W@2@@std@@$$BY0BAE@_W@v10@fmt@@ABV?$basic_string@_WU?$char_traits@_W@std@@V?$allocator@_W@2@@std@@AAY0BAE@$$CB_W@Z 10018c30 f i Pclass.obj
 0001:00017c30       ??$format@V?$basic_string@_WU?$char_traits@_W@std@@V?$allocator@_W@2@@std@@$$BY0DC@_W@far@@YA?A_PV?$basic_format_string@_WV?$basic_string@_WU?$char_traits@_W@std@@V?$allocator@_W@2@@std@@$$BY0DC@_W@v10@fmt@@ABV?$basic_string@_WU?$char_traits@_W@std@@V?$allocator@_W@2@@std@@AAY0DC@$$CB_W@Z 10018c30 f i Pclass.obj
 0001:00017cc0       ??$format@PB_WV?$basic_string@_WU?$char_traits@_W@std@@V?$allocator@_W@2@@std@@@far@@YA?A_PV?$basic_format_string@_WPB_WV?$basic_string@_WU?$char_traits@_W@std@@V?$allocator@_W@2@@std@@@v10@fmt@@ABQB_WABV?$basic_string@_WU?$char_traits@_W@std@@V?$allocator@_W@2@@std@@@Z 10018cc0 f i Pclass.obj
 0001:00017d50       ??$format@V?$basic_string@_WU?$char_traits@_W@std@@V?$allocator@_W@2@@std@@PBX@far@@YA?A_PV?$basic_format_string@_WV?$basic_string@_WU?$char_traits@_W@std@@V?$allocator@_W@2@@std@@PBX@v10@fmt@@ABV?$basic_string@_WU?$char_traits@_W@std@@V?$allocator@_W@2@@std@@ABQBX@Z 10018d50 f i Pclass.obj
 0001:00017df0       ??$format@V?$basic_string@_WU?$char_traits@_W@std@@V?$allocator@_W@2@@std@@KV12@@far@@YA?A_PV?$basic_format_string@_WV?$basic_string@_WU?$char_traits@_W@std@@V?$allocator@_W@2@@std@@KV12@@v10@fmt@@ABV?$basic_string@_WU?$char_traits@_W@std@@V?$allocator@_W@2@@std@@ABK1@Z 10018df0 f i Pclass.obj
 0001:00017eb0       ??$format@V?$basic_string@_WU?$char_traits@_W@std@@V?$allocator@_W@2@@std@@JV12@@far@@YA?A_PV?$basic_format_string@_WV?$basic_string@_WU?$char_traits@_W@std@@V?$allocator@_W@2@@std@@JV12@@v10@fmt@@ABV?$basic_string@_WU?$char_traits@_W@std@@V?$allocator@_W@2@@std@@ABJ1@Z 10018eb0 f i Pclass.obj
 0001:00017f70       ??$format@PB_WPB_WHPB_WPB_W@far@@YA?A_PV?$basic_format_string@_WPB_WPB_WHPB_WPB_W@v10@fmt@@ABQB_W1ABH11@Z 10018f70 f i Pclass.obj
 0001:00018040       ??1ProcessData@@QAE@XZ     10019040 f i Pclass.obj
 0001:000180e0       ?DeleteFiles@Plist@@QAEHPAUPluginPanelItem@@I_K@Z 100190e0 f   Pclass.obj
 0001:00018710       ?Reread@Plist@@AAEXXZ      10019710 f   Pclass.obj
 0001:000187a0       ?Connect@Plist@@QAE_NPB_W00@Z 100197a0 f   Pclass.obj
 0001:00018a20       ?ProcessKey@Plist@@QAEHPBU_INPUT_RECORD@@@Z 10019a20 f   Pclass.obj
 0001:0001a140       ??$format@PB_WPB_W@far@@YA?A_PV?$basic_format_string@_WPB_WPB_W@v10@fmt@@ABQB_W1@Z 1001b140 f i Pclass.obj
 0001:0001a1d0       ?DurationToText@@YA?AV?$basic_string@_WU?$char_traits@_W@std@@V?$allocator@_W@2@@std@@_K@Z 1001b1d0 f   Pclass.obj
 0001:0001a360       ?FileTimeDifferenceToText@@YA?AV?$basic_string@_WU?$char_traits@_W@std@@V?$allocator@_W@2@@std@@ABU_FILETIME@@0@Z 1001b360 f   Pclass.obj
 0001:0001a390       ?GetVersionInfo@Plist@@SA_NPB_WAAV?$unique_ptr@$$BY0A@DU?$default_delete@$$BY0A@D@std@@@std@@AAPB_W2@Z 1001b390 f   Pclass.obj
 0001:0001a6b0       ??$format@GG@far@@YA?A_PV?$basic_format_string@_WGG@v10@fmt@@ABG1@Z 1001b6b0 f i Pclass.obj
 0001:0001a740       ?ConnectWMI@Plist@@AAE_NXZ 1001b740 f   Pclass.obj
 0001:0001a800       ?PrintOwnerInfo@Plist@@AAEXPAXK@Z 1001b800 f   Pclass.obj
 0001:0001aaf0       ?Compare@Plist@@QBEHPBUPluginPanelItem@@0I@Z 1001baf0 f   Pclass.obj
 0001:0001acb0       ??$compare_numbers@_J@@YA?A_P_J0@Z 1001bcb0 f i Pclass.obj
 0001:0001ace0       ?WmiError@Plist@@ABEXXZ    1001bce0 f   Pclass.obj
 0001:0001ad10       ??1?$vector@IV?$allocator@I@std@@@std@@QAE@XZ 1001bd10 f i Pclass.obj
 0001:0001ad10       ??1?$vector@PAUHINSTANCE__@@V?$allocator@PAUHINSTANCE__@@@std@@@std@@QAE@XZ 1001bd10 f i Plist.obj
 0001:0001ad70       ??1?$vector@UFarMenuItem@@V?$allocator@UFarMenuItem@@@std@@@std@@QAE@XZ 1001bd70 f i Pclass.obj
 0001:0001add0       ??1?$vector@V?$basic_string@_WU?$char_traits@_W@std@@V?$allocator@_W@2@@std@@V?$allocator@V?$basic_string@_WU?$char_traits@_W@std@@V?$allocator@_W@2@@std@@@2@@std@@QAE@XZ 1001bdd0 f i Pclass.obj
 0001:0001ade0       ??1?$_Hash_vec@V?$allocator@V?$_List_unchecked_iterator@V?$_List_val@U?$_List_simple_types@U?$pair@$$CBKPAUHWND__@@@std@@@std@@@std@@@std@@@std@@@std@@QAE@XZ 1001bde0 f i Pclass.obj
 0001:0001ade0       ??1?$_Hash_vec@V?$allocator@V?$_List_unchecked_iterator@V?$_List_val@U?$_List_simple_types@U?$pair@$$CBKUProcessPerfData@@@std@@@std@@@std@@@std@@@std@@@std@@QAE@XZ 1001bde0 f i perfthread.obj
 0001:0001ae30       ??1?$list@U?$pair@$$CBKPAUHWND__@@@std@@V?$allocator@U?$pair@$$CBKPAUHWND__@@@std@@@2@@std@@QAE@XZ 1001be30 f i Pclass.obj
 0001:0001ae70       ??1?$scoped_lock@Vrefresh_lock@Plist@@@std@@QAE@XZ 1001be70 f i Pclass.obj
 0001:0001ae80       ??4?$vector@Umode@@V?$allocator@Umode@@@std@@@std@@QAEAAV01@V?$initializer_list@Umode@@@1@@Z 1001be80 f i Pclass.obj
 0001:0001afb0       ??1?$unique_ptr@VWMIConnection@@U?$default_delete@VWMIConnection@@@std@@@std@@QAE@XZ 1001bfb0 f i Pclass.obj
 0001:0001b050       ??1?$unique_ptr@VPerfThread@@U?$default_delete@VPerfThread@@@std@@@std@@QAE@XZ 1001c050 f i Pclass.obj
 0001:0001b070       ?clear@?$basic_string@_WU?$char_traits@_W@std@@V?$allocator@_W@2@@std@@QAEXXZ 1001c070 f i Pclass.obj
 0001:0001b090       ??R<lambda_1>@?1??insert@?$basic_string@_WU?$char_traits@_W@std@@V?$allocator@_W@2@@std@@QAEAAV23@II_W@Z@QBE@QA_WQB_WIII0@Z 1001c090 f i Pclass.obj
 0001:0001b100       ?append@?$basic_string@_WU?$char_traits@_W@std@@V?$allocator@_W@2@@std@@QAEAAV12@I_W@Z 1001c100 f i Pclass.obj
 0001:0001b2b0       ??Y?$basic_string@_WU?$char_traits@_W@std@@V?$allocator@_W@2@@std@@QAEAAV01@QB_W@Z 1001c2b0 f i Pclass.obj
 0001:0001b330       ??4?$basic_string@_WU?$char_traits@_W@std@@V?$allocator@_W@2@@std@@QAEAAV01@QB_W@Z 1001c330 f i Pclass.obj
 0001:0001b360       ?_Xlength@?$vector@UFarMenuItem@@V?$allocator@UFarMenuItem@@@std@@@std@@CAXXZ 1001c360 f i Pclass.obj
 0001:0001b360       ?_Xlength@?$vector@_WV?$allocator@_W@std@@@std@@CAXXZ 1001c360 f i perfthread.obj
 0001:0001b360       ?_Xlength@?$vector@V?$basic_string@_WU?$char_traits@_W@std@@V?$allocator@_W@2@@std@@V?$allocator@V?$basic_string@_WU?$char_traits@_W@std@@V?$allocator@_W@2@@std@@@2@@std@@CAXXZ 1001c360 f i Pclass.obj
 0001:0001b360       ?_Xlength@?$vector@UProcessPerfData@@V?$allocator@UProcessPerfData@@@std@@@std@@CAXXZ 1001c360 f i perfthread.obj
 0001:0001b360       ?_Xlength@?$vector@PB_WV?$allocator@PB_W@std@@@std@@CAXXZ 1001c360 f i Pclass.obj
 0001:0001b360       ?_Xlength@?$vector@EV?$allocator@E@std@@@std@@CAXXZ 1001c360 f i perfthread.obj
 0001:0001b360       ?_Xlength@?$vector@PAUHINSTANCE__@@V?$allocator@PAUHINSTANCE__@@@std@@@std@@CAXXZ 1001c360 f i Plist.obj
 0001:0001b360       ?_Xlength@?$vector@Umode@@V?$allocator@Umode@@@std@@@std@@CAXXZ 1001c360 f i Pclass.obj
 0001:0001b360       ?_Xlength@?$vector@IV?$allocator@I@std@@@std@@CAXXZ 1001c360 f i Pclass.obj
 0001:0001b370       ?_Reallocate_exactly@?$vector@IV?$allocator@I@std@@@std@@AAEXI@Z 1001c370 f i Pclass.obj
 0001:0001b3f0       ?_Reallocate_exactly@?$vector@UFarMenuItem@@V?$allocator@UFarMenuItem@@@std@@@std@@AAEXI@Z 1001c3f0 f i Pclass.obj
 0001:0001b470       ?_Tidy@?$vector@V?$basic_string@_WU?$char_traits@_W@std@@V?$allocator@_W@2@@std@@V?$allocator@V?$basic_string@_WU?$char_traits@_W@std@@V?$allocator@_W@2@@std@@@2@@std@@AAEXXZ 1001c470 f i Pclass.obj
 0001:0001b4e0       ?_Reallocate_exactly@?$vector@V?$basic_string@_WU?$char_traits@_W@std@@V?$allocator@_W@2@@std@@V?$allocator@V?$basic_string@_WU?$char_traits@_W@std@@V?$allocator@_W@2@@std@@@2@@std@@AAEXI@Z 1001c4e0 f i Pclass.obj
 0001:0001b530       ?reset@?$unique_ptr@VWMIConnection@@U?$default_delete@VWMIConnection@@@std@@@std@@QAEXPAVWMIConnection@@@Z 1001c530 f i Pclass.obj
 0001:0001b5e0       ?insert@?$basic_string@_WU?$char_traits@_W@std@@V?$allocator@_W@2@@std@@QAEAAV12@IQB_WI@Z 1001c5e0 f i Pclass.obj
 0001:0001b7a0       ?_Change_array@?$vector@IV?$allocator@I@std@@@std@@AAEXQAIII@Z 1001c7a0 f i Pclass.obj
 0001:0001b800       ?_Change_array@?$vector@UFarMenuItem@@V?$allocator@UFarMenuItem@@@std@@@std@@AAEXQAUFarMenuItem@@II@Z 1001c800 f i Pclass.obj
 0001:0001b860       ?allocate@?$allocator@UFarMenuItem@@@std@@QAEPAUFarMenuItem@@I@Z 1001c860 f i Pclass.obj
 0001:0001b8c0       ?deallocate@?$allocator@UFarMenuItem@@@std@@QAEXQAUFarMenuItem@@I@Z 1001c8c0 f i Pclass.obj
 0001:0001b900       ?_Change_array@?$vector@V?$basic_string@_WU?$char_traits@_W@std@@V?$allocator@_W@2@@std@@V?$allocator@V?$basic_string@_WU?$char_traits@_W@std@@V?$allocator@_W@2@@std@@@2@@std@@AAEXQAV?$basic_string@_WU?$char_traits@_W@std@@V?$allocator@_W@2@@2@II@Z 1001c900 f i Pclass.obj
 0001:0001b980       ?allocate@?$allocator@V?$basic_string@_WU?$char_traits@_W@std@@V?$allocator@_W@2@@std@@@std@@QAEPAV?$basic_string@_WU?$char_traits@_W@std@@V?$allocator@_W@2@@2@I@Z 1001c980 f i Pclass.obj
 0001:0001b9e0       ?deallocate@?$allocator@V?$basic_string@_WU?$char_traits@_W@std@@V?$allocator@_W@2@@std@@@std@@QAEXQAV?$basic_string@_WU?$char_traits@_W@std@@V?$allocator@_W@2@@2@I@Z 1001c9e0 f i Pclass.obj
 0001:0001ba20       ?_Assign_grow@?$_Hash_vec@V?$allocator@V?$_List_unchecked_iterator@V?$_List_val@U?$_List_simple_types@U?$pair@$$CBKPAUHWND__@@@std@@@std@@@std@@@std@@@std@@@std@@QAEXIV?$_List_unchecked_iterator@V?$_List_val@U?$_List_simple_types@U?$pair@$$CBKPAUHWND__@@@std@@@std@@@std@@@2@@Z 1001ca20 f i Pclass.obj
 0001:0001bb20       ?_Xran@?$_String_val@U?$_Simple_types@_W@std@@@std@@SAXXZ 1001cb20 f i Pclass.obj
 0001:0001bb30       ??$to_wstring@H@v10@fmt@@YA?AV?$basic_string@_WU?$char_traits@_W@std@@V?$allocator@_W@2@@std@@ABH@Z 1001cb30 f i Pclass.obj
 0001:0001bba0       ??$make_unique@VPerfThread@@PAVPlist@@$0A@@std@@YA?AV?$unique_ptr@VPerfThread@@U?$default_delete@VPerfThread@@@std@@@0@$$QAPAVPlist@@@Z 1001cba0 f i Pclass.obj
 0001:0001bc10       ??$?4U?$default_delete@VPerfThread@@@std@@$0A@@?$unique_ptr@VPerfThread@@U?$default_delete@VPerfThread@@@std@@@std@@QAEAAV01@$$QAV01@@Z 1001cc10 f i Pclass.obj
 0001:0001bc60       ??$construct@V?$basic_string@_WU?$char_traits@_W@std@@V?$allocator@_W@2@@std@@V12@@?$_Default_allocator_traits@V?$allocator@V?$basic_string@_WU?$char_traits@_W@std@@V?$allocator@_W@2@@std@@@std@@@std@@SAXAAV?$allocator@V?$basic_string@_WU?$char_traits@_W@std@@V?$allocator@_W@2@@std@@@1@QAV?$basic_string@_WU?$char_traits@_W@std@@V?$allocator@_W@2@@1@$$QAV31@@Z 1001cc60 f i Pclass.obj
 0001:0001bcf0       ??$_Emplace_reallocate@V?$basic_string@_WU?$char_traits@_W@std@@V?$allocator@_W@2@@std@@@?$vector@V?$basic_string@_WU?$char_traits@_W@std@@V?$allocator@_W@2@@std@@V?$allocator@V?$basic_string@_WU?$char_traits@_W@std@@V?$allocator@_W@2@@std@@@2@@std@@QAEPAV?$basic_string@_WU?$char_traits@_W@std@@V?$allocator@_W@2@@1@QAV21@$$QAV21@@Z 1001ccf0 f i Pclass.obj
 0001:0001be40       ??$?H_WU?$char_traits@_W@std@@V?$allocator@_W@1@@std@@YA?AV?$basic_string@_WU?$char_traits@_W@std@@V?$allocator@_W@2@@0@ABV10@$$QAV10@@Z 1001ce40 f i Pclass.obj
 0001:0001bef0       ??$_Emplace_reallocate@I@?$vector@IV?$allocator@I@std@@@std@@QAEPAIQAI$$QAI@Z 1001cef0 f i Pclass.obj
 0001:0001bef0       ??$_Emplace_reallocate@ABI@?$vector@IV?$allocator@I@std@@@std@@QAEPAIQAIABI@Z 1001cef0 f i Pclass.obj
 0001:0001bfc0       ??$_Emplace_reallocate@UFarMenuItem@@@?$vector@UFarMenuItem@@V?$allocator@UFarMenuItem@@@std@@@std@@QAEPAUFarMenuItem@@QAU2@$$QAU2@@Z 1001cfc0 f i Pclass.obj
 0001:0001c0a0       ??$_Try_emplace@ABK$$V@?$_Hash@V?$_Umap_traits@KPAUHWND__@@V?$_Uhash_compare@KU?$hash@K@std@@U?$equal_to@K@2@@std@@V?$allocator@U?$pair@$$CBKPAUHWND__@@@std@@@3@$0A@@std@@@std@@IAE?AU?$pair@PAU?$_List_node@U?$pair@$$CBKPAUHWND__@@@std@@PAX@std@@_N@1@ABK@Z 1001d0a0 f i Pclass.obj
 0001:0001c2a0       ??$_Destroy_range@V?$allocator@V?$basic_string@_WU?$char_traits@_W@std@@V?$allocator@_W@2@@std@@@std@@@std@@YAXPAV?$basic_string@_WU?$char_traits@_W@std@@V?$allocator@_W@2@@0@QAV10@AAV?$allocator@V?$basic_string@_WU?$char_traits@_W@std@@V?$allocator@_W@2@@std@@@0@@Z 1001d2a0 f i Pclass.obj
 0001:0001c310       ??$_Uninitialized_move@PAV?$basic_string@_WU?$char_traits@_W@std@@V?$allocator@_W@2@@std@@V?$allocator@V?$basic_string@_WU?$char_traits@_W@std@@V?$allocator@_W@2@@std@@@2@@std@@YAPAV?$basic_string@_WU?$char_traits@_W@std@@V?$allocator@_W@2@@0@QAV10@0PAV10@AAV?$allocator@V?$basic_string@_WU?$char_traits@_W@std@@V?$allocator@_W@2@@std@@@0@@Z 1001d310 f i Pclass.obj
 0001:0001c3c0       ??1?$_List_node_emplace_op2@V?$allocator@U?$_List_node@U?$pair@$$CBKPAUHWND__@@@std@@PAX@std@@@std@@@std@@QAE@XZ 1001d3c0 f i Pclass.obj
 0001:0001c3c0       ??1?$_Alloc_construct_ptr@V?$allocator@U?$_List_node@U?$pair@$$CBKPAUHWND__@@@std@@PAX@std@@@std@@@std@@QAE@XZ 1001d3c0 f i Pclass.obj
 0001:0001c3e0       ?_Clear_and_reserve_geometric@?$vector@Umode@@V?$allocator@Umode@@@std@@@std@@AAEXI@Z 1001d3e0 f i Pclass.obj
 0001:0001c540       ?_Forced_rehash@?$_Hash@V?$_Umap_traits@KPAUHWND__@@V?$_Uhash_compare@KU?$hash@K@std@@U?$equal_to@K@2@@std@@V?$allocator@U?$pair@$$CBKPAUHWND__@@@std@@@3@$0A@@std@@@std@@IAEXI@Z 1001d540 f i Pclass.obj
 0001:0001c6b0       ??$_Resize_reallocate@U_Value_init_tag@std@@@?$vector@PB_WV?$allocator@PB_W@std@@@std@@AAEXIABU_Value_init_tag@1@@Z 1001d6b0 f i Pclass.obj
 0001:0001c7e0       ??$_Find_last@K@?$_Hash@V?$_Umap_traits@KPAUHWND__@@V?$_Uhash_compare@KU?$hash@K@std@@U?$equal_to@K@2@@std@@V?$allocator@U?$pair@$$CBKPAUHWND__@@@std@@@3@$0A@@std@@@std@@IBE?AU?$_Hash_find_last_result@PAU?$_List_node@U?$pair@$$CBKPAUHWND__@@@std@@PAX@std@@@1@ABKI@Z 1001d7e0 f i Pclass.obj
 0001:0001c7e0       ??$_Find_last@K@?$_Hash@V?$_Umap_traits@KUProcessPerfData@@V?$_Uhash_compare@KU?$hash@K@std@@U?$equal_to@K@2@@std@@V?$allocator@U?$pair@$$CBKUProcessPerfData@@@std@@@3@$00@std@@@std@@IBE?AU?$_Hash_find_last_result@PAU?$_List_node@U?$pair@$$CBKUProcessPerfData@@@std@@PAX@std@@@1@ABKI@Z 1001d7e0 f i perfthread.obj
 0001:0001c850       ??$_Copy_unchecked@PBUmode@@PAU1@@std@@YAPAUmode@@PBU1@0PAU1@@Z 1001d850 f i Pclass.obj
 0001:0001c960       ??1?$_Uninitialized_backout_al@V?$allocator@Umode@@@std@@@std@@QAE@XZ 1001d960 f i Pclass.obj
 0001:0001c990       ??0mode@@QAE@ABU0@@Z       1001d990 f i Pclass.obj
 0001:0001ca60       ??0PerfThread@@QAE@PAVPlist@@PB_W11@Z 1001da60 f   perfthread.obj
 0001:0001d2a0       ??1?$unordered_multimap@KUProcessPerfData@@U?$hash@K@std@@U?$equal_to@K@3@V?$allocator@U?$pair@$$CBKUProcessPerfData@@@std@@@3@@std@@QAE@XZ 1001e2a0 f i perfthread.obj
 0001:0001d300       ??1PerfThread@@QAE@XZ      1001e300 f   perfthread.obj
 0001:0001d5b0       ?GetProcessData@PerfThread@@QAEPAUProcessPerfData@@KK@Z 1001e5b0 f   perfthread.obj
 0001:0001d690       ?RefreshImpl@PerfThread@@AAE_NXZ 1001e690 f   perfthread.obj
 0001:0001e670       ??1ProcessPerfData@@QAE@XZ 1001f670 f i perfthread.obj
 0001:0001e7e0       ??4ProcessPerfData@@QAEAAU0@ABU0@@Z 1001f7e0 f i perfthread.obj
 0001:0001e960       ?RefreshWMIData@PerfThread@@AAEXXZ 1001f960 f   perfthread.obj
 0001:0001efb0       ?WmiThreadProc@PerfThread@@AAEXXZ 1001ffb0 f   perfthread.obj
 0001:0001f0a0       ?ThreadProc@PerfThread@@CGKPAX@Z 100200a0 f   perfthread.obj
 0001:0001f120       ?WmiThreadProc@PerfThread@@CGKPAX@Z 10020120 f   perfthread.obj
 0001:0001f140       ??1?$vector@UProcessPerfData@@V?$allocator@UProcessPerfData@@@std@@@std@@QAE@XZ 10020140 f i perfthread.obj
 0001:0001f1c0       ??1?$vector@EV?$allocator@E@std@@@std@@QAE@XZ 100201c0 f i perfthread.obj
 0001:0001f210       ??1?$vector@_WV?$allocator@_W@std@@@std@@QAE@XZ 10020210 f i perfthread.obj
 0001:0001f270       ??0?$unordered_multimap@KUProcessPerfData@@U?$hash@K@std@@U?$equal_to@K@3@V?$allocator@U?$pair@$$CBKUProcessPerfData@@@std@@@3@@std@@QAE@XZ 10020270 f i perfthread.obj
 0001:0001f310       ??1?$list@U?$pair@$$CBKUProcessPerfData@@@std@@V?$allocator@U?$pair@$$CBKUProcessPerfData@@@std@@@2@@std@@QAE@XZ 10020310 f i perfthread.obj
 0001:0001f360       ?_Reallocate_exactly@?$vector@UProcessPerfData@@V?$allocator@UProcessPerfData@@@std@@@std@@AAEXI@Z 10020360 f i perfthread.obj
 0001:0001f3d0       ?_Change_array@?$vector@UProcessPerfData@@V?$allocator@UProcessPerfData@@@std@@@std@@AAEXQAUProcessPerfData@@II@Z 100203d0 f i perfthread.obj
 0001:0001f460       ?allocate@?$allocator@UProcessPerfData@@@std@@QAEPAUProcessPerfData@@I@Z 10020460 f i perfthread.obj
 0001:0001f4c0       ?_Assign_grow@?$_Hash_vec@V?$allocator@V?$_List_unchecked_iterator@V?$_List_val@U?$_List_simple_types@U?$pair@$$CBKUProcessPerfData@@@std@@@std@@@std@@@std@@@std@@@std@@QAEXIV?$_List_unchecked_iterator@V?$_List_val@U?$_List_simple_types@U?$pair@$$CBKUProcessPerfData@@@std@@@std@@@std@@@2@@Z 100204c0 f i perfthread.obj
 0001:0001f5b0       ?_Forced_rehash@?$_Hash@V?$_Umap_traits@KUProcessPerfData@@V?$_Uhash_compare@KU?$hash@K@std@@U?$equal_to@K@2@@std@@V?$allocator@U?$pair@$$CBKUProcessPerfData@@@std@@@3@$00@std@@@std@@IAEXI@Z 100205b0 f i perfthread.obj
 0001:0001f720       ?clear@?$_Hash@V?$_Umap_traits@KUProcessPerfData@@V?$_Uhash_compare@KU?$hash@K@std@@U?$equal_to@K@2@@std@@V?$allocator@U?$pair@$$CBKUProcessPerfData@@@std@@@3@$00@std@@@std@@QAEXXZ 10020720 f i perfthread.obj
 0001:0001f7b0       ?_Unchecked_erase@?$_Hash@V?$_Umap_traits@KUProcessPerfData@@V?$_Uhash_compare@KU?$hash@K@std@@U?$equal_to@K@2@@std@@V?$allocator@U?$pair@$$CBKUProcessPerfData@@@std@@@3@$00@std@@@std@@AAEPAU?$_List_node@U?$pair@$$CBKUProcessPerfData@@@std@@PAX@2@PAU32@QAU32@@Z 100207b0 f i perfthread.obj
 0001:0001fb50       ??0ProcessPerfData@@QAE@ABU0@@Z 10020b50 f i perfthread.obj
 0001:0001fca0       ??$uninitialized_fill@PAV?$_List_unchecked_iterator@V?$_List_val@U?$_List_simple_types@U?$pair@$$CBKUProcessPerfData@@@std@@@std@@@std@@@std@@V12@@std@@YAXQAV?$_List_unchecked_iterator@V?$_List_val@U?$_List_simple_types@U?$pair@$$CBKUProcessPerfData@@@std@@@std@@@std@@@0@0ABV10@@Z 10020ca0 f i perfthread.obj
 0001:0001fcc0       ??1?$_List_node_emplace_op2@V?$allocator@U?$_List_node@U?$pair@$$CBKUProcessPerfData@@@std@@PAX@std@@@std@@@std@@QAE@XZ 10020cc0 f i perfthread.obj
 0001:0001fcf0       ?_Rehash_for_1@?$_Hash@V?$_Umap_traits@KUProcessPerfData@@V?$_Uhash_compare@KU?$hash@K@std@@U?$equal_to@K@2@@std@@V?$allocator@U?$pair@$$CBKUProcessPerfData@@@std@@@3@$00@std@@@std@@IAEXXZ 10020cf0 f i perfthread.obj
 0001:0001fd80       ??1?$_Alloc_construct_ptr@V?$allocator@U?$_List_node@U?$pair@$$CBKUProcessPerfData@@@std@@PAX@std@@@std@@@std@@QAE@XZ 10020d80 f i perfthread.obj
 0001:0001fda0       ??$_Resize_reallocate@U_Value_init_tag@std@@@?$vector@EV?$allocator@E@std@@@std@@AAEXIABU_Value_init_tag@1@@Z 10020da0 f i perfthread.obj
 0001:0001fe70       ??$_Emplace_reallocate@UProcessPerfData@@@?$vector@UProcessPerfData@@V?$allocator@UProcessPerfData@@@std@@@std@@QAEPAUProcessPerfData@@QAU2@$$QAU2@@Z 10020e70 f i perfthread.obj
 0001:0001ffc0       ??0ProcessPerfData@@QAE@$$QAU0@@Z 10020fc0 f i perfthread.obj
 0001:000202a0       ??$format@II@far@@YA?A_PV?$basic_format_string@_WII@v10@fmt@@ABI1@Z 100212a0 f i Plist.obj
 0001:000203d0       ?OpenProcessForced@@YAPAXPAVDebugToken@@KKH@Z 100213d0 f   Plist.obj
 0001:00020420       ?GetPData@@YA_NAAUProcessData@@ABUProcessPerfData@@@Z 10021420 f   Plist.obj
 0001:00020630       ?GetList@@YA_NAAPAUPluginPanelItem@@AAIAAVPerfThread@@@Z 10021630 f   Plist.obj
 0001:00020a40       ?Enable@DebugToken@@QAE_NXZ 10021a40 f   Plist.obj
 0001:00020ad0       ?KillProcess@@YA_NKPAUHWND__@@@Z 10021ad0 f   Plist.obj
 0001:00020c80       ?PrintNTCurDirAndEnv@@YAXPAX0H@Z 10021c80 f   Plist.obj
 0001:00021260       ??$format@$$BY0BAE@_W@far@@YA?A_PV?$basic_format_string@_W$$BY0BAE@_W@v10@fmt@@AAY0BAE@$$CB_W@Z 10022260 f i Plist.obj
 0001:000212e0       ?PrintModules@@YAXPAXKAAUoptions@@@Z 100222e0 f   Plist.obj
 0001:00021750       ??1?$function@$$A6AXABUtagVARIANT@@@Z@std@@QAE@XZ 10022750 f i wmi.obj
 0001:00021750       ??1?$function@$$A6A_NPA_WI@Z@std@@QAE@XZ 10022750 f i Plist.obj
 0001:00021780       ?PrintModules@?$ipc_functions@$0A@@@SAXPAX0AAUoptions@@@Z 10022780 f i Plist.obj
 0001:000218a0       ?GetOpenProcessData@?$ipc_functions@$0A@@@SAXPAXPAV?$basic_string@_WU?$char_traits@_W@std@@V?$allocator@_W@2@@std@@1111@Z 100228a0 f i Plist.obj
 0001:00021ae0       ?PrintModules@?$ipc_functions@$00@@SAXPAX0AAUoptions@@@Z 10022ae0 f i Plist.obj
 0001:00021c60       ?GetOpenProcessData@?$ipc_functions@$00@@SAXPAXPAV?$basic_string@_WU?$char_traits@_W@std@@V?$allocator@_W@2@@std@@1111@Z 10022c60 f i Plist.obj
 0001:00021ef0       ?GetInternalProcessData@?$ipc_functions@$0A@@@SA_NPAXPAULDR_MODULE_SAME@detail@@AAPBD2_N@Z 10022ef0 f i Plist.obj
 0001:00021ff0       ?read_string@?$ipc_functions@$0A@@@SA?AV?$basic_string@_WU?$char_traits@_W@std@@V?$allocator@_W@2@@std@@PAXQBX@Z 10022ff0 f i Plist.obj
 0001:00022080       ?read_string@?$ipc_functions@$0A@@@SA?AV?$basic_string@_WU?$char_traits@_W@std@@V?$allocator@_W@2@@std@@PAXABUUNICODE_STRING_SAME@detail@@@Z 10023080 f i Plist.obj
 0001:000221b0       ?GetInternalProcessData@?$ipc_functions@$00@@SA_NPAXPAULDR_MODULE_64@detail@@AA_K2_N@Z 100231b0 f i Plist.obj
 0001:00022320       ?read_string@?$ipc_functions@$00@@SA?AV?$basic_string@_WU?$char_traits@_W@std@@V?$allocator@_W@2@@std@@PAX_K@Z 10023320 f i Plist.obj
 0001:000223c0       ?read_string@?$ipc_functions@$00@@SA?AV?$basic_string@_WU?$char_traits@_W@std@@V?$allocator@_W@2@@std@@PAXABUUNICODE_STRING_64@detail@@@Z 100233c0 f i Plist.obj
 0001:00022500       ?read_process_memory@?$ipc_functions@$00@@SA_NPAX_KQAXIQAI@Z 10023500 f i Plist.obj
 0001:000228b0       ??$format@_K@far@@YA?A_PV?$basic_format_string@_W_K@v10@fmt@@AB_K@Z 100238b0 f i Plist.obj
 0001:00022930       ??$_Resize_reallocate@U_Value_init_tag@std@@@?$vector@PAUHINSTANCE__@@V?$allocator@PAUHINSTANCE__@@@std@@@std@@AAEXIABU_Value_init_tag@1@@Z 10023930 f i Plist.obj
 0001:00022a10       ??$insert@V?$_List_unchecked_const_iterator@V?$_List_val@U?$_List_simple_types@U?$pair@$$CBKUProcessPerfData@@@std@@@std@@@std@@U_Iterator_base0@2@@std@@@?$_Hash@V?$_Umap_traits@KUProcessPerfData@@V?$_Uhash_compare@KU?$hash@K@std@@U?$equal_to@K@2@@std@@V?$allocator@U?$pair@$$CBKUProcessPerfData@@@std@@@3@$00@std@@@std@@QAEXV?$_List_unchecked_const_iterator@V?$_List_val@U?$_List_simple_types@U?$pair@$$CBKUProcessPerfData@@@std@@@std@@@std@@U_Iterator_base0@2@@1@0@Z 10023a10 f i Plist.obj
 0001:00022bd0       ?_Delete_this@?$_Func_impl_no_alloc@V<lambda_1>@?6??PrintModules@?$ipc_functions@$00@@SAXPAX0AAUoptions@@@Z@_NPA_WI@std@@EAEX_N@Z 10023bd0 f i Plist.obj
 0001:00022bd0       ?_Delete_this@?$_Func_impl_no_alloc@V<lambda_1>@?6??PrintModules@?$ipc_functions@$0A@@@SAXPAX0AAUoptions@@@Z@_NPA_WI@std@@EAEX_N@Z 10023bd0 f i Plist.obj
 0001:00022bf0       ?_Get@?$_Func_impl_no_alloc@V<lambda_1>@?6??PrintModules@?$ipc_functions@$00@@SAXPAX0AAUoptions@@@Z@_NPA_WI@std@@EBEPBXXZ 10023bf0 f i Plist.obj
 0001:00022bf0       ?_Get@?$_Func_impl_no_alloc@V<lambda_1>@?6??PrintModules@?$ipc_functions@$0A@@@SAXPAX0AAUoptions@@@Z@_NPA_WI@std@@EBEPBXXZ 10023bf0 f i Plist.obj
 0001:00022c00       ?_Target_type@?$_Func_impl_no_alloc@V<lambda_1>@?6??PrintModules@?$ipc_functions@$00@@SAXPAX0AAUoptions@@@Z@_NPA_WI@std@@EBEABVtype_info@@XZ 10023c00 f i Plist.obj
 0001:00022c10       ?_Do_call@?$_Func_impl_no_alloc@V<lambda_1>@?6??PrintModules@?$ipc_functions@$00@@SAXPAX0AAUoptions@@@Z@_NPA_WI@std@@EAE_N$$QAPA_W$$QAI@Z 10023c10 f i Plist.obj
 0001:00022c60       ?_Move@?$_Func_impl_no_alloc@V<lambda_1>@?6??PrintModules@?$ipc_functions@$00@@SAXPAX0AAUoptions@@@Z@_NPA_WI@std@@EAEPAV?$_Func_base@_NPA_WI@2@PAX@Z 10023c60 f i Plist.obj
 0001:00022c60       ?_Copy@?$_Func_impl_no_alloc@V<lambda_1>@?6??PrintModules@?$ipc_functions@$00@@SAXPAX0AAUoptions@@@Z@_NPA_WI@std@@EBEPAV?$_Func_base@_NPA_WI@2@PAX@Z 10023c60 f i Plist.obj
 0001:00022c80       ?_Target_type@?$_Func_impl_no_alloc@V<lambda_1>@?6??PrintModules@?$ipc_functions@$0A@@@SAXPAX0AAUoptions@@@Z@_NPA_WI@std@@EBEABVtype_info@@XZ 10023c80 f i Plist.obj
 0001:00022c90       ?_Do_call@?$_Func_impl_no_alloc@V<lambda_1>@?6??PrintModules@?$ipc_functions@$0A@@@SAXPAX0AAUoptions@@@Z@_NPA_WI@std@@EAE_N$$QAPA_W$$QAI@Z 10023c90 f i Plist.obj
 0001:00022cd0       ?_Copy@?$_Func_impl_no_alloc@V<lambda_1>@?6??PrintModules@?$ipc_functions@$0A@@@SAXPAX0AAUoptions@@@Z@_NPA_WI@std@@EBEPAV?$_Func_base@_NPA_WI@2@PAX@Z 10023cd0 f i Plist.obj
 0001:00022cd0       ?_Move@?$_Func_impl_no_alloc@V<lambda_1>@?6??PrintModules@?$ipc_functions@$0A@@@SAXPAX0AAUoptions@@@Z@_NPA_WI@std@@EAEPAV?$_Func_base@_NPA_WI@2@PAX@Z 10023cd0 f i Plist.obj
 0001:00022d50       ?GetMsg@@YAPB_WH@Z         10023d50 f   Pmix.obj
 0001:00022d60       ?ConvertDate@@YAXABU_FILETIME@@PA_W1@Z 10023d60 f   Pmix.obj
 0001:00022e10       ?WinError@@YAHPB_W@Z       10023e10 f   Pmix.obj
 0001:00023130       ??$_Traits_find_last_not_of@U?$char_traits@_W@std@@@std@@YAIQB_WII0IU?$integral_constant@_N$00@0@@Z 10024130 f i Pmix.obj
 0001:000232a0       ??1bstr@@QAE@XZ            100242a0 f i wmi.obj
 0001:00023370       ??0WMIConnection@@QAE@XZ   10024370 f   wmi.obj
 0001:00023410       ??1WMIConnection@@QAE@XZ   10024410 f   wmi.obj
 0001:000234a0       ?GetProcessOwner@WMIConnection@@QAE?AV?$basic_string@_WU?$char_traits@_W@std@@V?$allocator@_W@2@@std@@KPAV23@@Z 100244a0 f   wmi.obj
 0001:000236f0       ?GetProcessUserSid@WMIConnection@@QAE?AV?$basic_string@_WU?$char_traits@_W@std@@V?$allocator@_W@2@@std@@K@Z 100246f0 f   wmi.obj
 0001:000238e0       ?GetProcessSessionId@WMIConnection@@QAEKK@Z 100248e0 f   wmi.obj
 0001:00023970       ?ExecMethod@WMIConnection@@AAEHKPB_W0K@Z 10024970 f   wmi.obj
 0001:00023c30       ?GetProcessProperty@WMIConnection@@AAE_NKPB_WABV?$function@$$A6AXABUtagVARIANT@@@Z@std@@@Z 10024c30 f   wmi.obj
 0001:00023d50       ?GetProcessInt@WMIConnection@@AAEKKPB_W@Z 10024d50 f   wmi.obj
 0001:00023de0       ?GetProcessString@WMIConnection@@AAE?AV?$basic_string@_WU?$char_traits@_W@std@@V?$allocator@_W@2@@std@@KPB_W@Z 10024de0 f   wmi.obj
 0001:00023ea0       ?Connect@WMIConnection@@QAE_NPB_W00@Z 10024ea0 f   wmi.obj
 0001:00024080       ??1?$unique_ptr@UIWbemLocator@@Ucom_closer@@@std@@QAE@XZ 10025080 f i wmi.obj
 0001:00024080       ??1?$unique_ptr@UIWbemClassObject@@Ucom_closer@@@std@@QAE@XZ 10025080 f i wmi.obj
 0001:000240d0       ??1?$ptr_setter@V?$unique_ptr@UIWbemClassObject@@Ucom_closer@@@std@@@@QAE@XZ 100250d0 f i wmi.obj
 0001:000243b0       ?Message@@YAHIPB_WPAPB_WII@Z 100253b0 f   Proclist.obj
 0001:000243e0       _GetGlobalInfoW@4          100253e0 f   Proclist.obj
 0001:00024470       _SetStartupInfoW@4         10025470 f   Proclist.obj
 0001:000245a0       _OpenW@4                   100255a0 f   Proclist.obj
 0001:000246d0       _ClosePanelW@4             100256d0 f   Proclist.obj
 0001:000246f0       _GetFindDataW@4            100256f0 f   Proclist.obj
 0001:00024720       _FreeFindDataW@4           10025720 f   Proclist.obj
 0001:00024800       _GetPluginInfoW@4          10025800 f   Proclist.obj
 0001:000248c0       _GetOpenPanelInfoW@4       100258c0 f   Proclist.obj
 0001:000248e0       _GetFilesW@4               100258e0 f   Proclist.obj
 0001:00024910       _DeleteFilesW@4            10025910 f   Proclist.obj
 0001:00024930       _ProcessPanelEventW@4      10025930 f   Proclist.obj
 0001:00024a30       _ProcessPanelInputW@4      10025a30 f   Proclist.obj
 0001:00024a50       _ConfigureW@4              10025a50 f   Proclist.obj
 0001:00024a60       _CompareW@4                10025a60 f   Proclist.obj
 0001:00024a80       _ProcessSynchroEventW@4    10025a80 f   Proclist.obj
 0001:00024aa0       ??1?$unique_ptr@VPlist@@U?$default_delete@VPlist@@@std@@@std@@QAE@XZ 10025aa0 f i Proclist.obj
 0001:00024b60       _EncodePointerWrapper@4    10025b60 f   vc_crt_fix_impl.obj
 0001:00024c20       _DecodePointerWrapper@4    10025c20 f   vc_crt_fix_impl.obj
 0001:00024c70       _GetModuleHandleExWWrapper@12 10025c70 f   vc_crt_fix_impl.obj
 0001:00024fb0       _InitializeSListHeadWrapper@4 10025fb0 f   vc_crt_fix_impl.obj
 0001:00025000       _InterlockedFlushSListWrapper@4 10026000 f   vc_crt_fix_impl.obj
 0001:00025050       _InterlockedPopEntrySListWrapper@4 10026050 f   vc_crt_fix_impl.obj
 0001:000250a0       _InterlockedPushEntrySListWrapper@8 100260a0 f   vc_crt_fix_impl.obj
 0001:000250f0       _InterlockedPushListSListExWrapper@16 100260f0 f   vc_crt_fix_impl.obj
 0001:00025140       _RtlFirstEntrySListWrapper@4 10026140 f   vc_crt_fix_impl.obj
 0001:00025190       _QueryDepthSListWrapper@4  10026190 f   vc_crt_fix_impl.obj
 0001:000251e0       _GetNumaHighestNodeNumberWrapper@4 100261e0 f   vc_crt_fix_impl.obj
 0001:00025250       _GetLogicalProcessorInformationWrapper@8 10026250 f   vc_crt_fix_impl.obj
 0001:000252b0       _SetThreadStackGuaranteeWrapper@4 100262b0 f   vc_crt_fix_impl.obj
 0001:00025310       _InitializeCriticalSectionExWrapper@12 10026310 f   vc_crt_fix_impl.obj
 0001:00025390       _CompareStringExWrapper@36 10026390 f   vc_crt_fix_impl.obj
 0001:00025410       _LCMapStringExWrapper@36   10026410 f   vc_crt_fix_impl.obj
 0001:00025490       __Mbrtowc                  10026490 f   libcpmt:xmbtowc.obj
 0001:00025619       ??0_Init_locks@std@@QAE@XZ 10026619 f   libcpmt:xlock.obj
 0001:00025646       ??0_Lockit@std@@QAE@H@Z    10026646 f   libcpmt:xlock.obj
 0001:00025677       ??1_Init_locks@std@@QAE@XZ 10026677 f   libcpmt:xlock.obj
 0001:0002569e       ??1_Lockit@std@@QAE@XZ     1002669e f   libcpmt:xlock.obj
 0001:000256bd       ??0bad_alloc@std@@QAE@XZ   100266bd f i libcpmt:xthrow.obj
 0001:000256d5       ??0bad_function_call@std@@QAE@ABV01@@Z 100266d5 f i libcpmt:xthrow.obj
 0001:000256f0       ??0bad_function_call@std@@QAE@XZ 100266f0 f i libcpmt:xthrow.obj
 0001:00025701       ??0length_error@std@@QAE@ABV01@@Z 10026701 f i libcpmt:xthrow.obj
 0001:0002571c       ??0length_error@std@@QAE@PBD@Z 1002671c f i libcpmt:xthrow.obj
 0001:0002573b       ??0logic_error@std@@QAE@ABV01@@Z 1002673b f i libcpmt:xthrow.obj
 0001:00025756       ??0out_of_range@std@@QAE@ABV01@@Z 10026756 f i libcpmt:xthrow.obj
 0001:00025771       ??0out_of_range@std@@QAE@PBD@Z 10026771 f i libcpmt:xthrow.obj
 0001:00025790       ??_Gbad_exception@std@@UAEPAXI@Z 10026790 f i libvcruntime:frame.obj
 0001:00025790       ??_Eout_of_range@std@@UAEPAXI@Z 10026790 f i libcpmt:xthrow.obj
 0001:00025790       ??_Glogic_error@std@@UAEPAXI@Z 10026790 f i libcpmt:xthrow.obj
 0001:00025790       ??_Elength_error@std@@UAEPAXI@Z 10026790 f i libcpmt:xthrow.obj
 0001:00025790       ??_Ebad_exception@std@@UAEPAXI@Z 10026790 f i libvcruntime:frame.obj
 0001:00025790       ??_Glength_error@std@@UAEPAXI@Z 10026790 f i libcpmt:xthrow.obj
 0001:00025790       ??_Elogic_error@std@@UAEPAXI@Z 10026790 f i libcpmt:xthrow.obj
 0001:00025790       ??_Gbad_function_call@std@@UAEPAXI@Z 10026790 f i libcpmt:xthrow.obj
 0001:00025790       ??_Gout_of_range@std@@UAEPAXI@Z 10026790 f i libcpmt:xthrow.obj
 0001:00025790       ??_Ebad_function_call@std@@UAEPAXI@Z 10026790 f i libcpmt:xthrow.obj
 0001:000257bd       ?_Xbad_alloc@std@@YAXXZ    100267bd f   libcpmt:xthrow.obj
 0001:000257bd       ?__scrt_throw_std_bad_alloc@@YAXXZ 100267bd f   LIBCMT:throw_bad_alloc.obj
 0001:000257da       ?_Xbad_function_call@std@@YAXXZ 100267da f   libcpmt:xthrow.obj
 0001:000257f7       ?_Xlength_error@std@@YAXPBD@Z 100267f7 f   libcpmt:xthrow.obj
 0001:00025817       ?_Xout_of_range@std@@YAXPBD@Z 10026817 f   libcpmt:xthrow.obj
 0001:00025837       ?_Xruntime_error@std@@YAXPBD@Z 10026837 f   libcpmt:xthrow.obj
 0001:00025857       ?what@bad_function_call@std@@UBEPBDXZ 10026857 f i libcpmt:xthrow.obj
 0001:0002585d       ??0_Locimp@locale@std@@AAE@_N@Z 1002685d f i libcpmt:locale0.obj
 0001:0002589e       ??1_Fac_node@std@@QAE@XZ   1002689e f i libcpmt:locale0.obj
 0001:000258cf       ??1_Fac_tidy_reg_t@std@@QAE@XZ 100268cf f i libcpmt:locale0.obj
 0001:000258f6       ??1_Locimp@locale@std@@MAE@XZ 100268f6 f i libcpmt:locale0.obj
 0001:00025921       ??4?$_Yarn@D@std@@QAEAAV01@PBD@Z 10026921 f i libcpmt:locale0.obj
 0001:00025975       ??_E_Locimp@locale@std@@MAEPAXI@Z 10026975 f i libcpmt:locale0.obj
 0001:00025975       ??_G_Locimp@locale@std@@MAEPAXI@Z 10026975 f i libcpmt:locale0.obj
 0001:00025997       ?_Facet_Register@std@@YAXPAV_Facet_base@1@@Z 10026997 f   libcpmt:locale0.obj
 0001:000259c3       ?_Getgloballocale@locale@std@@CAPAV_Locimp@12@XZ 100269c3 f   libcpmt:locale0.obj
 0001:000259c9       ?_Init@locale@std@@CAPAV_Locimp@12@_N@Z 100269c9 f   libcpmt:locale0.obj
 0001:00025a59       ?_Locimp_dtor@_Locimp@locale@std@@CAXPAV123@@Z 10026a59 f   libcpmt:locale0.obj
 0001:00025ac9       ?_Locinfo_ctor@_Locinfo@std@@SAXPAV12@PBD@Z 10026ac9 f   libcpmt:locale0.obj
 0001:00025b14       ?_Locinfo_dtor@_Locinfo@std@@SAXPAV12@@Z 10026b14 f   libcpmt:locale0.obj
 0001:00025b2e       ?_New_Locimp@_Locimp@locale@std@@CAPAV123@_N@Z 10026b2e f   libcpmt:locale0.obj
 0001:00025b51       ?_Setgloballocale@locale@std@@CAXPAX@Z 10026b51 f   libcpmt:locale0.obj
 0001:00025b79       __Deletegloballocale       10026b79 f   libcpmt:locale0.obj
 0001:00025bde       __Getcvt                   10026bde f   libcpmt:xwctomb.obj
 0001:00025c51       __Mtxdst                   10026c51 f   libcpmt:xmtx.obj
 0001:00025c5f       __Mtxinit                  10026c5f f   libcpmt:xmtx.obj
 0001:00025c74       __Mtxlock                  10026c74 f   libcpmt:xmtx.obj
 0001:00025c82       __Mtxunlock                10026c82 f   libcpmt:xmtx.obj
 0001:00025c90       ??1_Init_atexit@@QAE@XZ    10026c90 f i libcpmt:iosptrs.obj
 0001:00025cf8       ?_Atexit@@YAXP6AXXZ@Z      10026cf8 f   libcpmt:iosptrs.obj
 0001:00025d27       __freea_crt                10026d27 f i libcpmt:StlLCMapStringA.obj
 0001:00025d45       @__security_check_cookie@4 10026d45 f   LIBCMT:secchk.obj
 0001:00025d97       ___scrt_acquire_startup_lock 10026d97 f   LIBCMT:utility.obj
 0001:00025dc9       ___scrt_dllmain_after_initialize_c 10026dc9 f   LIBCMT:utility.obj
 0001:00025df4       ___scrt_dllmain_before_initialize_c 10026df4 f   LIBCMT:utility.obj
 0001:00025e02       ___scrt_dllmain_crt_thread_attach 10026e02 f   LIBCMT:utility.obj
 0001:00025e21       ___scrt_dllmain_crt_thread_detach 10026e21 f   LIBCMT:utility.obj
 0001:00025e2e       ___scrt_dllmain_exception_filter 10026e2e f   LIBCMT:utility.obj
 0001:00025e62       ___scrt_dllmain_uninitialize_c 10026e62 f   LIBCMT:utility.obj
 0001:00025e85       ___scrt_dllmain_uninitialize_critical 10026e85 f   LIBCMT:utility.obj
 0001:00025e92       ___scrt_initialize_crt     10026e92 f   LIBCMT:utility.obj
 0001:00025ecb       ___scrt_initialize_onexit_tables 10026ecb f   LIBCMT:utility.obj
 0001:00025f52       ___scrt_is_nonwritable_in_current_image 10026f52 f   LIBCMT:utility.obj
 0001:00025fe6       ___scrt_release_startup_lock 10026fe6 f   LIBCMT:utility.obj
 0001:00026003       ___scrt_uninitialize_crt   10027003 f   LIBCMT:utility.obj
 0001:0002602b       __onexit                   1002702b f   LIBCMT:utility.obj
 0001:00026058       _atexit                    10027058 f   LIBCMT:utility.obj
 0001:0002606d       ??3@YAXPAX@Z               1002706d f   LIBCMT:delete_scalar.obj
 0001:00026072       ??3@YAXPAXI@Z              10027072 f   LIBCMT:delete_scalar_size.obj
 0001:00026080       ??2@YAPAXI@Z               10027080 f   LIBCMT:new_scalar.obj
 0001:000260b0       ??_Etype_info@@UAEPAXI@Z   100270b0 f i LIBCMT:std_type_info_static.obj
 0001:000260b0       ??_Gtype_info@@UAEPAXI@Z   100270b0 f i LIBCMT:std_type_info_static.obj
 0001:000260d3       ??_V@YAXPAX@Z              100270d3 f   LIBCMT:delete_array.obj
 0001:000260d8       ??_U@YAPAXI@Z              100270d8 f   LIBCMT:new_array.obj
 0001:000260e1       ___raise_securityfailure   100270e1 f   LIBCMT:gs_report.obj
 0001:00026109       ___report_gsfailure        10027109 f   LIBCMT:gs_report.obj
 0001:00026203       ___report_rangecheckfailure 10027203 f   LIBCMT:gs_report.obj
 0001:0002620f       ___report_securityfailure  1002720f f   LIBCMT:gs_report.obj
 0001:000262de       ??_M@YGXPAXIIP6EX0@Z@Z     100272de f   LIBCMT:ehvecdtr.obj
 0001:00026363       ?__ArrayUnwind@@YGXPAXIIP6EX0@Z@Z 10027363 f   LIBCMT:ehvecdtr.obj
 0001:00026733       __DllMainCRTStartup@12     10027733 f   LIBCMT:dll_dllmain.obj
 0001:00026756       __EH_epilog3               10027756 f   LIBCMT:ehprolg3.obj
 0001:0002676a       __EH_epilog3_GS            1002776a f   LIBCMT:ehprolg3.obj
 0001:00026779       __EH_prolog3               10027779 f   LIBCMT:ehprolg3.obj
 0001:000267ac       __EH_prolog3_GS            100277ac f   LIBCMT:ehprolg3.obj
 0001:000267e2       __EH_prolog3_catch         100277e2 f   LIBCMT:ehprolg3.obj
 0001:00026818       @_guard_check_icall_nop@4  10027818 f i LIBCMT:guard_support.obj
 0001:00026820       __allmul                   10027820 f   LIBCMT:llmul.obj
 0001:00026860       __alloca_probe_16          10027860 f   LIBCMT:alloca16.obj
 0001:00026876       __alloca_probe_8           10027876     LIBCMT:alloca16.obj
 0001:0002688c       ___isa_available_init      1002788c f   LIBCMT:cpu_disp.obj
 0001:00026a5d       __get_startup_argv_mode    10027a5d f   LIBCMT:argv_mode.obj
 0001:00026a61       ___scrt_is_ucrt_dll_in_use 10027a61 f   LIBCMT:ucrt_detection.obj
 0001:00026a6d       ___scrt_fastfail           10027a6d f   LIBCMT:utility_desktop.obj
 0001:00026b88       __crt_debugger_hook        10027b88 f   LIBCMT:utility_desktop.obj
 0001:00026b90       __SEH_prolog4              10027b90 f   LIBCMT:sehprolg4.obj
 0001:00026c22       ___security_init_cookie    10027c22 f   LIBCMT:gs_support.obj
 0001:00026c6d       _DllMain@12                10027c6d f   LIBCMT:dll_dllmain_stub.obj
 0001:00026c73       ?__scrt_initialize_type_info@@YAXXZ 10027c73 f   LIBCMT:tncleanup.obj
 0001:00026c7f       ?__scrt_uninitialize_type_info@@YAXXZ 10027c7f f   LIBCMT:tncleanup.obj
 0001:00026c8b       ___local_stdio_scanf_options 10027c8b f i LIBCMT:default_local_stdio_options.obj
 0001:00026c91       ___scrt_initialize_default_local_stdio_options 10027c91 f   LIBCMT:default_local_stdio_options.obj
 0001:00026cae       ___scrt_get_dyn_tls_init_callback 10027cae f   LIBCMT:dyn_tls_init.obj
 0001:00026cb4       __RTC_Initialize           10027cb4 f   LIBCMT:initsect.obj
 0001:00026ce0       __RTC_Terminate            10027ce0 f   LIBCMT:initsect.obj
 0001:00026d10       __alloca_probe             10027d10 f   LIBCMT:chkstk.obj
 0001:00026d10       __chkstk                   10027d10 f   LIBCMT:chkstk.obj
 0001:00026d3b       ?GetRangeOfTrysToCheck@__FrameHandler3@@SA?AU?$pair@Viterator@TryBlockMap@__FrameHandler3@@V123@@std@@AAVTryBlockMap@1@HPAXPBU_s_FuncInfo@@H@Z 10027d3b f   libvcruntime:trnsctrl.obj
 0001:00026dab       ?_CallCatchBlock2@@YAPAXPAUEHRegistrationNode@@PBU_s_FuncInfo@@PAXHK@Z 10027dab f   libvcruntime:trnsctrl.obj
 0001:00026e08       ?_CallSETranslator@@YAHPAUEHExceptionRecord@@PAUEHRegistrationNode@@PAX2PBU_s_FuncInfo@@H1@Z 10027e08 f   libvcruntime:trnsctrl.obj
 0001:00026efe       ?_JumpToContinuation@@YGXPAXPAUEHRegistrationNode@@@Z 10027efe f   libvcruntime:trnsctrl.obj
 0001:00026f2e       ?_UnwindNestedFrames@@YGXPAUEHRegistrationNode@@PAUEHExceptionRecord@@@Z 10027f2e f   libvcruntime:trnsctrl.obj
 0001:00026f81       __CatchGuardHandler        10027f81 f   libvcruntime:trnsctrl.obj
 0001:00026fb2       __CreateFrameInfo          10027fb2 f   libvcruntime:trnsctrl.obj
 0001:00026fd6       __FindAndUnlinkFrame       10027fd6 f   libvcruntime:trnsctrl.obj
 0001:0002701e       __TranslatorGuardHandler   1002801e f   libvcruntime:trnsctrl.obj
 0001:000270bb       ___CxxFrameHandler3        100280bb f   libvcruntime:trnsctrl.obj
 0001:000270f1       ___DestructExceptionObject 100280f1 f   libvcruntime:ehhelpers.obj
 0001:00027192       ?_CallMemberFunction0@@YGXQAX0@Z 10028192 f i libvcruntime:ehhelpers.obj
 0001:000271f7       __IsExceptionObjectToBeDestroyed 100281f7 f   libvcruntime:ehhelpers.obj
 0001:0002721d       ___AdjustPointer           1002821d f   libvcruntime:ehhelpers.obj
 0001:00027242       ___FrameUnwindFilter       10028242 f   libvcruntime:ehhelpers.obj
 0001:00027298       ___current_exception       10028298 f   libvcruntime:ehhelpers.obj
 0001:000272a1       ___current_exception_context 100282a1 f   libvcruntime:ehhelpers.obj
 0001:000272aa       ___std_terminate           100282aa f   libvcruntime:ehhelpers.obj
 0001:000272af       ___std_exception_copy      100282af f   libvcruntime:std_exception.obj
 0001:00027312       ___std_exception_destroy   10028312 f   libvcruntime:std_exception.obj
 0001:00027331       __get_purecall_handler     10028331 f   libvcruntime:purevirt.obj
 0001:00027337       __purecall                 10028337 f   libvcruntime:purevirt.obj
 0001:00027353       _wcschr                    10028353 f   libvcruntime:wcschr.obj
 0001:0002741a       __CxxThrowException@8      1002841a f   libvcruntime:throw.obj
 0001:00027490       _memmove                   10028490 f   libvcruntime:memmove.obj
 0001:00027490       _memcpy                    10028490 f   libvcruntime:memcpy.obj
 0001:00027a10       _memset                    10028a10 f   libvcruntime:memset.obj
 0001:00027b70       _memcmp                    10028b70 f   libvcruntime:memcmp.obj
 0001:00028a7c       ___vcrt_initialize         10029a7c f   libvcruntime:initialization.obj
 0001:00028a9b       ___vcrt_thread_attach      10029a9b f   libvcruntime:initialization.obj
 0001:00028aa6       ___vcrt_thread_detach      10029aa6 f   libvcruntime:initialization.obj
 0001:00028ab1       ___vcrt_uninitialize       10029ab1 f   libvcruntime:initialization.obj
 0001:00028ac8       ___vcrt_uninitialize_critical 10029ac8 f   libvcruntime:initialization.obj
 0001:00028b10       __except_handler4          10029b10 f   libvcruntime:chandler4.obj
 0001:00028c6e       ___std_type_info_compare   10029c6e f   libvcruntime:std_type_info.obj
 0001:00028caa       ___std_type_info_destroy_list 10029caa f   libvcruntime:std_type_info.obj
 0001:00028ccd       ___vcrt_freefls@4          10029ccd f   libvcruntime:per_thread_data.obj
 0001:00028ce9       ___vcrt_freeptd            10029ce9 f   libvcruntime:per_thread_data.obj
 0001:00028d1f       ___vcrt_getptd             10029d1f f   libvcruntime:per_thread_data.obj
 0001:00028d2d       ___vcrt_getptd_noexit      10029d2d f   libvcruntime:per_thread_data.obj
 0001:00028dbf       ___vcrt_initialize_ptd     10029dbf f   libvcruntime:per_thread_data.obj
 0001:00028df2       ___vcrt_uninitialize_ptd   10029df2 f   libvcruntime:per_thread_data.obj
 0001:00029544       ??$TypeMatchHelper@V__FrameHandler3@@@@YAHPBU_s_HandlerType@@PBU_s_CatchableType@@PBU_s_ThrowInfo@@@Z 1002a544 f i libvcruntime:frame.obj
 0001:000295d2       ??$__InternalCxxFrameHandler@V__FrameHandler3@@@@YA?AW4_EXCEPTION_DISPOSITION@@PAUEHExceptionRecord@@PAUEHRegistrationNode@@PAU_CONTEXT@@PAXPBU_s_FuncInfo@@H1E@Z 1002a5d2 f i libvcruntime:frame.obj
 0001:000296d4       ??0bad_exception@std@@QAE@ABV01@@Z 1002a6d4 f i libvcruntime:frame.obj
 0001:000296ef       ??0bad_exception@std@@QAE@XZ 1002a6ef f i libvcruntime:frame.obj
 0001:00029707       ??8type_info@@QBE_NABV0@@Z 1002a707 f i libvcruntime:frame.obj
 0001:00029973       ?FrameUnwindToEmptyState@__FrameHandler3@@SAXPAUEHRegistrationNode@@PAXPBU_s_FuncInfo@@@Z 1002a973 f   libvcruntime:frame.obj
 0001:0002998b       ?FrameUnwindToState@__FrameHandler3@@SAXPAUEHRegistrationNode@@PAXPBU_s_FuncInfo@@H@Z 1002a98b f   libvcruntime:frame.obj
 0001:00029b0d       ?_CallMemberFunction1@@YGXQAX00@Z 1002ab0d f i libvcruntime:frame.obj
 0001:00029b1d       ?_CallMemberFunction2@@YGXQAX00H@Z 1002ab1d f i libvcruntime:frame.obj
 0001:00029b30       ?getESTypes@__FrameHandler3@@SAPBU_s_ESTypeList@@PBU_s_FuncInfo@@@Z 1002ab30 f i libvcruntime:frame.obj
 0001:00029b40       __CallSettingFrame@12      1002ab40 f   libvcruntime:lowhelpr.obj
 0001:00029b67       __NLG_Return               1002ab67     libvcruntime:lowhelpr.obj
 0001:00029b8c       ___except_validate_context_record 1002ab8c f   libvcruntime:jbcxrval.obj
 0001:00029bbc       ___vcrt_initialize_locks   1002abbc f   libvcruntime:locks.obj
 0001:00029bf8       ___vcrt_uninitialize_locks 1002abf8 f   libvcruntime:locks.obj
 0001:00029c30       __local_unwind4            1002ac30 f   libvcruntime:exsup4.obj
 0001:00029d20       @_EH4_CallFilterFunc@8     1002ad20 f   libvcruntime:exsup4.obj
 0001:00029d40       @_EH4_TransferToHandler@8  1002ad40 f   libvcruntime:exsup4.obj
 0001:00029d60       @_EH4_GlobalUnwind2@8      1002ad60 f   libvcruntime:exsup4.obj
 0001:00029d80       @_EH4_LocalUnwind@16       1002ad80 f   libvcruntime:exsup4.obj
 0001:00029e7a       ___vcrt_FlsAlloc           1002ae7a f   libvcruntime:winapi_downlevel.obj
 0001:00029eb5       ___vcrt_FlsFree            1002aeb5 f   libvcruntime:winapi_downlevel.obj
 0001:00029ef0       ___vcrt_FlsGetValue        1002aef0 f   libvcruntime:winapi_downlevel.obj
 0001:00029f2b       ___vcrt_FlsSetValue        1002af2b f   libvcruntime:winapi_downlevel.obj
 0001:00029f69       ___vcrt_InitializeCriticalSectionEx 1002af69 f   libvcruntime:winapi_downlevel.obj
 0001:00029fb0       _unexpected                1002afb0 f   libvcruntime:unexpected.obj
 0001:00029fcd       ?GetCurrentState@__FrameHandler3@@SAHPAUEHRegistrationNode@@PAXPBU_s_FuncInfo@@@Z 1002afcd f   libvcruntime:ehstate.obj
 0001:00029fea       ?SetState@__FrameHandler3@@SAXPAUEHRegistrationNode@@PBU_s_FuncInfo@@H@Z 1002afea f   libvcruntime:ehstate.obj
 0001:0002a000       __NLG_Notify1              1002b000 f   libvcruntime:exsup.obj
 0001:0002a010       __NLG_Notify               1002b010 f   libvcruntime:exsup.obj
 0001:0002a027       __NLG_Dispatch2            1002b027     libvcruntime:exsup.obj
 0001:0002a027       __NLG_Dispatch             1002b027     libvcruntime:exsup.obj
 0001:0002a030       __NLG_Call                 1002b030 f   libvcruntime:exsup.obj
 0001:0002a032       __NLG_Return2              1002b032     libvcruntime:exsup.obj
 0001:0002a033       ___acrt_call_reportfault   1002b033 f   libucrt:invalid_parameter.obj
 0001:0002a16c       ___acrt_initialize_invalid_parameter_handler 1002b16c f   libucrt:invalid_parameter.obj
 0001:0002a17b       __invalid_parameter        1002b17b f   libucrt:invalid_parameter.obj
 0001:0002a1df       __invalid_parameter_noinfo 1002b1df f   libucrt:invalid_parameter.obj
 0001:0002a1ef       __invalid_parameter_noinfo_noreturn 1002b1ef f   libucrt:invalid_parameter.obj
 0001:0002a20c       __invoke_watson            1002b20c f   libucrt:invalid_parameter.obj
 0001:0002a240       _calloc                    1002b240 f   libucrt:calloc.obj
 0001:0002a24b       ___acrt_lowio_create_handle_array 1002b24b f   libucrt:osfinfo.obj
 0001:0002a2c6       ___acrt_lowio_destroy_handle_array 1002b2c6 f   libucrt:osfinfo.obj
 0001:0002a2fb       ___acrt_lowio_ensure_fh_exists 1002b2fb f   libucrt:osfinfo.obj
 0001:0002a399       ___acrt_lowio_lock_fh      1002b399 f   libucrt:osfinfo.obj
 0001:0002a3bc       ___acrt_lowio_unlock_fh    1002b3bc f   libucrt:osfinfo.obj
 0001:0002a3df       __free_osfhnd              1002b3df f   libucrt:osfinfo.obj
 0001:0002a470       __get_osfhandle            1002b470 f   libucrt:osfinfo.obj
 0001:0002a4da       ___acrt_initialize_stdio   1002b4da f   libucrt:_file.obj
 0001:0002a5a2       ___acrt_uninitialize_stdio 1002b5a2 f   libucrt:_file.obj
 0001:0002a5ee       __lock_file                1002b5ee f   libucrt:_file.obj
 0001:0002a602       __unlock_file              1002b602 f   libucrt:_file.obj
 0001:0002a616       __dclass                   1002b616 f   libucrt:nan.obj
 0001:0002a627       __dsign                    1002b627 f   libucrt:nan.obj
 0001:0002a637       ??0_LocaleUpdate@@QAE@QAU__crt_locale_pointers@@@Z 1002b637 f i libucrt:output.obj
 0001:0002a6ba       ??1_LocaleUpdate@@QAE@XZ   1002b6ba f i libucrt:output.obj
 0001:0002a6ca       ___acrt_locale_get_ctype_array_value 1002b6ca f i libucrt:output.obj
 0001:0002a6ec       __isatty                   1002b6ec f   libucrt:isatty.obj
 0001:0002a742       _terminate                 1002b742 f   libucrt:terminate.obj
 0001:0002a77e       _localeconv                1002b77e f   libucrt:localeconv.obj
 0001:0002a7a6       __fileno                   1002b7a6 f   libucrt:fileno.obj
 0001:0002a7cd       ___acrt_errno_from_os_error 1002b7cd f   libucrt:errno.obj
 0001:0002a810       ___acrt_errno_map_os_error 1002b810 f   libucrt:errno.obj
 0001:0002a833       ___doserrno                1002b833 f   libucrt:errno.obj
 0001:0002a846       __errno                    1002b846 f   libucrt:errno.obj
 0001:0002a859       _free                      1002b859 f   libucrt:free.obj
 0001:0002a874       _malloc                    1002b874 f   libucrt:malloc.obj
 0001:0002a880       _modf                      1002b880 f   libucrt:modf_pentium4.obj
 0001:0002a8c0       __modf_pentium4            1002b8c0 f   libucrt:modf_pentium4.obj
 0001:0002a9c8       __dlog                     1002b9c8 f   libucrt:log2d.obj
 0001:0002ab0f       _log2                      1002bb0f f   libucrt:log2d.obj
 0001:0002ab28       __isleadbyte_l             1002bb28 f i libucrt:_wctype.obj
 0001:0002ab62       _iswdigit                  1002bb62 f i libucrt:_wctype.obj
 0001:0002ab75       _wcspbrk                   1002bb75 f   libucrt:wcspbrk.obj
 0001:0002abc3       _wcstok                    1002bbc3 f   libucrt:wcstok.obj
 0001:0002abe8       _round                     1002bbe8 f   libucrt:round.obj
 0001:0002ad04       _wcsncpy_s                 1002bd04 f   libucrt:wcsncpy_s.obj
 0001:0002ad0f       _wcscspn                   1002bd0f f   libucrt:wcscspn.obj
 0001:0002ad68       ___acrt_initialize_locks   1002bd68 f   libucrt:locks.obj
 0001:0002ada9       ___acrt_lock               1002bda9 f   libucrt:locks.obj
 0001:0002adc0       ___acrt_uninitialize_locks 1002bdc0 f   libucrt:locks.obj
 0001:0002adf1       ___acrt_unlock             1002bdf1 f   libucrt:locks.obj
 0001:0002ae08       __lock_locales             1002be08 f   libucrt:locks.obj
 0001:0002ae16       __unlock_locales           1002be16 f   libucrt:locks.obj
 0001:0002b079       _setlocale                 1002c079 f   libucrt:setlocale.obj
 0001:0002b0b1       ____lc_codepage_func       1002c0b1 f   libucrt:initctype.obj
 0001:0002b0d6       ____lc_locale_name_func    1002c0d6 f   libucrt:initctype.obj
 0001:0002b0fd       ____mb_cur_max_func        1002c0fd f   libucrt:initctype.obj
 0001:0002b122       ___acrt_locale_initialize_ctype 1002c122 f   libucrt:initctype.obj
 0001:0002b580       ___pctype_func             1002c580 f   libucrt:ctype.obj
 0001:0002b5a4       ?unget@?$c_string_character_source@_W@__crt_strtox@@QAEX_W@Z 1002c5a4 f i libucrt:strtod.obj
 0001:0002b5d2       ?validate@?$c_string_character_source@_W@__crt_strtox@@QBE_NXZ 1002c5d2 f i libucrt:strtod.obj
 0001:0002b5f0       _strcspn                   1002c5f0 f   libucrt:strcspn.obj
 0001:0002b640       __CIpow                    1002c640 f   libucrt:pow_impl.obj
 0001:0002b67b       __CIpow_default            1002c67b f   libucrt:pow_impl.obj
 0001:0002b694       __pow_default              1002c694     libucrt:pow_impl.obj
 0001:0002b889       _abort                     1002c889 f   libucrt:abort.obj
 0001:0002b8cd       _wcsdup                    1002c8cd f   libucrt:wcsdup.obj
 0001:0002b8cd       __wcsdup                   1002c8cd f   libucrt:wcsdup.obj
 0001:0002b9de       ??$__acrt_mbs_to_wcs_cp@U__crt_win32_buffer_internal_dynamic_resizing@@@@YAHQBDAAV?$__crt_win32_buffer@_WU__crt_win32_buffer_internal_dynamic_resizing@@@@I@Z 1002c9de f i libucrt:strftime.obj
 0001:0002b9fb       ?_deallocate@?$__crt_win32_buffer@DU__crt_win32_buffer_internal_dynamic_resizing@@@@AAEXXZ 1002c9fb f i libucrt:argv_wildcards.obj
 0001:0002b9fb       ?_deallocate@?$__crt_win32_buffer@_WU__crt_win32_buffer_internal_dynamic_resizing@@@@AAEXXZ 1002c9fb f i libucrt:strftime.obj
 0001:0002ba15       ?allocate@?$__crt_win32_buffer@DU__crt_win32_buffer_no_resizing@@@@QAEHI@Z 1002ca15 f i libucrt:strftime.obj
 0001:0002ba3c       ?allocate@?$__crt_win32_buffer@_WU__crt_win32_buffer_internal_dynamic_resizing@@@@QAEHI@Z 1002ca3c f i libucrt:strftime.obj
 0001:0002ba7b       ?allocate@__crt_win32_buffer_internal_dynamic_resizing@@SAHQAPAXIABV__crt_win32_buffer_empty_debug_info@@@Z 1002ca7b f i libucrt:strftime.obj
 0001:0002ba9a       ?set_to_nullptr@?$__crt_win32_buffer@DU__crt_win32_buffer_no_resizing@@@@QAEXXZ 1002ca9a f i libucrt:strftime.obj
 0001:0002baae       ___strncnt                 1002caae f   libucrt:strncnt.obj
 0001:0002baca       _wcsnlen                   1002caca f   libucrt:strnlen.obj
 0001:0002bc7a       ___initialize_lconv_for_unsigned_char 1002cc7a f   libucrt:lconv_unsigned_char_initialization.obj
 0001:0002bca8       __seh_filter_dll           1002cca8 f   libucrt:exception_filter.obj
 0001:0002bcc8       __seh_filter_exe           1002ccc8 f   libucrt:exception_filter.obj
 0001:0002c096       ___acrt_initialize_thread_local_exit_callback 1002d096 f   libucrt:exit.obj
 0001:0002c0a5       __cexit                    1002d0a5 f   libucrt:exit.obj
 0001:0002c0b4       __exit                     1002d0b4 f   libucrt:exit.obj
 0001:0002c0ca       __is_c_termination_complete 1002d0ca f   libucrt:exit.obj
 0001:0002c37e       ___acrt_allocate_buffer_for_argv 1002d37e f   libucrt:argv_parsing.obj
 0001:0002c3cd       __configure_narrow_argv    1002d3cd f   libucrt:argv_parsing.obj
 0001:0002c52a       ??$uninitialize@A6AXAAPAPA_W@Z@?$dual_state_global@PAPA_W@__crt_state_management@@QAEXA6AXAAPAPA_W@Z@Z 1002d52a f i libucrt:environment_initialization.obj
 0001:0002c52a       ??$uninitialize@A6AXAAPAPAD@Z@?$dual_state_global@PAPAD@__crt_state_management@@QAEXA6AXAAPAPAD@Z@Z 1002d52a f i libucrt:environment_initialization.obj
 0001:0002c589       ___dcrt_uninitialize_environments_nolock 1002d589 f   libucrt:environment_initialization.obj
 0001:0002c5c0       __initialize_narrow_environment 1002d5c0 f   libucrt:environment_initialization.obj
 0001:0002c67b       ??$__crt_fast_encode_pointer@PAP6AXXZ@@YAPAP6AXXZQAP6AXXZ@Z 1002d67b f i libucrt:onexit.obj
 0001:0002c67b       ??$__crt_fast_encode_pointer@P6AHXZ@@YAP6AHXZQ6AHXZ@Z 1002d67b f i libucrt:onexit.obj
 0001:0002c67b       ??$__crt_fast_encode_pointer@PAX@@YAPAXQAX@Z 1002d67b f i libucrt:initialization.obj
 0001:0002c67b       ??$__crt_fast_encode_pointer@P6GHPA_WKJ@Z@@YAP6GHPA_WKJ@ZQ6GH0KJ@Z@Z 1002d67b f i libucrt:winapi_thunks.obj
 0001:0002c89d       __crt_atexit               1002d89d f   libucrt:onexit.obj
 0001:0002c8b3       __execute_onexit_table     1002d8b3 f   libucrt:onexit.obj
 0001:0002c8e0       __initialize_onexit_table  1002d8e0 f   libucrt:onexit.obj
 0001:0002c909       __register_onexit_function 1002d909 f   libucrt:onexit.obj
 0001:0002c93c       ___acrt_uninitialize_command_line 1002d93c f   libucrt:argv_data.obj
 0001:0002ca3a       ___acrt_initialize         1002da3a f   libucrt:initialization.obj
 0001:0002ca4c       ___acrt_thread_attach      1002da4c f   libucrt:initialization.obj
 0001:0002ca57       ___acrt_thread_detach      1002da57 f   libucrt:initialization.obj
 0001:0002ca5f       ___acrt_uninitialize       1002da5f f   libucrt:initialization.obj
 0001:0002ca8f       ___acrt_uninitialize_critical 1002da8f f   libucrt:initialization.obj
 0001:0002caa1       ___acrt_initialize_new_handler 1002daa1 f   libucrt:new_handler.obj
 0001:0002cab0       __callnewh                 1002dab0 f   libucrt:new_handler.obj
 0001:0002cadd       __query_new_handler        1002dadd f   libucrt:new_handler.obj
 0001:0002cb39       __initterm                 1002db39 f   libucrt:initterm.obj
 0001:0002cb7e       __initterm_e               1002db7e f   libucrt:initterm.obj
 0001:0002cbac       _strcpy_s                  1002dbac f   libucrt:strcpy_s.obj
 0001:0002cc06       ??$is_overflow_condition@K@__crt_strtox@@YA_NIK@Z 1002dc06 f i libucrt:atox.obj
 0001:0002cc37       ??$parse_integer@KV?$c_string_character_source@_W@__crt_strtox@@@__crt_strtox@@YAKQAU__crt_locale_pointers@@V?$c_string_character_source@_W@0@H_N@Z 1002dc37 f i libucrt:atox.obj
 0001:0002d23f       __wtol                     1002e23f f   libucrt:atox.obj
 0001:0002d270       _strncmp                   1002e270 f   libucrt:strncmp.obj
 0001:0002d2e8       _wcsncmp                   1002e2e8 f   libucrt:wcsncmp.obj
 0001:0002d660       ___acrt_freeptd            1002e660 f   libucrt:per_thread_data.obj
 0001:0002d68c       ___acrt_getptd             1002e68c f   libucrt:per_thread_data.obj
 0001:0002d749       ___acrt_getptd_head        1002e749 f   libucrt:per_thread_data.obj
 0001:0002d7e3       ___acrt_getptd_noexit      1002e7e3 f   libucrt:per_thread_data.obj
 0001:0002d898       ___acrt_initialize_ptd     1002e898 f   libucrt:per_thread_data.obj
 0001:0002d8c4       ___acrt_uninitialize_ptd   1002e8c4 f   libucrt:per_thread_data.obj
 0001:0002da48       ___acrt_initialize_lowio   1002ea48 f   libucrt:ioinit.obj
 0001:0002daa8       ___acrt_uninitialize_lowio 1002eaa8 f   libucrt:ioinit.obj
 0001:0002dad4       __calloc_base              1002ead4 f   libucrt:calloc_base.obj
 0001:0002db31       __query_app_type           1002eb31 f   libucrt:report_runtime_error.obj
 0001:0002db37       __free_base                1002eb37 f   libucrt:free_base.obj
 0001:0002de91       ___acrt_AppPolicyGetProcessTerminationMethodInternal@4 1002ee91 f   libucrt:winapi_thunks.obj
 0001:0002ded1       ___acrt_AreFileApisANSI@0  1002eed1 f   libucrt:winapi_thunks.obj
 0001:0002def0       ___acrt_EnumSystemLocalesEx@16 1002eef0 f   libucrt:winapi_thunks.obj
 0001:0002df44       ___acrt_FlsAlloc@4         1002ef44 f   libucrt:winapi_thunks.obj
 0001:0002df83       ___acrt_FlsFree@4          1002ef83 f   libucrt:winapi_thunks.obj
 0001:0002dfc5       ___acrt_FlsGetValue@4      1002efc5 f   libucrt:winapi_thunks.obj
 0001:0002e004       ___acrt_FlsSetValue@8      1002f004 f   libucrt:winapi_thunks.obj
 0001:0002e046       ___acrt_GetLocaleInfoEx@16 1002f046 f   libucrt:winapi_thunks.obj
 0001:0002e085       ___acrt_GetUserDefaultLocaleName@8 1002f085 f   libucrt:winapi_thunks.obj
 0001:0002e0c1       ___acrt_InitializeCriticalSectionEx@12 1002f0c1 f   libucrt:winapi_thunks.obj
 0001:0002e10c       ___acrt_IsValidLocaleName@4 1002f10c f   libucrt:winapi_thunks.obj
 0001:0002e144       ___acrt_LCIDToLocaleName@16 1002f144 f   libucrt:winapi_thunks.obj
 0001:0002e183       ___acrt_LCMapStringEx@36   1002f183 f   libucrt:winapi_thunks.obj
 0001:0002e1e0       ___acrt_LocaleNameToLCID@8 1002f1e0 f   libucrt:winapi_thunks.obj
 0001:0002e211       ___acrt_can_use_vista_locale_apis 1002f211 f   libucrt:winapi_thunks.obj
 0001:0002e21c       ___acrt_eagerly_load_locale_apis 1002f21c f   libucrt:winapi_thunks.obj
 0001:0002e253       ___acrt_initialize_winapi_thunks 1002f253 f   libucrt:winapi_thunks.obj
 0001:0002e27e       ___acrt_uninitialize_winapi_thunks 1002f27e f   libucrt:winapi_thunks.obj
 0001:0002e2b4       __fcloseall                1002f2b4 f   libucrt:closeall.obj
 0001:0002e53c       ___acrt_stdio_flush_nolock 1002f53c f   libucrt:fflush.obj
 0001:0002e5a1       __fflush_nolock            1002f5a1 f   libucrt:fflush.obj
 0001:0002e5e9       __flushall                 1002f5e9 f   libucrt:fflush.obj
 0001:0002e5f2       ___acrt_stdio_free_buffer_nolock 1002f5f2 f   libucrt:_freebuf.obj
 0001:0002e6aa       __d_int                    1002f6aa f   libucrt:_test.obj
 0001:0002e7b0       __dtest                    1002f7b0 f   libucrt:_test.obj
 0001:0002e814       __fdtest                   1002f814 f   libucrt:_test.obj
 0001:0002e862       __fperrraise               1002f862 f   libucrt:_test.obj
 0001:0002e883       __ldtest                   1002f883 f   libucrt:_test.obj
 0001:0002e88e       __malloc_base              1002f88e f   libucrt:malloc_base.obj
 0001:0002e8dc       __mbtowc_l                 1002f8dc f   libucrt:mbtowc.obj
 0001:0002ea1e       _mbtowc                    1002fa1e f   libucrt:mbtowc.obj
 0001:0002ea38       ___acrt_update_locale_info 1002fa38 f   libucrt:locale_update.obj
 0001:0002ea65       ___acrt_update_multibyte_info 1002fa65 f   libucrt:locale_update.obj
 0001:0002eb95       ??0_expandlocale_locale_name_cache@@QAE@QA_WIQAU__crt_qualified_locale_data@@@Z 1002fb95 f i libucrt:wsetlocale.obj
 0001:0002ebdf       ??1_expandlocale_locale_name_cache@@QAE@XZ 1002fbdf f i libucrt:wsetlocale.obj
 0001:0002ed77       ?commit_locale_name@_expandlocale_locale_name_cache@@QAEXQB_WI@Z 1002fd77 f i libucrt:wsetlocale.obj
 0001:0002edbb       ?commit_locale_name_cache_already_updated@_expandlocale_locale_name_cache@@QAEXQB_WI@Z 1002fdbb f i libucrt:wsetlocale.obj
 0001:0002edf0       ___acrt_copy_locale_name   1002fdf0 f   libucrt:wsetlocale.obj
 0001:0002ee50       ___acrt_set_locale_changed 1002fe50 f   libucrt:wsetlocale.obj
 0001:0002ee5b       ___acrt_uninitialize_locale 1002fe5b f   libucrt:wsetlocale.obj
 0001:0002ee82       ___lc_lctowcs              1002fe82 f   libucrt:wsetlocale.obj
 0001:0002eef2       ___lc_wcstolc              1002fef2 f   libucrt:wsetlocale.obj
 0001:0002f437       __wcscats                  10030437 f   libucrt:wsetlocale.obj
 0001:0002f478       __wsetlocale               10030478 f   libucrt:wsetlocale.obj
 0001:000308f6       __write                    100318f6 f   libucrt:write.obj
 0001:000309e8       __write_nolock             100319e8 f   libucrt:write.obj
 0001:00030bca       ___acrt_initialize_sse2    10031bca f   libucrt:mathfcns.obj
 0001:00030bda       __modf_default             10031bda f   libucrt:modf.obj
 0001:00030ce0       ___libm_error_support      10031ce0 f   libucrt:libm_error.obj
 0001:00030ed4       __dunscale                 10031ed4 f   libucrt:_unscale.obj
 0001:00030f6a       _iswctype                  10031f6a f   libucrt:iswctype.obj
 0001:00030fd3       ___acrt_wcstok_s_novalidation 10031fd3 f   libucrt:wcstok_s.obj
 0001:0003124f       __mbstowcs_s_l             1003224f f   libucrt:mbstowcs.obj
 0001:0003132f       _mbstowcs_s                1003232f f   libucrt:mbstowcs.obj
 0001:000315f8       __wcstombs_s_l             100325f8 f   libucrt:wcstombs.obj
 0001:000317a2       ___acrt_GetLocaleInfoA     100327a2 f   libucrt:getlocaleinfoa.obj
 0001:00031952       ___acrt_GetStringTypeA     10032952 f   libucrt:getstringtypea.obj
 0001:00031c3f       ___acrt_LCMapStringA       10032c3f f   libucrt:lcmapstringa.obj
 0001:00031c88       __errcode                  10032c88 f   libucrt:fpexcept.obj
 0001:00031cbc       __except1                  10032cbc f   libucrt:fpexcept.obj
 0001:00031d8a       __handle_exc               10032d8a f   libucrt:fpexcept.obj
 0001:00031f75       __raise_exc                10032f75 f   libucrt:fpexcept.obj
 0001:00031f98       __raise_exc_ex             10032f98 f   libucrt:fpexcept.obj
 0001:0003228e       __set_errno_from_matherr   1003328e f   libucrt:fpexcept.obj
 0001:000322bd       __umatherr                 100332bd f   libucrt:fpexcept.obj
 0001:0003235d       __decomp                   1003335d f   libucrt:util.obj
 0001:0003242f       __set_exp                  1003342f f   libucrt:util.obj
 0001:0003245c       __sptype                   1003345c f   libucrt:util.obj
 0001:000324ba       __clrfp                    100334ba f   libucrt:fpctrl.obj
 0001:000324cb       __ctrlfp                   100334cb f   libucrt:fpctrl.obj
 0001:000324f5       __set_statfp               100334f5 f   libucrt:fpctrl.obj
 0001:0003254e       __statfp                   1003354e f   libucrt:fpctrl.obj
 0001:0003255e       __copysign                 1003355e f   libucrt:ieeemisc.obj
 0001:00032581       __fpclass                  10033581 f   libucrt:ieeemisc.obj
 0001:00032625       __realloc_base             10033625 f   libucrt:realloc_base.obj
 0001:00032690       __CIpow_pentium4           10033690 f   libucrt:pow_pentium4.obj
 0001:000326a9       __pow_pentium4             100336a9     libucrt:pow_pentium4.obj
 0001:000331d0       __fFEXP                    100341d0 f   libucrt:87tran.obj
 0001:00033227       __rtinfpopse               10034227     libucrt:87tran.obj
 0001:00033229       __rtinfnpopse              10034229     libucrt:87tran.obj
 0001:00033239       __fFLN                     10034239     libucrt:87tran.obj
 0001:000332ee       __rtinfpop                 100342ee     libucrt:87tran.obj
 0001:000332f0       __rtinfnpop                100342f0     libucrt:87tran.obj
 0001:00033300       __rtforexpinf              10034300 f   libucrt:87tran.obj
 0001:0003330d       __ffexpm1                  1003430d     libucrt:87tran.obj
 0001:000333c0       __trandisp1                100343c0 f   libucrt:87disp.obj
 0001:00033435       __trandisp2                10034435 f   libucrt:87disp.obj
 0001:000334cf       __rttospopde               100344cf     libucrt:87disp.obj
 0001:000334d4       __rttospop                 100344d4     libucrt:87disp.obj
 0001:000334e0       __rtnospop                 100344e0 f   libucrt:87disp.obj
 0001:000334f0       __rttosnpop                100344f0 f   libucrt:87disp.obj
 0001:000334f1       __rtnospopde               100344f1     libucrt:87disp.obj
 0001:000334f8       __rtzeropop                100344f8     libucrt:87disp.obj
 0001:000334fa       __rtzeronpop               100344fa     libucrt:87disp.obj
 0001:00033500       __rtzerospop               10034500 f   libucrt:87disp.obj
 0001:0003350d       __rtonepop                 1003450d     libucrt:87disp.obj
 0001:00033510       __rtonenpop                10034510 f   libucrt:87disp.obj
 0001:00033520       __tosnan1                  10034520 f   libucrt:87disp.obj
 0001:00033550       __nosnan2                  10034550 f   libucrt:87disp.obj
 0001:00033560       __tosnan2                  10034560 f   libucrt:87disp.obj
 0001:00033590       __nan2                     10034590 f   libucrt:87disp.obj
 0001:000335d0       __rtindfpop                100345d0 f   libucrt:87disp.obj
 0001:000335d2       __rtindfnpop               100345d2     libucrt:87disp.obj
 0001:000335e3       __rttosnpopde              100345e3     libucrt:87disp.obj
 0001:000335f0       __rtatan2inf               100345f0 f   libucrt:87disp.obj
 0001:0003360d       __rtchsifneg               1003460d     libucrt:87disp.obj
 0001:00033620       __startTwoArgErrorHandling 10034620 f   libucrt:genexcep.obj
 0001:00033637       __startOneArgErrorHandling 10034637 f   libucrt:genexcep.obj
 0001:00033680       __twoToTOS                 10034680 f   libucrt:common.obj
 0001:00033695       __load_CW                  10034695 f   libucrt:common.obj
 0001:000336ac       __convertTOStoQNaN         100346ac f   libucrt:common.obj
 0001:000336c5       __fload_withFB             100346c5 f   libucrt:common.obj
 0001:00033708       __checkTOS_withFB          10034708 f   libucrt:common.obj
 0001:0003371e       __fast_exit                1003471e f   libucrt:common.obj
 0001:0003372b       __math_exit                1003472b f   libucrt:common.obj
 0001:00033755       __check_overflow_exit      10034755 f   libucrt:common.obj
 0001:00033769       __check_range_exit         10034769 f   libucrt:common.obj
 0001:0003380c       __d_inttype                1003480c f   libucrt:powhlp.obj
 0001:00033874       __powhlp                   10034874 f   libucrt:powhlp.obj
 0001:00033a6d       ___acrt_get_sigabrt_handler 10034a6d f   libucrt:signal.obj
 0001:00033a94       ___acrt_initialize_signal_handlers 10034a94 f   libucrt:signal.obj
 0001:00033ab2       ___fpecode                 10034ab2 f   libucrt:signal.obj
 0001:00033abb       _raise                     10034abb f   libucrt:signal.obj
 0001:00033cb6       _wcscpy_s                  10034cb6 f   libucrt:wcscpy_s.obj
 0001:00033d1a       ___acrt_MultiByteToWideChar 10034d1a f   libucrt:multibytetowidechar.obj
 0001:00033d96       ___acrt_WideCharToMultiByte 10034d96 f   libucrt:widechartomultibyte.obj
 0001:00033e43       ___ascii_wcsicmp           10034e43 f   libucrt:wcsicmp.obj
 0001:00033e80       __towlower_internal        10034e80 f i libucrt:wcsicmp.obj
 0001:00033ebf       __wcsicmp                  10034ebf f   libucrt:wcsicmp.obj
 0001:00033f08       __wcsicmp_l                10034f08 f   libucrt:wcsicmp.obj
 0001:00033fc0       ___acrt_initialize_timeset 10034fc0 f   libucrt:timeset.obj
 0001:00033feb       ___acrt_get_process_end_policy 10034feb f   libucrt:win_policies.obj
 0001:000345fa       ?__acrt_get_utf8_acp_compatibility_codepage@@YAIXZ 100355fa f i libucrt:argv_wildcards.obj
 0001:00034639       ?allocate@?$__crt_win32_buffer@DU__crt_win32_buffer_internal_dynamic_resizing@@@@QAEHI@Z 10035639 f i libucrt:argv_wildcards.obj
 0001:000346fc       ___acrt_expand_narrow_argv_wildcards 100356fc f   libucrt:argv_wildcards.obj
 0001:000347ce       ___acrt_GetModuleFileNameA 100357ce f   libucrt:getmodulefilenamea.obj
 0001:00034d8d       ___acrt_initialize_multibyte 10035d8d f   libucrt:mbctype.obj
 0001:00034dd5       ___acrt_update_thread_multibyte_data 10035dd5 f   libucrt:mbctype.obj
 0001:00034de8       __setmbcp_nolock           10035de8 f   libucrt:mbctype.obj
 0001:000350b3       __ismbblead                100360b3 f   libucrt:ismbbyte.obj
 0001:000350cb       ___acrt_initialize_command_line 100360cb f   libucrt:argv_data.obj
 0001:0003511b       ___dcrt_get_narrow_environment_from_os 1003611b f   libucrt:get_environment_from_os.obj
 0001:0003519f       __recalloc_base            1003619f f   libucrt:recalloc.obj
 0001:0003520c       ___acrt_initialize_heap    1003620c f   libucrt:heap_handle.obj
 0001:0003521d       ___acrt_uninitialize_heap  1003621d f   libucrt:heap_handle.obj
 0001:00035227       ___acrt_execute_initializers 10036227 f   libucrt:shared_initialization.obj
 0001:0003528f       ___acrt_execute_uninitializers 1003628f f   libucrt:shared_initialization.obj
 0001:000352c0       ___acrt_has_user_matherr   100362c0 f   libucrt:matherr.obj
 0001:000352d8       ___acrt_initialize_user_matherr 100362d8 f   libucrt:matherr.obj
 0001:000352e7       ___acrt_invoke_user_matherr 100362e7 f   libucrt:matherr.obj
 0001:00035319       ___acrt_add_locale_ref     10036319 f   libucrt:locale_refcounting.obj
 0001:00035396       ___acrt_free_locale        10036396 f   libucrt:locale_refcounting.obj
 0001:000354de       ___acrt_locale_add_lc_time_reference 100364de f   libucrt:locale_refcounting.obj
 0001:00035507       ___acrt_locale_free_lc_time_if_unreferenced 10036507 f   libucrt:locale_refcounting.obj
 0001:00035538       ___acrt_locale_release_lc_time_reference 10036538 f   libucrt:locale_refcounting.obj
 0001:00035561       ___acrt_release_locale_ref 10036561 f   libucrt:locale_refcounting.obj
 0001:000355e2       ___acrt_update_thread_locale_data 100365e2 f   libucrt:locale_refcounting.obj
 0001:00035663       __updatetlocinfoEx_nolock  10036663 f   libucrt:locale_refcounting.obj
 0001:0003572f       __lseeki64_nolock          1003672f f   libucrt:lseek.obj
 0001:0003574a       __query_new_mode           1003674a f   libucrt:new_mode.obj
 0001:00035751       _wcscat_s                  10036751 f   libucrt:wcscat_s.obj
 0001:00035816       ___acrt_DownlevelLCIDToLocaleName 10036816 f   libucrt:lcidtoname_downlevel.obj
 0001:000358c0       ___acrt_DownlevelLocaleNameToLCID 100368c0 f   libucrt:lcidtoname_downlevel.obj
 0001:000358ec       __fclose_nolock            100368ec f   libucrt:fclose.obj
 0001:00035963       _fclose                    10036963 f   libucrt:fclose.obj
 0001:00035a89       __commit                   10036a89 f   libucrt:commit.obj
 0001:00035b06       _fegetexceptflag           10036b06 f   libucrt:fegetexceptflag.obj
 0001:00035b37       _fesetexceptflag           10036b37 f   libucrt:fesetexceptflag.obj
 0001:00035b90       ___acrt_fenv_get_fp_status_word_from_exception_mask 10036b90 f   libucrt:_fenvutils.obj
 0001:00035baa       ___acrt_fenv_get_status    10036baa f   libucrt:_fenvutils.obj
 0001:00035c62       ___acrt_fenv_set_status    10036c62 f   libucrt:_fenvutils.obj
 0001:00035d85       ?__mbrtowc_utf8@__crt_mbstring@@YAIPA_WPBDIPAU_Mbstatet@@@Z 10036d85 f   libucrt:mbrtowc.obj
 0001:00035dc5       ?__mbsrtowcs_utf8@__crt_mbstring@@YAIPA_WPAPBDIPAU_Mbstatet@@@Z 10036dc5 f   libucrt:mbrtowc.obj
 0001:00035ec0       ?__c32rtomb_utf8@__crt_mbstring@@YAIPAD_UPAU_Mbstatet@@@Z 10036ec0 f   libucrt:c32rtomb.obj
 0001:00035f6b       ?return_illegal_sequence@__crt_mbstring@@YAIPAU_Mbstatet@@@Z 10036f6b f i libucrt:c32rtomb.obj
 0001:00035f8a       _c32rtomb                  10036f8a f   libucrt:c32rtomb.obj
 0001:00035f95       ___acrt_locale_free_monetary 10036f95 f   libucrt:initmon.obj
 0001:00036093       ___acrt_locale_initialize_monetary 10037093 f   libucrt:initmon.obj
 0001:0003644a       ___acrt_locale_free_numeric 1003744a f   libucrt:initnum.obj
 0001:000364b3       ___acrt_locale_initialize_numeric 100374b3 f   libucrt:initnum.obj
 0001:00036976       ___acrt_locale_free_time   10037976 f   libucrt:inittime.obj
 0001:00036a5a       ___acrt_locale_initialize_time 10037a5a f   libucrt:inittime.obj
 0001:00036bbc       _wcsncat_s                 10037bbc f   libucrt:wcsncat_s.obj
 0001:000372c3       ___acrt_get_qualified_locale 100382c3 f   libucrt:get_qualified_locale.obj
 0001:00037c24       ___acrt_get_qualified_locale_downlevel 10038c24 f   libucrt:getqloc_downlevel.obj
 0001:00037e19       __putwch_nolock            10038e19 f   libucrt:putwch.obj
 0001:00037e4b       __frnd                     10038e4b f   libucrt:frnd.obj
 0001:00037e5f       __dnorm                    10038e5f f   libucrt:_norm.obj
 0001:00037ff4       ___acrt_GetStringTypeW     10038ff4 f   libucrt:getstringtypew.obj
 0001:0003800d       ?__wcsrtombs_utf8@__crt_mbstring@@YAIPADPAPB_WIPAU_Mbstatet@@@Z 1003900d f   libucrt:wcrtomb.obj
 0001:000381be       _strncpy_s                 100391be f   libucrt:strncpy_s.obj
 0001:000381c9       __87except                 100391c9 f   libucrt:87except.obj
 0001:000382d3       __towlower_l               100392d3 f   libucrt:towlower.obj
 0001:000383c0       _qsort                     100393c0 f   libucrt:qsort.obj
 0001:00038810       _strpbrk                   10039810 f   libucrt:strpbrk.obj
 0001:00038850       __mbsdec                   10039850 f   libucrt:mbsdec.obj
 0001:00038867       __mbsdec_l                 10039867 f   libucrt:mbsdec.obj
 0001:00038903       __msize_base               10039903 f   libucrt:msize.obj
 0001:00038936       ___ascii_wcsnicmp          10039936 f   libucrt:wcsnicmp.obj
 0001:00038985       __wcsnicmp                 10039985 f   libucrt:wcsnicmp.obj
 0001:000389d1       __wcsnicmp_l               100399d1 f   libucrt:wcsnicmp.obj
 0001:00038b30       __close                    10039b30 f   libucrt:close.obj
 0001:00038bbd       __close_nolock             10039bbd f   libucrt:close.obj
 0001:00038c59       ?__acrt_stdio_free_stream@@YAXV__crt_stdio_stream@@@Z 10039c59 f   libucrt:stream.obj
 0001:00038c94       _fetestexcept              10039c94 f   libucrt:fetestexcept.obj
 0001:00038cb4       ?__mbrtoc32_utf8@__crt_mbstring@@YAIPA_UPBDIPAU_Mbstatet@@@Z 10039cb4 f   libucrt:mbrtoc32.obj
 0001:00038e60       __CIlog10                  10039e60 f   libucrt:log10_impl.obj
 0001:00038e9b       __CIlog10_default          10039e9b f   libucrt:log10_impl.obj
 0001:00038eaf       __log10_default            10039eaf     libucrt:log10_impl.obj
 0001:00038f70       _ceil                      10039f70 f   libucrt:ceil_pentium4.obj
 0001:00038fb0       __ceil_pentium4            10039fb0 f   libucrt:ceil_pentium4.obj
 0001:000391b2       __itow_s                   1003a1b2 f   libucrt:xtoa.obj
 0001:00039204       ___dcrt_lowio_ensure_console_output_initialized 1003a204 f   libucrt:initcon.obj
 0001:00039223       ___dcrt_terminate_console_output 1003a223 f   libucrt:initcon.obj
 0001:0003923a       ___dcrt_write_console      1003a23a f   libucrt:initcon.obj
 0001:0003928f       ?__c16rtomb_utf8@__crt_mbstring@@YAIPAD_SPAU_Mbstatet@@@Z 1003a28f f   libucrt:c16rtomb.obj
 0001:00039329       ___acrt_LCMapStringW       1003a329 f   libucrt:lcmapstringw.obj
 0001:00039370       __CIlog10_pentium4         1003a370 f   libucrt:log10_pentium4.obj
 0001:00039388       __log10_pentium4           1003a388     libucrt:log10_pentium4.obj
 0001:00039600       __ceil_default             1003a600 f   libucrt:ceil.obj
 0001:000396c0       ___ascii_strnicmp          1003a6c0 f   libucrt:_strnicm.obj
 0001:00039730       __FindPESection            1003a730 f   LIBCMT:pesect.obj
 0001:00039780       __IsNonwritableInCurrentImage 1003a780 f   LIBCMT:pesect.obj
 0001:00039840       __ValidateImageBase        1003a840 f   LIBCMT:pesect.obj
 0001:00039880       __aulldvrm                 1003a880 f   LIBCMT:ulldvrm.obj
 0001:00039920       __allshl                   1003a920 f   LIBCMT:llshl.obj
 0001:00039940       __aullshr                  1003a940 f   LIBCMT:ullshr.obj
 0001:00039960       __ftol2_sse                1003a960 f   LIBCMT:ftol2.obj
 0001:00039970       __ftoi2                    1003a970 f   LIBCMT:ftol2.obj
 0001:000399f0       __ftol2                    1003a9f0 f   LIBCMT:ftol2.obj
 0001:00039aa0       __filter_x86_sse2_floating_point_exception 1003aaa0 f   LIBCMT:x86_exception_filter.obj
 0001:00039aa0       __filter_x86_sse2_floating_point_exception_default 1003aaa0 f   LIBCMT:x86_exception_filter.obj
 0001:00039b20       __alldiv                   1003ab20 f   LIBCMT:lldiv.obj
 0001:00039bca       __fdclass                  1003abca f   libucrt:nanf.obj
 0001:00039bdb       __ldclass                  1003abdb f   libucrt:nanl.obj
 0002:00000000       __imp__LookupPrivilegeValueW@12 1003d000     advapi32:ADVAPI32.dll
 0002:00000004       __imp__AdjustTokenPrivileges@24 1003d004     advapi32:ADVAPI32.dll
 0002:00000008       __imp__OpenProcessToken@12 1003d008     advapi32:ADVAPI32.dll
 0002:0000000c       __imp__SetThreadToken@8    1003d00c     advapi32:ADVAPI32.dll
 0002:00000010       __imp__DuplicateTokenEx@24 1003d010     advapi32:ADVAPI32.dll
 0002:00000014       __imp__OpenThreadToken@16  1003d014     advapi32:ADVAPI32.dll
 0002:00000018       __imp__RegCloseKey@4       1003d018     advapi32:ADVAPI32.dll
 0002:0000001c       __imp__RegConnectRegistryW@12 1003d01c     advapi32:ADVAPI32.dll
 0002:00000020       __imp__RegQueryValueExW@24 1003d020     advapi32:ADVAPI32.dll
 0002:00000024       __imp__ConvertSidToStringSidW@8 1003d024     advapi32:ADVAPI32.dll
 0002:00000028       __imp__GetUserNameW@8      1003d028     advapi32:ADVAPI32.dll
 0002:0000002c       __imp__LookupAccountNameW@28 1003d02c     advapi32:ADVAPI32.dll
 0002:00000030       \177ADVAPI32_NULL_THUNK_DATA 1003d030     advapi32:ADVAPI32.dll
 0002:00000034       __imp__lstrlenW@4          1003d034     kernel32:KERNEL32.dll
 0002:00000038       __imp__SetLastError@4      1003d038     kernel32:KERNEL32.dll
 0002:0000003c       __imp__SetPriorityClass@8  1003d03c     kernel32:KERNEL32.dll
 0002:00000040       __imp__lstrcpynW@12        1003d040     kernel32:KERNEL32.dll
 0002:00000044       __imp__CreateFileW@28      1003d044     kernel32:KERNEL32.dll
 0002:00000048       __imp__GetCurrentThreadId@0 1003d048     kernel32:KERNEL32.dll
 0002:0000004c       __imp__SetEvent@4          1003d04c     kernel32:KERNEL32.dll
 0002:00000050       __imp__FileTimeToSystemTime@8 1003d050     kernel32:KERNEL32.dll
 0002:00000054       __imp__GetLocalTime@4      1003d054     kernel32:KERNEL32.dll
 0002:00000058       __imp__GetPriorityClass@4  1003d058     kernel32:KERNEL32.dll
 0002:0000005c       __imp__SystemTimeToTzSpecificLocalTime@12 1003d05c     kernel32:KERNEL32.dll
 0002:00000060       __imp__GetSystemTimeAsFileTime@4 1003d060     kernel32:KERNEL32.dll
 0002:00000064       __imp__GetTickCount@0      1003d064     kernel32:KERNEL32.dll
 0002:00000068       __imp__lstrcmpW@8          1003d068     kernel32:KERNEL32.dll
 0002:0000006c       __imp__WaitForMultipleObjects@16 1003d06c     kernel32:KERNEL32.dll
 0002:00000070       __imp__CreateMutexW@12     1003d070     kernel32:KERNEL32.dll
 0002:00000074       __imp__ReleaseMutex@4      1003d074     kernel32:KERNEL32.dll
 0002:00000078       __imp__CreateEventW@16     1003d078     kernel32:KERNEL32.dll
 0002:0000007c       __imp__ResetEvent@4        1003d07c     kernel32:KERNEL32.dll
 0002:00000080       __imp__GetProcessTimes@20  1003d080     kernel32:KERNEL32.dll
 0002:00000084       __imp__GetFileType@4       1003d084     kernel32:KERNEL32.dll
 0002:00000088       __imp__OpenProcess@12      1003d088     kernel32:KERNEL32.dll
 0002:0000008c       __imp__GetLastError@0      1003d08c     kernel32:KERNEL32.dll
 0002:00000090       __imp__GetCurrentThread@0  1003d090     kernel32:KERNEL32.dll
 0002:00000094       __imp__ReadProcessMemory@20 1003d094     kernel32:KERNEL32.dll
 0002:00000098       __imp__FormatMessageW@28   1003d098     kernel32:KERNEL32.dll
 0002:0000009c       __imp__FileTimeToLocalFileTime@8 1003d09c     kernel32:KERNEL32.dll
 0002:000000a0       __imp__GetTimeFormatW@24   1003d0a0     kernel32:KERNEL32.dll
 0002:000000a4       __imp__GetModuleHandleW@4  1003d0a4     kernel32:KERNEL32.dll
 0002:000000a8       __imp__GetDateFormatW@24   1003d0a8     kernel32:KERNEL32.dll
 0002:000000ac       __imp__GetProcAddress@8    1003d0ac     kernel32:KERNEL32.dll
 0002:000000b0       __imp__CompareStringW@24   1003d0b0     kernel32:KERNEL32.dll
 0002:000000b4       __imp__EnterCriticalSection@4 1003d0b4     kernel32:KERNEL32.dll
 0002:000000b8       __imp__GetModuleFileNameW@12 1003d0b8     kernel32:KERNEL32.dll
 0002:000000bc       __imp__LeaveCriticalSection@4 1003d0bc     kernel32:KERNEL32.dll
 0002:000000c0       __imp__InitializeCriticalSection@4 1003d0c0     kernel32:KERNEL32.dll
 0002:000000c4       __imp__LoadLibraryW@4      1003d0c4     kernel32:KERNEL32.dll
 0002:000000c8       __imp__DeleteCriticalSection@4 1003d0c8     kernel32:KERNEL32.dll
 0002:000000cc       __imp__LCMapStringW@24     1003d0cc     kernel32:KERNEL32.dll
 0002:000000d0       __imp__GetThreadTimes@20   1003d0d0     kernel32:KERNEL32.dll
 0002:000000d4       __imp__VirtualQuery@12     1003d0d4     kernel32:KERNEL32.dll
 0002:000000d8       __imp__GetCurrentProcessId@0 1003d0d8     kernel32:KERNEL32.dll
 0002:000000dc       __imp__LocalFree@4         1003d0dc     kernel32:KERNEL32.dll
 0002:000000e0       __imp__CreateThread@24     1003d0e0     kernel32:KERNEL32.dll
 0002:000000e4       __imp__CloseHandle@4       1003d0e4     kernel32:KERNEL32.dll
 0002:000000e8       __imp__TerminateThread@8   1003d0e8     kernel32:KERNEL32.dll
 0002:000000ec       __imp__DuplicateHandle@28  1003d0ec     kernel32:KERNEL32.dll
 0002:000000f0       __imp__WaitForSingleObject@8 1003d0f0     kernel32:KERNEL32.dll
 0002:000000f4       __imp__VirtualAlloc@16     1003d0f4     kernel32:KERNEL32.dll
 0002:000000f8       __imp__GetCurrentProcess@0 1003d0f8     kernel32:KERNEL32.dll
 0002:000000fc       __imp__VirtualFree@12      1003d0fc     kernel32:KERNEL32.dll
 0002:00000100       __imp__WriteConsoleW@20    1003d100     kernel32:KERNEL32.dll
 0002:00000104       __imp__TerminateProcess@8  1003d104     kernel32:KERNEL32.dll
 0002:00000108       __imp__WriteFile@20        1003d108     kernel32:KERNEL32.dll
 0002:0000010c       __imp__FlushFileBuffers@4  1003d10c     kernel32:KERNEL32.dll
 0002:00000110       __imp__GetProcessHeap@0    1003d110     kernel32:KERNEL32.dll
 0002:00000114       __imp__FreeEnvironmentStringsW@4 1003d114     kernel32:KERNEL32.dll
 0002:00000118       __imp__GetEnvironmentStringsW@0 1003d118     kernel32:KERNEL32.dll
 0002:0000011c       __imp__GetCommandLineW@0   1003d11c     kernel32:KERNEL32.dll
 0002:00000120       __imp__HeapSize@12         1003d120     kernel32:KERNEL32.dll
 0002:00000124       __imp__GetCommandLineA@0   1003d124     kernel32:KERNEL32.dll
 0002:00000128       __imp__GetOEMCP@0          1003d128     kernel32:KERNEL32.dll
 0002:0000012c       __imp__GetACP@0            1003d12c     kernel32:KERNEL32.dll
 0002:00000130       __imp__IsValidCodePage@4   1003d130     kernel32:KERNEL32.dll
 0002:00000134       __imp__FindNextFileW@8     1003d134     kernel32:KERNEL32.dll
 0002:00000138       __imp__FindFirstFileExW@24 1003d138     kernel32:KERNEL32.dll
 0002:0000013c       __imp__FindClose@4         1003d13c     kernel32:KERNEL32.dll
 0002:00000140       __imp__HeapReAlloc@16      1003d140     kernel32:KERNEL32.dll
 0002:00000144       __imp__GetConsoleMode@8    1003d144     kernel32:KERNEL32.dll
 0002:00000148       __imp__GetConsoleCP@0      1003d148     kernel32:KERNEL32.dll
 0002:0000014c       __imp__EnumSystemLocalesW@8 1003d14c     kernel32:KERNEL32.dll
 0002:00000150       __imp__GetUserDefaultLCID@0 1003d150     kernel32:KERNEL32.dll
 0002:00000154       __imp__IsValidLocale@8     1003d154     kernel32:KERNEL32.dll
 0002:00000158       __imp__GetLocaleInfoW@16   1003d158     kernel32:KERNEL32.dll
 0002:0000015c       __imp__HeapFree@12         1003d15c     kernel32:KERNEL32.dll
 0002:00000160       __imp__HeapAlloc@12        1003d160     kernel32:KERNEL32.dll
 0002:00000164       __imp__GetStdHandle@4      1003d164     kernel32:KERNEL32.dll
 0002:00000168       __imp__SetFilePointerEx@20 1003d168     kernel32:KERNEL32.dll
 0002:0000016c       __imp__ExitProcess@4       1003d16c     kernel32:KERNEL32.dll
 0002:00000170       __imp__MultiByteToWideChar@24 1003d170     kernel32:KERNEL32.dll
 0002:00000174       __imp__WideCharToMultiByte@32 1003d174     kernel32:KERNEL32.dll
 0002:00000178       __imp__GetStringTypeW@16   1003d178     kernel32:KERNEL32.dll
 0002:0000017c       __imp__GetCPInfo@8         1003d17c     kernel32:KERNEL32.dll
 0002:00000180       __imp__UnhandledExceptionFilter@4 1003d180     kernel32:KERNEL32.dll
 0002:00000184       __imp__SetUnhandledExceptionFilter@4 1003d184     kernel32:KERNEL32.dll
 0002:00000188       __imp__IsProcessorFeaturePresent@4 1003d188     kernel32:KERNEL32.dll
 0002:0000018c       __imp__IsDebuggerPresent@0 1003d18c     kernel32:KERNEL32.dll
 0002:00000190       __imp__GetStartupInfoW@4   1003d190     kernel32:KERNEL32.dll
 0002:00000194       __imp__QueryPerformanceCounter@4 1003d194     kernel32:KERNEL32.dll
 0002:00000198       __imp__RtlUnwind@16        1003d198     kernel32:KERNEL32.dll
 0002:0000019c       __imp__RaiseException@16   1003d19c     kernel32:KERNEL32.dll
 0002:000001a0       __imp__InitializeCriticalSectionAndSpinCount@8 1003d1a0     kernel32:KERNEL32.dll
 0002:000001a4       __imp__TlsAlloc@0          1003d1a4     kernel32:KERNEL32.dll
 0002:000001a8       __imp__TlsGetValue@4       1003d1a8     kernel32:KERNEL32.dll
 0002:000001ac       __imp__TlsSetValue@8       1003d1ac     kernel32:KERNEL32.dll
 0002:000001b0       __imp__TlsFree@4           1003d1b0     kernel32:KERNEL32.dll
 0002:000001b4       __imp__FreeLibrary@4       1003d1b4     kernel32:KERNEL32.dll
 0002:000001b8       __imp__LoadLibraryExW@12   1003d1b8     kernel32:KERNEL32.dll
 0002:000001bc       __imp__SetStdHandle@8      1003d1bc     kernel32:KERNEL32.dll
 0002:000001c0       \177KERNEL32_NULL_THUNK_DATA 1003d1c0     kernel32:KERNEL32.dll
 0002:000001c4       __imp__WNetCancelConnection2W@12 1003d1c4     mpr:MPR.dll
 0002:000001c8       __imp__WNetAddConnection2W@16 1003d1c8     mpr:MPR.dll
 0002:000001cc       \177MPR_NULL_THUNK_DATA    1003d1cc     mpr:MPR.dll
 0002:000001d0       __imp__VariantClear@4      1003d1d0     oleaut32:OLEAUT32.dll
 0002:000001d4       __imp__SysAllocString@4    1003d1d4     oleaut32:OLEAUT32.dll
 0002:000001d8       __imp__SysFreeString@4     1003d1d8     oleaut32:OLEAUT32.dll
 0002:000001dc       \177OLEAUT32_NULL_THUNK_DATA 1003d1dc     oleaut32:OLEAUT32.dll
 0002:000001e0       __imp__GetModuleInformation@16 1003d1e0     psapi:PSAPI.DLL
 0002:000001e4       __imp__GetModuleFileNameExW@16 1003d1e4     psapi:PSAPI.DLL
 0002:000001e8       \177PSAPI_NULL_THUNK_DATA  1003d1e8     psapi:PSAPI.DLL
 0002:000001ec       __imp__SetForegroundWindow@4 1003d1ec     user32:USER32.dll
 0002:000001f0       __imp__GetParent@4         1003d1f0     user32:USER32.dll
 0002:000001f4       __imp__CharUpperBuffW@8    1003d1f4     user32:USER32.dll
 0002:000001f8       __imp__GetAncestor@8       1003d1f8     user32:USER32.dll
 0002:000001fc       __imp__GetWindowTextW@12   1003d1fc     user32:USER32.dll
 0002:00000200       __imp__ShowWindowAsync@8   1003d200     user32:USER32.dll
 0002:00000204       __imp__IsIconic@4          1003d204     user32:USER32.dll
 0002:00000208       __imp__EnumWindows@8       1003d208     user32:USER32.dll
 0002:0000020c       __imp__GetWindowLongW@8    1003d20c     user32:USER32.dll
 0002:00000210       __imp__GetWindowThreadProcessId@8 1003d210     user32:USER32.dll
 0002:00000214       __imp__GetLastActivePopup@4 1003d214     user32:USER32.dll
 0002:00000218       __imp__IsWindowVisible@4   1003d218     user32:USER32.dll
 0002:0000021c       \177USER32_NULL_THUNK_DATA 1003d21c     user32:USER32.dll
 0002:00000220       __imp__VerQueryValueW@16   1003d220     version:VERSION.dll
 0002:00000224       __imp__GetFileVersionInfoSizeW@8 1003d224     version:VERSION.dll
 0002:00000228       __imp__GetFileVersionInfoW@16 1003d228     version:VERSION.dll
 0002:0000022c       \177VERSION_NULL_THUNK_DATA 1003d22c     version:VERSION.dll
 0002:00000230       __imp__CoUninitialize@0    1003d230     ole32:ole32.dll
 0002:00000234       __imp__CoInitialize@4      1003d234     ole32:ole32.dll
 0002:00000238       __imp__CoCreateInstance@20 1003d238     ole32:ole32.dll
 0002:0000023c       \177ole32_NULL_THUNK_DATA  1003d23c     ole32:ole32.dll
 0002:00000240       ___guard_check_icall_fptr  1003d240     LIBCMT:guard_support.obj
 0002:00000244       ___xc_a                    1003d244     LIBCMT:initializers.obj
 0002:00000268       ___xc_z                    1003d268     LIBCMT:initializers.obj
 0002:0000026c       ___xi_a                    1003d26c     LIBCMT:initializers.obj
 0002:00000274       ___acrt_stdio_initializer  1003d274     libucrt:stdio_initializer.obj
 0002:00000278       ___acrt_tran_sse2_initializer 1003d278     libucrt:sse2_initializer.obj
 0002:0000027c       ___acrt_timeset_initializer 1003d27c     libucrt:timeset_initializer.obj
 0002:00000280       ___acrt_multibyte_initializer 1003d280     libucrt:multibyte_initializer.obj
 0002:00000284       ___xi_z                    1003d284     LIBCMT:initializers.obj
 0002:00000288       ___xp_a                    1003d288     LIBCMT:initializers.obj
 0002:0000028c       ___acrt_locale_terminator  1003d28c     libucrt:locale_initializer.obj
 0002:00000290       ___dcrt_console_output_terminator 1003d290     libucrt:console_output_initializer.obj
 0002:00000294       ___acrt_stdio_terminator   1003d294     libucrt:stdio_initializer.obj
 0002:00000298       ___xp_z                    1003d298     LIBCMT:initializers.obj
 0002:0000029c       ___xt_a                    1003d29c     LIBCMT:initializers.obj
 0002:000002a0       ___xt_z                    1003d2a0     LIBCMT:initializers.obj
 0002:000002b0       __imp__EncodePointer@4     1003d2b0     vc_crt_fix.obj
 0002:000002b4       __imp__DecodePointer@4     1003d2b4     vc_crt_fix.obj
 0002:000002b8       __imp__GetModuleHandleExW@12 1003d2b8     vc_crt_fix.obj
 0002:000002bc       __imp__InitializeSListHead@4 1003d2bc     vc_crt_fix.obj
 0002:000002c0       __imp__InterlockedFlushSList@4 1003d2c0     vc_crt_fix.obj
 0002:000002c4       __imp__InterlockedPopEntrySList@4 1003d2c4     vc_crt_fix.obj
 0002:000002c8       __imp__InterlockedPushEntrySList@8 1003d2c8     vc_crt_fix.obj
 0002:000002cc       __imp__InterlockedPushListSListEx@16 1003d2cc     vc_crt_fix.obj
 0002:000002d0       __imp__RtlFirstEntrySList@4 1003d2d0     vc_crt_fix.obj
 0002:000002d4       __imp__QueryDepthSList@4   1003d2d4     vc_crt_fix.obj
 0002:000002d8       __imp__GetNumaHighestNodeNumber@4 1003d2d8     vc_crt_fix.obj
 0002:000002dc       __imp__GetLogicalProcessorInformation@8 1003d2dc     vc_crt_fix.obj
 0002:000002e0       __imp__SetThreadStackGuarantee@4 1003d2e0     vc_crt_fix.obj
 0002:000002e4       __imp__InitializeCriticalSectionEx@12 1003d2e4     vc_crt_fix.obj
 0002:000002e8       __imp__CompareStringEx@36  1003d2e8     vc_crt_fix.obj
 0002:000002ec       __imp__LCMapStringEx@36    1003d2ec     vc_crt_fix.obj
 0002:000002f0       _CLSID_WbemLocator         1003d2f0     wbemuuid:wbemcli_i.obj
 0002:00000300       _IID_IWbemLocator          1003d300     wbemuuid:wbemcli_i.obj
 0002:00000314       ??_7exception@std@@6B@     1003d314     libcpmt:xthrow.obj
 0002:00000320       ??_7bad_alloc@std@@6B@     1003d320     libcpmt:xthrow.obj
 0002:00000328       ??_C@_0P@GHFPNOJB@bad?5allocation@ 1003d328     libcpmt:xthrow.obj
 0002:0000033c       ??_7bad_function_call@std@@6B@ 1003d33c     libcpmt:xthrow.obj
 0002:00000344       ??_C@_0BC@DPJNKNAF@bad?5function?5call@ 1003d344     libcpmt:xthrow.obj
 0002:0000035c       ??_7logic_error@std@@6B@   1003d35c     libcpmt:xthrow.obj
 0002:00000368       ??_7length_error@std@@6B@  1003d368     libcpmt:xthrow.obj
 0002:00000374       ??_7out_of_range@std@@6B@  1003d374     libcpmt:xthrow.obj
 0002:00000380       ??_7runtime_error@std@@6B@ 1003d380     libcpmt:xthrow.obj
 0002:0000038c       ??_7_Facet_base@std@@6B@   1003d38c     libcpmt:locale0.obj
 0002:0000039c       ??_7_Locimp@locale@std@@6B@ 1003d39c     libcpmt:locale0.obj
 0002:000003a8       ??_C@_01NBENCBCI@?$CK@     1003d3a8     libcpmt:locale0.obj
 0002:000003ac       ??_C@_01GFHCPBMG@C@        1003d3ac     libcpmt:locale0.obj
 0002:00000898       ??_C@_0BN@LKKBCCDB@address?5family?5not?5supported@ 1003d898     libcpmt:syserror.obj
 0002:000008b8       ??_C@_0P@LDMLAFHI@address?5in?5use@ 1003d8b8     libcpmt:syserror.obj
 0002:000008c8       ??_C@_0BG@DHPCNBJB@address?5not?5available@ 1003d8c8     libcpmt:syserror.obj
 0002:000008e0       ??_C@_0BC@DFIBIBIL@already?5connected@ 1003d8e0     libcpmt:syserror.obj
 0002:000008f4       ??_C@_0BH@CAKOHOMI@argument?5list?5too?5long@ 1003d8f4     libcpmt:syserror.obj
 0002:0000090c       ??_C@_0BH@CGIMPKIM@argument?5out?5of?5domain@ 1003d90c     libcpmt:syserror.obj
 0002:00000924       ??_C@_0M@KGHGGJGL@bad?5address@ 1003d924     libcpmt:syserror.obj
 0002:00000930       ??_C@_0BE@MPJPGCEO@bad?5file?5descriptor@ 1003d930     libcpmt:syserror.obj
 0002:00000944       ??_C@_0M@PMMIEFCP@bad?5message@ 1003d944     libcpmt:syserror.obj
 0002:00000950       ??_C@_0M@KPHOFDBE@broken?5pipe@ 1003d950     libcpmt:syserror.obj
 0002:0000095c       ??_C@_0BD@MGNDDEGM@connection?5aborted@ 1003d95c     libcpmt:syserror.obj
 0002:00000970       ??_C@_0BP@KAIHPOGN@connection?5already?5in?5progress@ 1003d970     libcpmt:syserror.obj
 0002:00000990       ??_C@_0BD@PJLIIJEL@connection?5refused@ 1003d990     libcpmt:syserror.obj
 0002:000009a4       ??_C@_0BB@IECNJNOI@connection?5reset@ 1003d9a4     libcpmt:syserror.obj
 0002:000009b8       ??_C@_0BC@PPHBOELF@cross?5device?5link@ 1003d9b8     libcpmt:syserror.obj
 0002:000009cc       ??_C@_0BN@KDMIFEIP@destination?5address?5required@ 1003d9cc     libcpmt:syserror.obj
 0002:000009ec       ??_C@_0BI@NGCEHDD@device?5or?5resource?5busy@ 1003d9ec     libcpmt:syserror.obj
 0002:00000a04       ??_C@_0BE@JIDOCPHM@directory?5not?5empty@ 1003da04     libcpmt:syserror.obj
 0002:00000a18       ??_C@_0BI@BNCLIGPB@executable?5format?5error@ 1003da18     libcpmt:syserror.obj
 0002:00000a30       ??_C@_0M@MIDIAGJP@file?5exists@ 1003da30     libcpmt:syserror.obj
 0002:00000a3c       ??_C@_0P@DNAJLBJK@file?5too?5large@ 1003da3c     libcpmt:syserror.obj
 0002:00000a4c       ??_C@_0BC@EJHOMAAK@filename?5too?5long@ 1003da4c     libcpmt:syserror.obj
 0002:00000a60       ??_C@_0BH@KEFGLDAF@function?5not?5supported@ 1003da60     libcpmt:syserror.obj
 0002:00000a78       ??_C@_0BB@DHFDFGDM@host?5unreachable@ 1003da78     libcpmt:syserror.obj
 0002:00000a8c       ??_C@_0BD@JPHBMONG@identifier?5removed@ 1003da8c     libcpmt:syserror.obj
 0002:00000aa0       ??_C@_0BG@CDNPAGJK@illegal?5byte?5sequence@ 1003daa0     libcpmt:syserror.obj
 0002:00000ab8       ??_C@_0CD@BNPLBMNA@inappropriate?5io?5control?5operat@ 1003dab8     libcpmt:syserror.obj
 0002:00000adc       ??_C@_0M@EGEKIIMP@interrupted@ 1003dadc     libcpmt:syserror.obj
 0002:00000ae8       ??_C@_0BB@FCMFBGOM@invalid?5argument@ 1003dae8     libcpmt:syserror.obj
 0002:00000afc       ??_C@_0N@OHAFKDEK@invalid?5seek@ 1003dafc     libcpmt:syserror.obj
 0002:00000b0c       ??_C@_08GLNPIFBN@io?5error@ 1003db0c     libcpmt:syserror.obj
 0002:00000b18       ??_C@_0P@FLLDBIDK@is?5a?5directory@ 1003db18     libcpmt:syserror.obj
 0002:00000b28       ??_C@_0N@IFLPBIOP@message?5size@ 1003db28     libcpmt:syserror.obj
 0002:00000b38       ??_C@_0N@KIIEAAIO@network?5down@ 1003db38     libcpmt:syserror.obj
 0002:00000b48       ??_C@_0O@FNPDBHEE@network?5reset@ 1003db48     libcpmt:syserror.obj
 0002:00000b58       ??_C@_0BE@IFNCKGE@network?5unreachable@ 1003db58     libcpmt:syserror.obj
 0002:00000b6c       ??_C@_0BA@PFFCAOFK@no?5buffer?5space@ 1003db6c     libcpmt:syserror.obj
 0002:00000b7c       ??_C@_0BB@IEPBLJHK@no?5child?5process@ 1003db7c     libcpmt:syserror.obj
 0002:00000b90       ??_C@_07PLECNNKG@no?5link@ 1003db90     libcpmt:syserror.obj
 0002:00000b98       ??_C@_0BC@NJECKMKE@no?5lock?5available@ 1003db98     libcpmt:syserror.obj
 0002:00000bac       ??_C@_0BF@PBGGPKKE@no?5message?5available@ 1003dbac     libcpmt:syserror.obj
 0002:00000bc4       ??_C@_0L@EDOLMPAK@no?5message@ 1003dbc4     libcpmt:syserror.obj
 0002:00000bd0       ??_C@_0BD@EAMBFIDF@no?5protocol?5option@ 1003dbd0     libcpmt:syserror.obj
 0002:00000be4       ??_C@_0BD@IJDJKDEA@no?5space?5on?5device@ 1003dbe4     libcpmt:syserror.obj
 0002:00000bf8       ??_C@_0BE@MKFDAFMP@no?5stream?5resources@ 1003dbf8     libcpmt:syserror.obj
 0002:00000c0c       ??_C@_0BK@IMCPHCBI@no?5such?5device?5or?5address@ 1003dc0c     libcpmt:syserror.obj
 0002:00000c28       ??_C@_0P@FDINDDOK@no?5such?5device@ 1003dc28     libcpmt:syserror.obj
 0002:00000c38       ??_C@_0BK@NDOCBPGE@no?5such?5file?5or?5directory@ 1003dc38     libcpmt:syserror.obj
 0002:00000c54       ??_C@_0BA@ENLPPKBN@no?5such?5process@ 1003dc54     libcpmt:syserror.obj
 0002:00000c64       ??_C@_0BA@DOCPFFJG@not?5a?5directory@ 1003dc64     libcpmt:syserror.obj
 0002:00000c74       ??_C@_0N@POEIPGGF@not?5a?5socket@ 1003dc74     libcpmt:syserror.obj
 0002:00000c84       ??_C@_0N@LGAPMMPI@not?5a?5stream@ 1003dc84     libcpmt:syserror.obj
 0002:00000c94       ??_C@_0O@GLMIBBEG@not?5connected@ 1003dc94     libcpmt:syserror.obj
 0002:00000ca4       ??_C@_0BC@ENOOLCNF@not?5enough?5memory@ 1003dca4     libcpmt:syserror.obj
 0002:00000cb8       ??_C@_0O@NHEDABJP@not?5supported@ 1003dcb8     libcpmt:syserror.obj
 0002:00000cc8       ??_C@_0BD@MOLBPMEA@operation?5canceled@ 1003dcc8     libcpmt:syserror.obj
 0002:00000cdc       ??_C@_0BG@KDKHOPCO@operation?5in?5progress@ 1003dcdc     libcpmt:syserror.obj
 0002:00000cf4       ??_C@_0BI@OHIEJAAB@operation?5not?5permitted@ 1003dcf4     libcpmt:syserror.obj
 0002:00000d0c       ??_C@_0BI@LNEGIFLN@operation?5not?5supported@ 1003dd0c     libcpmt:syserror.obj
 0002:00000d24       ??_C@_0BG@OEMDKMEE@operation?5would?5block@ 1003dd24     libcpmt:syserror.obj
 0002:00000d3c       ??_C@_0L@BLPOFLNJ@owner?5dead@ 1003dd3c     libcpmt:syserror.obj
 0002:00000d48       ??_C@_0BC@CIJDGCDI@permission?5denied@ 1003dd48     libcpmt:syserror.obj
 0002:00000d5c       ??_C@_0P@FNPOCJBE@protocol?5error@ 1003dd5c     libcpmt:syserror.obj
 0002:00000d6c       ??_C@_0BH@JPPPLHJB@protocol?5not?5supported@ 1003dd6c     libcpmt:syserror.obj
 0002:00000d84       ??_C@_0BG@EICBIHDP@read?5only?5file?5system@ 1003dd84     libcpmt:syserror.obj
 0002:00000d9c       ??_C@_0BO@BJBOMOEJ@resource?5deadlock?5would?5occur@ 1003dd9c     libcpmt:syserror.obj
 0002:00000dbc       ??_C@_0BP@LKNGHENJ@resource?5unavailable?5try?5again@ 1003ddbc     libcpmt:syserror.obj
 0002:00000ddc       ??_C@_0BE@GOIPJJHG@result?5out?5of?5range@ 1003dddc     libcpmt:syserror.obj
 0002:00000df0       ??_C@_0BG@MPLKFPAE@state?5not?5recoverable@ 1003ddf0     libcpmt:syserror.obj
 0002:00000e08       ??_C@_0P@DIIFGFCG@stream?5timeout@ 1003de08     libcpmt:syserror.obj
 0002:00000e18       ??_C@_0P@IPFDMIFL@text?5file?5busy@ 1003de18     libcpmt:syserror.obj
 0002:00000e28       ??_C@_09KJPPMAOI@timed?5out@ 1003de28     libcpmt:syserror.obj
 0002:00000e34       ??_C@_0BO@HACHBEKI@too?5many?5files?5open?5in?5system@ 1003de34     libcpmt:syserror.obj
 0002:00000e54       ??_C@_0BE@GHAFMPAH@too?5many?5files?5open@ 1003de54     libcpmt:syserror.obj
 0002:00000e68       ??_C@_0P@HCOMKFCC@too?5many?5links@ 1003de68     libcpmt:syserror.obj
 0002:00000e78       ??_C@_0BO@EFGOJEF@too?5many?5symbolic?5link?5levels@ 1003de78     libcpmt:syserror.obj
 0002:00000e98       ??_C@_0BA@KGKGOOJA@value?5too?5large@ 1003de98     libcpmt:syserror.obj
 0002:00000ea8       ??_C@_0BE@MIEJDDNH@wrong?5protocol?5type@ 1003dea8     libcpmt:syserror.obj
 0002:00000ec0       ??_7bad_array_new_length@std@@6B@ 1003dec0     libcpmt:locale.obj
 0002:00000fcc       ??_7?$numpunct@_W@std@@6B@ 1003dfcc     libcpmt:wlocale.obj
 0002:00000fec       ??_C@_13IMODFHAA@?$AA?9@   1003dfec     libcpmt:wlocale.obj
 0002:00000ff0       ??_C@_01JOAMLHOP@?9@       1003dff0     libcpmt:wlocale.obj
 0002:00001098       ??_7type_info@@6B@         1003e098     LIBCMT:std_type_info_static.obj
 0002:000010a4       __pRawDllMain              1003e0a4     LIBCMT:dll_dllmain.obj
 0002:000010a4       __pDefaultRawDllMain       1003e0a4     LIBCMT:dll_dllmain.obj
 0002:000010a8       __pDestructExceptionObject 1003e0a8     libvcruntime:ehhelpers.obj
 0002:000010b0       ??_7bad_exception@std@@6B@ 1003e0b0     libvcruntime:frame.obj
 0002:000010b8       ??_C@_0O@DPKOEFFH@bad?5exception@ 1003e0b8     libvcruntime:frame.obj
 0002:00001448       ??_C@_08EHJDFFNH@__based?$CI@ 1003e448     libvcruntime:undname.obj
 0002:00001454       ??_C@_07KOLFKCDI@__cdecl@  1003e454     libvcruntime:undname.obj
 0002:0000145c       ??_C@_08GHMPAG@__pascal@   1003e45c     libvcruntime:undname.obj
 0002:00001468       ??_C@_09IFJBGAPI@__stdcall@ 1003e468     libvcruntime:undname.obj
 0002:00001474       ??_C@_0L@NPHFGOKO@__thiscall@ 1003e474     libvcruntime:undname.obj
 0002:00001480       ??_C@_0L@JMKHOMEK@__fastcall@ 1003e480     libvcruntime:undname.obj
 0002:0000148c       ??_C@_0N@BCKKPABJ@__vectorcall@ 1003e48c     libvcruntime:undname.obj
 0002:0000149c       ??_C@_09HIJEGCPM@__clrcall@ 1003e49c     libvcruntime:undname.obj
 0002:000014a8       ??_C@_06GHPCKEAG@__eabi@   1003e4a8     libvcruntime:undname.obj
 0002:000014b0       ??_C@_09IOPIDJLG@__swift_1@ 1003e4b0     libvcruntime:undname.obj
 0002:000014bc       ??_C@_09KFNFGKHF@__swift_2@ 1003e4bc     libvcruntime:undname.obj
 0002:000014c8       ??_C@_07JOMMBBKO@__ptr64@  1003e4c8     libvcruntime:undname.obj
 0002:000014d0       ??_C@_0L@PILCLIHE@__restrict@ 1003e4d0     libvcruntime:undname.obj
 0002:000014dc       ??_C@_0M@GFIIJFMG@__unaligned@ 1003e4dc     libvcruntime:undname.obj
 0002:000014e8       ??_C@_09DHDLOLLB@restrict?$CI@ 1003e4e8     libvcruntime:undname.obj
 0002:000014f4       ??_C@_04NIHEBCM@?5new@     1003e4f4     libvcruntime:undname.obj
 0002:000014fc       ??_C@_07FPCDHGMM@?5delete@ 1003e4fc     libvcruntime:undname.obj
 0002:00001504       ??_C@_01NEMOKFLO@?$DN@     1003e504     libvcruntime:undname.obj
 0002:00001508       ??_C@_02GPIOPFAK@?$DO?$DO@ 1003e508     libvcruntime:undname.obj
 0002:0000150c       ??_C@_02FODMEDOG@?$DM?$DM@ 1003e50c     libvcruntime:undname.obj
 0002:00001510       ??_C@_01DCLJPIOD@?$CB@     1003e510     libvcruntime:undname.obj
 0002:00001514       ??_C@_02EGOFBIJA@?$DN?$DN@ 1003e514     libvcruntime:undname.obj
 0002:00001518       ??_C@_02FDNJECIE@?$CB?$DN@ 1003e518     libvcruntime:undname.obj
 0002:0000151c       ??_C@_02GPECMEKF@?$FL?$FN@ 1003e51c     libvcruntime:undname.obj
 0002:00001520       ??_C@_08LHJFAFGD@operator@ 1003e520     libvcruntime:undname.obj
 0002:0000152c       ??_C@_02HBOOOICD@?9?$DO@   1003e52c     libvcruntime:undname.obj
 0002:00001530       ??_C@_02ECNGHCIF@?$CL?$CL@ 1003e530     libvcruntime:undname.obj
 0002:00001534       ??_C@_02BAABKJLB@?9?9@     1003e534     libvcruntime:undname.obj
 0002:00001538       ??_C@_01MIFGBAGJ@?$CL@     1003e538     libvcruntime:undname.obj
 0002:0000153c       ??_C@_01HNPIGOCE@?$CG@     1003e53c     libvcruntime:undname.obj
 0002:00001540       ??_C@_03MNHNFDLC@?9?$DO?$CK@ 1003e540     libvcruntime:undname.obj
 0002:00001544       ??_C@_01KMDKNFGN@?1@       1003e544     libvcruntime:undname.obj
 0002:00001548       ??_C@_01FGNFDNOH@?$CF@     1003e548     libvcruntime:undname.obj
 0002:0000154c       ??_C@_01MNNFJEPP@?$DM@     1003e54c     libvcruntime:undname.obj
 0002:00001550       ??_C@_02EHCHHCKH@?$DM?$DN@ 1003e550     libvcruntime:undname.obj
 0002:00001554       ??_C@_01PPODPGHN@?$DO@     1003e554     libvcruntime:undname.obj
 0002:00001558       ??_C@_02EEKDKGMJ@?$DO?$DN@ 1003e558     libvcruntime:undname.obj
 0002:0000155c       ??_C@_01IHBHIGKO@?0@       1003e55c     libvcruntime:undname.obj
 0002:00001560       ??_C@_02HCKGKOFO@?$CI?$CJ@ 1003e560     libvcruntime:undname.obj
 0002:00001564       ??_C@_01PJKLJHI@?$HO@      1003e564     libvcruntime:undname.obj
 0002:00001568       ??_C@_01JKBOJNNK@?$FO@     1003e568     libvcruntime:undname.obj
 0002:0000156c       ??_C@_01DNKMNLPK@?$HM@     1003e56c     libvcruntime:undname.obj
 0002:00001570       ??_C@_02PPKAJPJL@?$CG?$CG@ 1003e570     libvcruntime:undname.obj
 0002:00001574       ??_C@_02NONPIBCD@?$HM?$HM@ 1003e574     libvcruntime:undname.obj
 0002:00001578       ??_C@_02FPIMKNGF@?$CK?$DN@ 1003e578     libvcruntime:undname.obj
 0002:0000157c       ??_C@_02FOEOMHFC@?$CL?$DN@ 1003e57c     libvcruntime:undname.obj
 0002:00001580       ??_C@_02FKMDLLOA@?9?$DN@   1003e580     libvcruntime:undname.obj
 0002:00001584       ??_C@_02FJEHGPIO@?1?$DN@   1003e584     libvcruntime:undname.obj
 0002:00001588       ??_C@_02FENAOKFI@?$CF?$DN@ 1003e588     libvcruntime:undname.obj
 0002:0000158c       ??_C@_03IKFCCPFF@?$DO?$DO?$DN@ 1003e58c     libvcruntime:undname.obj
 0002:00001590       ??_C@_03CDNPDDLA@?$DM?$DM?$DN@ 1003e590     libvcruntime:undname.obj
 0002:00001594       ??_C@_02FGJGFEAB@?$CG?$DN@ 1003e594     libvcruntime:undname.obj
 0002:00001598       ??_C@_02DHLNPPGH@?$HM?$DN@ 1003e598     libvcruntime:undname.obj
 0002:0000159c       ??_C@_02MHEGNOJ@?$FO?$DN@  1003e59c     libvcruntime:undname.obj
 0002:000015a0       ??_C@_09IFPLHPGF@?$GAvftable?8@ 1003e5a0     libvcruntime:undname.obj
 0002:000015ac       ??_C@_09BLBHBJP@?$GAvbtable?8@ 1003e5ac     libvcruntime:undname.obj
 0002:000015b8       ??_C@_07FEEIOKP@?$GAvcall?8@ 1003e5b8     libvcruntime:undname.obj
 0002:000015c0       ??_C@_08LLFFHHDJ@?$GAtypeof?8@ 1003e5c0     libvcruntime:undname.obj
 0002:000015cc       ??_C@_0BF@KDPPACIK@?$GAlocal?5static?5guard?8@ 1003e5cc     libvcruntime:undname.obj
 0002:000015e4       ??_C@_08OBABFOLI@?$GAstring?8@ 1003e5e4     libvcruntime:undname.obj
 0002:000015f0       ??_C@_0BD@JDLKDPAB@?$GAvbase?5destructor?8@ 1003e5f0     libvcruntime:undname.obj
 0002:00001604       ??_C@_0BN@DEGPLNFK@?$GAvector?5deleting?5destructor?8@ 1003e604     libvcruntime:undname.obj
 0002:00001624       ??_C@_0BO@OBMKPJIG@?$GAdefault?5constructor?5closure?8@ 1003e624     libvcruntime:undname.obj
 0002:00001644       ??_C@_0BN@IMDCHIKM@?$GAscalar?5deleting?5destructor?8@ 1003e644     libvcruntime:undname.obj
 0002:00001664       ??_C@_0BO@PFGOCPJJ@?$GAvector?5constructor?5iterator?8@ 1003e664     libvcruntime:undname.obj
 0002:00001684       ??_C@_0BN@LFPFMEDL@?$GAvector?5destructor?5iterator?8@ 1003e684     libvcruntime:undname.obj
 0002:000016a4       ??_C@_0CE@IKBNEHA@?$GAvector?5vbase?5constructor?5itera@ 1003e6a4     libvcruntime:undname.obj
 0002:000016c8       ??_C@_0BL@NILFHHPC@?$GAvirtual?5displacement?5map?8@ 1003e6c8     libvcruntime:undname.obj
 0002:000016e4       ??_C@_0CB@JONCMFFK@?$GAeh?5vector?5constructor?5iterator@ 1003e6e4     libvcruntime:undname.obj
 0002:00001708       ??_C@_0CA@GCEOPDGL@?$GAeh?5vector?5destructor?5iterator?8@ 1003e708     libvcruntime:undname.obj
 0002:00001728       ??_C@_0CH@OOJPLCPH@?$GAeh?5vector?5vbase?5constructor?5it@ 1003e728     libvcruntime:undname.obj
 0002:00001750       ??_C@_0BL@LLKPOHJI@?$GAcopy?5constructor?5closure?8@ 1003e750     libvcruntime:undname.obj
 0002:0000176c       ??_C@_0BA@KBCDOMBN@?$GAudt?5returning?8@ 1003e76c     libvcruntime:undname.obj
 0002:0000177c       ??_C@_03KLGMFNMG@?$GAEH@   1003e77c     libvcruntime:undname.obj
 0002:00001780       ??_C@_05KHLCHHI@?$GARTTI@  1003e780     libvcruntime:undname.obj
 0002:00001788       ??_C@_0BA@KKLDJDLB@?$GAlocal?5vftable?8@ 1003e788     libvcruntime:undname.obj
 0002:00001798       ??_C@_0CE@IIHCMGGL@?$GAlocal?5vftable?5constructor?5clos@ 1003e798     libvcruntime:undname.obj
 0002:000017bc       ??_C@_06FHBGPFGH@?5new?$FL?$FN@ 1003e7bc     libvcruntime:undname.obj
 0002:000017c4       ??_C@_09LBNFPBCA@?5delete?$FL?$FN@ 1003e7c4     libvcruntime:undname.obj
 0002:000017d0       ??_C@_0P@HJKNJFNN@?$GAomni?5callsig?8@ 1003e7d0     libvcruntime:undname.obj
 0002:000017e0       ??_C@_0BL@CNOONJFP@?$GAplacement?5delete?5closure?8@ 1003e7e0     libvcruntime:undname.obj
 0002:000017fc       ??_C@_0BN@CKNJLHMB@?$GAplacement?5delete?$FL?$FN?5closure?8@ 1003e7fc     libvcruntime:undname.obj
 0002:0000181c       ??_C@_0CG@CFDHKGGD@?$GAmanaged?5vector?5constructor?5ite@ 1003e81c     libvcruntime:undname.obj
 0002:00001844       ??_C@_0CF@IMGKMJNO@?$GAmanaged?5vector?5destructor?5iter@ 1003e844     libvcruntime:undname.obj
 0002:0000186c       ??_C@_0CG@HLDDJMAG@?$GAeh?5vector?5copy?5constructor?5ite@ 1003e86c     libvcruntime:undname.obj
 0002:00001894       ??_C@_0CM@FCBBDIGB@?$GAeh?5vector?5vbase?5copy?5construct@ 1003e894     libvcruntime:undname.obj
 0002:000018c0       ??_C@_0BL@CLIPGLGB@?$GAdynamic?5initializer?5for?5?8@ 1003e8c0     libvcruntime:undname.obj
 0002:000018dc       ??_C@_0CB@PDBIFEP@?$GAdynamic?5atexit?5destructor?5for?5@ 1003e8dc     libvcruntime:undname.obj
 0002:00001900       ??_C@_0CD@CGAJBKEJ@?$GAvector?5copy?5constructor?5iterat@ 1003e900     libvcruntime:undname.obj
 0002:00001924       ??_C@_0CJ@GJELGAMM@?$GAvector?5vbase?5copy?5constructor?5@ 1003e924     libvcruntime:undname.obj
 0002:00001950       ??_C@_0CL@FGIJHLCE@?$GAmanaged?5vector?5copy?5constructo@ 1003e950     libvcruntime:undname.obj
 0002:0000197c       ??_C@_0BM@PMGGMLDN@?$GAlocal?5static?5thread?5guard?8@ 1003e97c     libvcruntime:undname.obj
 0002:00001998       ??_C@_0N@BDNMDMOL@operator?5?$CC?$CC?5@ 1003e998     libvcruntime:undname.obj
 0002:000019a8       ??_C@_0BC@GGEBGALA@operator?5co_await@ 1003e9a8     libvcruntime:undname.obj
 0002:000019bc       ??_C@_0M@GAAIMMOH@operator?$DM?$DN?$DO@ 1003e9bc     libvcruntime:undname.obj
 0002:000019c8       ??_C@_0BC@DAFEJGAK@?5Type?5Descriptor?8@ 1003e9c8     libvcruntime:undname.obj
 0002:000019dc       ??_C@_0BM@LDKODKLH@?5Base?5Class?5Descriptor?5at?5?$CI@ 1003e9dc     libvcruntime:undname.obj
 0002:000019f8       ??_C@_0BD@LGICGFMM@?5Base?5Class?5Array?8@ 1003e9f8     libvcruntime:undname.obj
 0002:00001a0c       ??_C@_0BN@MECKDCOJ@?5Class?5Hierarchy?5Descriptor?8@ 1003ea0c     libvcruntime:undname.obj
 0002:00001a2c       ??_C@_0BK@CFCOFLF@?5Complete?5Object?5Locator?8@ 1003ea2c     libvcruntime:undname.obj
 0002:00001a48       ??_C@_0BG@JNJLAMPM@?$GAanonymous?5namespace?8@ 1003ea48     libvcruntime:undname.obj
 0002:00001a6c       ??_C@_1DM@KHCHBNEB@?$AAa?$AAp?$AAi?$AA?9?$AAm?$AAs?$AA?9?$AAw?$AAi?$AAn?$AA?9?$AAc?$AAo?$AAr?$AAe@ 1003ea6c     libvcruntime:winapi_downlevel.obj
 0002:00001aa8       ??_C@_1DK@LPPGFMPP@?$AAa?$AAp?$AAi?$AA?9?$AAm?$AAs?$AA?9?$AAw?$AAi?$AAn?$AA?9?$AAc?$AAo?$AAr?$AAe@ 1003eaa8     libvcruntime:winapi_downlevel.obj
 0002:00001ae4       ??_C@_1BA@PFFKHIOG@?$AAa?$AAp?$AAi?$AA?9?$AAm?$AAs?$AA?9@ 1003eae4     libvcruntime:winapi_downlevel.obj
 0002:00001afc       ??_C@_08KNHFBNJ@FlsAlloc@  1003eafc     libvcruntime:winapi_downlevel.obj
 0002:00001b10       ??_C@_07PEJMOBNF@FlsFree@  1003eb10     libvcruntime:winapi_downlevel.obj
 0002:00001b20       ??_C@_0M@GDNOONDI@FlsGetValue@ 1003eb20     libvcruntime:winapi_downlevel.obj
 0002:00001b34       ??_C@_0M@JCPCPOEF@FlsSetValue@ 1003eb34     libvcruntime:winapi_downlevel.obj
 0002:00001cf0       __real@3e54ae0bf85ddf44    1003ecf0     libucrt:log2d.obj
 0002:00001cf8       __real@3e5526e50e32a6ab    1003ecf8     libucrt:log2d.obj
 0002:00001d00       __real@3e7427de7fbcc47c    1003ed00     libucrt:log2d.obj
 0002:00001d08       __real@3e7f7d1cf79abc9e    1003ed08     libucrt:log2d.obj
 0002:00001d10       __real@3fc2f8d8bf29def7    1003ed10     libucrt:log2d.obj
 0002:00001d18       __real@3fc3991accfeb3f4    1003ed18     libucrt:log2d.obj
 0002:00001d20       __real@3fc7466fd968cb62    1003ed20     libucrt:log2d.obj
 0002:00001d28       __real@3fcc71c4da12c9c6    1003ed28     libucrt:log2d.obj
 0002:00001d30       __real@3fd24924948ae94a    1003ed30     libucrt:log2d.obj
 0002:00001d38       __real@3fd3441300000000    1003ed38     libucrt:log2d.obj
 0002:00001d40       __real@3fd9999999975ff7    1003ed40     libucrt:log2d.obj
 0002:00001d48       __real@3fdbcb7b00000000    1003ed48     libucrt:log2d.obj
 0002:00001d50       __real@3fdbcb7b1526e50e    1003ed50     libucrt:log2d.obj
 0002:00001d58       __real@3fe55555555555bc    1003ed58     libucrt:log2d.obj
 0002:00001d60       __real@3fe62e42c0000000    1003ed60     libucrt:log2d.obj
 0002:00001d68       __real@3fe6a09e667f3bcd    1003ed68     libucrt:log2d.obj
 0002:00001d70       __real@3ff0000000000000    1003ed70     libucrt:log2d.obj
 0002:00001d78       __real@3ff7154760000000    1003ed78     libucrt:log2d.obj
 0002:00001d80       __real@3ff71547652b82fe    1003ed80     libucrt:log2d.obj
 0002:00001d88       ___newctype                1003ed88     libucrt:ctype.obj
 0002:00002088       ___newclmap                1003f088     libucrt:ctype.obj
 0002:00002208       ___newcumap                1003f208     libucrt:ctype.obj
 0002:00002388       __wctype                   1003f388     libucrt:ctype.obj
 0002:00002594       __half                     1003f594     libucrt:pow_impl.obj
 0002:000025a0       ___acrt_exception_action_table 1003f5a0     libucrt:exception_filter.obj
 0002:00002630       ___acrt_signal_action_table_count 1003f630     libucrt:exception_filter.obj
 0002:00002634       ___acrt_signal_action_first_fpe_index 1003f634     libucrt:exception_filter.obj
 0002:00002638       ___acrt_signal_action_fpe_count 1003f638     libucrt:exception_filter.obj
 0002:0000263c       ??_C@_1BI@BGOHAHKC@?$AAm?$AAs?$AAc?$AAo?$AAr?$AAe?$AAe?$AA?4?$AAd?$AAl?$AAl@ 1003f63c     libucrt:exit.obj
 0002:00002654       ??_C@_0P@MIGLKIOC@CorExitProcess@ 1003f654     libucrt:exit.obj
 0002:00002738       ??_C@_1EA@JGEFHKEI@?$AAa?$AAp?$AAi?$AA?9?$AAm?$AAs?$AA?9?$AAw?$AAi?$AAn?$AA?9?$AAc?$AAo?$AAr?$AAe@ 1003f738     libucrt:winapi_thunks.obj
 0002:00002778       ??_C@_1DI@IJCEHOCB@?$AAa?$AAp?$AAi?$AA?9?$AAm?$AAs?$AA?9?$AAw?$AAi?$AAn?$AA?9?$AAc?$AAo?$AAr?$AAe@ 1003f778     libucrt:winapi_thunks.obj
 0002:000027b0       ??_C@_1EI@MPIAOHOC@?$AAa?$AAp?$AAi?$AA?9?$AAm?$AAs?$AA?9?$AAw?$AAi?$AAn?$AA?9?$AAc?$AAo?$AAr?$AAe@ 1003f7b0     libucrt:winapi_thunks.obj
 0002:000027f8       ??_C@_1FK@FPHCKFIE@?$AAa?$AAp?$AAi?$AA?9?$AAm?$AAs?$AA?9?$AAw?$AAi?$AAn?$AA?9?$AAc?$AAo?$AAr?$AAe@ 1003f7f8     libucrt:winapi_thunks.obj
 0002:00002858       ??_C@_1EM@DILCGIIO@?$AAa?$AAp?$AAi?$AA?9?$AAm?$AAs?$AA?9?$AAw?$AAi?$AAn?$AA?9?$AAc?$AAo?$AAr?$AAe@ 1003f858     libucrt:winapi_thunks.obj
 0002:000028a4       ??_C@_1DM@LNCGDDPN@?$AAa?$AAp?$AAi?$AA?9?$AAm?$AAs?$AA?9?$AAw?$AAi?$AAn?$AA?9?$AAc?$AAo?$AAr?$AAe@ 1003f8a4     libucrt:winapi_thunks.obj
 0002:000028e0       ??_C@_1DO@FPAPJEMD@?$AAa?$AAp?$AAi?$AA?9?$AAm?$AAs?$AA?9?$AAw?$AAi?$AAn?$AA?9?$AAc?$AAo?$AAr?$AAe@ 1003f8e0     libucrt:winapi_thunks.obj
 0002:00002920       ??_C@_1DK@NDHNAHIO@?$AAa?$AAp?$AAi?$AA?9?$AAm?$AAs?$AA?9?$AAw?$AAi?$AAn?$AA?9?$AAc?$AAo?$AAr?$AAe@ 1003f920     libucrt:winapi_thunks.obj
 0002:0000295c       ??_C@_1DM@KGHDGBCM@?$AAa?$AAp?$AAi?$AA?9?$AAm?$AAs?$AA?9?$AAw?$AAi?$AAn?$AA?9?$AAc?$AAo?$AAr?$AAe@ 1003f95c     libucrt:winapi_thunks.obj
 0002:00002998       ??_C@_1EO@IJIOEFOH@?$AAa?$AAp?$AAi?$AA?9?$AAm?$AAs?$AA?9?$AAw?$AAi?$AAn?$AA?9?$AAr?$AAt?$AAc?$AAo@ 1003f998     libucrt:winapi_thunks.obj
 0002:000029e8       ??_C@_1FG@HHGEKANL@?$AAa?$AAp?$AAi?$AA?9?$AAm?$AAs?$AA?9?$AAw?$AAi?$AAn?$AA?9?$AAs?$AAe?$AAc?$AAu@ 1003f9e8     libucrt:winapi_thunks.obj
 0002:00002a40       ??_C@_1EG@DBIOJECG@?$AAe?$AAx?$AAt?$AA?9?$AAm?$AAs?$AA?9?$AAw?$AAi?$AAn?$AA?9?$AAn?$AAt?$AAu?$AAs@ 1003fa40     libucrt:winapi_thunks.obj
 0002:00002a88       ??_C@_1EO@FIHMJCLF@?$AAe?$AAx?$AAt?$AA?9?$AAm?$AAs?$AA?9?$AAw?$AAi?$AAn?$AA?9?$AAn?$AAt?$AAu?$AAs@ 1003fa88     libucrt:winapi_thunks.obj
 0002:00002ad8       ??_C@_1EG@DPGNFKGC@?$AAa?$AAp?$AAi?$AA?9?$AAm?$AAs?$AA?9?$AAw?$AAi?$AAn?$AA?9?$AAa?$AAp?$AAp?$AAm@ 1003fad8     libucrt:winapi_thunks.obj
 0002:00002b20       ??_C@_1BA@IAIFMGEF@?$AAe?$AAx?$AAt?$AA?9?$AAm?$AAs?$AA?9@ 1003fb20     libucrt:winapi_thunks.obj
 0002:00002b34       ??_C@_0BA@FHFNEAED@AreFileApisANSI@ 1003fb34     libucrt:winapi_thunks.obj
 0002:00002b54       ??_C@_0BE@LJANKFHF@EnumSystemLocalesEx@ 1003fb54     libucrt:winapi_thunks.obj
 0002:00002b90       ??_C@_0BA@EPCJIIPD@GetDateFormatEx@ 1003fb90     libucrt:winapi_thunks.obj
 0002:00002ba8       ??_C@_0BA@ONOKGCMP@GetLocaleInfoEx@ 1003fba8     libucrt:winapi_thunks.obj
 0002:00002bc0       ??_C@_0BA@CIJJKCJJ@GetTimeFormatEx@ 1003fbc0     libucrt:winapi_thunks.obj
 0002:00002bd8       ??_C@_0BJ@PBCCBIPI@GetUserDefaultLocaleName@ 1003fbd8     libucrt:winapi_thunks.obj
 0002:00002c04       ??_C@_0BC@CELBKLLA@IsValidLocaleName@ 1003fc04     libucrt:winapi_thunks.obj
 0002:00002c20       ??_C@_0O@KKBNKAPF@LCMapStringEx@ 1003fc20     libucrt:winapi_thunks.obj
 0002:00002c38       ??_C@_0BB@CDHDDLLP@LCIDToLocaleName@ 1003fc38     libucrt:winapi_thunks.obj
 0002:00002c54       ??_C@_0BB@HBDEELFH@LocaleNameToLCID@ 1003fc54     libucrt:winapi_thunks.obj
 0002:00002c6c       ??_C@_0CF@OJOFEIGO@AppPolicyGetProcessTerminationM@ 1003fc6c     libucrt:winapi_thunks.obj
 0002:00002cc8       __Inf_C                    1003fcc8     libucrt:_values.obj
 0002:00002cd0       __Nan_C                    1003fcd0     libucrt:_values.obj
 0002:00002d58       ___lc_category             1003fd58     libucrt:wsetlocale.obj
 0002:00002da0       ??_C@_1O@GIFLHMA@?$AAL?$AAC?$AA_?$AAA?$AAL?$AAL@ 1003fda0     libucrt:wsetlocale.obj
 0002:00002db0       ??_C@_1BG@PPOMIBNJ@?$AAL?$AAC?$AA_?$AAC?$AAO?$AAL?$AAL?$AAA?$AAT?$AAE@ 1003fdb0     libucrt:wsetlocale.obj
 0002:00002dc8       ??_C@_1BC@FFJGAPJM@?$AAL?$AAC?$AA_?$AAC?$AAT?$AAY?$AAP?$AAE@ 1003fdc8     libucrt:wsetlocale.obj
 0002:00002ddc       ??_C@_1BI@PCKFNJFB@?$AAL?$AAC?$AA_?$AAM?$AAO?$AAN?$AAE?$AAT?$AAA?$AAR?$AAY@ 1003fddc     libucrt:wsetlocale.obj
 0002:00002df4       ??_C@_1BG@ENIEDKID@?$AAL?$AAC?$AA_?$AAN?$AAU?$AAM?$AAE?$AAR?$AAI?$AAC@ 1003fdf4     libucrt:wsetlocale.obj
 0002:00002e0c       ??_C@_1BA@HAAOMIIG@?$AAL?$AAC?$AA_?$AAT?$AAI?$AAM?$AAE@ 1003fe0c     libucrt:wsetlocale.obj
 0002:00002e1c       ??_C@_15NBPDDFIP@?$AA?$DN?$AA?$DL@ 1003fe1c     libucrt:wsetlocale.obj
 0002:00002e24       ??_C@_13PJJBFPED@?$AA?$DL@ 1003fe24     libucrt:wsetlocale.obj
 0002:00002e28       ??_C@_13NMPKAAJP@?$AA?$DN@ 1003fe28     libucrt:wsetlocale.obj
 0002:00002e2c       ??_C@_17EFJLDFDO@?$AA?9?$AA_?$AA?4@ 1003fe2c     libucrt:wsetlocale.obj
 0002:00002e34       ??_C@_13FHBKNHDA@?$AAC@    1003fe34     libucrt:wsetlocale.obj
 0002:00002e38       ??_C@_17MBJJLFDM@?$AA_?$AA?4?$AA?0@ 1003fe38     libucrt:wsetlocale.obj
 0002:00002e40       ??_C@_13ENNFDPBH@?$AA_@    1003fe40     libucrt:wsetlocale.obj
 0002:00002e48       ___lc_time_c               1003fe48     libucrt:nlsdata.obj
 0002:00002fac       ??_C@_03KOEHGMDN@Sun@      1003ffac     libucrt:nlsdata.obj
 0002:00002fb0       ??_C@_03PDAGKDH@Mon@       1003ffb0     libucrt:nlsdata.obj
 0002:00002fb4       ??_C@_03NAGEINEP@Tue@      1003ffb4     libucrt:nlsdata.obj
 0002:00002fb8       ??_C@_03MHOMLAJA@Wed@      1003ffb8     libucrt:nlsdata.obj
 0002:00002fbc       ??_C@_03IOFIKPDN@Thu@      1003ffbc     libucrt:nlsdata.obj
 0002:00002fc0       ??_C@_03IDIOELNC@Fri@      1003ffc0     libucrt:nlsdata.obj
 0002:00002fc4       ??_C@_03FEFJNEK@Sat@       1003ffc4     libucrt:nlsdata.obj
 0002:00002fc8       ??_C@_06OOPIFAJ@Sunday@    1003ffc8     libucrt:nlsdata.obj
 0002:00002fd0       ??_C@_06JLEDEDGH@Monday@   1003ffd0     libucrt:nlsdata.obj
 0002:00002fd8       ??_C@_07BAAGCFCM@Tuesday@  1003ffd8     libucrt:nlsdata.obj
 0002:00002fe0       ??_C@_09DLIGFAKA@Wednesday@ 1003ffe0     libucrt:nlsdata.obj
 0002:00002fec       ??_C@_08HACCIKIA@Thursday@ 1003ffec     libucrt:nlsdata.obj
 0002:00002ff8       ??_C@_06JECMNKMI@Friday@   1003fff8     libucrt:nlsdata.obj
 0002:00003000       ??_C@_08INBOOONO@Saturday@ 10040000     libucrt:nlsdata.obj
 0002:0000300c       ??_C@_03JIHJHPIE@Jan@      1004000c     libucrt:nlsdata.obj
 0002:00003010       ??_C@_03HJBDCHOM@Feb@      10040010     libucrt:nlsdata.obj
 0002:00003014       ??_C@_03ODNJBKGA@Mar@      10040014     libucrt:nlsdata.obj
 0002:00003018       ??_C@_03LEOLGMJP@Apr@      10040018     libucrt:nlsdata.obj
 0002:0000301c       ??_C@_03CNMDKL@May@        1004001c     libucrt:nlsdata.obj
 0002:00003020       ??_C@_03IDFGHECI@Jun@      10040020     libucrt:nlsdata.obj
 0002:00003024       ??_C@_03LBGABGKK@Jul@      10040024     libucrt:nlsdata.obj
 0002:00003028       ??_C@_03IFJFEIGA@Aug@      10040028     libucrt:nlsdata.obj
 0002:0000302c       ??_C@_03GGCAPAJC@Sep@      1004002c     libucrt:nlsdata.obj
 0002:00003030       ??_C@_03BMAOKBAD@Oct@      10040030     libucrt:nlsdata.obj
 0002:00003034       ??_C@_03JPJOFNIA@Nov@      10040034     libucrt:nlsdata.obj
 0002:00003038       ??_C@_03MKABNOCG@Dec@      10040038     libucrt:nlsdata.obj
 0002:0000303c       ??_C@_07CGJPFGJA@January@  1004003c     libucrt:nlsdata.obj
 0002:00003044       ??_C@_08GNJGEPFN@February@ 10040044     libucrt:nlsdata.obj
 0002:00003050       ??_C@_05HPCKOFNC@March@    10040050     libucrt:nlsdata.obj
 0002:00003058       ??_C@_05DMJDNLEJ@April@    10040058     libucrt:nlsdata.obj
 0002:00003060       ??_C@_04CNLMGBGM@June@     10040060     libucrt:nlsdata.obj
 0002:00003068       ??_C@_04MIEPOIFP@July@     10040068     libucrt:nlsdata.obj
 0002:00003070       ??_C@_06LBBHFDDG@August@   10040070     libucrt:nlsdata.obj
 0002:00003078       ??_C@_09BHHEALKD@September@ 10040078     libucrt:nlsdata.obj
 0002:00003084       ??_C@_07JJNFCEND@October@  10040084     libucrt:nlsdata.obj
 0002:0000308c       ??_C@_08HCHEGEOA@November@ 1004008c     libucrt:nlsdata.obj
 0002:00003098       ??_C@_08EDHMEBNP@December@ 10040098     libucrt:nlsdata.obj
 0002:000030a4       ??_C@_02DEDBPAFC@AM@       100400a4     libucrt:nlsdata.obj
 0002:000030a8       ??_C@_02CJNFDJBF@PM@       100400a8     libucrt:nlsdata.obj
 0002:000030ac       ??_C@_08BPBNCDIB@MM?1dd?1yy@ 100400ac     libucrt:nlsdata.obj
 0002:000030b8       ??_C@_0BE@CKGJFCPC@dddd?0?5MMMM?5dd?0?5yyyy@ 100400b8     libucrt:nlsdata.obj
 0002:000030cc       ??_C@_08JCCMCCIL@HH?3mm?3ss@ 100400cc     libucrt:nlsdata.obj
 0002:000030d8       ??_C@_17MBGCMIPB@?$AAS?$AAu?$AAn@ 100400d8     libucrt:nlsdata.obj
 0002:000030e0       ??_C@_17KBOMKBF@?$AAM?$AAo?$AAn@ 100400e0     libucrt:nlsdata.obj
 0002:000030e8       ??_C@_17BMKGEGOJ@?$AAT?$AAu?$AAe@ 100400e8     libucrt:nlsdata.obj
 0002:000030f0       ??_C@_17CJEDCEPE@?$AAW?$AAe?$AAd@ 100400f0     libucrt:nlsdata.obj
 0002:000030f8       ??_C@_17PDPHAADD@?$AAT?$AAh?$AAu@ 100400f8     libucrt:nlsdata.obj
 0002:00003100       ??_C@_17HFOLPPLP@?$AAF?$AAr?$AAi@ 10040100     libucrt:nlsdata.obj
 0002:00003108       ??_C@_17GGIBDPIH@?$AAS?$AAa?$AAt@ 10040108     libucrt:nlsdata.obj
 0002:00003110       ??_C@_1O@IHNHDHPB@?$AAS?$AAu?$AAn?$AAd?$AAa?$AAy@ 10040110     libucrt:nlsdata.obj
 0002:00003120       ??_C@_1O@MMNBFLIA@?$AAM?$AAo?$AAn?$AAd?$AAa?$AAy@ 10040120     libucrt:nlsdata.obj
 0002:00003130       ??_C@_1BA@ENFBFFEK@?$AAT?$AAu?$AAe?$AAs?$AAd?$AAa?$AAy@ 10040130     libucrt:nlsdata.obj
 0002:00003140       ??_C@_1BE@EBOGMDOH@?$AAW?$AAe?$AAd?$AAn?$AAe?$AAs?$AAd?$AAa?$AAy@ 10040140     libucrt:nlsdata.obj
 0002:00003154       ??_C@_1BC@HHMNLIHE@?$AAT?$AAh?$AAu?$AAr?$AAs?$AAd?$AAa?$AAy@ 10040154     libucrt:nlsdata.obj
 0002:00003168       ??_C@_1O@PDICJHAG@?$AAF?$AAr?$AAi?$AAd?$AAa?$AAy@ 10040168     libucrt:nlsdata.obj
 0002:00003178       ??_C@_1BC@ENMNNPAJ@?$AAS?$AAa?$AAt?$AAu?$AAr?$AAd?$AAa?$AAy@ 10040178     libucrt:nlsdata.obj
 0002:0000318c       ??_C@_17DKNBKCHM@?$AAJ?$AAa?$AAn@ 1004018c     libucrt:nlsdata.obj
 0002:00003194       ??_C@_17LMDJEKJN@?$AAF?$AAe?$AAb@ 10040194     libucrt:nlsdata.obj
 0002:0000319c       ??_C@_17CKNLEDEC@?$AAM?$AAa?$AAr@ 1004019c     libucrt:nlsdata.obj
 0002:000031a4       ??_C@_17LFPOIHDD@?$AAA?$AAp?$AAr@ 100401a4     libucrt:nlsdata.obj
 0002:000031ac       ??_C@_17PNNKMEED@?$AAM?$AAa?$AAy@ 100401ac     libucrt:nlsdata.obj
 0002:000031b4       ??_C@_17KCJGOCPB@?$AAJ?$AAu?$AAn@ 100401b4     libucrt:nlsdata.obj
 0002:000031bc       ??_C@_17IJPCKHK@?$AAJ?$AAu?$AAl@ 100401bc     libucrt:nlsdata.obj
 0002:000031c4       ??_C@_17ICPELBCN@?$AAA?$AAu?$AAg@ 100401c4     libucrt:nlsdata.obj
 0002:000031cc       ??_C@_17HCHCOKMG@?$AAS?$AAe?$AAp@ 100401cc     libucrt:nlsdata.obj
 0002:000031d4       ??_C@_17FNLKOI@?$AAO?$AAc?$AAt@ 100401d4     libucrt:nlsdata.obj
 0002:000031dc       ??_C@_17BBDMLCIG@?$AAN?$AAo?$AAv@ 100401dc     libucrt:nlsdata.obj
 0002:000031e4       ??_C@_17EGKACKIF@?$AAD?$AAe?$AAc@ 100401e4     libucrt:nlsdata.obj
 0002:000031ec       ??_C@_1BA@EFMEIEBA@?$AAJ?$AAa?$AAn?$AAu?$AAa?$AAr?$AAy@ 100401ec     libucrt:nlsdata.obj
 0002:000031fc       ??_C@_1BC@JGDDFFAM@?$AAF?$AAe?$AAb?$AAr?$AAu?$AAa?$AAr?$AAy@ 100401fc     libucrt:nlsdata.obj
 0002:00003210       ??_C@_1M@IKEENEDF@?$AAM?$AAa?$AAr?$AAc?$AAh@ 10040210     libucrt:nlsdata.obj
 0002:0000321c       ??_C@_1M@GJNLMHFD@?$AAA?$AAp?$AAr?$AAi?$AAl@ 1004021c     libucrt:nlsdata.obj
 0002:00003228       ??_C@_19EPFLPGAP@?$AAJ?$AAu?$AAn?$AAe@ 10040228     libucrt:nlsdata.obj
 0002:00003234       ??_C@_19BIFMLPCD@?$AAJ?$AAu?$AAl?$AAy@ 10040234     libucrt:nlsdata.obj
 0002:00003240       ??_C@_1O@PAHLKOAC@?$AAA?$AAu?$AAg?$AAu?$AAs?$AAt@ 10040240     libucrt:nlsdata.obj
 0002:00003250       ??_C@_1BE@DKAAMBJL@?$AAS?$AAe?$AAp?$AAt?$AAe?$AAm?$AAb?$AAe?$AAr@ 10040250     libucrt:nlsdata.obj
 0002:00003264       ??_C@_1BA@EPANDLNG@?$AAO?$AAc?$AAt?$AAo?$AAb?$AAe?$AAr@ 10040264     libucrt:nlsdata.obj
 0002:00003274       ??_C@_1BC@BGLIFPF@?$AAN?$AAo?$AAv?$AAe?$AAm?$AAb?$AAe?$AAr@ 10040274     libucrt:nlsdata.obj
 0002:00003288       ??_C@_1BC@FEMKIFH@?$AAD?$AAe?$AAc?$AAe?$AAm?$AAb?$AAe?$AAr@ 10040288     libucrt:nlsdata.obj
 0002:0000329c       ??_C@_15ODEHAHHF@?$AAA?$AAM@ 1004029c     libucrt:nlsdata.obj
 0002:000032a4       ??_C@_15CLMNNGEL@?$AAP?$AAM@ 100402a4     libucrt:nlsdata.obj
 0002:000032ac       ??_C@_1BC@IEBCMHCM@?$AAM?$AAM?$AA?1?$AAd?$AAd?$AA?1?$AAy?$AAy@ 100402ac     libucrt:nlsdata.obj
 0002:000032c0       ??_C@_1CI@KNAKOEBC@?$AAd?$AAd?$AAd?$AAd?$AA?0?$AA?5?$AAM?$AAM?$AAM?$AAM?$AA?5?$AAd?$AAd?$AA?0?$AA?5@ 100402c0     libucrt:nlsdata.obj
 0002:000032e8       ??_C@_1BC@GDGBMEMK@?$AAH?$AAH?$AA?3?$AAm?$AAm?$AA?3?$AAs?$AAs@ 100402e8     libucrt:nlsdata.obj
 0002:000032fc       ??_C@_1M@BMHNFIME@?$AAe?$AAn?$AA?9?$AAU?$AAS@ 100402fc     libucrt:nlsdata.obj
 0002:00003308       ??_C@_03MGHMBJCF@log@      10040308     libucrt:libm_error.obj
 0002:0000330c       ??_C@_05HGHHAHAP@log10@    1004030c     libucrt:libm_error.obj
 0002:00003314       ??_C@_03KHJOGHMM@exp@      10040314     libucrt:libm_error.obj
 0002:00003318       ??_C@_03JGHBODFD@pow@      10040318     libucrt:libm_error.obj
 0002:0000331c       ??_C@_04FIHNOPOL@asin@     1004031c     libucrt:libm_error.obj
 0002:00003324       ??_C@_04PDIFKINK@acos@     10040324     libucrt:libm_error.obj
 0002:0000332c       ??_C@_04EIAKFFMI@sqrt@     1004032c     libucrt:libm_error.obj
 0002:00003420       ??_C@_04COOMCNPB@sinh@     10040420     libucrt:fpexcept.obj
 0002:00003428       ??_C@_04HPJJNFIM@cosh@     10040428     libucrt:fpexcept.obj
 0002:00003430       ??_C@_04FJHINJAO@tanh@     10040430     libucrt:fpexcept.obj
 0002:00003438       ??_C@_04MLLJIGOK@atan@     10040438     libucrt:fpexcept.obj
 0002:00003440       ??_C@_05KNGEOGJB@atan2@    10040440     libucrt:fpexcept.obj
 0002:00003448       ??_C@_03BLEJJJBH@sin@      10040448     libucrt:fpexcept.obj
 0002:0000344c       ??_C@_03LALBNOCG@cos@      1004044c     libucrt:fpexcept.obj
 0002:00003450       ??_C@_03IIINPABG@tan@      10040450     libucrt:fpexcept.obj
 0002:00003454       ??_C@_04GFPJNGEK@ceil@     10040454     libucrt:fpexcept.obj
 0002:0000345c       ??_C@_05PBJFFIGL@floor@    1004045c     libucrt:fpexcept.obj
 0002:00003464       ??_C@_04ODHECPBC@fabs@     10040464     libucrt:fpexcept.obj
 0002:0000346c       ??_C@_04EHEDPDJG@modf@     1004046c     libucrt:fpexcept.obj
 0002:00003474       ??_C@_05CEJMAHNP@ldexp@    10040474     libucrt:fpexcept.obj
 0002:0000347c       ??_C@_05KBKMEMPO@_cabs@    1004047c     libucrt:fpexcept.obj
 0002:00003484       ??_C@_06MEIMCGCF@_hypot@   10040484     libucrt:fpexcept.obj
 0002:0000348c       ??_C@_04KEPJIHGP@fmod@     1004048c     libucrt:fpexcept.obj
 0002:00003494       ??_C@_05GKKHEGJL@frexp@    10040494     libucrt:fpexcept.obj
 0002:0000349c       ??_C@_03MJLDFKDL@_y0@      1004049c     libucrt:fpexcept.obj
 0002:000034a0       ??_C@_03NAKIGLHK@_y1@      100404a0     libucrt:fpexcept.obj
 0002:000034a4       ??_C@_03ONILCKOB@_yn@      100404a4     libucrt:fpexcept.obj
 0002:000034a8       ??_C@_05JGDBENOH@_logb@    100404a8     libucrt:fpexcept.obj
 0002:000034b0       ??_C@_0L@KDOEJCKC@_nextafter@ 100404b0     libucrt:fpexcept.obj
 0002:000034c0       __d_inf                    100404c0     libucrt:util.obj
 0002:000034c8       __d_ind                    100404c8     libucrt:util.obj
 0002:000034d0       __d_max                    100404d0     libucrt:util.obj
 0002:000034d8       __d_mzero                  100404d8     libucrt:util.obj
 0002:000035c0       __infinity                 100405c0     libucrt:87tran.obj
 0002:000035ca       __minfinity                100405ca     libucrt:87tran.obj
 0002:000035d4       __logemax                  100405d4     libucrt:87tran.obj
 0002:000035fa       __OP_EXPjmptab             100405fa     libucrt:87tran.obj
 0002:00003620       __indefinite               10040620     libucrt:87disp.obj
 0002:0000362a       __piby2                    1004062a     libucrt:87disp.obj
 0002:00003634       __piby4                    10040634     libucrt:87disp.obj
 0002:00003668       __DEFAULT_CW_in_mem        10040668     libucrt:common.obj
 0002:0000366a       __pi_by_2_to_61            1004066a     libucrt:common.obj
 0002:000036b4       ??_C@_1M@HPNHIDJI@?$AAj?$AAa?$AA?9?$AAJ?$AAP@ 100406b4     libucrt:mbctype.obj
 0002:000036c0       ??_C@_1M@BIBDDEMK@?$AAz?$AAh?$AA?9?$AAC?$AAN@ 100406c0     libucrt:mbctype.obj
 0002:000036cc       ??_C@_1M@JLOOOEGK@?$AAk?$AAo?$AA?9?$AAK?$AAR@ 100406cc     libucrt:mbctype.obj
 0002:000036d8       ??_C@_1M@CLNBBOPM@?$AAz?$AAh?$AA?9?$AAT?$AAW@ 100406d8     libucrt:mbctype.obj
 0002:00003e08       ??_C@_15EMKDOKLE@?$AAa?$AAr@ 10040e08     libucrt:lcidtoname_downlevel.obj
 0002:00003e10       ??_C@_15KNPADPLH@?$AAb?$AAg@ 10040e10     libucrt:lcidtoname_downlevel.obj
 0002:00003e18       ??_C@_15EDMHLDMO@?$AAc?$AAa@ 10040e18     libucrt:lcidtoname_downlevel.obj
 0002:00003e20       ??_C@_1O@BPEAJADD@?$AAz?$AAh?$AA?9?$AAC?$AAH?$AAS@ 10040e20     libucrt:lcidtoname_downlevel.obj
 0002:00003e30       ??_C@_15LJNHCMNK@?$AAc?$AAs@ 10040e30     libucrt:lcidtoname_downlevel.obj
 0002:00003e38       ??_C@_15FOMCIDHG@?$AAd?$AAa@ 10040e38     libucrt:lcidtoname_downlevel.obj
 0002:00003e40       ??_C@_15NBKABECB@?$AAd?$AAe@ 10040e40     libucrt:lcidtoname_downlevel.obj
 0002:00003e48       ??_C@_15GHPEIIAO@?$AAe?$AAl@ 10040e48     libucrt:lcidtoname_downlevel.obj
 0002:00003e50       ??_C@_15MNPNEAIF@?$AAe?$AAn@ 10040e50     libucrt:lcidtoname_downlevel.obj
 0002:00003e58       ??_C@_15GPIOMPMH@?$AAe?$AAs@ 10040e58     libucrt:lcidtoname_downlevel.obj
 0002:00003e60       ??_C@_15NGLOAKJC@?$AAf?$AAi@ 10040e60     libucrt:lcidtoname_downlevel.obj
 0002:00003e68       ??_C@_15FBKGNKAM@?$AAf?$AAr@ 10040e68     libucrt:lcidtoname_downlevel.obj
 0002:00003e70       ??_C@_15KGGCNEFK@?$AAh?$AAe@ 10040e70     libucrt:lcidtoname_downlevel.obj
 0002:00003e78       ??_C@_15PGHLIDMF@?$AAh?$AAu@ 10040e78     libucrt:lcidtoname_downlevel.obj
 0002:00003e80       ??_C@_15BIEMAPLM@?$AAi?$AAs@ 10040e80     libucrt:lcidtoname_downlevel.obj
 0002:00003e88       ??_C@_15IFJLDHAF@?$AAi?$AAt@ 10040e88     libucrt:lcidtoname_downlevel.obj
 0002:00003e90       ??_C@_15GEMIOCAG@?$AAj?$AAa@ 10040e90     libucrt:lcidtoname_downlevel.obj
 0002:00003e98       ??_C@_15EPELEGJA@?$AAk?$AAo@ 10040e98     libucrt:lcidtoname_downlevel.obj
 0002:00003ea0       ??_C@_15NDDHIMN@?$AAn?$AAl@ 10040ea0     libucrt:lcidtoname_downlevel.obj
 0002:00003ea8       ??_C@_15BPIGNHCD@?$AAn?$AAo@ 10040ea8     libucrt:lcidtoname_downlevel.obj
 0002:00003eb0       ??_C@_15DEOPBLCG@?$AAp?$AAl@ 10040eb0     libucrt:lcidtoname_downlevel.obj
 0002:00003eb8       ??_C@_15KBECGEFG@?$AAp?$AAt@ 10040eb8     libucrt:lcidtoname_downlevel.obj
 0002:00003ec0       ??_C@_15GLJCBFMD@?$AAr?$AAo@ 10040ec0     libucrt:lcidtoname_downlevel.obj
 0002:00003ec8       ??_C@_15FEDGKCDI@?$AAr?$AAu@ 10040ec8     libucrt:lcidtoname_downlevel.obj
 0002:00003ed0       ??_C@_15GLKMLLHM@?$AAh?$AAr@ 10040ed0     libucrt:lcidtoname_downlevel.obj
 0002:00003ed8       ??_C@_15CPKMFBDB@?$AAs?$AAk@ 10040ed8     libucrt:lcidtoname_downlevel.obj
 0002:00003ee0       ??_C@_15BAAIOGMK@?$AAs?$AAq@ 10040ee0     libucrt:lcidtoname_downlevel.obj
 0002:00003ee8       ??_C@_15INNPNOHD@?$AAs?$AAv@ 10040ee8     libucrt:lcidtoname_downlevel.obj
 0002:00003ef0       ??_C@_15CABMMOGH@?$AAt?$AAh@ 10040ef0     libucrt:lcidtoname_downlevel.obj
 0002:00003ef8       ??_C@_15BPLIHJJM@?$AAt?$AAr@ 10040ef8     libucrt:lcidtoname_downlevel.obj
 0002:00003f00       ??_C@_15NEOEKKDJ@?$AAu?$AAr@ 10040f00     libucrt:lcidtoname_downlevel.obj
 0002:00003f08       ??_C@_15NFICGAJK@?$AAi?$AAd@ 10040f08     libucrt:lcidtoname_downlevel.obj
 0002:00003f10       ??_C@_15PJPFLCCM@?$AAu?$AAk@ 10040f10     libucrt:lcidtoname_downlevel.obj
 0002:00003f18       ??_C@_15HPJPHDM@?$AAb?$AAe@ 10040f18     libucrt:lcidtoname_downlevel.obj
 0002:00003f20       ??_C@_15LCHLGJII@?$AAs?$AAl@ 10040f20     libucrt:lcidtoname_downlevel.obj
 0002:00003f28       ??_C@_15PCFJPHHO@?$AAe?$AAt@ 10040f28     libucrt:lcidtoname_downlevel.obj
 0002:00003f30       ??_C@_15HPFPGODN@?$AAl?$AAv@ 10040f30     libucrt:lcidtoname_downlevel.obj
 0002:00003f38       ??_C@_15NFFGKGLG@?$AAl?$AAt@ 10040f38     libucrt:lcidtoname_downlevel.obj
 0002:00003f40       ??_C@_15BDAKCCHN@?$AAf?$AAa@ 10040f40     libucrt:lcidtoname_downlevel.obj
 0002:00003f48       ??_C@_15NFGIAIAJ@?$AAv?$AAi@ 10040f48     libucrt:lcidtoname_downlevel.obj
 0002:00003f50       ??_C@_15LMKNDMHN@?$AAh?$AAy@ 10040f50     libucrt:lcidtoname_downlevel.obj
 0002:00003f58       ??_C@_15IJBHMCFL@?$AAa?$AAz@ 10040f58     libucrt:lcidtoname_downlevel.obj
 0002:00003f60       ??_C@_15EKOFJABL@?$AAe?$AAu@ 10040f60     libucrt:lcidtoname_downlevel.obj
 0002:00003f68       ??_C@_15BGHADCNK@?$AAm?$AAk@ 10040f68     libucrt:lcidtoname_downlevel.obj
 0002:00003f70       ??_C@_15JDNICKHM@?$AAa?$AAf@ 10040f70     libucrt:lcidtoname_downlevel.obj
 0002:00003f78       ??_C@_15KPJEDBKD@?$AAk?$AAa@ 10040f78     libucrt:lcidtoname_downlevel.obj
 0002:00003f80       ??_C@_15PDNFFFEO@?$AAf?$AAo@ 10040f80     libucrt:lcidtoname_downlevel.obj
 0002:00003f88       ??_C@_15OMLEGLOC@?$AAh?$AAi@ 10040f88     libucrt:lcidtoname_downlevel.obj
 0002:00003f90       ??_C@_15IDNNENKK@?$AAm?$AAs@ 10040f90     libucrt:lcidtoname_downlevel.obj
 0002:00003f98       ??_C@_15MACJNBMH@?$AAk?$AAk@ 10040f98     libucrt:lcidtoname_downlevel.obj
 0002:00003fa0       ??_C@_15DKDJEOND@?$AAk?$AAy@ 10040fa0     libucrt:lcidtoname_downlevel.obj
 0002:00003fa8       ??_C@_15DFGDLJBG@?$AAs?$AAw@ 10040fa8     libucrt:lcidtoname_downlevel.obj
 0002:00003fb0       ??_C@_15BBFAICNG@?$AAu?$AAz@ 10040fb0     libucrt:lcidtoname_downlevel.obj
 0002:00003fb8       ??_C@_15DKNDCGEA@?$AAt?$AAt@ 10040fb8     libucrt:lcidtoname_downlevel.obj
 0002:00003fc0       ??_C@_15MGIFMDPL@?$AAp?$AAa@ 10040fc0     libucrt:lcidtoname_downlevel.obj
 0002:00003fc8       ??_C@_15HCNDBBA@?$AAg?$AAu@ 10040fc8     libucrt:lcidtoname_downlevel.obj
 0002:00003fd0       ??_C@_15FNBEIBON@?$AAt?$AAa@ 10040fd0     libucrt:lcidtoname_downlevel.obj
 0002:00003fd8       ??_C@_15NCHGBGLK@?$AAt?$AAe@ 10040fd8     libucrt:lcidtoname_downlevel.obj
 0002:00003fe0       ??_C@_15PHPHCBPF@?$AAk?$AAn@ 10040fe0     libucrt:lcidtoname_downlevel.obj
 0002:00003fe8       ??_C@_15DLGBCKMP@?$AAm?$AAr@ 10040fe8     libucrt:lcidtoname_downlevel.obj
 0002:00003ff0       ??_C@_15EABBLBFF@?$AAs?$AAa@ 10040ff0     libucrt:lcidtoname_downlevel.obj
 0002:00003ff8       ??_C@_15CBKOMCOI@?$AAm?$AAn@ 10040ff8     libucrt:lcidtoname_downlevel.obj
 0002:00004000       ??_C@_15CKDMCJAF@?$AAg?$AAl@ 10041000     libucrt:lcidtoname_downlevel.obj
 0002:00004008       ??_C@_17CNJFBPG@?$AAk?$AAo?$AAk@ 10041008     libucrt:lcidtoname_downlevel.obj
 0002:00004010       ??_C@_17FFBJICPL@?$AAs?$AAy?$AAr@ 10041010     libucrt:lcidtoname_downlevel.obj
 0002:00004018       ??_C@_17KPNDCPAF@?$AAd?$AAi?$AAv@ 10041018     libucrt:lcidtoname_downlevel.obj
 0002:00004020       ??_C@_1M@OKAHONE@?$AAa?$AAr?$AA?9?$AAS?$AAA@ 10041020     libucrt:lcidtoname_downlevel.obj
 0002:0000402c       ??_C@_1M@FFFIGIGK@?$AAb?$AAg?$AA?9?$AAB?$AAG@ 1004102c     libucrt:lcidtoname_downlevel.obj
 0002:00004038       ??_C@_1M@BJNKEDC@?$AAc?$AAa?$AA?9?$AAE?$AAS@ 10041038     libucrt:lcidtoname_downlevel.obj
 0002:00004044       ??_C@_1M@IJJHFJHA@?$AAc?$AAs?$AA?9?$AAC?$AAZ@ 10041044     libucrt:lcidtoname_downlevel.obj
 0002:00004050       ??_C@_1M@CLPEOBGI@?$AAd?$AAa?$AA?9?$AAD?$AAK@ 10041050     libucrt:lcidtoname_downlevel.obj
 0002:0000405c       ??_C@_1M@MCMADGCB@?$AAd?$AAe?$AA?9?$AAD?$AAE@ 1004105c     libucrt:lcidtoname_downlevel.obj
 0002:00004068       ??_C@_1M@OOCKEMAM@?$AAe?$AAl?$AA?9?$AAG?$AAR@ 10041068     libucrt:lcidtoname_downlevel.obj
 0002:00004074       ??_C@_1M@DDNJFGID@?$AAf?$AAi?$AA?9?$AAF?$AAI@ 10041074     libucrt:lcidtoname_downlevel.obj
 0002:00004080       ??_C@_1M@GLIPPMAC@?$AAf?$AAr?$AA?9?$AAF?$AAR@ 10041080     libucrt:lcidtoname_downlevel.obj
 0002:0000408c       ??_C@_1M@GFMCHPE@?$AAh?$AAe?$AA?9?$AAI?$AAL@ 1004108c     libucrt:lcidtoname_downlevel.obj
 0002:00004098       ??_C@_1M@MHLPGNKM@?$AAh?$AAu?$AA?9?$AAH?$AAU@ 10041098     libucrt:lcidtoname_downlevel.obj
 0002:000040a4       ??_C@_1M@LPDDNNPN@?$AAi?$AAs?$AA?9?$AAI?$AAS@ 100410a4     libucrt:lcidtoname_downlevel.obj
 0002:000040b0       ??_C@_1M@MADIPODN@?$AAi?$AAt?$AA?9?$AAI?$AAT@ 100410b0     libucrt:lcidtoname_downlevel.obj
 0002:000040bc       ??_C@_1M@IHBJJGG@?$AAn?$AAl?$AA?9?$AAN?$AAL@ 100410bc     libucrt:lcidtoname_downlevel.obj
 0002:000040c8       ??_C@_1M@EANAGDL@?$AAn?$AAb?$AA?9?$AAN?$AAO@ 100410c8     libucrt:lcidtoname_downlevel.obj
 0002:000040d4       ??_C@_1M@NEIEMEGP@?$AAp?$AAl?$AA?9?$AAP?$AAL@ 100410d4     libucrt:lcidtoname_downlevel.obj
 0002:000040e0       ??_C@_1M@BOCFIGEP@?$AAp?$AAt?$AA?9?$AAB?$AAR@ 100410e0     libucrt:lcidtoname_downlevel.obj
 0002:000040ec       ??_C@_1M@IMPFOPBG@?$AAr?$AAo?$AA?9?$AAR?$AAO@ 100410ec     libucrt:lcidtoname_downlevel.obj
 0002:000040f8       ??_C@_1M@IDNNEJMM@?$AAr?$AAu?$AA?9?$AAR?$AAU@ 100410f8     libucrt:lcidtoname_downlevel.obj
 0002:00004104       ??_C@_1M@LILEEOGM@?$AAh?$AAr?$AA?9?$AAH?$AAR@ 10041104     libucrt:lcidtoname_downlevel.obj
 0002:00004110       ??_C@_1M@FKIFEHPB@?$AAs?$AAk?$AA?9?$AAS?$AAK@ 10041110     libucrt:lcidtoname_downlevel.obj
 0002:0000411c       ??_C@_1M@LJMAMNPJ@?$AAs?$AAq?$AA?9?$AAA?$AAL@ 1004111c     libucrt:lcidtoname_downlevel.obj
 0002:00004128       ??_C@_1M@GIAKDKJK@?$AAs?$AAv?$AA?9?$AAS?$AAE@ 10041128     libucrt:lcidtoname_downlevel.obj
 0002:00004134       ??_C@_1M@MKJKIKCL@?$AAt?$AAh?$AA?9?$AAT?$AAH@ 10041134     libucrt:lcidtoname_downlevel.obj
 0002:00004140       ??_C@_1M@MFLCCMPB@?$AAt?$AAr?$AA?9?$AAT?$AAR@ 10041140     libucrt:lcidtoname_downlevel.obj
 0002:0000414c       ??_C@_1M@OIJHDKJN@?$AAu?$AAr?$AA?9?$AAP?$AAK@ 1004114c     libucrt:lcidtoname_downlevel.obj
 0002:00004158       ??_C@_1M@LHIPCIEK@?$AAi?$AAd?$AA?9?$AAI?$AAD@ 10041158     libucrt:lcidtoname_downlevel.obj
 0002:00004164       ??_C@_1M@MFMOBGI@?$AAu?$AAk?$AA?9?$AAU?$AAA@ 10041164     libucrt:lcidtoname_downlevel.obj
 0002:00004170       ??_C@_1M@OBGLJIPL@?$AAb?$AAe?$AA?9?$AAB?$AAY@ 10041170     libucrt:lcidtoname_downlevel.obj
 0002:0000417c       ??_C@_1M@BCFAJEAD@?$AAs?$AAl?$AA?9?$AAS?$AAI@ 1004117c     libucrt:lcidtoname_downlevel.obj
 0002:00004188       ??_C@_1M@FKFFEDDN@?$AAe?$AAt?$AA?9?$AAE?$AAE@ 10041188     libucrt:lcidtoname_downlevel.obj
 0002:00004194       ??_C@_1M@KGKKAACI@?$AAl?$AAv?$AA?9?$AAL?$AAV@ 10041194     libucrt:lcidtoname_downlevel.obj
 0002:000041a0       ??_C@_1M@IFGBIJO@?$AAl?$AAt?$AA?9?$AAL?$AAT@ 100411a0     libucrt:lcidtoname_downlevel.obj
 0002:000041ac       ??_C@_1M@FGEAHEDM@?$AAf?$AAa?$AA?9?$AAI?$AAR@ 100411ac     libucrt:lcidtoname_downlevel.obj
 0002:000041b8       ??_C@_1M@KBMAIBFN@?$AAv?$AAi?$AA?9?$AAV?$AAN@ 100411b8     libucrt:lcidtoname_downlevel.obj
 0002:000041c4       ??_C@_1M@GPCBKDJK@?$AAh?$AAy?$AA?9?$AAA?$AAM@ 100411c4     libucrt:lcidtoname_downlevel.obj
 0002:000041d0       ??_C@_1BG@BECMDDJB@?$AAa?$AAz?$AA?9?$AAA?$AAZ?$AA?9?$AAL?$AAa?$AAt?$AAn@ 100411d0     libucrt:lcidtoname_downlevel.obj
 0002:000041e8       ??_C@_1M@MAOFCAEA@?$AAe?$AAu?$AA?9?$AAE?$AAS@ 100411e8     libucrt:lcidtoname_downlevel.obj
 0002:000041f4       ??_C@_1M@IGHABKPI@?$AAm?$AAk?$AA?9?$AAM?$AAK@ 100411f4     libucrt:lcidtoname_downlevel.obj
 0002:00004200       ??_C@_1M@IAIGNEJG@?$AAt?$AAn?$AA?9?$AAZ?$AAA@ 10041200     libucrt:lcidtoname_downlevel.obj
 0002:0000420c       ??_C@_1M@IIJCOJFA@?$AAx?$AAh?$AA?9?$AAZ?$AAA@ 1004120c     libucrt:lcidtoname_downlevel.obj
 0002:00004218       ??_C@_1M@LGPJHNJH@?$AAz?$AAu?$AA?9?$AAZ?$AAA@ 10041218     libucrt:lcidtoname_downlevel.obj
 0002:00004224       ??_C@_1M@HOKAOIO@?$AAa?$AAf?$AA?9?$AAZ?$AAA@ 10041224     libucrt:lcidtoname_downlevel.obj
 0002:00004230       ??_C@_1M@DPCLHLIE@?$AAk?$AAa?$AA?9?$AAG?$AAE@ 10041230     libucrt:lcidtoname_downlevel.obj
 0002:0000423c       ??_C@_1M@BLKMHJBI@?$AAf?$AAo?$AA?9?$AAF?$AAO@ 1004123c     libucrt:lcidtoname_downlevel.obj
 0002:00004248       ??_C@_1M@LGGJAPPB@?$AAh?$AAi?$AA?9?$AAI?$AAN@ 10041248     libucrt:lcidtoname_downlevel.obj
 0002:00004254       ??_C@_1M@FIKPIHFE@?$AAm?$AAt?$AA?9?$AAM?$AAT@ 10041254     libucrt:lcidtoname_downlevel.obj
 0002:00004260       ??_C@_1M@HEGGPBFA@?$AAs?$AAe?$AA?9?$AAN?$AAO@ 10041260     libucrt:lcidtoname_downlevel.obj
 0002:0000426c       ??_C@_1M@EIBJEEPA@?$AAm?$AAs?$AA?9?$AAM?$AAY@ 1004126c     libucrt:lcidtoname_downlevel.obj
 0002:00004278       ??_C@_1M@FHLBGMPP@?$AAk?$AAk?$AA?9?$AAK?$AAZ@ 10041278     libucrt:lcidtoname_downlevel.obj
 0002:00004284       ??_C@_1M@NGJJLCGI@?$AAk?$AAy?$AA?9?$AAK?$AAG@ 10041284     libucrt:lcidtoname_downlevel.obj
 0002:00004290       ??_C@_1M@GIENNBFC@?$AAs?$AAw?$AA?9?$AAK?$AAE@ 10041290     libucrt:lcidtoname_downlevel.obj
 0002:0000429c       ??_C@_1BG@NDGMJIMJ@?$AAu?$AAz?$AA?9?$AAU?$AAZ?$AA?9?$AAL?$AAa?$AAt?$AAn@ 1004129c     libucrt:lcidtoname_downlevel.obj
 0002:000042b4       ??_C@_1M@IDCCIHBC@?$AAt?$AAt?$AA?9?$AAR?$AAU@ 100412b4     libucrt:lcidtoname_downlevel.obj
 0002:000042c0       ??_C@_1M@LOICPMOJ@?$AAb?$AAn?$AA?9?$AAI?$AAN@ 100412c0     libucrt:lcidtoname_downlevel.obj
 0002:000042cc       ??_C@_1M@KPKKNEAH@?$AAp?$AAa?$AA?9?$AAI?$AAN@ 100412cc     libucrt:lcidtoname_downlevel.obj
 0002:000042d8       ??_C@_1M@PJGPPBOG@?$AAg?$AAu?$AA?9?$AAI?$AAN@ 100412d8     libucrt:lcidtoname_downlevel.obj
 0002:000042e4       ??_C@_1M@KMKMOPHI@?$AAt?$AAa?$AA?9?$AAI?$AAN@ 100412e4     libucrt:lcidtoname_downlevel.obj
 0002:000042f0       ??_C@_1M@KFEHEPAC@?$AAt?$AAe?$AA?9?$AAI?$AAN@ 100412f0     libucrt:lcidtoname_downlevel.obj
 0002:000042fc       ??_C@_1M@CDCLMGHI@?$AAk?$AAn?$AA?9?$AAI?$AAN@ 100412fc     libucrt:lcidtoname_downlevel.obj
 0002:00004308       ??_C@_1M@MIODLDKF@?$AAm?$AAl?$AA?9?$AAI?$AAN@ 10041308     libucrt:lcidtoname_downlevel.obj
 0002:00004314       ??_C@_1M@PBIEACPO@?$AAm?$AAr?$AA?9?$AAI?$AAN@ 10041314     libucrt:lcidtoname_downlevel.obj
 0002:00004320       ??_C@_1M@NIDEAGPH@?$AAs?$AAa?$AA?9?$AAI?$AAN@ 10041320     libucrt:lcidtoname_downlevel.obj
 0002:0000432c       ??_C@_1M@FHIHCBIO@?$AAm?$AAn?$AA?9?$AAM?$AAN@ 1004132c     libucrt:lcidtoname_downlevel.obj
 0002:00004338       ??_C@_1M@JAIJPENP@?$AAc?$AAy?$AA?9?$AAG?$AAB@ 10041338     libucrt:lcidtoname_downlevel.obj
 0002:00004344       ??_C@_1M@PHGFBEPN@?$AAg?$AAl?$AA?9?$AAE?$AAS@ 10041344     libucrt:lcidtoname_downlevel.obj
 0002:00004350       ??_C@_1O@KPIPDNCP@?$AAk?$AAo?$AAk?$AA?9?$AAI?$AAN@ 10041350     libucrt:lcidtoname_downlevel.obj
 0002:00004360       ??_C@_1O@KNHJLDJA@?$AAs?$AAy?$AAr?$AA?9?$AAS?$AAY@ 10041360     libucrt:lcidtoname_downlevel.obj
 0002:00004370       ??_C@_1O@MKEKBLAH@?$AAd?$AAi?$AAv?$AA?9?$AAM?$AAV@ 10041370     libucrt:lcidtoname_downlevel.obj
 0002:00004380       ??_C@_1O@OHDCKDDF@?$AAq?$AAu?$AAz?$AA?9?$AAB?$AAO@ 10041380     libucrt:lcidtoname_downlevel.obj
 0002:00004390       ??_C@_1M@LEPJNLFD@?$AAn?$AAs?$AA?9?$AAZ?$AAA@ 10041390     libucrt:lcidtoname_downlevel.obj
 0002:0000439c       ??_C@_1M@OMLEIIJB@?$AAm?$AAi?$AA?9?$AAN?$AAZ@ 1004139c     libucrt:lcidtoname_downlevel.obj
 0002:000043a8       ??_C@_1M@PMPEAILG@?$AAa?$AAr?$AA?9?$AAI?$AAQ@ 100413a8     libucrt:lcidtoname_downlevel.obj
 0002:000043b4       ??_C@_1M@CNKPNOEE@?$AAd?$AAe?$AA?9?$AAC?$AAH@ 100413b4     libucrt:lcidtoname_downlevel.obj
 0002:000043c0       ??_C@_1M@LKMGMLKO@?$AAe?$AAn?$AA?9?$AAG?$AAB@ 100413c0     libucrt:lcidtoname_downlevel.obj
 0002:000043cc       ??_C@_1M@PGKJFFGL@?$AAe?$AAs?$AA?9?$AAM?$AAX@ 100413cc     libucrt:lcidtoname_downlevel.obj
 0002:000043d8       ??_C@_1M@DNNANBDC@?$AAf?$AAr?$AA?9?$AAB?$AAE@ 100413d8     libucrt:lcidtoname_downlevel.obj
 0002:000043e4       ??_C@_1M@HLGMDFHM@?$AAi?$AAt?$AA?9?$AAC?$AAH@ 100413e4     libucrt:lcidtoname_downlevel.obj
 0002:000043f0       ??_C@_1M@CLLBGJH@?$AAn?$AAl?$AA?9?$AAB?$AAE@ 100413f0     libucrt:lcidtoname_downlevel.obj
 0002:000043fc       ??_C@_1M@BODBOGLF@?$AAn?$AAn?$AA?9?$AAN?$AAO@ 100413fc     libucrt:lcidtoname_downlevel.obj
 0002:00004408       ??_C@_1M@HFFAHKAD@?$AAp?$AAt?$AA?9?$AAP?$AAT@ 10041408     libucrt:lcidtoname_downlevel.obj
 0002:00004414       ??_C@_1BG@LNOAKHIE@?$AAs?$AAr?$AA?9?$AAS?$AAP?$AA?9?$AAL?$AAa?$AAt?$AAn@ 10041414     libucrt:lcidtoname_downlevel.obj
 0002:0000442c       ??_C@_1M@HBMHBGAK@?$AAs?$AAv?$AA?9?$AAF?$AAI@ 1004142c     libucrt:lcidtoname_downlevel.obj
 0002:00004438       ??_C@_1BG@DGCJGJBE@?$AAa?$AAz?$AA?9?$AAA?$AAZ?$AA?9?$AAC?$AAy?$AAr?$AAl@ 10041438     libucrt:lcidtoname_downlevel.obj
 0002:00004450       ??_C@_1M@KEJDAAHB@?$AAs?$AAe?$AA?9?$AAS?$AAE@ 10041450     libucrt:lcidtoname_downlevel.obj
 0002:0000445c       ??_C@_1M@HEIBJJAD@?$AAm?$AAs?$AA?9?$AAB?$AAN@ 1004145c     libucrt:lcidtoname_downlevel.obj
 0002:00004468       ??_C@_1BG@PBGJMCEM@?$AAu?$AAz?$AA?9?$AAU?$AAZ?$AA?9?$AAC?$AAy?$AAr?$AAl@ 10041468     libucrt:lcidtoname_downlevel.obj
 0002:00004480       ??_C@_1O@LAOBCMDF@?$AAq?$AAu?$AAz?$AA?9?$AAE?$AAC@ 10041480     libucrt:lcidtoname_downlevel.obj
 0002:00004490       ??_C@_1M@POEEMAIO@?$AAa?$AAr?$AA?9?$AAE?$AAG@ 10041490     libucrt:lcidtoname_downlevel.obj
 0002:0000449c       ??_C@_1M@EFAKDEDL@?$AAz?$AAh?$AA?9?$AAH?$AAK@ 1004149c     libucrt:lcidtoname_downlevel.obj
 0002:000044a8       ??_C@_1M@HKKIJHGI@?$AAd?$AAe?$AA?9?$AAA?$AAT@ 100414a8     libucrt:lcidtoname_downlevel.obj
 0002:000044b4       ??_C@_1M@KBFBEHJF@?$AAe?$AAn?$AA?9?$AAA?$AAU@ 100414b4     libucrt:lcidtoname_downlevel.obj
 0002:000044c0       ??_C@_1M@MNPLFAAH@?$AAe?$AAs?$AA?9?$AAE?$AAS@ 100414c0     libucrt:lcidtoname_downlevel.obj
 0002:000044cc       ??_C@_1M@HJOOJFMA@?$AAf?$AAr?$AA?9?$AAC?$AAA@ 100414cc     libucrt:lcidtoname_downlevel.obj
 0002:000044d8       ??_C@_1BG@JPOFPNAB@?$AAs?$AAr?$AA?9?$AAS?$AAP?$AA?9?$AAC?$AAy?$AAr?$AAl@ 100414d8     libucrt:lcidtoname_downlevel.obj
 0002:000044f0       ??_C@_1M@LNFOCMOB@?$AAs?$AAe?$AA?9?$AAF?$AAI@ 100414f0     libucrt:lcidtoname_downlevel.obj
 0002:000044fc       ??_C@_1O@MGJBOAMB@?$AAq?$AAu?$AAz?$AA?9?$AAP?$AAE@ 100414fc     libucrt:lcidtoname_downlevel.obj
 0002:0000450c       ??_C@_1M@GJINLBOK@?$AAa?$AAr?$AA?9?$AAL?$AAY@ 1004150c     libucrt:lcidtoname_downlevel.obj
 0002:00004518       ??_C@_1M@GGMNHJNL@?$AAz?$AAh?$AA?9?$AAS?$AAG@ 10041518     libucrt:lcidtoname_downlevel.obj
 0002:00004524       ??_C@_1M@HOIKODND@?$AAd?$AAe?$AA?9?$AAL?$AAU@ 10041524     libucrt:lcidtoname_downlevel.obj
 0002:00004530       ??_C@_1M@DDOCCGFG@?$AAe?$AAn?$AA?9?$AAC?$AAA@ 10041530     libucrt:lcidtoname_downlevel.obj
 0002:0000453c       ??_C@_1M@BNOEMJLF@?$AAe?$AAs?$AA?9?$AAG?$AAT@ 1004153c     libucrt:lcidtoname_downlevel.obj
 0002:00004548       ??_C@_1M@EOGNKEK@?$AAf?$AAr?$AA?9?$AAC?$AAH@ 10041548     libucrt:lcidtoname_downlevel.obj
 0002:00004554       ??_C@_1M@FLIDJFHL@?$AAh?$AAr?$AA?9?$AAB?$AAA@ 10041554     libucrt:lcidtoname_downlevel.obj
 0002:00004560       ??_C@_1O@FMCELNAJ@?$AAs?$AAm?$AAj?$AA?9?$AAN?$AAO@ 10041560     libucrt:lcidtoname_downlevel.obj
 0002:00004570       ??_C@_1M@JHGLJMGJ@?$AAa?$AAr?$AA?9?$AAD?$AAZ@ 10041570     libucrt:lcidtoname_downlevel.obj
 0002:0000457c       ??_C@_1M@JKKFDCNP@?$AAz?$AAh?$AA?9?$AAM?$AAO@ 1004157c     libucrt:lcidtoname_downlevel.obj
 0002:00004588       ??_C@_1M@GEEFALPE@?$AAd?$AAe?$AA?9?$AAL?$AAI@ 10041588     libucrt:lcidtoname_downlevel.obj
 0002:00004594       ??_C@_1M@IGEOFBG@?$AAe?$AAn?$AA?9?$AAN?$AAZ@ 10041594     libucrt:lcidtoname_downlevel.obj
 0002:000045a0       ??_C@_1M@KDBONEHP@?$AAe?$AAs?$AA?9?$AAC?$AAR@ 100415a0     libucrt:lcidtoname_downlevel.obj
 0002:000045ac       ??_C@_1M@FHMDOHNN@?$AAf?$AAr?$AA?9?$AAL?$AAU@ 100415ac     libucrt:lcidtoname_downlevel.obj
 0002:000045b8       ??_C@_1BG@NFKKMAFG@?$AAb?$AAs?$AA?9?$AAB?$AAA?$AA?9?$AAL?$AAa?$AAt?$AAn@ 100415b8     libucrt:lcidtoname_downlevel.obj
 0002:000045d0       ??_C@_1O@IMNBEMCI@?$AAs?$AAm?$AAj?$AA?9?$AAS?$AAE@ 100415d0     libucrt:lcidtoname_downlevel.obj
 0002:000045e0       ??_C@_1M@DHHMBNDP@?$AAa?$AAr?$AA?9?$AAM?$AAA@ 100415e0     libucrt:lcidtoname_downlevel.obj
 0002:000045ec       ??_C@_1M@BNBLJCGH@?$AAe?$AAn?$AA?9?$AAI?$AAE@ 100415ec     libucrt:lcidtoname_downlevel.obj
 0002:000045f8       ??_C@_1M@GEPAFMDL@?$AAe?$AAs?$AA?9?$AAP?$AAA@ 100415f8     libucrt:lcidtoname_downlevel.obj
 0002:00004604       ??_C@_1M@OJONDMDL@?$AAf?$AAr?$AA?9?$AAM?$AAC@ 10041604     libucrt:lcidtoname_downlevel.obj
 0002:00004610       ??_C@_1BG@OBCNFJB@?$AAs?$AAr?$AA?9?$AAB?$AAA?$AA?9?$AAL?$AAa?$AAt?$AAn@ 10041610     libucrt:lcidtoname_downlevel.obj
 0002:00004628       ??_C@_1O@KEMEEGPO@?$AAs?$AAm?$AAa?$AA?9?$AAN?$AAO@ 10041628     libucrt:lcidtoname_downlevel.obj
 0002:00004638       ??_C@_1M@ELMGFODK@?$AAa?$AAr?$AA?9?$AAT?$AAN@ 10041638     libucrt:lcidtoname_downlevel.obj
 0002:00004644       ??_C@_1M@BHDLHFAF@?$AAe?$AAn?$AA?9?$AAZ?$AAA@ 10041644     libucrt:lcidtoname_downlevel.obj
 0002:00004650       ??_C@_1M@BMGIGLIF@?$AAe?$AAs?$AA?9?$AAD?$AAO@ 10041650     libucrt:lcidtoname_downlevel.obj
 0002:0000465c       ??_C@_1BG@CMBHIPBE@?$AAs?$AAr?$AA?9?$AAB?$AAA?$AA?9?$AAC?$AAy?$AAr?$AAl@ 1004165c     libucrt:lcidtoname_downlevel.obj
 0002:00004674       ??_C@_1O@HEDBLHNP@?$AAs?$AAm?$AAa?$AA?9?$AAS?$AAE@ 10041674     libucrt:lcidtoname_downlevel.obj
 0002:00004684       ??_C@_1M@DAGCADIM@?$AAa?$AAr?$AA?9?$AAO?$AAM@ 10041684     libucrt:lcidtoname_downlevel.obj
 0002:00004690       ??_C@_1M@FODLMICG@?$AAe?$AAn?$AA?9?$AAJ?$AAM@ 10041690     libucrt:lcidtoname_downlevel.obj
 0002:0000469c       ??_C@_1M@DNMLCIHB@?$AAe?$AAs?$AA?9?$AAV?$AAE@ 1004169c     libucrt:lcidtoname_downlevel.obj
 0002:000046a8       ??_C@_1O@EOKHMKJK@?$AAs?$AAm?$AAs?$AA?9?$AAF?$AAI@ 100416a8     libucrt:lcidtoname_downlevel.obj
 0002:000046b8       ??_C@_1M@CAFJMKOF@?$AAa?$AAr?$AA?9?$AAY?$AAE@ 100416b8     libucrt:lcidtoname_downlevel.obj
 0002:000046c4       ??_C@_1M@CBFHIJLI@?$AAe?$AAn?$AA?9?$AAC?$AAB@ 100416c4     libucrt:lcidtoname_downlevel.obj
 0002:000046d0       ??_C@_1M@BGNFLDN@?$AAe?$AAs?$AA?9?$AAC?$AAO@ 100416d0     libucrt:lcidtoname_downlevel.obj
 0002:000046dc       ??_C@_1O@JMPHMAMC@?$AAs?$AAm?$AAn?$AA?9?$AAF?$AAI@ 100416dc     libucrt:lcidtoname_downlevel.obj
 0002:000046ec       ??_C@_1M@JLANABKE@?$AAa?$AAr?$AA?9?$AAS?$AAY@ 100416ec     libucrt:lcidtoname_downlevel.obj
 0002:000046f8       ??_C@_1M@HPKGCFGN@?$AAe?$AAn?$AA?9?$AAB?$AAZ@ 100416f8     libucrt:lcidtoname_downlevel.obj
 0002:00004704       ??_C@_1M@OLJCMLGM@?$AAe?$AAs?$AA?9?$AAP?$AAE@ 10041704     libucrt:lcidtoname_downlevel.obj
 0002:00004710       ??_C@_1M@MKKGFKLE@?$AAa?$AAr?$AA?9?$AAJ?$AAO@ 10041710     libucrt:lcidtoname_downlevel.obj
 0002:0000471c       ??_C@_1M@EKPGLDNI@?$AAe?$AAn?$AA?9?$AAT?$AAT@ 1004171c     libucrt:lcidtoname_downlevel.obj
 0002:00004728       ??_C@_1M@OONGHFHE@?$AAe?$AAs?$AA?9?$AAA?$AAR@ 10041728     libucrt:lcidtoname_downlevel.obj
 0002:00004734       ??_C@_1M@OOJFGBHE@?$AAa?$AAr?$AA?9?$AAL?$AAB@ 10041734     libucrt:lcidtoname_downlevel.obj
 0002:00004740       ??_C@_1M@GCEJHNEG@?$AAe?$AAn?$AA?9?$AAZ?$AAW@ 10041740     libucrt:lcidtoname_downlevel.obj
 0002:0000474c       ??_C@_1M@JNOCAHJI@?$AAe?$AAs?$AA?9?$AAE?$AAC@ 1004174c     libucrt:lcidtoname_downlevel.obj
 0002:00004758       ??_C@_1M@JEFHPGGB@?$AAa?$AAr?$AA?9?$AAK?$AAW@ 10041758     libucrt:lcidtoname_downlevel.obj
 0002:00004764       ??_C@_1M@MLKIBJOJ@?$AAe?$AAn?$AA?9?$AAP?$AAH@ 10041764     libucrt:lcidtoname_downlevel.obj
 0002:00004770       ??_C@_1M@BDNIPEND@?$AAe?$AAs?$AA?9?$AAC?$AAL@ 10041770     libucrt:lcidtoname_downlevel.obj
 0002:0000477c       ??_C@_1M@MPNMEKBD@?$AAa?$AAr?$AA?9?$AAA?$AAE@ 1004177c     libucrt:lcidtoname_downlevel.obj
 0002:00004788       ??_C@_1M@KBJALCPI@?$AAe?$AAs?$AA?9?$AAU?$AAY@ 10041788     libucrt:lcidtoname_downlevel.obj
 0002:00004794       ??_C@_1M@LLCCOAGA@?$AAa?$AAr?$AA?9?$AAB?$AAH@ 10041794     libucrt:lcidtoname_downlevel.obj
 0002:000047a0       ??_C@_1M@PBFNCDEL@?$AAe?$AAs?$AA?9?$AAP?$AAY@ 100417a0     libucrt:lcidtoname_downlevel.obj
 0002:000047ac       ??_C@_1M@EDGINPNP@?$AAa?$AAr?$AA?9?$AAQ?$AAA@ 100417ac     libucrt:lcidtoname_downlevel.obj
 0002:000047b8       ??_C@_1M@MKDBIIJI@?$AAe?$AAs?$AA?9?$AAB?$AAO@ 100417b8     libucrt:lcidtoname_downlevel.obj
 0002:000047c4       ??_C@_1M@CPKKEBLD@?$AAe?$AAs?$AA?9?$AAS?$AAV@ 100417c4     libucrt:lcidtoname_downlevel.obj
 0002:000047d0       ??_C@_1M@NDBGMMJL@?$AAe?$AAs?$AA?9?$AAH?$AAN@ 100417d0     libucrt:lcidtoname_downlevel.obj
 0002:000047dc       ??_C@_1M@JIJIBHDP@?$AAe?$AAs?$AA?9?$AAN?$AAI@ 100417dc     libucrt:lcidtoname_downlevel.obj
 0002:000047e8       ??_C@_1M@CGFMKEEK@?$AAe?$AAs?$AA?9?$AAP?$AAR@ 100417e8     libucrt:lcidtoname_downlevel.obj
 0002:000047f4       ??_C@_1O@ICJHKIIK@?$AAz?$AAh?$AA?9?$AAC?$AAH?$AAT@ 100417f4     libucrt:lcidtoname_downlevel.obj
 0002:00004804       ??_C@_15CLNEJCE@?$AAs?$AAr@ 10041804     libucrt:lcidtoname_downlevel.obj
 0002:00004f30       ??_C@_1M@KAHEKEIG@?$AAa?$AAf?$AA?9?$AAz?$AAa@ 10041f30     libucrt:lcidtoname_downlevel.obj
 0002:00004f3c       ??_C@_1M@GIECOABL@?$AAa?$AAr?$AA?9?$AAa?$AAe@ 10041f3c     libucrt:lcidtoname_downlevel.obj
 0002:00004f48       ??_C@_1M@BMLMEKGI@?$AAa?$AAr?$AA?9?$AAb?$AAh@ 10041f48     libucrt:lcidtoname_downlevel.obj
 0002:00004f54       ??_C@_1M@DAPFDGGB@?$AAa?$AAr?$AA?9?$AAd?$AAz@ 10041f54     libucrt:lcidtoname_downlevel.obj
 0002:00004f60       ??_C@_1M@FJNKGKIG@?$AAa?$AAr?$AA?9?$AAe?$AAg@ 10041f60     libucrt:lcidtoname_downlevel.obj
 0002:00004f6c       ??_C@_1M@FLGKKCLO@?$AAa?$AAr?$AA?9?$AAi?$AAq@ 10041f6c     libucrt:lcidtoname_downlevel.obj
 0002:00004f78       ??_C@_1M@GNDIPALM@?$AAa?$AAr?$AA?9?$AAj?$AAo@ 10041f78     libucrt:lcidtoname_downlevel.obj
 0002:00004f84       ??_C@_1M@DDMJFMGJ@?$AAa?$AAr?$AA?9?$AAk?$AAw@ 10041f84     libucrt:lcidtoname_downlevel.obj
 0002:00004f90       ??_C@_1M@EJALMLHM@?$AAa?$AAr?$AA?9?$AAl?$AAb@ 10041f90     libucrt:lcidtoname_downlevel.obj
 0002:00004f9c       ??_C@_1M@MOBDBLOC@?$AAa?$AAr?$AA?9?$AAl?$AAy@ 10041f9c     libucrt:lcidtoname_downlevel.obj
 0002:00004fa8       ??_C@_1M@JAOCLHDH@?$AAa?$AAr?$AA?9?$AAm?$AAa@ 10041fa8     libucrt:lcidtoname_downlevel.obj
 0002:00004fb4       ??_C@_1M@JHPMKJIE@?$AAa?$AAr?$AA?9?$AAo?$AAm@ 10041fb4     libucrt:lcidtoname_downlevel.obj
 0002:00004fc0       ??_C@_1M@OEPGHFNH@?$AAa?$AAr?$AA?9?$AAq?$AAa@ 10041fc0     libucrt:lcidtoname_downlevel.obj
 0002:00004fcc       ??_C@_1M@KJDONENM@?$AAa?$AAr?$AA?9?$AAs?$AAa@ 10041fcc     libucrt:lcidtoname_downlevel.obj
 0002:00004fd8       ??_C@_1M@DMJDKLKM@?$AAa?$AAr?$AA?9?$AAs?$AAy@ 10041fd8     libucrt:lcidtoname_downlevel.obj
 0002:00004fe4       ??_C@_1M@OMFIPEDC@?$AAa?$AAr?$AA?9?$AAt?$AAn@ 10041fe4     libucrt:lcidtoname_downlevel.obj
 0002:00004ff0       ??_C@_1M@IHMHGAON@?$AAa?$AAr?$AA?9?$AAy?$AAe@ 10041ff0     libucrt:lcidtoname_downlevel.obj
 0002:00004ffc       ??_C@_1BG@KDCPGJGB@?$AAa?$AAz?$AA?9?$AAa?$AAz?$AA?9?$AAc?$AAy?$AAr?$AAl@ 10041ffc     libucrt:lcidtoname_downlevel.obj
 0002:00005014       ??_C@_1BG@IBCKDDOE@?$AAa?$AAz?$AA?9?$AAa?$AAz?$AA?9?$AAl?$AAa?$AAt?$AAn@ 10042014     libucrt:lcidtoname_downlevel.obj
 0002:0000502c       ??_C@_1M@EGPFDCPD@?$AAb?$AAe?$AA?9?$AAb?$AAy@ 1004202c     libucrt:lcidtoname_downlevel.obj
 0002:00005038       ??_C@_1M@PCMGMCGC@?$AAb?$AAg?$AA?9?$AAb?$AAg@ 10042038     libucrt:lcidtoname_downlevel.obj
 0002:00005044       ??_C@_1M@BJBMFGOB@?$AAb?$AAn?$AA?9?$AAi?$AAn@ 10042044     libucrt:lcidtoname_downlevel.obj
 0002:00005050       ??_C@_1BG@EAKMMACD@?$AAb?$AAs?$AA?9?$AAb?$AAa?$AA?9?$AAl?$AAa?$AAt?$AAn@ 10042050     libucrt:lcidtoname_downlevel.obj
 0002:00005068       ??_C@_1M@KGADAODK@?$AAc?$AAa?$AA?9?$AAe?$AAs@ 10042068     libucrt:lcidtoname_downlevel.obj
 0002:00005074       ??_C@_1M@COAJPDHI@?$AAc?$AAs?$AA?9?$AAc?$AAz@ 10042074     libucrt:lcidtoname_downlevel.obj
 0002:00005080       ??_C@_1M@DHBHFONH@?$AAc?$AAy?$AA?9?$AAg?$AAb@ 10042080     libucrt:lcidtoname_downlevel.obj
 0002:0000508c       ??_C@_1M@IMGKELGA@?$AAd?$AAa?$AA?9?$AAd?$AAk@ 1004208c     libucrt:lcidtoname_downlevel.obj
 0002:00005098       ??_C@_1M@NNDGDNGA@?$AAd?$AAe?$AA?9?$AAa?$AAt@ 10042098     libucrt:lcidtoname_downlevel.obj
 0002:000050a4       ??_C@_1M@IKDBHEEM@?$AAd?$AAe?$AA?9?$AAc?$AAh@ 100420a4     libucrt:lcidtoname_downlevel.obj
 0002:000050b0       ??_C@_1M@GFFOJMCJ@?$AAd?$AAe?$AA?9?$AAd?$AAe@ 100420b0     libucrt:lcidtoname_downlevel.obj
 0002:000050bc       ??_C@_1M@MDNLKBPM@?$AAd?$AAe?$AA?9?$AAl?$AAi@ 100420bc     libucrt:lcidtoname_downlevel.obj
 0002:000050c8       ??_C@_1M@NJBEEJNL@?$AAd?$AAe?$AA?9?$AAl?$AAu@ 100420c8     libucrt:lcidtoname_downlevel.obj
 0002:000050d4       ??_C@_1O@GNNELBAP@?$AAd?$AAi?$AAv?$AA?9?$AAm?$AAv@ 100420d4     libucrt:lcidtoname_downlevel.obj
 0002:000050e4       ??_C@_1M@EJLEOGAE@?$AAe?$AAl?$AA?9?$AAg?$AAr@ 100420e4     libucrt:lcidtoname_downlevel.obj
 0002:000050f0       ??_C@_1M@GMPONJN@?$AAe?$AAn?$AA?9?$AAa?$AAu@ 100420f0     libucrt:lcidtoname_downlevel.obj
 0002:000050fc       ??_C@_1M@NIDIIPGF@?$AAe?$AAn?$AA?9?$AAb?$AAz@ 100420fc     libucrt:lcidtoname_downlevel.obj
 0002:00005108       ??_C@_1M@JEHMIMFO@?$AAe?$AAn?$AA?9?$AAc?$AAa@ 10042108     libucrt:lcidtoname_downlevel.obj
 0002:00005114       ??_C@_1M@IGMJCDLA@?$AAe?$AAn?$AA?9?$AAc?$AAb@ 10042114     libucrt:lcidtoname_downlevel.obj
 0002:00005120       ??_C@_1M@BNFIGBKG@?$AAe?$AAn?$AA?9?$AAg?$AAb@ 10042120     libucrt:lcidtoname_downlevel.obj
 0002:0000512c       ??_C@_1M@LKIFDIGP@?$AAe?$AAn?$AA?9?$AAi?$AAe@ 1004212c     libucrt:lcidtoname_downlevel.obj
 0002:00005138       ??_C@_1M@PJKFGCCO@?$AAe?$AAn?$AA?9?$AAj?$AAm@ 10042138     libucrt:lcidtoname_downlevel.obj
 0002:00005144       ??_C@_1M@KPPKEPBO@?$AAe?$AAn?$AA?9?$AAn?$AAz@ 10042144     libucrt:lcidtoname_downlevel.obj
 0002:00005150       ??_C@_1M@GMDGLDOB@?$AAe?$AAn?$AA?9?$AAp?$AAh@ 10042150     libucrt:lcidtoname_downlevel.obj
 0002:0000515c       ??_C@_1M@ONGIBJNA@?$AAe?$AAn?$AA?9?$AAt?$AAt@ 1004215c     libucrt:lcidtoname_downlevel.obj
 0002:00005168       ??_C@_1M@LLODPCMM@?$AAe?$AAn?$AA?9?$AAu?$AAs@ 10042168     libucrt:lcidtoname_downlevel.obj
 0002:00005174       ??_C@_1M@LAKFNPAN@?$AAe?$AAn?$AA?9?$AAz?$AAa@ 10042174     libucrt:lcidtoname_downlevel.obj
 0002:00005180       ??_C@_1M@MFNHNHEO@?$AAe?$AAn?$AA?9?$AAz?$AAw@ 10042180     libucrt:lcidtoname_downlevel.obj
 0002:0000518c       ??_C@_1M@EJEINPHM@?$AAe?$AAs?$AA?9?$AAa?$AAr@ 1004218c     libucrt:lcidtoname_downlevel.obj
 0002:00005198       ??_C@_1M@GNKPCCJA@?$AAe?$AAs?$AA?9?$AAb?$AAo@ 10042198     libucrt:lcidtoname_downlevel.obj
 0002:000051a4       ??_C@_1M@LEEGFONL@?$AAe?$AAs?$AA?9?$AAc?$AAl@ 100421a4     libucrt:lcidtoname_downlevel.obj
 0002:000051b0       ??_C@_1M@KGPDPBDF@?$AAe?$AAs?$AA?9?$AAc?$AAo@ 100421b0     libucrt:lcidtoname_downlevel.obj
 0002:000051bc       ??_C@_1M@EIAHOHH@?$AAe?$AAs?$AA?9?$AAc?$AAr@ 100421bc     libucrt:lcidtoname_downlevel.obj
 0002:000051c8       ??_C@_1M@LLPGMBIN@?$AAe?$AAs?$AA?9?$AAd?$AAo@ 100421c8     libucrt:lcidtoname_downlevel.obj
 0002:000051d4       ??_C@_1M@DKHMKNJA@?$AAe?$AAs?$AA?9?$AAe?$AAc@ 100421d4     libucrt:lcidtoname_downlevel.obj
 0002:000051e0       ??_C@_1M@GKGFPKAP@?$AAe?$AAs?$AA?9?$AAe?$AAs@ 100421e0     libucrt:lcidtoname_downlevel.obj
 0002:000051ec       ??_C@_1M@LKHKGDLN@?$AAe?$AAs?$AA?9?$AAg?$AAt@ 100421ec     libucrt:lcidtoname_downlevel.obj
 0002:000051f8       ??_C@_1M@HEIIGGJD@?$AAe?$AAs?$AA?9?$AAh?$AAn@ 100421f8     libucrt:lcidtoname_downlevel.obj
 0002:00005204       ??_C@_1M@FBDHPPGD@?$AAe?$AAs?$AA?9?$AAm?$AAx@ 10042204     libucrt:lcidtoname_downlevel.obj
 0002:00005210       ??_C@_1M@DPAGLNDH@?$AAe?$AAs?$AA?9?$AAn?$AAi@ 10042210     libucrt:lcidtoname_downlevel.obj
 0002:0000521c       ??_C@_1M@MDGOPGDD@?$AAe?$AAs?$AA?9?$AAp?$AAa@ 1004221c     libucrt:lcidtoname_downlevel.obj
 0002:00005228       ??_C@_1M@EMAMGBGE@?$AAe?$AAs?$AA?9?$AAp?$AAe@ 10042228     libucrt:lcidtoname_downlevel.obj
 0002:00005234       ??_C@_1M@IBMCAOEC@?$AAe?$AAs?$AA?9?$AAp?$AAr@ 10042234     libucrt:lcidtoname_downlevel.obj
 0002:00005240       ??_C@_1M@FGMDIJED@?$AAe?$AAs?$AA?9?$AAp?$AAy@ 10042240     libucrt:lcidtoname_downlevel.obj
 0002:0000524c       ??_C@_1M@IIDEOLLL@?$AAe?$AAs?$AA?9?$AAs?$AAv@ 1004224c     libucrt:lcidtoname_downlevel.obj
 0002:00005258       ??_C@_1M@GAOBIPA@?$AAe?$AAs?$AA?9?$AAu?$AAy@ 10042258     libucrt:lcidtoname_downlevel.obj
 0002:00005264       ??_C@_1M@JKFFICHJ@?$AAe?$AAs?$AA?9?$AAv?$AAe@ 10042264     libucrt:lcidtoname_downlevel.obj
 0002:00005270       ??_C@_1M@PNMLOJDF@?$AAe?$AAt?$AA?9?$AAe?$AAe@ 10042270     libucrt:lcidtoname_downlevel.obj
 0002:0000527c       ??_C@_1M@GHHLIKEI@?$AAe?$AAu?$AA?9?$AAe?$AAs@ 1004227c     libucrt:lcidtoname_downlevel.obj
 0002:00005288       ??_C@_1M@PBNONODE@?$AAf?$AAa?$AA?9?$AAi?$AAr@ 10042288     libucrt:lcidtoname_downlevel.obj
 0002:00005294       ??_C@_1M@JEEHPMIL@?$AAf?$AAi?$AA?9?$AAf?$AAi@ 10042294     libucrt:lcidtoname_downlevel.obj
 0002:000052a0       ??_C@_1M@LMDCNDBA@?$AAf?$AAo?$AA?9?$AAf?$AAo@ 100422a0     libucrt:lcidtoname_downlevel.obj
 0002:000052ac       ??_C@_1M@JKEOHLDK@?$AAf?$AAr?$AA?9?$AAb?$AAe@ 100422ac     libucrt:lcidtoname_downlevel.obj
 0002:000052b8       ??_C@_1M@NOHADPMI@?$AAf?$AAr?$AA?9?$AAc?$AAa@ 100422b8     libucrt:lcidtoname_downlevel.obj
 0002:000052c4       ??_C@_1M@KDHIHAEC@?$AAf?$AAr?$AA?9?$AAc?$AAh@ 100422c4     libucrt:lcidtoname_downlevel.obj
 0002:000052d0       ??_C@_1M@MMBBFGAK@?$AAf?$AAr?$AA?9?$AAf?$AAr@ 100422d0     libucrt:lcidtoname_downlevel.obj
 0002:000052dc       ??_C@_1M@PAFNENNF@?$AAf?$AAr?$AA?9?$AAl?$AAu@ 100422dc     libucrt:lcidtoname_downlevel.obj
 0002:000052e8       ??_C@_1M@EOHDJGDD@?$AAf?$AAr?$AA?9?$AAm?$AAc@ 100422e8     libucrt:lcidtoname_downlevel.obj
 0002:000052f4       ??_C@_1M@FAPLLOPF@?$AAg?$AAl?$AA?9?$AAe?$AAs@ 100422f4     libucrt:lcidtoname_downlevel.obj
 0002:00005300       ??_C@_1M@FOPBFLOO@?$AAg?$AAu?$AA?9?$AAi?$AAn@ 10042300     libucrt:lcidtoname_downlevel.obj
 0002:0000530c       ??_C@_1M@KBMCINPM@?$AAh?$AAe?$AA?9?$AAi?$AAl@ 1004230c     libucrt:lcidtoname_downlevel.obj
 0002:00005318       ??_C@_1M@BBPHKFPJ@?$AAh?$AAi?$AA?9?$AAi?$AAn@ 10042318     libucrt:lcidtoname_downlevel.obj
 0002:00005324       ??_C@_1M@PMBNDPHD@?$AAh?$AAr?$AA?9?$AAb?$AAa@ 10042324     libucrt:lcidtoname_downlevel.obj
 0002:00005330       ??_C@_1M@BPCKOEGE@?$AAh?$AAr?$AA?9?$AAh?$AAr@ 10042330     libucrt:lcidtoname_downlevel.obj
 0002:0000533c       ??_C@_1M@GACBMHKE@?$AAh?$AAu?$AA?9?$AAh?$AAu@ 1004233c     libucrt:lcidtoname_downlevel.obj
 0002:00005348       ??_C@_1M@MILPAJJC@?$AAh?$AAy?$AA?9?$AAa?$AAm@ 10042348     libucrt:lcidtoname_downlevel.obj
 0002:00005354       ??_C@_1M@BABBICEC@?$AAi?$AAd?$AA?9?$AAi?$AAd@ 10042354     libucrt:lcidtoname_downlevel.obj
 0002:00005360       ??_C@_1M@BIKNHHPF@?$AAi?$AAs?$AA?9?$AAi?$AAs@ 10042360     libucrt:lcidtoname_downlevel.obj
 0002:0000536c       ??_C@_1M@NMPCJPHE@?$AAi?$AAt?$AA?9?$AAc?$AAh@ 1004236c     libucrt:lcidtoname_downlevel.obj
 0002:00005378       ??_C@_1M@GHKGFEDF@?$AAi?$AAt?$AA?9?$AAi?$AAt@ 10042378     libucrt:lcidtoname_downlevel.obj
 0002:00005384       ??_C@_1M@NIEJCJJA@?$AAj?$AAa?$AA?9?$AAj?$AAp@ 10042384     libucrt:lcidtoname_downlevel.obj
 0002:00005390       ??_C@_1M@JILFNBIM@?$AAk?$AAa?$AA?9?$AAg?$AAe@ 10042390     libucrt:lcidtoname_downlevel.obj
 0002:0000539c       ??_C@_1M@PACPMGPH@?$AAk?$AAk?$AA?9?$AAk?$AAz@ 1004239c     libucrt:lcidtoname_downlevel.obj
 0002:000053a8       ??_C@_1M@IELFGMHA@?$AAk?$AAn?$AA?9?$AAi?$AAn@ 100423a8     libucrt:lcidtoname_downlevel.obj
 0002:000053b4       ??_C@_1O@IBBJHCH@?$AAk?$AAo?$AAk?$AA?9?$AAi?$AAn@ 100423b4     libucrt:lcidtoname_downlevel.obj
 0002:000053c4       ??_C@_1M@DMHAEOGC@?$AAk?$AAo?$AA?9?$AAk?$AAr@ 100423c4     libucrt:lcidtoname_downlevel.obj
 0002:000053d0       ??_C@_1M@HBAHBIGA@?$AAk?$AAy?$AA?9?$AAk?$AAg@ 100423d0     libucrt:lcidtoname_downlevel.obj
 0002:000053dc       ??_C@_1M@KPMILCJG@?$AAl?$AAt?$AA?9?$AAl?$AAt@ 100423dc     libucrt:lcidtoname_downlevel.obj
 0002:000053e8       ??_C@_1M@BDEKKCA@?$AAl?$AAv?$AA?9?$AAl?$AAv@ 100423e8     libucrt:lcidtoname_downlevel.obj
 0002:000053f4       ??_C@_1M@ELCKCCJJ@?$AAm?$AAi?$AA?9?$AAn?$AAz@ 100423f4     libucrt:lcidtoname_downlevel.obj
 0002:00005400       ??_C@_1M@CBOOLAPA@?$AAm?$AAk?$AA?9?$AAm?$AAk@ 10042400     libucrt:lcidtoname_downlevel.obj
 0002:0000540c       ??_C@_1M@GPHNBJKN@?$AAm?$AAl?$AA?9?$AAi?$AAn@ 1004240c     libucrt:lcidtoname_downlevel.obj
 0002:00005418       ??_C@_1M@PABJILIG@?$AAm?$AAn?$AA?9?$AAm?$AAn@ 10042418     libucrt:lcidtoname_downlevel.obj
 0002:00005424       ??_C@_1M@FGBKKIPG@?$AAm?$AAr?$AA?9?$AAi?$AAn@ 10042424     libucrt:lcidtoname_downlevel.obj
 0002:00005430       ??_C@_1M@NDBPDDAL@?$AAm?$AAs?$AA?9?$AAb?$AAn@ 10042430     libucrt:lcidtoname_downlevel.obj
 0002:0000543c       ??_C@_1M@OPIHOOPI@?$AAm?$AAs?$AA?9?$AAm?$AAy@ 1004243c     libucrt:lcidtoname_downlevel.obj
 0002:00005448       ??_C@_1M@PPDBCNFM@?$AAm?$AAt?$AA?9?$AAm?$AAt@ 10042448     libucrt:lcidtoname_downlevel.obj
 0002:00005454       ??_C@_1M@KDJDKMDD@?$AAn?$AAb?$AA?9?$AAn?$AAo@ 10042454     libucrt:lcidtoname_downlevel.obj
 0002:00005460       ??_C@_1M@KFCFLMJP@?$AAn?$AAl?$AA?9?$AAb?$AAe@ 10042460     libucrt:lcidtoname_downlevel.obj
 0002:0000546c       ??_C@_1M@KPOPDDGO@?$AAn?$AAl?$AA?9?$AAn?$AAl@ 1004246c     libucrt:lcidtoname_downlevel.obj
 0002:00005478       ??_C@_1M@LJKPEMLN@?$AAn?$AAn?$AA?9?$AAn?$AAo@ 10042478     libucrt:lcidtoname_downlevel.obj
 0002:00005484       ??_C@_1M@BDGHHBFL@?$AAn?$AAs?$AA?9?$AAz?$AAa@ 10042484     libucrt:lcidtoname_downlevel.obj
 0002:00005490       ??_C@_1M@IDEHOAP@?$AAp?$AAa?$AA?9?$AAi?$AAn@ 10042490     libucrt:lcidtoname_downlevel.obj
 0002:0000549c       ??_C@_1M@HDBKGOGH@?$AAp?$AAl?$AA?9?$AAp?$AAl@ 1004249c     libucrt:lcidtoname_downlevel.obj
 0002:000054a8       ??_C@_1M@LJLLCMEH@?$AAp?$AAt?$AA?9?$AAb?$AAr@ 100424a8     libucrt:lcidtoname_downlevel.obj
 0002:000054b4       ??_C@_1M@NCMONAAL@?$AAp?$AAt?$AA?9?$AAp?$AAt@ 100424b4     libucrt:lcidtoname_downlevel.obj
 0002:000054c0       ??_C@_1O@EAKMAJDN@?$AAq?$AAu?$AAz?$AA?9?$AAb?$AAo@ 100424c0     libucrt:lcidtoname_downlevel.obj
 0002:000054d0       ??_C@_1O@BHHPIGDN@?$AAq?$AAu?$AAz?$AA?9?$AAe?$AAc@ 100424d0     libucrt:lcidtoname_downlevel.obj
 0002:000054e0       ??_C@_1O@GBAPEKMJ@?$AAq?$AAu?$AAz?$AA?9?$AAp?$AAe@ 100424e0     libucrt:lcidtoname_downlevel.obj
 0002:000054f0       ??_C@_1M@CLGLEFBO@?$AAr?$AAo?$AA?9?$AAr?$AAo@ 100424f0     libucrt:lcidtoname_downlevel.obj
 0002:000054fc       ??_C@_1M@CEEDODME@?$AAr?$AAu?$AA?9?$AAr?$AAu@ 100424fc     libucrt:lcidtoname_downlevel.obj
 0002:00005508       ??_C@_1M@HPKKKMPP@?$AAs?$AAa?$AA?9?$AAi?$AAn@ 10042508     libucrt:lcidtoname_downlevel.obj
 0002:00005514       ??_C@_1M@BKMAIGOJ@?$AAs?$AAe?$AA?9?$AAf?$AAi@ 10042514     libucrt:lcidtoname_downlevel.obj
 0002:00005520       ??_C@_1M@NDPIFLFI@?$AAs?$AAe?$AA?9?$AAn?$AAo@ 10042520     libucrt:lcidtoname_downlevel.obj
 0002:0000552c       ??_C@_1M@DANKKHJ@?$AAs?$AAe?$AA?9?$AAs?$AAe@ 1004252c     libucrt:lcidtoname_downlevel.obj
 0002:00005538       ??_C@_1M@PNBLONPJ@?$AAs?$AAk?$AA?9?$AAs?$AAk@ 10042538     libucrt:lcidtoname_downlevel.obj
 0002:00005544       ??_C@_1M@LFMODOAL@?$AAs?$AAl?$AA?9?$AAs?$AAi@ 10042544     libucrt:lcidtoname_downlevel.obj
 0002:00005550       ??_C@_1O@DFKOMPG@?$AAs?$AAm?$AAa?$AA?9?$AAn?$AAo@ 10042550     libucrt:lcidtoname_downlevel.obj
 0002:00005560       ??_C@_1O@NDKPBNNH@?$AAs?$AAm?$AAa?$AA?9?$AAs?$AAe@ 10042560     libucrt:lcidtoname_downlevel.obj
 0002:00005570       ??_C@_1O@PLLKBHAB@?$AAs?$AAm?$AAj?$AA?9?$AAn?$AAo@ 10042570     libucrt:lcidtoname_downlevel.obj
 0002:00005580       ??_C@_1O@CLEPOGCA@?$AAs?$AAm?$AAj?$AA?9?$AAs?$AAe@ 10042580     libucrt:lcidtoname_downlevel.obj
 0002:00005590       ??_C@_1O@DLGJGKMK@?$AAs?$AAm?$AAn?$AA?9?$AAf?$AAi@ 10042590     libucrt:lcidtoname_downlevel.obj
 0002:000055a0       ??_C@_1O@OJDJGAJC@?$AAs?$AAm?$AAs?$AA?9?$AAf?$AAi@ 100425a0     libucrt:lcidtoname_downlevel.obj
 0002:000055b0       ??_C@_1M@BOFOGHPB@?$AAs?$AAq?$AA?9?$AAa?$AAl@ 100425b0     libucrt:lcidtoname_downlevel.obj
 0002:000055bc       ??_C@_1BG@LJBBIPGB@?$AAs?$AAr?$AA?9?$AAb?$AAa?$AA?9?$AAc?$AAy?$AAr?$AAl@ 100425bc     libucrt:lcidtoname_downlevel.obj
 0002:000055d4       ??_C@_1BG@JLBENFOE@?$AAs?$AAr?$AA?9?$AAb?$AAa?$AA?9?$AAl?$AAa?$AAt?$AAn@ 100425d4     libucrt:lcidtoname_downlevel.obj
 0002:000055ec       ??_C@_1BG@KODPNHE@?$AAs?$AAr?$AA?9?$AAs?$AAp?$AA?9?$AAc?$AAy?$AAr?$AAl@ 100425ec     libucrt:lcidtoname_downlevel.obj
 0002:00005604       ??_C@_1BG@CIOGKHPB@?$AAs?$AAr?$AA?9?$AAs?$AAp?$AA?9?$AAl?$AAa?$AAt?$AAn@ 10042604     libucrt:lcidtoname_downlevel.obj
 0002:0000561c       ??_C@_1M@NGFJLMAC@?$AAs?$AAv?$AA?9?$AAf?$AAi@ 1004261c     libucrt:lcidtoname_downlevel.obj
 0002:00005628       ??_C@_1M@MPJEJAJC@?$AAs?$AAv?$AA?9?$AAs?$AAe@ 10042628     libucrt:lcidtoname_downlevel.obj
 0002:00005634       ??_C@_1M@MPNDHLFK@?$AAs?$AAw?$AA?9?$AAk?$AAe@ 10042634     libucrt:lcidtoname_downlevel.obj
 0002:00005640       ??_C@_1O@KOHBJJI@?$AAs?$AAy?$AAr?$AA?9?$AAs?$AAy@ 10042640     libucrt:lcidtoname_downlevel.obj
 0002:00005650       ??_C@_1M@LDCEFHA@?$AAt?$AAa?$AA?9?$AAi?$AAn@ 10042650     libucrt:lcidtoname_downlevel.obj
 0002:0000565c       ??_C@_1M@CNJOFAK@?$AAt?$AAe?$AA?9?$AAi?$AAn@ 1004265c     libucrt:lcidtoname_downlevel.obj
 0002:00005668       ??_C@_1M@GNAECACD@?$AAt?$AAh?$AA?9?$AAt?$AAh@ 10042668     libucrt:lcidtoname_downlevel.obj
 0002:00005674       ??_C@_1M@CHBIHOJO@?$AAt?$AAn?$AA?9?$AAz?$AAa@ 10042674     libucrt:lcidtoname_downlevel.obj
 0002:00005680       ??_C@_1M@GCCMIGPJ@?$AAt?$AAr?$AA?9?$AAt?$AAr@ 10042680     libucrt:lcidtoname_downlevel.obj
 0002:0000568c       ??_C@_1M@CELMCNBK@?$AAt?$AAt?$AA?9?$AAr?$AAu@ 1004268c     libucrt:lcidtoname_downlevel.obj
 0002:00005698       ??_C@_1M@KLMCELGA@?$AAu?$AAk?$AA?9?$AAu?$AAa@ 10042698     libucrt:lcidtoname_downlevel.obj
 0002:000056a4       ??_C@_1M@EPAJJAJF@?$AAu?$AAr?$AA?9?$AAp?$AAk@ 100426a4     libucrt:lcidtoname_downlevel.obj
 0002:000056b0       ??_C@_1BG@GEGPMCDJ@?$AAu?$AAz?$AA?9?$AAu?$AAz?$AA?9?$AAc?$AAy?$AAr?$AAl@ 100426b0     libucrt:lcidtoname_downlevel.obj
 0002:000056c8       ??_C@_1BG@EGGKJILM@?$AAu?$AAz?$AA?9?$AAu?$AAz?$AA?9?$AAl?$AAa?$AAt?$AAn@ 100426c8     libucrt:lcidtoname_downlevel.obj
 0002:000056e0       ??_C@_1M@GFOCLFF@?$AAv?$AAi?$AA?9?$AAv?$AAn@ 100426e0     libucrt:lcidtoname_downlevel.obj
 0002:000056ec       ??_C@_1M@CPAMEDFI@?$AAx?$AAh?$AA?9?$AAz?$AAa@ 100426ec     libucrt:lcidtoname_downlevel.obj
 0002:000056f8       ??_C@_1O@EBKIFIGN@?$AAz?$AAh?$AA?9?$AAc?$AAh?$AAs@ 100426f8     libucrt:lcidtoname_downlevel.obj
 0002:00005708       ??_C@_1O@NMHPGANE@?$AAz?$AAh?$AA?9?$AAc?$AAh?$AAt@ 10042708     libucrt:lcidtoname_downlevel.obj
 0002:00005718       ??_C@_1M@LPINJOMC@?$AAz?$AAh?$AA?9?$AAc?$AAn@ 10042718     libucrt:lcidtoname_downlevel.obj
 0002:00005724       ??_C@_1M@OCJEJODD@?$AAz?$AAh?$AA?9?$AAh?$AAk@ 10042724     libucrt:lcidtoname_downlevel.obj
 0002:00005730       ??_C@_1M@DNDLJINH@?$AAz?$AAh?$AA?9?$AAm?$AAo@ 10042730     libucrt:lcidtoname_downlevel.obj
 0002:0000573c       ??_C@_1M@MBFDNDND@?$AAz?$AAh?$AA?9?$AAs?$AAg@ 1004273c     libucrt:lcidtoname_downlevel.obj
 0002:00005748       ??_C@_1M@IMEPLEPE@?$AAz?$AAh?$AA?9?$AAt?$AAw@ 10042748     libucrt:lcidtoname_downlevel.obj
 0002:00005754       ??_C@_1M@BBGHNHJP@?$AAz?$AAu?$AA?9?$AAz?$AAa@ 10042754     libucrt:lcidtoname_downlevel.obj
 0002:00005760       ___acrt_rg_language        10042760     libucrt:get_qualified_locale.obj
 0002:00005a6c       ___acrt_rg_language_count  10042a6c     libucrt:get_qualified_locale.obj
 0002:00005a70       ___acrt_rg_country         10042a70     libucrt:get_qualified_locale.obj
 0002:00005b84       ___acrt_rg_country_count   10042b84     libucrt:get_qualified_locale.obj
 0002:00005b88       ??_C@_1BC@LLOKLNP@?$AAa?$AAm?$AAe?$AAr?$AAi?$AAc?$AAa?$AAn@ 10042b88     libucrt:get_qualified_locale.obj
 0002:00005b9c       ??_C@_1CC@HEIGCDGG@?$AAa?$AAm?$AAe?$AAr?$AAi?$AAc?$AAa?$AAn?$AA?5?$AAe?$AAn?$AAg?$AAl?$AAi?$AAs@ 10042b9c     libucrt:get_qualified_locale.obj
 0002:00005bc0       ??_C@_1CC@IHCNOMIN@?$AAa?$AAm?$AAe?$AAr?$AAi?$AAc?$AAa?$AAn?$AA?9?$AAe?$AAn?$AAg?$AAl?$AAi?$AAs@ 10042bc0     libucrt:get_qualified_locale.obj
 0002:00005be4       ??_C@_1BG@GKAGPCGG@?$AAa?$AAu?$AAs?$AAt?$AAr?$AAa?$AAl?$AAi?$AAa?$AAn@ 10042be4     libucrt:get_qualified_locale.obj
 0002:00005bfc       ??_C@_1BA@GMENCENF@?$AAb?$AAe?$AAl?$AAg?$AAi?$AAa?$AAn@ 10042bfc     libucrt:get_qualified_locale.obj
 0002:00005c0c       ??_C@_1BC@PJMIIAAN@?$AAc?$AAa?$AAn?$AAa?$AAd?$AAi?$AAa?$AAn@ 10042c0c     libucrt:get_qualified_locale.obj
 0002:00005c20       ??_C@_17NOIMNFBF@?$AAc?$AAh?$AAh@ 10042c20     libucrt:get_qualified_locale.obj
 0002:00005c28       ??_C@_17GGDALCHA@?$AAc?$AAh?$AAi@ 10042c28     libucrt:get_qualified_locale.obj
 0002:00005c30       ??_C@_1BA@NPNJKIBL@?$AAc?$AAh?$AAi?$AAn?$AAe?$AAs?$AAe@ 10042c30     libucrt:get_qualified_locale.obj
 0002:00005c40       ??_C@_1CC@DINBAMMJ@?$AAc?$AAh?$AAi?$AAn?$AAe?$AAs?$AAe?$AA?9?$AAh?$AAo?$AAn?$AAg?$AAk?$AAo?$AAn@ 10042c40     libucrt:get_qualified_locale.obj
 0002:00005c64       ??_C@_1CG@IOBJPACO@?$AAc?$AAh?$AAi?$AAn?$AAe?$AAs?$AAe?$AA?9?$AAs?$AAi?$AAm?$AAp?$AAl?$AAi?$AAf@ 10042c64     libucrt:get_qualified_locale.obj
 0002:00005c8c       ??_C@_1CE@GAJNDCKG@?$AAc?$AAh?$AAi?$AAn?$AAe?$AAs?$AAe?$AA?9?$AAs?$AAi?$AAn?$AAg?$AAa?$AAp?$AAo@ 10042c8c     libucrt:get_qualified_locale.obj
 0002:00005cb0       ??_C@_1CI@PAJPIOOD@?$AAc?$AAh?$AAi?$AAn?$AAe?$AAs?$AAe?$AA?9?$AAt?$AAr?$AAa?$AAd?$AAi?$AAt?$AAi@ 10042cb0     libucrt:get_qualified_locale.obj
 0002:00005cd8       ??_C@_1BM@NILJBMMD@?$AAd?$AAu?$AAt?$AAc?$AAh?$AA?9?$AAb?$AAe?$AAl?$AAg?$AAi?$AAa?$AAn@ 10042cd8     libucrt:get_qualified_locale.obj
 0002:00005cf4       ??_C@_1CC@OOJPJNEJ@?$AAe?$AAn?$AAg?$AAl?$AAi?$AAs?$AAh?$AA?9?$AAa?$AAm?$AAe?$AAr?$AAi?$AAc?$AAa@ 10042cf4     libucrt:get_qualified_locale.obj
 0002:00005d18       ??_C@_1BI@IOLFEEM@?$AAe?$AAn?$AAg?$AAl?$AAi?$AAs?$AAh?$AA?9?$AAa?$AAu?$AAs@ 10042d18     libucrt:get_qualified_locale.obj
 0002:00005d30       ??_C@_1BO@HFFNLENJ@?$AAe?$AAn?$AAg?$AAl?$AAi?$AAs?$AAh?$AA?9?$AAb?$AAe?$AAl?$AAi?$AAz?$AAe@ 10042d30     libucrt:get_qualified_locale.obj
 0002:00005d50       ??_C@_1BI@HAPKJMPO@?$AAe?$AAn?$AAg?$AAl?$AAi?$AAs?$AAh?$AA?9?$AAc?$AAa?$AAn@ 10042d50     libucrt:get_qualified_locale.obj
 0002:00005d68       ??_C@_1CE@HLNDMIOJ@?$AAe?$AAn?$AAg?$AAl?$AAi?$AAs?$AAh?$AA?9?$AAc?$AAa?$AAr?$AAi?$AAb?$AAb?$AAe@ 10042d68     libucrt:get_qualified_locale.obj
 0002:00005d8c       ??_C@_1BI@LDHJHHAC@?$AAe?$AAn?$AAg?$AAl?$AAi?$AAs?$AAh?$AA?9?$AAi?$AAr?$AAe@ 10042d8c     libucrt:get_qualified_locale.obj
 0002:00005da4       ??_C@_1CA@NJMMCFOC@?$AAe?$AAn?$AAg?$AAl?$AAi?$AAs?$AAh?$AA?9?$AAj?$AAa?$AAm?$AAa?$AAi?$AAc?$AAa@ 10042da4     libucrt:get_qualified_locale.obj
 0002:00005dc4       ??_C@_1BG@BHJEBBGG@?$AAe?$AAn?$AAg?$AAl?$AAi?$AAs?$AAh?$AA?9?$AAn?$AAz@ 10042dc4     libucrt:get_qualified_locale.obj
 0002:00005ddc       ??_C@_1CK@FGOEJJCO@?$AAe?$AAn?$AAg?$AAl?$AAi?$AAs?$AAh?$AA?9?$AAs?$AAo?$AAu?$AAt?$AAh?$AA?5?$AAa@ 10042ddc     libucrt:get_qualified_locale.obj
 0002:00005e08       ??_C@_1DE@PDBJPCJ@?$AAe?$AAn?$AAg?$AAl?$AAi?$AAs?$AAh?$AA?9?$AAt?$AAr?$AAi?$AAn?$AAi?$AAd?$AAa@ 10042e08     libucrt:get_qualified_locale.obj
 0002:00005e3c       ??_C@_1BG@JGCANDME@?$AAe?$AAn?$AAg?$AAl?$AAi?$AAs?$AAh?$AA?9?$AAu?$AAk@ 10042e3c     libucrt:get_qualified_locale.obj
 0002:00005e54       ??_C@_1BG@DINKMLE@?$AAe?$AAn?$AAg?$AAl?$AAi?$AAs?$AAh?$AA?9?$AAu?$AAs@ 10042e54     libucrt:get_qualified_locale.obj
 0002:00005e6c       ??_C@_1BI@NMFDBHJE@?$AAe?$AAn?$AAg?$AAl?$AAi?$AAs?$AAh?$AA?9?$AAu?$AAs?$AAa@ 10042e6c     libucrt:get_qualified_locale.obj
 0002:00005e84       ??_C@_1BO@OIHKJKII@?$AAf?$AAr?$AAe?$AAn?$AAc?$AAh?$AA?9?$AAb?$AAe?$AAl?$AAg?$AAi?$AAa?$AAn@ 10042e84     libucrt:get_qualified_locale.obj
 0002:00005ea4       ??_C@_1CA@NKAELJKI@?$AAf?$AAr?$AAe?$AAn?$AAc?$AAh?$AA?9?$AAc?$AAa?$AAn?$AAa?$AAd?$AAi?$AAa?$AAn@ 10042ea4     libucrt:get_qualified_locale.obj
 0002:00005ec4       ??_C@_1CE@MGKCNLGN@?$AAf?$AAr?$AAe?$AAn?$AAc?$AAh?$AA?9?$AAl?$AAu?$AAx?$AAe?$AAm?$AAb?$AAo?$AAu@ 10042ec4     libucrt:get_qualified_locale.obj
 0002:00005ee8       ??_C@_1BK@CEGEAILM@?$AAf?$AAr?$AAe?$AAn?$AAc?$AAh?$AA?9?$AAs?$AAw?$AAi?$AAs?$AAs@ 10042ee8     libucrt:get_qualified_locale.obj
 0002:00005f04       ??_C@_1CA@PAFKEOCC@?$AAg?$AAe?$AAr?$AAm?$AAa?$AAn?$AA?9?$AAa?$AAu?$AAs?$AAt?$AAr?$AAi?$AAa?$AAn@ 10042f04     libucrt:get_qualified_locale.obj
 0002:00005f24       ??_C@_1CI@HCFHGOFD@?$AAg?$AAe?$AAr?$AAm?$AAa?$AAn?$AA?9?$AAl?$AAi?$AAc?$AAh?$AAt?$AAe?$AAn?$AAs@ 10042f24     libucrt:get_qualified_locale.obj
 0002:00005f4c       ??_C@_1CE@FEDDNPDG@?$AAg?$AAe?$AAr?$AAm?$AAa?$AAn?$AA?9?$AAl?$AAu?$AAx?$AAe?$AAm?$AAb?$AAo?$AAu@ 10042f4c     libucrt:get_qualified_locale.obj
 0002:00005f70       ??_C@_1BK@LIMINNMN@?$AAg?$AAe?$AAr?$AAm?$AAa?$AAn?$AA?9?$AAs?$AAw?$AAi?$AAs?$AAs@ 10042f70     libucrt:get_qualified_locale.obj
 0002:00005f8c       ??_C@_1BM@LGMDBEPD@?$AAi?$AAr?$AAi?$AAs?$AAh?$AA?9?$AAe?$AAn?$AAg?$AAl?$AAi?$AAs?$AAh@ 10042f8c     libucrt:get_qualified_locale.obj
 0002:00005fa8       ??_C@_1BM@NNCFBAEE@?$AAi?$AAt?$AAa?$AAl?$AAi?$AAa?$AAn?$AA?9?$AAs?$AAw?$AAi?$AAs?$AAs@ 10042fa8     libucrt:get_qualified_locale.obj
 0002:00005fc4       ??_C@_1BE@FEDJNPIB@?$AAn?$AAo?$AAr?$AAw?$AAe?$AAg?$AAi?$AAa?$AAn@ 10042fc4     libucrt:get_qualified_locale.obj
 0002:00005fd8       ??_C@_1CC@CILKDEIE@?$AAn?$AAo?$AAr?$AAw?$AAe?$AAg?$AAi?$AAa?$AAn?$AA?9?$AAb?$AAo?$AAk?$AAm?$AAa@ 10042fd8     libucrt:get_qualified_locale.obj
 0002:00005ffc       ??_C@_1CE@DHMMHEPL@?$AAn?$AAo?$AAr?$AAw?$AAe?$AAg?$AAi?$AAa?$AAn?$AA?9?$AAn?$AAy?$AAn?$AAo?$AAr@ 10042ffc     libucrt:get_qualified_locale.obj
 0002:00006020       ??_C@_1CK@OPNMHECD@?$AAp?$AAo?$AAr?$AAt?$AAu?$AAg?$AAu?$AAe?$AAs?$AAe?$AA?9?$AAb?$AAr?$AAa?$AAz@ 10043020     libucrt:get_qualified_locale.obj
 0002:0000604c       ??_C@_1CE@KEEHCDB@?$AAs?$AAp?$AAa?$AAn?$AAi?$AAs?$AAh?$AA?9?$AAa?$AAr?$AAg?$AAe?$AAn?$AAt?$AAi@ 1004304c     libucrt:get_qualified_locale.obj
 0002:00006070       ??_C@_1CA@GIAOLHJD@?$AAs?$AAp?$AAa?$AAn?$AAi?$AAs?$AAh?$AA?9?$AAb?$AAo?$AAl?$AAi?$AAv?$AAi?$AAa@ 10043070     libucrt:get_qualified_locale.obj
 0002:00006090       ??_C@_1BM@OJNDFNPD@?$AAs?$AAp?$AAa?$AAn?$AAi?$AAs?$AAh?$AA?9?$AAc?$AAh?$AAi?$AAl?$AAe@ 10043090     libucrt:get_qualified_locale.obj
 0002:000060ac       ??_C@_1CC@OCOLPALL@?$AAs?$AAp?$AAa?$AAn?$AAi?$AAs?$AAh?$AA?9?$AAc?$AAo?$AAl?$AAo?$AAm?$AAb?$AAi@ 100430ac     libucrt:get_qualified_locale.obj
 0002:000060d0       ??_C@_1CG@BPOFMKBB@?$AAs?$AAp?$AAa?$AAn?$AAi?$AAs?$AAh?$AA?9?$AAc?$AAo?$AAs?$AAt?$AAa?$AA?5?$AAr@ 100430d0     libucrt:get_qualified_locale.obj
 0002:000060f8       ??_C@_1DG@IGOBAPBB@?$AAs?$AAp?$AAa?$AAn?$AAi?$AAs?$AAh?$AA?9?$AAd?$AAo?$AAm?$AAi?$AAn?$AAi?$AAc@ 100430f8     libucrt:get_qualified_locale.obj
 0002:00006130       ??_C@_1CA@JHAPGEGI@?$AAs?$AAp?$AAa?$AAn?$AAi?$AAs?$AAh?$AA?9?$AAe?$AAc?$AAu?$AAa?$AAd?$AAo?$AAr@ 10043130     libucrt:get_qualified_locale.obj
 0002:00006150       ??_C@_1CI@LAPALJPP@?$AAs?$AAp?$AAa?$AAn?$AAi?$AAs?$AAh?$AA?9?$AAe?$AAl?$AA?5?$AAs?$AAa?$AAl?$AAv@ 10043150     libucrt:get_qualified_locale.obj
 0002:00006178       ??_C@_1CE@PDGBOFOM@?$AAs?$AAp?$AAa?$AAn?$AAi?$AAs?$AAh?$AA?9?$AAg?$AAu?$AAa?$AAt?$AAe?$AAm?$AAa@ 10043178     libucrt:get_qualified_locale.obj
 0002:0000619c       ??_C@_1CC@NBEBAODI@?$AAs?$AAp?$AAa?$AAn?$AAi?$AAs?$AAh?$AA?9?$AAh?$AAo?$AAn?$AAd?$AAu?$AAr?$AAa@ 1004319c     libucrt:get_qualified_locale.obj
 0002:000061c0       ??_C@_1CA@LLKGHBMF@?$AAs?$AAp?$AAa?$AAn?$AAi?$AAs?$AAh?$AA?9?$AAm?$AAe?$AAx?$AAi?$AAc?$AAa?$AAn@ 100431c0     libucrt:get_qualified_locale.obj
 0002:000061e0       ??_C@_1BO@LKNDOIGD@?$AAs?$AAp?$AAa?$AAn?$AAi?$AAs?$AAh?$AA?9?$AAm?$AAo?$AAd?$AAe?$AAr?$AAn@ 100431e0     libucrt:get_qualified_locale.obj
 0002:00006200       ??_C@_1CE@NMDMOEEB@?$AAs?$AAp?$AAa?$AAn?$AAi?$AAs?$AAh?$AA?9?$AAn?$AAi?$AAc?$AAa?$AAr?$AAa?$AAg@ 10043200     libucrt:get_qualified_locale.obj
 0002:00006224       ??_C@_1BO@LLCBEJGB@?$AAs?$AAp?$AAa?$AAn?$AAi?$AAs?$AAh?$AA?9?$AAp?$AAa?$AAn?$AAa?$AAm?$AAa@ 10043224     libucrt:get_qualified_locale.obj
 0002:00006244       ??_C@_1CC@FKPGGIHO@?$AAs?$AAp?$AAa?$AAn?$AAi?$AAs?$AAh?$AA?9?$AAp?$AAa?$AAr?$AAa?$AAg?$AAu?$AAa@ 10043244     libucrt:get_qualified_locale.obj
 0002:00006268       ??_C@_1BK@CDEIHOOP@?$AAs?$AAp?$AAa?$AAn?$AAi?$AAs?$AAh?$AA?9?$AAp?$AAe?$AAr?$AAu@ 10043268     libucrt:get_qualified_locale.obj
 0002:00006284       ??_C@_1CI@GAHAKKGP@?$AAs?$AAp?$AAa?$AAn?$AAi?$AAs?$AAh?$AA?9?$AAp?$AAu?$AAe?$AAr?$AAt?$AAo?$AA?5@ 10043284     libucrt:get_qualified_locale.obj
 0002:000062ac       ??_C@_1CA@NKJBCAGP@?$AAs?$AAp?$AAa?$AAn?$AAi?$AAs?$AAh?$AA?9?$AAu?$AAr?$AAu?$AAg?$AAu?$AAa?$AAy@ 100432ac     libucrt:get_qualified_locale.obj
 0002:000062cc       ??_C@_1CE@ODILCONM@?$AAs?$AAp?$AAa?$AAn?$AAi?$AAs?$AAh?$AA?9?$AAv?$AAe?$AAn?$AAe?$AAz?$AAu?$AAe@ 100432cc     libucrt:get_qualified_locale.obj
 0002:000062f0       ??_C@_1CA@OBNMCGFO@?$AAs?$AAw?$AAe?$AAd?$AAi?$AAs?$AAh?$AA?9?$AAf?$AAi?$AAn?$AAl?$AAa?$AAn?$AAd@ 100432f0     libucrt:get_qualified_locale.obj
 0002:00006310       ??_C@_1M@PIPDDPPI@?$AAs?$AAw?$AAi?$AAs?$AAs@ 10043310     libucrt:get_qualified_locale.obj
 0002:0000631c       ??_C@_15GMFIMNFM@?$AAu?$AAs@ 1004331c     libucrt:get_qualified_locale.obj
 0002:00006324       ??_C@_17HAEBFAGL@?$AAu?$AAs?$AAa@ 10043324     libucrt:get_qualified_locale.obj
 0002:0000632c       ??_C@_1BA@DPFJEPHB@?$AAa?$AAm?$AAe?$AAr?$AAi?$AAc?$AAa@ 1004332c     libucrt:get_qualified_locale.obj
 0002:0000633c       ??_C@_1BA@ELOGGFK@?$AAb?$AAr?$AAi?$AAt?$AAa?$AAi?$AAn@ 1004333c     libucrt:get_qualified_locale.obj
 0002:0000634c       ??_C@_1M@GHBGIGDA@?$AAc?$AAh?$AAi?$AAn?$AAa@ 1004334c     libucrt:get_qualified_locale.obj
 0002:00006358       ??_C@_1M@NCHEJOPO@?$AAc?$AAz?$AAe?$AAc?$AAh@ 10043358     libucrt:get_qualified_locale.obj
 0002:00006364       ??_C@_1BA@BKPAPBLA@?$AAe?$AAn?$AAg?$AAl?$AAa?$AAn?$AAd@ 10043364     libucrt:get_qualified_locale.obj
 0002:00006374       ??_C@_1BM@HKBCKIPC@?$AAg?$AAr?$AAe?$AAa?$AAt?$AA?5?$AAb?$AAr?$AAi?$AAt?$AAa?$AAi?$AAn@ 10043374     libucrt:get_qualified_locale.obj
 0002:00006390       ??_C@_1BA@PPCHPGJB@?$AAh?$AAo?$AAl?$AAl?$AAa?$AAn?$AAd@ 10043390     libucrt:get_qualified_locale.obj
 0002:000063a0       ??_C@_1BE@JBMPEGDG@?$AAh?$AAo?$AAn?$AAg?$AA?9?$AAk?$AAo?$AAn?$AAg@ 100433a0     libucrt:get_qualified_locale.obj
 0002:000063b4       ??_C@_1BI@KOELBBPJ@?$AAn?$AAe?$AAw?$AA?9?$AAz?$AAe?$AAa?$AAl?$AAa?$AAn?$AAd@ 100433b4     libucrt:get_qualified_locale.obj
 0002:000063cc       ??_C@_15HIEBHAIO@?$AAn?$AAz@ 100433cc     libucrt:get_qualified_locale.obj
 0002:000063d4       ??_C@_1BC@CHBCPFPI@?$AAp?$AAr?$AA?5?$AAc?$AAh?$AAi?$AAn?$AAa@ 100433d4     libucrt:get_qualified_locale.obj
 0002:000063e8       ??_C@_1BC@JAOIIFKD@?$AAp?$AAr?$AA?9?$AAc?$AAh?$AAi?$AAn?$AAa@ 100433e8     libucrt:get_qualified_locale.obj
 0002:000063fc       ??_C@_1BI@BEHPPHKC@?$AAp?$AAu?$AAe?$AAr?$AAt?$AAo?$AA?9?$AAr?$AAi?$AAc?$AAo@ 100433fc     libucrt:get_qualified_locale.obj
 0002:00006414       ??_C@_1O@PAEOFKDI@?$AAs?$AAl?$AAo?$AAv?$AAa?$AAk@ 10043414     libucrt:get_qualified_locale.obj
 0002:00006424       ??_C@_1BK@FIHMCKAM@?$AAs?$AAo?$AAu?$AAt?$AAh?$AA?5?$AAa?$AAf?$AAr?$AAi?$AAc?$AAa@ 10043424     libucrt:get_qualified_locale.obj
 0002:00006440       ??_C@_1BI@NAEOODKB@?$AAs?$AAo?$AAu?$AAt?$AAh?$AA?5?$AAk?$AAo?$AAr?$AAe?$AAa@ 10043440     libucrt:get_qualified_locale.obj
 0002:00006458       ??_C@_1BK@FBDGGIFF@?$AAs?$AAo?$AAu?$AAt?$AAh?$AA?9?$AAa?$AAf?$AAr?$AAi?$AAc?$AAa@ 10043458     libucrt:get_qualified_locale.obj
 0002:00006474       ??_C@_1BI@GHLEJDPK@?$AAs?$AAo?$AAu?$AAt?$AAh?$AA?9?$AAk?$AAo?$AAr?$AAe?$AAa@ 10043474     libucrt:get_qualified_locale.obj
 0002:0000648c       ??_C@_1CE@PLHLOMJF@?$AAt?$AAr?$AAi?$AAn?$AAi?$AAd?$AAa?$AAd?$AA?5?$AA?$CG?$AA?5?$AAt?$AAo?$AAb?$AAa@ 1004348c     libucrt:get_qualified_locale.obj
 0002:000064b0       ??_C@_1BO@MODIMHHI@?$AAu?$AAn?$AAi?$AAt?$AAe?$AAd?$AA?9?$AAk?$AAi?$AAn?$AAg?$AAd?$AAo?$AAm@ 100434b0     libucrt:get_qualified_locale.obj
 0002:000064d0       ??_C@_1BM@FFHJONBJ@?$AAu?$AAn?$AAi?$AAt?$AAe?$AAd?$AA?9?$AAs?$AAt?$AAa?$AAt?$AAe?$AAs@ 100434d0     libucrt:get_qualified_locale.obj
 0002:000064ec       ??_C@_19MPDNHKDG@?$AAu?$AAt?$AAf?$AA8@ 100434ec     libucrt:get_qualified_locale.obj
 0002:000064f8       ??_C@_17DNCLJFIF@?$AAA?$AAC?$AAP@ 100434f8     libucrt:get_qualified_locale.obj
 0002:00006500       ??_C@_1M@FPEIIFAM@?$AAu?$AAt?$AAf?$AA?9?$AA8@ 10043500     libucrt:get_qualified_locale.obj
 0002:0000650c       ??_C@_17CIKBIHLH@?$AAO?$AAC?$AAP@ 1004350c     libucrt:get_qualified_locale.obj
 0002:00006514       ___rglangidNotDefault      10043514     libucrt:getqloc_downlevel.obj
 0002:00006528       ___acrt_pow_rcp_t1         10043528     libucrt:pow_tables.obj
 0002:00006940       ___acrt_pow_log2_t1        10043940     libucrt:pow_tables.obj
 0002:00007150       ___acrt_pow_rcp_t2         10044150     libucrt:pow_tables.obj
 0002:00007560       ___acrt_pow_log2_t2        10044560     libucrt:pow_tables.obj
 0002:00007d70       ___acrt_pow_rcp_t3         10044d70     libucrt:pow_tables.obj
 0002:00008580       ___acrt_pow_log2_t3        10045580     libucrt:pow_tables.obj
 0002:00009590       ___acrt_pow_clv            10046590     libucrt:pow_tables.obj
 0002:000095b0       ___acrt_pow_exp2_tbl       100465b0     libucrt:pow_tables.obj
 0002:00009e08       ??_C@_1BA@BALFACEM@?$AAC?$AAO?$AAN?$AAO?$AAU?$AAT?$AA$@ 10046e08     libucrt:initcon.obj
 0002:00009f20       ___acrt_log10_table_t      10046f20     libucrt:log10_tables.obj
 0002:0000a330       ___acrt_log10_table_cb     10047330     libucrt:log10_tables.obj
 0002:0000a74c       ??_C@_0BC@EOODALEL@Unknown?5exception@ 1004774c     format.obj
 0002:0000a760       ??_C@_0BF@KINCDENJ@bad?5array?5new?5length@ 10047760     format.obj
 0002:0000a778       ??_C@_0BA@JFNIOLAK@string?5too?5long@ 10047778     format.obj
 0002:0000a788       ??_C@_00CNPNBAHC@@         10047788     format.obj
 0002:0000a790       ??_C@_0MJ@HFBCCPGP@0001020304050607080910111213141@ 10047790     format.obj
 0002:0000a85c       ??_C@_0BC@MDEIBHGE@number?5is?5too?5big@ 1004785c     format.obj
 0002:0000a870       ??_C@_0BA@ELKIONDK@bad?5locale?5name@ 10047870     format.obj
 0002:0000a880       ??_C@_05LAPONLG@false@     10047880     format.obj
 0002:0000a888       ??_C@_04LOAJBDKD@true@     10047888     format.obj
 0002:0000a890       ??_C@_0BP@NMGMJOEM@unmatched?5?8?$HN?8?5in?5format?5string@ 10047890     format.obj
 0002:0000a8b0       ??_C@_0BG@PEJKJNLA@invalid?5format?5string@ 100478b0     format.obj
 0002:0000a8c8       ??_C@_0BJ@JNDNOEDN@unknown?5format?5specifier@ 100478c8     format.obj
 0002:0000a8e4       ??_C@_0BN@JNLAGDD@missing?5?8?$HN?8?5in?5format?5string@ 100478e4     format.obj
 0002:0000a904       ??_C@_0BD@DBEDGLNA@argument?5not?5found@ 10047904     format.obj
 0002:0000a918       ??_C@_0DJ@GHJONFIH@cannot?5switch?5from?5manual?5to?5au@ 10047918     format.obj
 0002:0000a954       ??_C@_0BJ@KLNHPFKH@invalid?5format?5specifier@ 10047954     format.obj
 0002:0000a970       ??_C@_0CL@CFEEEDMP@format?5specifier?5requires?5numer@ 10047970     format.obj
 0002:0000a99c       ??_C@_0BL@KNEDAEPA@invalid?5fill?5character?5?8?$HL?8@ 1004799c     format.obj
 0002:0000a9b8       ??_C@_0DJ@LMIJFHJI@cannot?5switch?5from?5automatic?5to@ 100479b8     format.obj
 0002:0000a9f4       ??_C@_0CC@ELFJMMCC@invalid?5format?5specifier?5for?5ch@ 100479f4     format.obj
 0002:0000aa18       ??_C@_0BC@CFECDNCP@invalid?5precision@ 10047a18     format.obj
 0002:0000aa2c       ??_C@_0BH@IEEDMHI@string?5pointer?5is?5null@ 10047a2c     format.obj
 0002:0000aa44       ??_C@_0P@DAPDPGEO@negative?5width@ 10047a44     format.obj
 0002:0000aa54       ??_C@_0BD@PKKFPMLC@negative?5precision@ 10047a54     format.obj
 0002:0000aa68       ??_C@_04MKAMHODJ@?$BP?$BP?$AA?$AB@ 10047a68     format.obj
 0002:0000aa70       ??_C@_04CILMHOGK@?$AA?$BP?$AA?$AB@ 10047a70     format.obj
 0002:0000aa78       ??_C@_03LKNCIKJB@NAN@      10047a78     format.obj
 0002:0000aa7c       ??_C@_03LHCJEHON@nan@      10047a7c     format.obj
 0002:0000aa80       ??_C@_03OEIAHPBN@INF@      10047a80     format.obj
 0002:0000aa84       ??_C@_03OJHLLCGB@inf@      10047a84     format.obj
 0002:0000aa88       ??_C@_0BF@KEAPHPPE@width?5is?5not?5integer@ 10047a88     format.obj
 0002:0000aaa0       ??_C@_0BJ@KKLAKOOL@precision?5is?5not?5integer@ 10047aa0     format.obj
 0002:0000aabc       ??_C@_04MKBJPCKC@?$AA?9?$CL?5@ 10047abc     format.obj
 0002:0000aad0       ??_C@_0BB@JGGOGLEG@0123456789ABCDEF@ 10047ad0     format.obj
 0002:0000aaf0       ??_C@_0BB@JCEFLFJE@0123456789abcdef@ 10047af0     format.obj
 0002:0000ac4c       ??_7?$basic_memory_buffer@I$0CA@V?$allocator@I@std@@@v10@fmt@@6B@ 10047c4c     format.obj
 0002:0000ac50       ?powers_of_5_64@?1??get_cached_power@?$cache_accessor@N@dragonbox@detail@v10@fmt@@SA?AVuint128_fallback@456@H@Z@4QB_KB 10047c50     format.obj
 0002:0000ad28       ?bsr2log10@?1??do_count_digits@detail@v10@fmt@@YAH_K@Z@4QBEB 10047d28     format.obj
 0002:0000ad6c       ??_7?$basic_memory_buffer@D$0BPE@V?$allocator@D@std@@@v10@fmt@@6B@ 10047d6c     format.obj
 0002:0000ad70       ?fractional_part_rounding_thresholds@?$basic_data@X@detail@v10@fmt@@2QBIB 10047d70     format.obj
 0002:0000ad90       ?zero_or_powers_of_10@?1??do_count_digits@detail@v10@fmt@@YAH_K@Z@4QB_KB 10047d90     format.obj
 0002:0000b0f8       ?pow10_significands@?1??get_cached_power@?$cache_accessor@M@dragonbox@detail@v10@fmt@@SA_KH@Z@4QB_KB 100480f8     format.obj
 0002:0000b36c       ??_7?$basic_memory_buffer@_W$0BPE@V?$allocator@_W@std@@@v10@fmt@@6B@ 1004836c     format.obj
 0002:0000b4f0       ?pow10_significands@?1??get_cached_power@?$cache_accessor@N@dragonbox@detail@v10@fmt@@SA?AVuint128_fallback@456@H@Z@4QBV7456@B 100484f0     format.obj
 0002:0000b674       ??_7format_error@v10@fmt@@6B@ 10048674     format.obj
 0002:0000b680       ?table@?1??do_count_digits@detail@v10@fmt@@YAHI@Z@4QB_KB 10048680     format.obj
 0002:0000b784       ??_7?$basic_memory_buffer@H$0BPE@V?$allocator@H@std@@@v10@fmt@@6B@ 10048784     format.obj
 0002:0000b788       ??_C@_1O@ECECHNAE@?$AA?$DM?$AAp?$AAi?$AAp?$AAe?$AA?$DO@ 10048788     handles.obj
 0002:0000b798       ??_C@_1O@HIMECKKA@?$AA?$DM?$AAc?$AAh?$AAa?$AAr?$AA?$DO@ 10048798     handles.obj
 0002:0000b7a8       ??_C@_1BC@FBIGGGKE@?$AA?$DM?$AAr?$AAe?$AAm?$AAo?$AAt?$AAe?$AA?$DO@ 100487a8     handles.obj
 0002:0000b7bc       ??_C@_1BE@ELICABCK@?$AA?$DM?$AAu?$AAn?$AAk?$AAn?$AAo?$AAw?$AAn?$AA?$DO@ 100487bc     handles.obj
 0002:0000b7d0       ??_C@_1BO@MHBBMPMP@?$AA?$DM?$AAu?$AAn?$AAk?$AAn?$AAo?$AAw?$AAn?$AA?$DO?$AA?5?$AA?$CI?$AA?$HL?$AA?$HN?$AA?$CJ@ 100487d0     handles.obj
 0002:0000b7f0       ??_C@_11LOCGONAA@@         100487f0     handles.obj
 0002:0000b7f4       ??_C@_1BA@NMDNJJOO@?$AAP?$AAr?$AAo?$AAc?$AAe?$AAs?$AAs@ 100487f4     handles.obj
 0002:0000b804       ??_C@_1O@CDOGJPJJ@?$AAT?$AAh?$AAr?$AAe?$AAa?$AAd@ 10048804     handles.obj
 0002:0000b814       ??_C@_17KACEIPNC@?$AAK?$AAe?$AAy@ 10048814     handles.obj
 0002:0000b81c       ??_C@_19DDLLJDOO@?$AAF?$AAi?$AAl?$AAe@ 1004881c     handles.obj
 0002:0000b828       ??_C@_1BA@BEGLAEKB@?$AA?$HL?$AA?$HN?$AA?5?$AA?$CI?$AA?$HL?$AA?$HN?$AA?$CJ@ 10048828     handles.obj
 0002:0000b838       ??_C@_1BA@KNLBEBJD@?$AAT?$AAI?$AAD?$AA?3?$AA?5?$AA?$HL?$AA?$HN@ 10048838     handles.obj
 0002:0000b848       ??_C@_1BG@OKCBELMP@?$AA?2?$AAR?$AAE?$AAG?$AAI?$AAS?$AAT?$AAR?$AAY?$AA?2@ 10048848     handles.obj
 0002:0000b860       ??_C@_19KGHAHCFG@?$AAU?$AAS?$AAE?$AAR@ 10048860     handles.obj
 0002:0000b86c       ??_C@_1DC@OIDKFHBF@?$AAM?$AAA?$AAC?$AAH?$AAI?$AAN?$AAE?$AA?2?$AAS?$AAO?$AAF?$AAT?$AAW?$AAA?$AAR@ 1004886c     handles.obj
 0002:0000b8a0       ??_C@_1BA@INBMCOAP@?$AAM?$AAA?$AAC?$AAH?$AAI?$AAN?$AAE@ 100488a0     handles.obj
 0002:0000b8b0       ??_C@_1BC@DCCOJFBE@?$AA_?$AAC?$AAL?$AAA?$AAS?$AAS?$AAE?$AAS@ 100488b0     handles.obj
 0002:0000b8c4       ??_C@_13FPGAJAPJ@?$AA?2@   100488c4     handles.obj
 0002:0000b8c8       ??_C@_19DIHHCHDI@?$AAH?$AAK?$AAU?$AA?2@ 100488c8     handles.obj
 0002:0000b8d4       ??_C@_19JAPAIJDE@?$AAH?$AAK?$AAC?$AAU@ 100488d4     handles.obj
 0002:0000b8e0       ??_C@_1BK@OEABCBLA@?$AAH?$AAK?$AAC?$AAU?$AA?2?$AAC?$AAl?$AAa?$AAs?$AAs?$AAe?$AAs@ 100488e0     handles.obj
 0002:0000b8fc       ??_C@_17PJOJPMPB@?$AAH?$AAK?$AAU@ 100488fc     handles.obj
 0002:0000b904       ??_C@_19NCHLBIN@?$AAH?$AAK?$AAC?$AAR@ 10048904     handles.obj
 0002:0000b910       ??_C@_19PEALEEJB@?$AAH?$AAK?$AAL?$AAM@ 10048910     handles.obj
 0002:0000b91c       ??_C@_1DC@EMNPLNEM@?$AA?6?$AA?$HL?$AA?$HN?$AA?3?$AA?6?$AA?$HL?$AA?3?$AA6?$AA?$HN?$AA?5?$AA?$HL?$AA?3?$AA8?$AA?$HN?$AA?5@ 1004891c     handles.obj
 0002:0000b950       ??_C@_1CO@HBDELFCB@?$AA?$HL?$AA?3?$AA6?$AAX?$AA?$HN?$AA?5?$AA?$HL?$AA?3?$AA0?$AA8?$AAX?$AA?$HN?$AA?5?$AA?$HL?$AA?3@ 10048950     handles.obj
 0002:0000b994       ??_C@_1O@BJPKKLLM@?$AAC?$AAo?$AAn?$AAf?$AAi?$AAg@ 10048994     Pcfg.obj
 0002:0000b9a4       ??_C@_1BO@NGDOFANC@?$AAA?$AAd?$AAd?$AAT?$AAo?$AAD?$AAi?$AAs?$AAk?$AAs?$AAM?$AAe?$AAn?$AAu@ 100489a4     Pcfg.obj
 0002:0000b9c4       ??_C@_1CC@PNNAOHJC@?$AAA?$AAd?$AAd?$AAT?$AAo?$AAP?$AAl?$AAu?$AAg?$AAi?$AAn?$AAs?$AAM?$AAe?$AAn@ 100489c4     Pcfg.obj
 0002:0000b9e8       ??_C@_1CE@JIPJNDMD@?$AAE?$AAx?$AAp?$AAo?$AAr?$AAt?$AAE?$AAn?$AAv?$AAi?$AAr?$AAo?$AAn?$AAm?$AAe@ 100489e8     Pcfg.obj
 0002:0000ba0c       ??_C@_1CC@OABICAMP@?$AAE?$AAx?$AAp?$AAo?$AAr?$AAt?$AAM?$AAo?$AAd?$AAu?$AAl?$AAe?$AAI?$AAn?$AAf@ 10048a0c     Pcfg.obj
 0002:0000ba30       ??_C@_1CI@OFLGHPDG@?$AAE?$AAx?$AAp?$AAo?$AAr?$AAt?$AAM?$AAo?$AAd?$AAu?$AAl?$AAe?$AAV?$AAe?$AAr@ 10048a30     Pcfg.obj
 0002:0000ba58       ??_C@_1CE@GNMOKOAL@?$AAE?$AAx?$AAp?$AAo?$AAr?$AAt?$AAP?$AAe?$AAr?$AAf?$AAo?$AAr?$AAm?$AAa?$AAn@ 10048a58     Pcfg.obj
 0002:0000ba7c       ??_C@_1BM@KMCHODLM@?$AAE?$AAx?$AAp?$AAo?$AAr?$AAt?$AAH?$AAa?$AAn?$AAd?$AAl?$AAe?$AAs@ 10048a7c     Pcfg.obj
 0002:0000ba98       ??_C@_1CK@CLFOOHFA@?$AAE?$AAx?$AAp?$AAo?$AAr?$AAt?$AAH?$AAa?$AAn?$AAd?$AAl?$AAe?$AAs?$AAU?$AAn@ 10048a98     Pcfg.obj
 0002:0000bac4       ??_C@_1BE@PKILIDFH@?$AAE?$AAn?$AAa?$AAb?$AAl?$AAe?$AAW?$AAM?$AAI@ 10048ac4     Pcfg.obj
 0002:0000badc       ??_7PluginCheckBoxBinding@@6B@ 10048adc     Pcfg.obj
 0002:0000bae4       ??_C@_1BK@GMMKGKID@?$AA?$HL?$AA0?$AA?$HN?$AA?4?$AA?$HL?$AA1?$AA?3?$AA0?$AA?$HL?$AA2?$AA?$HN?$AA?$HN@ 10048ae4     Pclass.obj
 0002:0000bb00       ??_C@_1BA@BHJJFMCM@?$AAB?$AAK?$AAM?$AAG?$AAT?$AAP?$AAE@ 10048b00     Pclass.obj
 0002:0000bb10       ??_C@_19LPDLLMEB@?$AA?$HL?$AA0?$AA?$HN?$AA?3@ 10048b10     Pclass.obj
 0002:0000bb1c       ??_C@_1BC@HGOMHBK@?$AA?$HL?$AA0?$AA?3?$AA?$DM?$AA2?$AA1?$AA?$HN?$AA?5@ 10048b1c     Pclass.obj
 0002:0000bb30       ??_C@_1BC@IALIJCAM@?$AAS?$AAo?$AAr?$AAt?$AAM?$AAo?$AAd?$AAe@ 10048b30     Pclass.obj
 0002:0000bb44       ??_C@_1BO@OMKAPLPJ@?$AAS?$AAt?$AAa?$AAr?$AAt?$AAP?$AAa?$AAn?$AAe?$AAl?$AAM?$AAo?$AAd?$AAe@ 10048b44     Pclass.obj
 0002:0000bb64       ??_C@_1CM@KGJLHHPG@?$AAN?$AA?0?$AAX?$AA1?$AA5?$AAF?$AA?0?$AAX?$AA1?$AA6?$AAF?$AA?0?$AAX?$AA1?$AA7@ 10048b64     Pclass.obj
 0002:0000bb90       ??_C@_1BG@MNPGDOEP@?$AA1?$AA2?$AA?0?$AA0?$AA?0?$AA0?$AA?0?$AA0?$AA?0?$AA4@ 10048b90     Pclass.obj
 0002:0000bba8       ??_C@_1CG@OHFJBKLN@?$AAN?$AA?0?$AAX?$AAI?$AA?0?$AAX?$AAB?$AA?0?$AAX?$AAP?$AA?0?$AAX?$AA0?$AAS?$AA?0@ 10048ba8     Pclass.obj
 0002:0000bbd0       ??_C@_1BI@EFANNANC@?$AA0?$AA?0?$AA6?$AA?0?$AA2?$AA?0?$AA2?$AA?0?$AA3?$AA?0?$AA9@ 10048bd0     Pclass.obj
 0002:0000bbe8       ??_C@_17KNGPBKAK@?$AAN?$AA?0?$AAN@ 10048be8     Pclass.obj
 0002:0000bbf0       ??_C@_17JPFFEOAH@?$AA0?$AA?0?$AA0@ 10048bf0     Pclass.obj
 0002:0000bbf8       ??_C@_1BO@JAFIOFIL@?$AAN?$AA?0?$AAX?$AAI?$AA?0?$AAX?$AAB?$AA?0?$AAX?$AAC?$AA?0?$AAD?$AA?0?$AAT@ 10048bf8     Pclass.obj
 0002:0000bc18       ??_C@_1BI@LFIMKDME@?$AA0?$AA?0?$AA6?$AA?0?$AA2?$AA?0?$AA6?$AA?0?$AA0?$AA?0?$AA0@ 10048c18     Pclass.obj
 0002:0000bc30       ??_C@_1BK@IEHCCPMO@?$AAN?$AA?0?$AAX?$AAI?$AA?0?$AAX?$AA4?$AAF?$AA?0?$AAX?$AA6?$AAF@ 10048c30     Pclass.obj
 0002:0000bc4c       ??_C@_1BA@MMHHFCDG@?$AA0?$AA?0?$AA6?$AA?0?$AA9?$AA?0?$AA9@ 10048c4c     Pclass.obj
 0002:0000bc60       ??_C@_1EA@CMHCGANC@?$AAN?$AA?0?$AAX?$AAI?$AA?0?$AAX?$AA4?$AAF?$AA?0?$AAX?$AA6?$AAF?$AA?0?$AAX?$AA1@ 10048c60     Pclass.obj
 0002:0000bca0       ??_C@_1CE@LPFIEDMN@?$AA0?$AA?0?$AA6?$AA?0?$AA9?$AA?0?$AA9?$AA?0?$AA9?$AA?0?$AA9?$AA?0?$AA8?$AA?0?$AA8@ 10048ca0     Pclass.obj
 0002:0000bcc4       ??_C@_19ILLMDDHI@?$AAN?$AA?0?$AAZ?$AAD@ 10048cc4     Pclass.obj
 0002:0000bcd0       ??_C@_19NMOJBHGD@?$AA1?$AA2?$AA?0?$AA0@ 10048cd0     Pclass.obj
 0002:0000bce0       ??_C@_1EC@OFLHMCFD@?$AAN?$AA?0?$AAX?$AAP?$AA?0?$AAX?$AA0?$AAS?$AA?0?$AAX?$AA1?$AAS?$AA?0?$AAX?$AA2@ 10048ce0     Pclass.obj
 0002:0000bd24       ??_C@_1CA@MGMNHCLL@?$AA0?$AA?0?$AA2?$AA?0?$AA3?$AA?0?$AA2?$AA?0?$AA2?$AA?0?$AA3?$AA?0?$AA4?$AA?0?$AA3@ 10048d24     Pclass.obj
 0002:0000bd44       ??_C@_1O@JGFFCAGM@?$AAN?$AA?0?$AAX?$AAI?$AA?0?$AAO@ 10048d44     Pclass.obj
 0002:0000bd54       ??_C@_1O@FLEOANAI@?$AA0?$AA?0?$AA6?$AA?0?$AA1?$AA5@ 10048d54     Pclass.obj
 0002:0000bd64       ??_C@_1CC@FANCGEGE@?$AAN?$AA?0?$AAX?$AAI?$AA?0?$AAX?$AAT?$AA?0?$AAX?$AA3?$AA?0?$AAX?$AAG?$AA?0?$AAX@ 10048d64     Pclass.obj
 0002:0000bd88       ??_C@_1BI@PMPHDFGH@?$AA0?$AA?0?$AA6?$AA?0?$AA3?$AA?0?$AA4?$AA?0?$AA4?$AA?0?$AA4@ 10048d88     Pclass.obj
 0002:0000bda0       ??_C@_1BG@COBJEPBB@?$AAN?$AA?0?$AAX?$AAI?$AA?0?$AAX?$AAT?$AA?0?$AAX?$AA3@ 10048da0     Pclass.obj
 0002:0000bdb8       ??_C@_1BA@KPNNJGCD@?$AA0?$AA?0?$AA6?$AA?0?$AA3?$AA?0?$AA4@ 10048db8     Pclass.obj
 0002:0000bdc8       ??_C@_1BA@JOLGFBLP@?$AAM?$AAo?$AAd?$AAe?$AA?$HL?$AA0?$AA?$HN@ 10048dc8     Pclass.obj
 0002:0000bdd8       ??_C@_1CA@HLBJOHGN@?$AAF?$AAu?$AAl?$AAl?$AAS?$AAc?$AAr?$AAe?$AAe?$AAn?$AAL?$AAo?$AAc?$AAa?$AAl@ 10048dd8     Pclass.obj
 0002:0000bdf8       ??_C@_1CC@EBBNDNOD@?$AAF?$AAu?$AAl?$AAl?$AAS?$AAc?$AAr?$AAe?$AAe?$AAn?$AAR?$AAe?$AAm?$AAo?$AAt@ 10048df8     Pclass.obj
 0002:0000be1c       ??_C@_1BK@HMOODHKK@?$AAC?$AAo?$AAl?$AAu?$AAm?$AAn?$AAs?$AAL?$AAo?$AAc?$AAa?$AAl@ 10048e1c     Pclass.obj
 0002:0000be38       ??_C@_1BM@EDHFKJEJ@?$AAC?$AAo?$AAl?$AAu?$AAm?$AAn?$AAs?$AAR?$AAe?$AAm?$AAo?$AAt?$AAe@ 10048e38     Pclass.obj
 0002:0000be54       ??_C@_1BI@FOOHDOCI@?$AAW?$AAi?$AAd?$AAt?$AAh?$AAs?$AAL?$AAo?$AAc?$AAa?$AAl@ 10048e54     Pclass.obj
 0002:0000be6c       ??_C@_1BK@DDBMMJCN@?$AAW?$AAi?$AAd?$AAt?$AAh?$AAs?$AAR?$AAe?$AAm?$AAo?$AAt?$AAe@ 10048e6c     Pclass.obj
 0002:0000be88       ??_C@_13DEFPDAGF@?$AA?0@   10048e88     Pclass.obj
 0002:0000be8c       ??_C@_15LNKNCLHH@?$AAS?$AAs@ 10048e8c     Pclass.obj
 0002:0000be94       ??_C@_19LFJMKILO@?$AA?5?$AA?$HL?$AA?$HN?$AA?5@ 10048e94     Pclass.obj
 0002:0000bea0       ??_C@_1BA@JMJLAOEC@?$AA?$HL?$AA?$HN?$AA?3?$AA?5?$AA?$HL?$AA?$HN?$AA?5@ 10048ea0     Pclass.obj
 0002:0000beb0       ??_C@_15JOGBDECP@?$AA?0?$AA?5@ 10048eb0     Pclass.obj
 0002:0000beb8       ??_C@_15DNHPCDHG@?$AAT?$AAt@ 10048eb8     Pclass.obj
 0002:0000bec0       ??_C@_15IJHBBPPC@?$AAF?$AAf@ 10048ec0     Pclass.obj
 0002:0000bec8       ??_C@_1BC@OMEIHGFC@?$AAW?$AAS?$AA_?$AAP?$AAO?$AAP?$AAU?$AAP@ 10048ec8     Pclass.obj
 0002:0000bedc       ??_C@_1BC@ONEEOLLM@?$AAW?$AAS?$AA_?$AAC?$AAH?$AAI?$AAL?$AAD@ 10048edc     Pclass.obj
 0002:0000bef0       ??_C@_1BI@GHDIGAD@?$AAW?$AAS?$AA_?$AAM?$AAI?$AAN?$AAI?$AAM?$AAI?$AAZ?$AAE@ 10048ef0     Pclass.obj
 0002:0000bf08       ??_C@_1BG@KLPFHNBP@?$AAW?$AAS?$AA_?$AAV?$AAI?$AAS?$AAI?$AAB?$AAL?$AAE@ 10048f08     Pclass.obj
 0002:0000bf20       ??_C@_1BI@NKODCGOF@?$AAW?$AAS?$AA_?$AAD?$AAI?$AAS?$AAA?$AAB?$AAL?$AAE?$AAD@ 10048f20     Pclass.obj
 0002:0000bf38       ??_C@_1CA@PCFJBBHH@?$AAW?$AAS?$AA_?$AAC?$AAL?$AAI?$AAP?$AAS?$AAI?$AAB?$AAL?$AAI?$AAN?$AAG?$AAS@ 10048f38     Pclass.obj
 0002:0000bf58       ??_C@_1CA@MPLGGIO@?$AAW?$AAS?$AA_?$AAC?$AAL?$AAI?$AAP?$AAC?$AAH?$AAI?$AAL?$AAD?$AAR?$AAE?$AAN@ 10048f58     Pclass.obj
 0002:0000bf78       ??_C@_1BI@OLBAGOJG@?$AAW?$AAS?$AA_?$AAM?$AAA?$AAX?$AAI?$AAM?$AAI?$AAZ?$AAE@ 10048f78     Pclass.obj
 0002:0000bf90       ??_C@_1BE@DAMMEKNP@?$AAW?$AAS?$AA_?$AAB?$AAO?$AAR?$AAD?$AAE?$AAR@ 10048f90     Pclass.obj
 0002:0000bfa4       ??_C@_1BI@EDHINADK@?$AAW?$AAS?$AA_?$AAD?$AAL?$AAG?$AAF?$AAR?$AAA?$AAM?$AAE@ 10048fa4     Pclass.obj
 0002:0000bfbc       ??_C@_1BG@CKCLFGFA@?$AAW?$AAS?$AA_?$AAV?$AAS?$AAC?$AAR?$AAO?$AAL?$AAL@ 10048fbc     Pclass.obj
 0002:0000bfd4       ??_C@_1BG@OMIOJOGF@?$AAW?$AAS?$AA_?$AAH?$AAS?$AAC?$AAR?$AAO?$AAL?$AAL@ 10048fd4     Pclass.obj
 0002:0000bfec       ??_C@_1BG@KJOBMDJC@?$AAW?$AAS?$AA_?$AAS?$AAY?$AAS?$AAM?$AAE?$AAN?$AAU@ 10048fec     Pclass.obj
 0002:0000c004       ??_C@_1BM@GPNNOPCH@?$AAW?$AAS?$AA_?$AAT?$AAH?$AAI?$AAC?$AAK?$AAF?$AAR?$AAA?$AAM?$AAE@ 10049004     Pclass.obj
 0002:0000c020       ??_C@_1BO@FODKBODI@?$AAW?$AAS?$AA_?$AAM?$AAI?$AAN?$AAI?$AAM?$AAI?$AAZ?$AAE?$AAB?$AAO?$AAX@ 10049020     Pclass.obj
 0002:0000c040       ??_C@_1BO@IDJMAOMI@?$AAW?$AAS?$AA_?$AAM?$AAA?$AAX?$AAI?$AAM?$AAI?$AAZ?$AAE?$AAB?$AAO?$AAX@ 10049040     Pclass.obj
 0002:0000c060       ??_C@_1CI@PKBCIOPN@?$AAW?$AAS?$AA_?$AAE?$AAX?$AA_?$AAD?$AAL?$AAG?$AAM?$AAO?$AAD?$AAA?$AAL?$AAF@ 10049060     Pclass.obj
 0002:0000c088       ??_C@_1CK@KJECLHMG@?$AAW?$AAS?$AA_?$AAE?$AAX?$AA_?$AAN?$AAO?$AAP?$AAA?$AAR?$AAE?$AAN?$AAT?$AAN@ 10049088     Pclass.obj
 0002:0000c0b4       ??_C@_1BM@OCBKBALE@?$AAW?$AAS?$AA_?$AAE?$AAX?$AA_?$AAT?$AAO?$AAP?$AAM?$AAO?$AAS?$AAT@ 100490b4     Pclass.obj
 0002:0000c0d0       ??_C@_1CE@JIDMMICL@?$AAW?$AAS?$AA_?$AAE?$AAX?$AA_?$AAA?$AAC?$AAC?$AAE?$AAP?$AAT?$AAF?$AAI?$AAL@ 100490d0     Pclass.obj
 0002:0000c0f4       ??_C@_1CE@PFFPBMCF@?$AAW?$AAS?$AA_?$AAE?$AAX?$AA_?$AAT?$AAR?$AAA?$AAN?$AAS?$AAP?$AAA?$AAR?$AAE@ 100490f4     Pclass.obj
 0002:0000c118       ??_C@_1BO@MEOEJPLO@?$AAW?$AAS?$AA_?$AAE?$AAX?$AA_?$AAM?$AAD?$AAI?$AAC?$AAH?$AAI?$AAL?$AAD@ 10049118     Pclass.obj
 0002:0000c138       ??_C@_1CC@IEIGGJGG@?$AAW?$AAS?$AA_?$AAE?$AAX?$AA_?$AAT?$AAO?$AAO?$AAL?$AAW?$AAI?$AAN?$AAD?$AAO@ 10049138     Pclass.obj
 0002:0000c15c       ??_C@_1CC@PLPNIKGL@?$AAW?$AAS?$AA_?$AAE?$AAX?$AA_?$AAW?$AAI?$AAN?$AAD?$AAO?$AAW?$AAE?$AAD?$AAG@ 1004915c     Pclass.obj
 0002:0000c180       ??_C@_1CC@IAPGCLEG@?$AAW?$AAS?$AA_?$AAE?$AAX?$AA_?$AAC?$AAL?$AAI?$AAE?$AAN?$AAT?$AAE?$AAD?$AAG@ 10049180     Pclass.obj
 0002:0000c1a4       ??_C@_1CE@EANKNCIF@?$AAW?$AAS?$AA_?$AAE?$AAX?$AA_?$AAC?$AAO?$AAN?$AAT?$AAE?$AAX?$AAT?$AAH?$AAE@ 100491a4     Pclass.obj
 0002:0000c1c8       ??_C@_1BI@GFIADCMK@?$AAW?$AAS?$AA_?$AAE?$AAX?$AA_?$AAR?$AAI?$AAG?$AAH?$AAT@ 100491c8     Pclass.obj
 0002:0000c1e0       ??_C@_1CC@JOFCJJPB@?$AAW?$AAS?$AA_?$AAE?$AAX?$AA_?$AAR?$AAT?$AAL?$AAR?$AAE?$AAA?$AAD?$AAI?$AAN@ 100491e0     Pclass.obj
 0002:0000c204       ??_C@_1CI@EFLDECAB@?$AAW?$AAS?$AA_?$AAE?$AAX?$AA_?$AAL?$AAE?$AAF?$AAT?$AAS?$AAC?$AAR?$AAO?$AAL@ 10049204     Pclass.obj
 0002:0000c22c       ??_C@_1CI@CIFGFFJB@?$AAW?$AAS?$AA_?$AAE?$AAX?$AA_?$AAC?$AAO?$AAN?$AAT?$AAR?$AAO?$AAL?$AAP?$AAA@ 1004922c     Pclass.obj
 0002:0000c254       ??_C@_1CC@BGEPLDCA@?$AAW?$AAS?$AA_?$AAE?$AAX?$AA_?$AAS?$AAT?$AAA?$AAT?$AAI?$AAC?$AAE?$AAD?$AAG@ 10049254     Pclass.obj
 0002:0000c278       ??_C@_1CA@DOAIHHLO@?$AAW?$AAS?$AA_?$AAE?$AAX?$AA_?$AAA?$AAP?$AAP?$AAW?$AAI?$AAN?$AAD?$AAO?$AAW@ 10049278     Pclass.obj
 0002:0000c298       ??_C@_1BM@FAODAMGD@?$AAW?$AAS?$AA_?$AAE?$AAX?$AA_?$AAL?$AAA?$AAY?$AAE?$AAR?$AAE?$AAD@ 10049298     Pclass.obj
 0002:0000c2b4       ??_C@_1CM@DJKNBOGD@?$AAW?$AAS?$AA_?$AAE?$AAX?$AA_?$AAN?$AAO?$AAI?$AAN?$AAH?$AAE?$AAR?$AAI?$AAT@ 100492b4     Pclass.obj
 0002:0000c2e0       ??_C@_1CA@KMHLBMFI@?$AAW?$AAS?$AA_?$AAE?$AAX?$AA_?$AAL?$AAA?$AAY?$AAO?$AAU?$AAT?$AAR?$AAT?$AAL@ 100492e0     Pclass.obj
 0002:0000c300       ??_C@_1CC@LOFMDOPL@?$AAW?$AAS?$AA_?$AAE?$AAX?$AA_?$AAN?$AAO?$AAA?$AAC?$AAT?$AAI?$AAV?$AAA?$AAT@ 10049300     Pclass.obj
 0002:0000c324       ??_C@_1O@EEMHCPPG@?$AA?$HL?$AA?3?$AA2?$AA0?$AA?$HN?$AA?6@ 10049324     Pclass.obj
 0002:0000c334       ??_C@_1BM@LABJMFIE@?$AA?$HL?$AA?3?$AA?$DO?$AA2?$AA0?$AA?$HN?$AA?5?$AA?$HL?$AA?3?$AA7?$AA?$HN?$AA?$CF?$AA?6@ 10049334     Pclass.obj
 0002:0000c350       ??_C@_1BO@HALKGPHE@?$AA?$HL?$AA?3?$AA2?$AA0?$AA?$HN?$AA?5?$AA?5?$AA?$HL?$AA?3?$AA7?$AA?$HN?$AA?$HL?$AA?$HN?$AA?6@ 10049350     Pclass.obj
 0002:0000c370       ??_C@_19GGNHIDOH@?$AA?4?$AAt?$AAx?$AAt@ 10049370     Pclass.obj
 0002:0000c37c       ??_C@_1BI@KNPOOCNP@?$AA?$HL?$AA?$HN?$AA?$HL?$AA?$HN?$AA?0?$AA?5?$AA?$HL?$AA?$HN?$AA?$HL?$AA?$HN?$AA?6@ 1004937c     Pclass.obj
 0002:0000c394       ??_C@_1M@PLHOGBPP@?$AA?$HL?$AA?$HN?$AA?$HL?$AA?$HN?$AA?6@ 10049394     Pclass.obj
 0002:0000c3a0       ??_C@_1BE@IFNNBPIG@?$AA?$HL?$AA?$HN?$AA?5?$AA?5?$AA?$CI?$AA?$HL?$AA?$HN?$AA?$CJ?$AA?6@ 100493a0     Pclass.obj
 0002:0000c3b4       ??_C@_17LDOGFDCL@?$AA?$HL?$AA?$HN?$AA?6@ 100493b4     Pclass.obj
 0002:0000c3bc       ??_C@_1BE@DMHIKKPF@?$AA?6?$AA?$HL?$AA?$HN?$AA?$HL?$AA?$HN?$AA?5?$AA?$HL?$AA?$HN?$AA?6@ 100493bc     Pclass.obj
 0002:0000c3d0       ??_C@_1O@IDCHAEMM@?$AA?6?$AA?$HL?$AA?$HN?$AA?$HL?$AA?$HN?$AA?6@ 100493d0     Pclass.obj
 0002:0000c3e0       ??_C@_1BC@JCEOJDJG@?$AA?6?$AA?$HL?$AA?$HN?$AA?3?$AA?6?$AA?$HL?$AA?$HN?$AA?6@ 100493e0     Pclass.obj
 0002:0000c3f4       ??_C@_19OPNPIOHE@?$AAH?$AAW?$AAN?$AAD@ 100493f4     Pclass.obj
 0002:0000c400       ??_C@_1BK@HEHCIBBK@?$AA?$HL?$AA?$HN?$AA?$HL?$AA?3?$AA0?$AA8?$AAX?$AA?$HN?$AA?5?$AA?$HL?$AA?$HN?$AA?6@ 10049400     Pclass.obj
 0002:0000c41c       ??_C@_1CM@NMKGACPH@?$AA?6?$AA?$HL?$AA?$HN?$AA?3?$AA?6?$AA?$HL?$AA?3?$AA?$DM?$AA?$HL?$AA?$HN?$AA?$HN?$AA?5?$AA?$HL?$AA?3?$AA?$DM@ 1004941c     Pclass.obj
 0002:0000c448       ??_C@_15GKIJICBO@?$AAZ?$AAC@ 10049448     Pclass.obj
 0002:0000c450       ??_C@_17JJIMNMHK@?$AA?5?$AA?$CG?$AA?$FO@ 10049450     Pclass.obj
 0002:0000c458       ??_C@_13HOIJIPNN@?$AA?5@   10049458     Pclass.obj
 0002:0000c45c       ??_C@_15LEKKCGMK@?$AA?2?$AA?2@ 1004945c     Pclass.obj
 0002:0000c464       ??_C@_15DDHGOCBH@?$AA?4?$AA?4@ 10049464     Pclass.obj
 0002:0000c46c       ??_C@_17FJPEEFCB@?$AAp?$AAr?$AAc@ 1004946c     Pclass.obj
 0002:0000c474       ??_C@_1BC@ENICKDH@?$AAC?$AAo?$AAn?$AAt?$AAe?$AAn?$AAt?$AAs@ 10049474     Pclass.obj
 0002:0000c488       ??_C@_1CK@DGKCELDD@?$AAP?$AAr?$AAo?$AAc?$AAe?$AAs?$AAs?$AAL?$AAi?$AAs?$AAt?$AA?4?$AAC?$AAo?$AAm@ 10049488     Pclass.obj
 0002:0000c4b4       ??_C@_1CK@ECJCGOEK@?$AAP?$AAr?$AAo?$AAc?$AAe?$AAs?$AAs?$AAL?$AAi?$AAs?$AAt?$AA?4?$AAU?$AAs?$AAe@ 100494b4     Pclass.obj
 0002:0000c4e0       ??_C@_19LEMHLIAI@?$AA?$CF?$AA?5?$AA?$HL?$AA?$HN@ 100494e0     Pclass.obj
 0002:0000c4ec       ??_C@_19NNDJOIOE@?$AA?$HL?$AA?$HN?$AA?$HL?$AA?$HN@ 100494ec     Pclass.obj
 0002:0000c4f8       ??_C@_1DG@GNDNNFLA@?$AA?$HL?$AA?$HN?$AA?5?$AA?$HL?$AA?3?$AA0?$AA2?$AA?$HN?$AA?3?$AA?$HL?$AA?3?$AA0?$AA2?$AA?$HN?$AA?3@ 100494f8     Pclass.obj
 0002:0000c530       ??_C@_1DA@IEGGOAFB@?$AA?$HL?$AA?3?$AA0?$AA2?$AA?$HN?$AA?3?$AA?$HL?$AA?3?$AA0?$AA2?$AA?$HN?$AA?3?$AA?$HL?$AA?3?$AA0@ 10049530     Pclass.obj
 0002:0000c560       ??_C@_19JHEHLFPM@?$AA?2?$AA?$DP?$AA?$DP?$AA?2@ 10049560     Pclass.obj
 0002:0000c56c       ??_C@_1DC@HCLBMGIA@?$AA?2?$AAV?$AAa?$AAr?$AAF?$AAi?$AAl?$AAe?$AAI?$AAn?$AAf?$AAo?$AA?2?$AAT?$AAr@ 1004956c     Pclass.obj
 0002:0000c5a0       ??_C@_1DM@LKEGNDCP@?$AA?2?$AAS?$AAt?$AAr?$AAi?$AAn?$AAg?$AAF?$AAi?$AAl?$AAe?$AAI?$AAn?$AAf?$AAo@ 100495a0     Pclass.obj
 0002:0000c5dc       ??_C@_1BI@HCCAONKE@?$AAF?$AAi?$AAl?$AAe?$AAV?$AAe?$AAr?$AAs?$AAi?$AAo?$AAn@ 100495dc     Pclass.obj
 0002:0000c5f4       ??_C@_1CA@JGBAIPOO@?$AAF?$AAi?$AAl?$AAe?$AAD?$AAe?$AAs?$AAc?$AAr?$AAi?$AAp?$AAt?$AAi?$AAo?$AAn@ 100495f4     Pclass.obj
 0002:0000c614       ??_C@_17FNIAADFF@?$AA?$HL?$AA?$HN?$AA?2@ 10049614     Pclass.obj
 0002:0000c61c       ??_C@_1M@FLCNNCCB@?$AA?5?$AA?$CI?$AA?$HL?$AA?$HN?$AA?$CJ@ 1004961c     Pclass.obj
 0002:0000c628       ??_C@_1BC@OMEIBLAI@?$AAw?$AAb?$AAe?$AAm?$AAc?$AAo?$AAm?$AAn@ 10049628     Pclass.obj
 0002:0000c63c       ??_C@_0BA@FOIKENOD@vector?5too?5long@ 1004963c     Pclass.obj
 0002:0000c64c       ??_C@_0BI@CFPLBAOH@invalid?5string?5position@ 1004964c     Pclass.obj
 0002:0000c664       ??_C@_15LGINNLBP@?$AA?$HL?$AA?$HN@ 10049664     Pclass.obj
 0002:0000c66c       ??_C@_0BL@GOIGLPKN@unordered_map?1set?5too?5long@ 1004966c     Pclass.obj
 0002:0000c688       ??_C@_0BK@OGNNAFAB@invalid?5hash?5bucket?5count@ 10049688     Pclass.obj
 0002:0000c780       ??_7PluginEditFieldBinding@@6B@ 10049780     Pclass.obj
 0002:0000c8e0       ?Counters@@3QBUcounters@@B 100498e0     perfthread.obj
 0002:0000c9e8       ??_C@_1CC@DNHMJIKH@?$AA?$CF?$AA?5?$AAP?$AAr?$AAo?$AAc?$AAe?$AAs?$AAs?$AAo?$AAr?$AA?5?$AAT?$AAi?$AAm@ 100499e8     perfthread.obj
 0002:0000ca0c       ??_C@_1CE@FNEMIHOD@?$AA?$CF?$AA?5?$AAP?$AAr?$AAi?$AAv?$AAi?$AAl?$AAe?$AAg?$AAe?$AAd?$AA?5?$AAT?$AAi@ 10049a0c     perfthread.obj
 0002:0000ca30       ??_C@_1BI@IIOPEKIO@?$AA?$CF?$AA?5?$AAU?$AAs?$AAe?$AAr?$AA?5?$AAT?$AAi?$AAm?$AAe@ 10049a30     perfthread.obj
 0002:0000ca48       ??_C@_1BK@FAAJNJIB@?$AAH?$AAa?$AAn?$AAd?$AAl?$AAe?$AA?5?$AAC?$AAo?$AAu?$AAn?$AAt@ 10049a48     perfthread.obj
 0002:0000ca64       ??_C@_1CA@KJMNGIDJ@?$AAP?$AAa?$AAg?$AAe?$AA?5?$AAF?$AAi?$AAl?$AAe?$AA?5?$AAB?$AAy?$AAt?$AAe?$AAs@ 10049a64     perfthread.obj
 0002:0000ca84       ??_C@_1CK@FGGMBBIH@?$AAP?$AAa?$AAg?$AAe?$AA?5?$AAF?$AAi?$AAl?$AAe?$AA?5?$AAB?$AAy?$AAt?$AAe?$AAs@ 10049a84     perfthread.obj
 0002:0000cab0       ??_C@_1BI@GCOMDKEO@?$AAW?$AAo?$AAr?$AAk?$AAi?$AAn?$AAg?$AA?5?$AAS?$AAe?$AAt@ 10049ab0     perfthread.obj
 0002:0000cac8       ??_C@_1CC@OFJLEPCP@?$AAW?$AAo?$AAr?$AAk?$AAi?$AAn?$AAg?$AA?5?$AAS?$AAe?$AAt?$AA?5?$AAP?$AAe?$AAa@ 10049ac8     perfthread.obj
 0002:0000caec       ??_C@_1CI@LLKMGPEG@?$AAP?$AAo?$AAo?$AAl?$AA?5?$AAN?$AAo?$AAn?$AAp?$AAa?$AAg?$AAe?$AAd?$AA?5?$AAB@ 10049aec     perfthread.obj
 0002:0000cb14       ??_C@_1CC@IMBAECJF@?$AAP?$AAo?$AAo?$AAl?$AA?5?$AAP?$AAa?$AAg?$AAe?$AAd?$AA?5?$AAB?$AAy?$AAt?$AAe@ 10049b14     perfthread.obj
 0002:0000cb38       ??_C@_1BM@DGDPAMAA@?$AAP?$AAr?$AAi?$AAv?$AAa?$AAt?$AAe?$AA?5?$AAB?$AAy?$AAt?$AAe?$AAs@ 10049b38     perfthread.obj
 0002:0000cb54       ??_C@_1CA@GADAGCME@?$AAP?$AAa?$AAg?$AAe?$AA?5?$AAF?$AAa?$AAu?$AAl?$AAt?$AAs?$AA?1?$AAs?$AAe?$AAc@ 10049b54     perfthread.obj
 0002:0000cb74       ??_C@_1BM@FMIOMJAE@?$AAV?$AAi?$AAr?$AAt?$AAu?$AAa?$AAl?$AA?5?$AAB?$AAy?$AAt?$AAe?$AAs@ 10049b74     perfthread.obj
 0002:0000cb90       ??_C@_1CG@KJOKFONA@?$AAV?$AAi?$AAr?$AAt?$AAu?$AAa?$AAl?$AA?5?$AAB?$AAy?$AAt?$AAe?$AAs?$AA?5?$AAP@ 10049b90     perfthread.obj
 0002:0000cbb8       ??_C@_1CE@DFDFLLAO@?$AAI?$AAO?$AA?5?$AAD?$AAa?$AAt?$AAa?$AA?5?$AAB?$AAy?$AAt?$AAe?$AAs?$AA?1?$AAs@ 10049bb8     perfthread.obj
 0002:0000cbdc       ??_C@_1CE@EFLEKJAB@?$AAI?$AAO?$AA?5?$AAR?$AAe?$AAa?$AAd?$AA?5?$AAB?$AAy?$AAt?$AAe?$AAs?$AA?1?$AAs@ 10049bdc     perfthread.obj
 0002:0000cc00       ??_C@_1CG@MEJHKKKF@?$AAI?$AAO?$AA?5?$AAW?$AAr?$AAi?$AAt?$AAe?$AA?5?$AAB?$AAy?$AAt?$AAe?$AAs?$AA?1@ 10049c00     perfthread.obj
 0002:0000cc28       ??_C@_1CG@LBBBPCJA@?$AAI?$AAO?$AA?5?$AAO?$AAt?$AAh?$AAe?$AAr?$AA?5?$AAB?$AAy?$AAt?$AAe?$AAs?$AA?1@ 10049c28     perfthread.obj
 0002:0000cc50       ??_C@_1CO@LIEOHDCC@?$AAI?$AAO?$AA?5?$AAD?$AAa?$AAt?$AAa?$AA?5?$AAO?$AAp?$AAe?$AAr?$AAa?$AAt?$AAi@ 10049c50     perfthread.obj
 0002:0000cc80       ??_C@_1CO@LIIKBHDH@?$AAI?$AAO?$AA?5?$AAR?$AAe?$AAa?$AAd?$AA?5?$AAO?$AAp?$AAe?$AAr?$AAa?$AAt?$AAi@ 10049c80     perfthread.obj
 0002:0000ccb0       ??_C@_1DA@HICMAFKK@?$AAI?$AAO?$AA?5?$AAW?$AAr?$AAi?$AAt?$AAe?$AA?5?$AAO?$AAp?$AAe?$AAr?$AAa?$AAt@ 10049cb0     perfthread.obj
 0002:0000cce0       ??_C@_1DA@BEHINMGJ@?$AAI?$AAO?$AA?5?$AAO?$AAt?$AAh?$AAe?$AAr?$AA?5?$AAO?$AAp?$AAe?$AAr?$AAa?$AAt@ 10049ce0     perfthread.obj
 0002:0000cd10       ??_C@_1BA@MGJGGMO@?$AAC?$AAo?$AAu?$AAn?$AAt?$AAe?$AAr@ 10049d10     perfthread.obj
 0002:0000cd20       ??_C@_1BG@NKNJPBCD@?$AAI?$AAD?$AA?5?$AAP?$AAr?$AAo?$AAc?$AAe?$AAs?$AAs@ 10049d20     perfthread.obj
 0002:0000cd38       ??_C@_1BM@KCAKLHJN@?$AAP?$AAr?$AAi?$AAo?$AAr?$AAi?$AAt?$AAy?$AA?5?$AAB?$AAa?$AAs?$AAe@ 10049d38     perfthread.obj
 0002:0000cd54       ??_C@_1BK@KCHPPKHP@?$AAT?$AAh?$AAr?$AAe?$AAa?$AAd?$AA?5?$AAC?$AAo?$AAu?$AAn?$AAt@ 10049d54     perfthread.obj
 0002:0000cd70       ??_C@_1CI@FNIEMNAI@?$AAC?$AAr?$AAe?$AAa?$AAt?$AAi?$AAn?$AAg?$AA?5?$AAP?$AAr?$AAo?$AAc?$AAe?$AAs@ 10049d70     perfthread.obj
 0002:0000cd98       ??_C@_1BK@IKAFHKBD@?$AAE?$AAl?$AAa?$AAp?$AAs?$AAe?$AAd?$AA?5?$AAT?$AAi?$AAm?$AAe@ 10049d98     perfthread.obj
 0002:0000cdb4       ??_C@_19DOGDICKI@?$AA?4?$AAe?$AAx?$AAe@ 10049db4     perfthread.obj
 0002:0000cdc0       ??_C@_19DLCFHDFF@?$AAP?$AAE?$AAR?$AAF@ 10049dc0     perfthread.obj
 0002:0000cdcc       ??_C@_1O@NKAIMMPD@?$AA_?$AAT?$AAo?$AAt?$AAa?$AAl@ 10049dcc     Plist.obj
 0002:0000cddc       ??_C@_1CC@DMDJMJLM@?$AAS?$AAe?$AAD?$AAe?$AAb?$AAu?$AAg?$AAP?$AAr?$AAi?$AAv?$AAi?$AAl?$AAe?$AAg@ 10049ddc     Plist.obj
 0002:0000ce00       ??_C@_1BA@LGLNCAB@?$AA?$HL?$AA?$HN?$AA?3?$AA?6?$AA?$HL?$AA?$HN?$AA?6@ 10049e00     Plist.obj
 0002:0000ce10       ??_C@_1M@JNLNOPHA@?$AA?6?$AA?$HL?$AA?$HN?$AA?3?$AA?6@ 10049e10     Plist.obj
 0002:0000ce1c       ??_C@_1BC@LCLKNDBE@?$AA?$HL?$AA?$HN?$AA?5?$AA?$HL?$AA?3?$AA8?$AAX?$AA?$HN@ 10049e1c     Plist.obj
 0002:0000ce30       ??_C@_17JLBLMHID@?$AA?5?$AA?$HL?$AA?$HN@ 10049e30     Plist.obj
 0002:0000ce38       ??_C@_1BA@LLEFIMNA@?$AA?$HL?$AA?3?$AA0?$AA?$HL?$AA?$HN?$AAX?$AA?$HN@ 10049e38     Plist.obj
 0002:0000ce48       ??_C@_1BA@EGCKMFAC@?$AA?$HL?$AA?3?$AA0?$AA1?$AA6?$AAX?$AA?$HN@ 10049e48     Plist.obj
 0002:0000ce5c       ??_7?$_Func_impl_no_alloc@V<lambda_1>@?6??PrintModules@?$ipc_functions@$00@@SAXPAX0AAUoptions@@@Z@_NPA_WI@std@@6B@ 10049e5c     Plist.obj
 0002:0000ce78       ??_7?$_Func_impl_no_alloc@V<lambda_1>@?6??PrintModules@?$ipc_functions@$0A@@@SAXPAX0AAUoptions@@@Z@_NPA_WI@std@@6B@ 10049e78     Plist.obj
 0002:0000ceac       ??_C@_1CA@CCAFOKCB@?$AAE?$AAr?$AAr?$AAo?$AAr?$AA?5?$AA0?$AAx?$AA?$HL?$AA0?$AA?3?$AA0?$AA8?$AAX?$AA?$HN@ 10049eac     Pmix.obj
 0002:0000cecc       ??_C@_15JNBOKNOG@?$AA?$AN?$AA?6@ 10049ecc     Pmix.obj
 0002:0000ced4       ??_C@_1DC@LAIEFOLO@?$AAW?$AAi?$AAn?$AA3?$AA2?$AA_?$AAP?$AAr?$AAo?$AAc?$AAe?$AAs?$AAs?$AA?4?$AAH@ 10049ed4     wmi.obj
 0002:0000cf08       ??_C@_1BO@CLCOBGDE@?$AAE?$AAx?$AAe?$AAc?$AAu?$AAt?$AAa?$AAb?$AAl?$AAe?$AAP?$AAa?$AAt?$AAh@ 10049f08     wmi.obj
 0002:0000cf28       ??_C@_1BI@LPJNJKGA@?$AAC?$AAo?$AAm?$AAm?$AAa?$AAn?$AAd?$AAL?$AAi?$AAn?$AAe@ 10049f28     wmi.obj
 0002:0000cf40       ??_C@_1BC@JHNNEHFE@?$AAP?$AAr?$AAi?$AAo?$AAr?$AAi?$AAt?$AAy@ 10049f40     wmi.obj
 0002:0000cf54       ??_C@_1BC@HJJANEGO@?$AAG?$AAe?$AAt?$AAO?$AAw?$AAn?$AAe?$AAr@ 10049f54     wmi.obj
 0002:0000cf68       ??_C@_19PIJILKAI@?$AAU?$AAs?$AAe?$AAr@ 10049f68     wmi.obj
 0002:0000cf74       ??_C@_1O@OAMNPMOM@?$AAD?$AAo?$AAm?$AAa?$AAi?$AAn@ 10049f74     wmi.obj
 0002:0000cf84       ??_C@_1BI@OIPNMPCL@?$AAG?$AAe?$AAt?$AAO?$AAw?$AAn?$AAe?$AAr?$AAS?$AAi?$AAd@ 10049f84     wmi.obj
 0002:0000cf9c       ??_C@_17NKMLOKHF@?$AAS?$AAi?$AAd@ 10049f9c     wmi.obj
 0002:0000cfa4       ??_C@_1BE@CFEJJKFE@?$AAS?$AAe?$AAs?$AAs?$AAi?$AAo?$AAn?$AAI?$AAd@ 10049fa4     wmi.obj
 0002:0000cfb8       ??_C@_1BM@MLGLIGHJ@?$AAW?$AAi?$AAn?$AA3?$AA2?$AA_?$AAP?$AAr?$AAo?$AAc?$AAe?$AAs?$AAs@ 10049fb8     wmi.obj
 0002:0000cfd4       ??_C@_1BI@FLOHINJE@?$AAR?$AAe?$AAt?$AAu?$AAr?$AAn?$AAV?$AAa?$AAl?$AAu?$AAe@ 10049fd4     wmi.obj
 0002:0000cfec       ??_C@_1BI@NKNJJIDM@?$AAS?$AAe?$AAt?$AAP?$AAr?$AAi?$AAo?$AAr?$AAi?$AAt?$AAy@ 10049fec     wmi.obj
 0002:0000d004       ??_C@_1O@GGHBFGJC@?$AAR?$AAe?$AAa?$AAs?$AAo?$AAn@ 1004a004     wmi.obj
 0002:0000d014       ??_C@_1BE@PBPGMODO@?$AAT?$AAe?$AAr?$AAm?$AAi?$AAn?$AAa?$AAt?$AAe@ 1004a014     wmi.obj
 0002:0000d028       ??_C@_13JOFGPIOO@?$AA?4@   1004a028     wmi.obj
 0002:0000d02c       ??_C@_1CC@OGNCBAIB@?$AA?2?$AA?2?$AA?$HL?$AA0?$AA?$HN?$AA?2?$AAr?$AAo?$AAo?$AAt?$AA?2?$AAc?$AAi?$AAm?$AAv@ 1004a02c     wmi.obj
 0002:0000d088       _MainGuid                  1004a088     Proclist.obj
 0002:0000d098       _ConfigDialogGuid          1004a098     Proclist.obj
 0002:0000d0a8       ??_C@_1M@OAIMIKLP@?$AAn?$AAt?$AAd?$AAl?$AAl@ 1004a0a8     Proclist.obj
 0002:0000d0b4       ??_C@_0BK@EGDDIFMK@NtQueryInformationProcess@ 1004a0b4     Proclist.obj
 0002:0000d0d0       ??_C@_0BJ@HKKELGGC@NtQueryInformationThread@ 1004a0d0     Proclist.obj
 0002:0000d0ec       ??_C@_0O@IFMDHOMC@NtQueryObject@ 1004a0ec     Proclist.obj
 0002:0000d0fc       ??_C@_0BJ@NDLOPGCH@NtQuerySystemInformation@ 1004a0fc     Proclist.obj
 0002:0000d118       ??_C@_0BH@DLPGICA@NtQueryInformationFile@ 1004a118     Proclist.obj
 0002:0000d130       ??_C@_0CB@GDPHBMJN@NtWow64QueryInformationProcess6@ 1004a130     Proclist.obj
 0002:0000d154       ??_C@_0BL@NJDHCDMK@NtWow64ReadVirtualMemory64@ 1004a154     Proclist.obj
 0002:0000d170       ??_C@_1BC@GDMECMAK@?$AAk?$AAe?$AAr?$AAn?$AAe?$AAl?$AA3?$AA2@ 1004a170     Proclist.obj
 0002:0000d184       ??_C@_0P@LKABJJMO@IsWow64Process@ 1004a184     Proclist.obj
 0002:0000d194       ??_C@_1BC@DNHGCMLG@?$AAa?$AAd?$AAv?$AAa?$AAp?$AAi?$AA3?$AA2@ 1004a194     Proclist.obj
 0002:0000d1a8       ??_C@_0L@KJHKJIPF@IsValidSid@ 1004a1a8     Proclist.obj
 0002:0000d1b4       ??_C@_0BK@FIHGNING@GetSidIdentifierAuthority@ 1004a1b4     Proclist.obj
 0002:0000d1d0       ??_C@_0BI@LPFJALDI@GetSidSubAuthorityCount@ 1004a1d0     Proclist.obj
 0002:0000d1e8       ??_C@_0BD@LMGFHOAE@GetSidSubAuthority@ 1004a1e8     Proclist.obj
 0002:0000d1fc       ??_C@_1O@BCCLBEOE@?$AAu?$AAs?$AAe?$AAr?$AA3?$AA2@ 1004a1fc     Proclist.obj
 0002:0000d20c       ??_C@_0BA@FKGDNIJG@GetGuiResources@ 1004a20c     Proclist.obj
 0002:0000d21c       ??_C@_1M@FFPAMFOB@?$AAo?$AAl?$AAe?$AA3?$AA2@ 1004a21c     Proclist.obj
 0002:0000d228       ??_C@_0BC@IOEGILCE@CoSetProxyBlanket@ 1004a228     Proclist.obj
 0002:0000d23c       ??_C@_1M@OMFDJDJC@?$AAp?$AAs?$AAa?$AAp?$AAi@ 1004a23c     Proclist.obj
 0002:0000d248       ??_C@_0BF@LEEEDPDK@EnumProcessModulesEx@ 1004a248     Proclist.obj
 0002:0000d260       ??_C@_1BC@PDEABLIN@?$AAP?$AAr?$AAo?$AAc?$AAL?$AAi?$AAs?$AAt@ 1004a260     Proclist.obj
 0002:0000d274       ??_C@_1DK@DCAMPEPJ@?$AAP?$AAr?$AAo?$AAc?$AAe?$AAs?$AAs?$AA?5?$AAL?$AAi?$AAs?$AAt?$AA?5?$AAf?$AAo@ 1004a274     Proclist.obj
 0002:0000d2b0       ??_C@_1DE@BGKMIKPD@?$AAE?$AAu?$AAg?$AAe?$AAn?$AAe?$AA?5?$AAR?$AAo?$AAs?$AAh?$AAa?$AAl?$AA?5?$AA?$CG@ 1004a2b0     Proclist.obj
 0002:0000d2e4       ??_C@_1M@MNPEKPKO@?$AAp?$AAl?$AAi?$AAs?$AAt@ 1004a2e4     Proclist.obj
 0002:0000d2f0       _MenuGuid                  1004a2f0     Proclist.obj
 0002:0000d300       ??_C@_0O@NLDKAIKN@EncodePointer@ 1004a300     vc_crt_fix_impl.obj
 0002:0000d310       ??_C@_0O@KBPMFGHI@DecodePointer@ 1004a310     vc_crt_fix_impl.obj
 0002:0000d320       ??_C@_0BD@GIGEJCNH@GetModuleHandleExW@ 1004a320     vc_crt_fix_impl.obj
 0002:0000d334       ??_C@_0BE@NBEJPEJA@InitializeSListHead@ 1004a334     vc_crt_fix_impl.obj
 0002:0000d348       ??_C@_0BG@PLLPFLHB@InterlockedFlushSList@ 1004a348     vc_crt_fix_impl.obj
 0002:0000d360       ??_C@_0BJ@PNEEKDOK@InterlockedPopEntrySList@ 1004a360     vc_crt_fix_impl.obj
 0002:0000d37c       ??_C@_0BK@JFGGAIOA@InterlockedPushEntrySList@ 1004a37c     vc_crt_fix_impl.obj
 0002:0000d398       ??_C@_0BL@FOECAEGO@InterlockedPushListSListEx@ 1004a398     vc_crt_fix_impl.obj
 0002:0000d3b4       ??_C@_0BD@FHMMIGCI@RtlFirstEntrySList@ 1004a3b4     vc_crt_fix_impl.obj
 0002:0000d3c8       ??_C@_0BA@FGPHPMJB@QueryDepthSList@ 1004a3c8     vc_crt_fix_impl.obj
 0002:0000d3d8       ??_C@_0BJ@NLNFLAMA@GetNumaHighestNodeNumber@ 1004a3d8     vc_crt_fix_impl.obj
 0002:0000d3f4       ??_C@_0BP@KHGALBC@GetLogicalProcessorInformation@ 1004a3f4     vc_crt_fix_impl.obj
 0002:0000d414       ??_C@_0BI@BKLFFAPO@SetThreadStackGuarantee@ 1004a414     vc_crt_fix_impl.obj
 0002:0000d42c       ??_C@_0BM@HCFOFFN@InitializeCriticalSectionEx@ 1004a42c     vc_crt_fix_impl.obj
 0002:0000d448       ??_C@_0BA@IHGNDAEB@CompareStringEx@ 1004a448     vc_crt_fix_impl.obj
 0002:0000d478       __real@3fe0000000000000    1004a478     perfthread.obj
 0002:0000d480       __real@4024000000000000    1004a480     Pclass.obj
 0002:0000d488       __real@41f0000000000000    1004a488     Pclass.obj
 0002:0000d490       __real@43e0000000000000    1004a490     Pclass.obj
 0002:0000d498       __real@4f800000            1004a498     Pclass.obj
 0002:0000d4f0       __load_config_used         1004a4f0     LIBCMT:loadcfg.obj
 0002:0000d5c0       ??_R4bad_function_call@std@@6B@ 1004a5c0     libcpmt:xthrow.obj
 0002:0000d5d4       ??_R3bad_function_call@std@@8 1004a5d4     libcpmt:xthrow.obj
 0002:0000d5e4       ??_R2bad_function_call@std@@8 1004a5e4     libcpmt:xthrow.obj
 0002:0000d5f0       ??_R1A@?0A@EA@bad_function_call@std@@8 1004a5f0     libcpmt:xthrow.obj
 0002:0000d60c       ??_R4logic_error@std@@6B@  1004a60c     libcpmt:xthrow.obj
 0002:0000d620       ??_R3logic_error@std@@8    1004a620     libcpmt:xthrow.obj
 0002:0000d630       ??_R2logic_error@std@@8    1004a630     libcpmt:xthrow.obj
 0002:0000d63c       ??_R1A@?0A@EA@logic_error@std@@8 1004a63c     libcpmt:xthrow.obj
 0002:0000d658       ??_R4length_error@std@@6B@ 1004a658     libcpmt:xthrow.obj
 0002:0000d66c       ??_R3length_error@std@@8   1004a66c     libcpmt:xthrow.obj
 0002:0000d67c       ??_R2length_error@std@@8   1004a67c     libcpmt:xthrow.obj
 0002:0000d68c       ??_R1A@?0A@EA@length_error@std@@8 1004a68c     libcpmt:xthrow.obj
 0002:0000d6a8       ??_R4out_of_range@std@@6B@ 1004a6a8     libcpmt:xthrow.obj
 0002:0000d6bc       ??_R3out_of_range@std@@8   1004a6bc     libcpmt:xthrow.obj
 0002:0000d6cc       ??_R2out_of_range@std@@8   1004a6cc     libcpmt:xthrow.obj
 0002:0000d6dc       ??_R1A@?0A@EA@out_of_range@std@@8 1004a6dc     libcpmt:xthrow.obj
 0002:0000d6f8       ??_R4_Locimp@locale@std@@6B@ 1004a6f8     libcpmt:locale0.obj
 0002:0000d70c       ??_R3_Locimp@locale@std@@8 1004a70c     libcpmt:locale0.obj
 0002:0000d71c       ??_R2_Locimp@locale@std@@8 1004a71c     libcpmt:locale0.obj
 0002:0000d730       ??_R1A@?0A@EA@_Locimp@locale@std@@8 1004a730     libcpmt:locale0.obj
 0002:0000d74c       ??_R4type_info@@6B@        1004a74c     LIBCMT:std_type_info_static.obj
 0002:0000d760       ??_R3type_info@@8          1004a760     LIBCMT:std_type_info_static.obj
 0002:0000d770       ??_R2type_info@@8          1004a770     LIBCMT:std_type_info_static.obj
 0002:0000d778       ??_R1A@?0A@EA@type_info@@8 1004a778     LIBCMT:std_type_info_static.obj
 0002:0000d794       ??_R4bad_exception@std@@6B@ 1004a794     libvcruntime:frame.obj
 0002:0000d7a8       ??_R3bad_exception@std@@8  1004a7a8     libvcruntime:frame.obj
 0002:0000d7b8       ??_R2bad_exception@std@@8  1004a7b8     libvcruntime:frame.obj
 0002:0000d7c4       ??_R1A@?0A@EA@bad_exception@std@@8 1004a7c4     libvcruntime:frame.obj
 0002:0000d7e0       ??_R3?$buffer@_W@detail@v10@fmt@@8 1004a7e0     format.obj
 0002:0000d7f0       ??_R4?$basic_memory_buffer@_W$0BPE@V?$allocator@_W@std@@@v10@fmt@@6B@ 1004a7f0     format.obj
 0002:0000d804       ??_R4exception@std@@6B@    1004a804     format.obj
 0002:0000d818       ??_R2bad_array_new_length@std@@8 1004a818     format.obj
 0002:0000d828       ??_R4runtime_error@std@@6B@ 1004a828     format.obj
 0002:0000d83c       ??_R3_Facet_base@std@@8    1004a83c     format.obj
 0002:0000d84c       ??_R2?$basic_memory_buffer@H$0BPE@V?$allocator@H@std@@@v10@fmt@@8 1004a84c     format.obj
 0002:0000d858       ??_R2?$buffer@I@detail@v10@fmt@@8 1004a858     format.obj
 0002:0000d860       ??_R2bad_alloc@std@@8      1004a860     format.obj
 0002:0000d86c       ??_R3?$buffer@D@detail@v10@fmt@@8 1004a86c     format.obj
 0002:0000d87c       ??_R3_Crt_new_delete@std@@8 1004a87c     format.obj
 0002:0000d88c       ??_R1A@?0A@EA@runtime_error@std@@8 1004a88c     format.obj
 0002:0000d8a8       ??_R13?0A@EA@_Crt_new_delete@std@@8 1004a8a8     format.obj
 0002:0000d8c4       ??_R3format_error@v10@fmt@@8 1004a8c4     format.obj
 0002:0000d8d4       ??_R3?$basic_memory_buffer@I$0CA@V?$allocator@I@std@@@v10@fmt@@8 1004a8d4     format.obj
 0002:0000d8e4       ??_R4?$basic_memory_buffer@H$0BPE@V?$allocator@H@std@@@v10@fmt@@6B@ 1004a8e4     format.obj
 0002:0000d8f8       ??_R1A@?0A@EA@exception@std@@8 1004a8f8     format.obj
 0002:0000d914       ??_R1A@?0A@EA@?$basic_memory_buffer@H$0BPE@V?$allocator@H@std@@@v10@fmt@@8 1004a914     format.obj
 0002:0000d930       ??_R2?$numpunct@_W@std@@8  1004a930     format.obj
 0002:0000d944       ??_R1A@?0A@EA@_Facet_base@std@@8 1004a944     format.obj
 0002:0000d960       ??_R1A@?0A@EA@bad_alloc@std@@8 1004a960     format.obj
 0002:0000d97c       ??_R3?$buffer@H@detail@v10@fmt@@8 1004a97c     format.obj
 0002:0000d98c       ??_R2?$basic_memory_buffer@_W$0BPE@V?$allocator@_W@std@@@v10@fmt@@8 1004a98c     format.obj
 0002:0000d998       ??_R1A@?0A@EA@?$basic_memory_buffer@_W$0BPE@V?$allocator@_W@std@@@v10@fmt@@8 1004a998     format.obj
 0002:0000d9b4       ??_R1A@?0A@EA@?$buffer@D@detail@v10@fmt@@8 1004a9b4     format.obj
 0002:0000d9d0       ??_R4?$basic_memory_buffer@I$0CA@V?$allocator@I@std@@@v10@fmt@@6B@ 1004a9d0     format.obj
 0002:0000d9e4       ??_R2exception@std@@8      1004a9e4     format.obj
 0002:0000d9ec       ??_R1A@?0A@EA@format_error@v10@fmt@@8 1004a9ec     format.obj
 0002:0000da08       ??_R2?$buffer@H@detail@v10@fmt@@8 1004aa08     format.obj
 0002:0000da10       ??_R4format_error@v10@fmt@@6B@ 1004aa10     format.obj
 0002:0000da24       ??_R1A@?0A@EA@facet@locale@std@@8 1004aa24     format.obj
 0002:0000da40       ??_R2format_error@v10@fmt@@8 1004aa40     format.obj
 0002:0000da50       ??_R3?$basic_memory_buffer@H$0BPE@V?$allocator@H@std@@@v10@fmt@@8 1004aa50     format.obj
 0002:0000da60       ??_R3?$numpunct@_W@std@@8  1004aa60     format.obj
 0002:0000da70       ??_R2?$buffer@_W@detail@v10@fmt@@8 1004aa70     format.obj
 0002:0000da78       ??_R1A@?0A@EA@?$numpunct@_W@std@@8 1004aa78     format.obj
 0002:0000da94       ??_R2?$basic_memory_buffer@D$0BPE@V?$allocator@D@std@@@v10@fmt@@8 1004aa94     format.obj
 0002:0000daa0       ??_R3?$basic_memory_buffer@D$0BPE@V?$allocator@D@std@@@v10@fmt@@8 1004aaa0     format.obj
 0002:0000dab0       ??_R3exception@std@@8      1004aab0     format.obj
 0002:0000dac0       ??_R3facet@locale@std@@8   1004aac0     format.obj
 0002:0000dad0       ??_R3?$buffer@I@detail@v10@fmt@@8 1004aad0     format.obj
 0002:0000dae0       ??_R4bad_alloc@std@@6B@    1004aae0     format.obj
 0002:0000daf4       ??_R1A@?0A@EA@_Crt_new_delete@std@@8 1004aaf4     format.obj
 0002:0000db10       ??_R3bad_array_new_length@std@@8 1004ab10     format.obj
 0002:0000db20       ??_R3bad_alloc@std@@8      1004ab20     format.obj
 0002:0000db30       ??_R1A@?0A@EA@?$buffer@_W@detail@v10@fmt@@8 1004ab30     format.obj
 0002:0000db4c       ??_R4_Facet_base@std@@6B@  1004ab4c     format.obj
 0002:0000db60       ??_R3?$basic_memory_buffer@_W$0BPE@V?$allocator@_W@std@@@v10@fmt@@8 1004ab60     format.obj
 0002:0000db70       ??_R2?$basic_memory_buffer@I$0CA@V?$allocator@I@std@@@v10@fmt@@8 1004ab70     format.obj
 0002:0000db7c       ??_R2runtime_error@std@@8  1004ab7c     format.obj
 0002:0000db88       ??_R4?$numpunct@_W@std@@6B@ 1004ab88     format.obj
 0002:0000db9c       ??_R4bad_array_new_length@std@@6B@ 1004ab9c     format.obj
 0002:0000dbb0       ??_R1A@?0A@EA@?$buffer@H@detail@v10@fmt@@8 1004abb0     format.obj
 0002:0000dbcc       ??_R1A@?0A@EA@?$basic_memory_buffer@I$0CA@V?$allocator@I@std@@@v10@fmt@@8 1004abcc     format.obj
 0002:0000dbe8       ??_R2_Crt_new_delete@std@@8 1004abe8     format.obj
 0002:0000dbf0       ??_R1A@?0A@EA@bad_array_new_length@std@@8 1004abf0     format.obj
 0002:0000dc0c       ??_R4?$basic_memory_buffer@D$0BPE@V?$allocator@D@std@@@v10@fmt@@6B@ 1004ac0c     format.obj
 0002:0000dc20       ??_R1A@?0A@EA@?$buffer@I@detail@v10@fmt@@8 1004ac20     format.obj
 0002:0000dc3c       ??_R2_Facet_base@std@@8    1004ac3c     format.obj
 0002:0000dc44       ??_R2facet@locale@std@@8   1004ac44     format.obj
 0002:0000dc54       ??_R1A@?0A@EA@?$basic_memory_buffer@D$0BPE@V?$allocator@D@std@@@v10@fmt@@8 1004ac54     format.obj
 0002:0000dc70       ??_R3runtime_error@std@@8  1004ac70     format.obj
 0002:0000dc80       ??_R2?$buffer@D@detail@v10@fmt@@8 1004ac80     format.obj
 0002:0000dc88       ??_R3DialogAPIBinding@@8   1004ac88     Pcfg.obj
 0002:0000dc98       ??_R1A@?0A@EA@PluginCheckBoxBinding@@8 1004ac98     Pcfg.obj
 0002:0000dcb4       ??_R3PluginCheckBoxBinding@@8 1004acb4     Pcfg.obj
 0002:0000dcc4       ??_R2DialogAPIBinding@@8   1004acc4     Pcfg.obj
 0002:0000dccc       ??_R4PluginCheckBoxBinding@@6B@ 1004accc     Pcfg.obj
 0002:0000dce0       ??_R2PluginCheckBoxBinding@@8 1004ace0     Pcfg.obj
 0002:0000dcec       ??_R1A@?0A@EA@DialogAPIBinding@@8 1004acec     Pcfg.obj
 0002:0000dd08       ??_R2PluginEditFieldBinding@@8 1004ad08     Pclass.obj
 0002:0000dd14       ??_R4PluginEditFieldBinding@@6B@ 1004ad14     Pclass.obj
 0002:0000dd28       ??_R3PluginEditFieldBinding@@8 1004ad28     Pclass.obj
 0002:0000dd38       ??_R1A@?0A@EA@PluginEditFieldBinding@@8 1004ad38     Pclass.obj
 0002:0000dd54       ??_R3?$_Func_impl_no_alloc@V<lambda_1>@?6??PrintModules@?$ipc_functions@$0A@@@SAXPAX0AAUoptions@@@Z@_NPA_WI@std@@8 1004ad54     Plist.obj
 0002:0000dd64       ??_R2?$_Func_impl_no_alloc@V<lambda_1>@?6??PrintModules@?$ipc_functions@$00@@SAXPAX0AAUoptions@@@Z@_NPA_WI@std@@8 1004ad64     Plist.obj
 0002:0000dd70       ??_R2?$_Func_base@_NPA_WI@std@@8 1004ad70     Plist.obj
 0002:0000dd78       ??_R1A@?0A@EA@?$_Func_impl_no_alloc@V<lambda_1>@?6??PrintModules@?$ipc_functions@$00@@SAXPAX0AAUoptions@@@Z@_NPA_WI@std@@8 1004ad78     Plist.obj
 0002:0000dd94       ??_R3?$_Func_impl_no_alloc@V<lambda_1>@?6??PrintModules@?$ipc_functions@$00@@SAXPAX0AAUoptions@@@Z@_NPA_WI@std@@8 1004ad94     Plist.obj
 0002:0000dda4       ??_R4?$_Func_impl_no_alloc@V<lambda_1>@?6??PrintModules@?$ipc_functions@$0A@@@SAXPAX0AAUoptions@@@Z@_NPA_WI@std@@6B@ 1004ada4     Plist.obj
 0002:0000ddb8       ??_R3?$_Func_base@_NPA_WI@std@@8 1004adb8     Plist.obj
 0002:0000ddc8       ??_R1A@?0A@EA@?$_Func_impl_no_alloc@V<lambda_1>@?6??PrintModules@?$ipc_functions@$0A@@@SAXPAX0AAUoptions@@@Z@_NPA_WI@std@@8 1004adc8     Plist.obj
 0002:0000de08       ??_R1A@?0A@EA@?$_Func_base@_NPA_WI@std@@8 1004ae08     Plist.obj
 0002:0000de40       ??_R2?$_Func_impl_no_alloc@V<lambda_1>@?6??PrintModules@?$ipc_functions@$0A@@@SAXPAX0AAUoptions@@@Z@_NPA_WI@std@@8 1004ae40     Plist.obj
 0002:0000de4c       ??_R4?$_Func_impl_no_alloc@V<lambda_1>@?6??PrintModules@?$ipc_functions@$00@@SAXPAX0AAUoptions@@@Z@_NPA_WI@std@@6B@ 1004ae4c     Plist.obj
 0002:0000de80       ??_R1A@?0A@EA@?$_Func_base@XABUtagVARIANT@@@std@@8 1004ae80     wmi.obj
 0002:0000de9c       ??_R3?$_Func_base@XABUtagVARIANT@@@std@@8 1004ae9c     wmi.obj
 0002:0000df00       ??_R2?$_Func_base@XABUtagVARIANT@@@std@@8 1004af00     wmi.obj
 0002:0000df38       ___safe_se_handler_table   1004af38     <linker-defined>
 0002:0000e0e4       ___volatile_metadata       1004b0e4     <linker-defined>
 0002:0000e4b8       ___rtc_iaa                 1004b4b8     LIBCMT:initsect.obj
 0002:0000e4bc       ___rtc_izz                 1004b4bc     LIBCMT:initsect.obj
 0002:0000e4c0       ___rtc_taa                 1004b4c0     LIBCMT:initsect.obj
 0002:0000e4c4       ___rtc_tzz                 1004b4c4     LIBCMT:initsect.obj
 0002:00010218       __TI2?AVbad_alloc@std@@    1004d218     libcpmt:xthrow.obj
 0002:00010228       __CTA2?AVbad_alloc@std@@   1004d228     libcpmt:xthrow.obj
 0002:00010234       __CT??_R0?AVlogic_error@std@@@8??0logic_error@std@@QAE@ABV01@@Z12 1004d234     libcpmt:xthrow.obj
 0002:00010250       __TI3?AVlength_error@std@@ 1004d250     libcpmt:xthrow.obj
 0002:00010260       __CTA3?AVlength_error@std@@ 1004d260     libcpmt:xthrow.obj
 0002:00010270       __CT??_R0?AVlength_error@std@@@8??0length_error@std@@QAE@ABV01@@Z12 1004d270     libcpmt:xthrow.obj
 0002:0001028c       __TI3?AVout_of_range@std@@ 1004d28c     libcpmt:xthrow.obj
 0002:0001029c       __CTA3?AVout_of_range@std@@ 1004d29c     libcpmt:xthrow.obj
 0002:000102ac       __CT??_R0?AVout_of_range@std@@@8??0out_of_range@std@@QAE@ABV01@@Z12 1004d2ac     libcpmt:xthrow.obj
 0002:000102c8       __TI2?AVbad_function_call@std@@ 1004d2c8     libcpmt:xthrow.obj
 0002:000102d8       __CTA2?AVbad_function_call@std@@ 1004d2d8     libcpmt:xthrow.obj
 0002:000102e4       __CT??_R0?AVbad_function_call@std@@@8??0bad_function_call@std@@QAE@ABV01@@Z12 1004d2e4     libcpmt:xthrow.obj
 0002:000104fc       __TI2?AVbad_exception@std@@ 1004d4fc     libvcruntime:frame.obj
 0002:0001050c       __CTA2?AVbad_exception@std@@ 1004d50c     libvcruntime:frame.obj
 0002:00010518       __CT??_R0?AVbad_exception@std@@@8??0bad_exception@std@@QAE@ABV01@@Z12 1004d518     libvcruntime:frame.obj
 0002:0001091c       __TI2?AVruntime_error@std@@ 1004d91c     format.obj
 0002:0001092c       __CTA3?AVbad_array_new_length@std@@ 1004d92c     format.obj
 0002:0001093c       __CT??_R0?AVbad_alloc@std@@@8??0bad_alloc@std@@QAE@ABV01@@Z12 1004d93c     format.obj
 0002:00010958       __CT??_R0?AVformat_error@v10@fmt@@@8??0format_error@v10@fmt@@QAE@ABV012@@Z12 1004d958     format.obj
 0002:00010974       __CTA3?AVformat_error@v10@fmt@@ 1004d974     format.obj
 0002:00010984       __CTA2?AVruntime_error@std@@ 1004d984     format.obj
 0002:00010990       __CT??_R0?AVruntime_error@std@@@8??0runtime_error@std@@QAE@ABV01@@Z12 1004d990     format.obj
 0002:000109ac       __CT??_R0?AVexception@std@@@8??0exception@std@@QAE@ABV01@@Z12 1004d9ac     format.obj
 0002:000109c8       __TI3?AVformat_error@v10@fmt@@ 1004d9c8     format.obj
 0002:000109d8       __TI3?AVbad_array_new_length@std@@ 1004d9d8     format.obj
 0002:000109e8       __CT??_R0?AVbad_array_new_length@std@@@8??0bad_array_new_length@std@@QAE@ABV01@@Z12 1004d9e8     format.obj
 0002:00010bb0       __IMPORT_DESCRIPTOR_KERNEL32 1004dbb0     kernel32:KERNEL32.dll
 0002:00010bc4       __IMPORT_DESCRIPTOR_ADVAPI32 1004dbc4     advapi32:ADVAPI32.dll
 0002:00010bd8       __IMPORT_DESCRIPTOR_USER32 1004dbd8     user32:USER32.dll
 0002:00010bec       __IMPORT_DESCRIPTOR_MPR    1004dbec     mpr:MPR.dll
 0002:00010c00       __IMPORT_DESCRIPTOR_ole32  1004dc00     ole32:ole32.dll
 0002:00010c14       __IMPORT_DESCRIPTOR_OLEAUT32 1004dc14     oleaut32:OLEAUT32.dll
 0002:00010c28       __IMPORT_DESCRIPTOR_PSAPI  1004dc28     psapi:PSAPI.DLL
 0002:00010c3c       __IMPORT_DESCRIPTOR_VERSION 1004dc3c     version:VERSION.dll
 0002:00010c50       __NULL_IMPORT_DESCRIPTOR   1004dc50     kernel32:KERNEL32.dll
 0003:00000008       ___do_unsigned_char_lconv_initialization 1004f008     LIBCMT:lconv_unsigned_char.obj
 0003:0000000c       ___scrt_native_dllmain_reason 1004f00c     LIBCMT:utility.obj
 0003:00000010       ___security_cookie_complement 1004f010     LIBCMT:gs_cookie.obj
 0003:00000014       ___security_cookie         1004f014     LIBCMT:gs_cookie.obj
 0003:00000018       __fltused                  1004f018     LIBCMT:fltused.obj
 0003:00000020       ___isa_enabled             1004f020     LIBCMT:cpu_disp.obj
 0003:00000040       __NLG_Destination          1004f040     libvcruntime:exsup.obj
 0003:00000050       __iob                      1004f050     libucrt:_file.obj
 0003:000000f8       ___acrt_lconv_c            1004f0f8     libucrt:localeconv.obj
 0003:00000148       ___acrt_lconv              1004f148     libucrt:localeconv.obj
 0003:0000014c       ___acrt_lconv_static_decimal 1004f14c     libucrt:localeconv.obj
 0003:00000150       ___acrt_lconv_static_W_decimal 1004f150     libucrt:localeconv.obj
 0003:00000160       __pctype                   1004f160     libucrt:ctype.obj
 0003:00000164       __pwctype                  1004f164     libucrt:ctype.obj
 0003:00000170       ___abort_behavior          1004f170     libucrt:abort.obj
 0003:00000188       ___acrt_initial_locale_data 1004f188     libucrt:nlsdata.obj
 0003:00000240       ___acrt_initial_locale_pointers 1004f240     libucrt:nlsdata.obj
 0003:00000248       ___acrt_wide_c_locale_string 1004f248     libucrt:nlsdata.obj
 0003:0000024c       ___mb_cur_max              1004f24c     libucrt:nlsdata.obj
 0003:00000254       ___globallocalestatus      1004f254     libucrt:glstatus.obj
 0003:000002e8       ___acrt_initial_multibyte_data 1004f2e8     libucrt:mbctype.obj
 0003:00000808       __lookuptrailbytes         1004f808     libucrt:read.obj
 0003:0000098c       ?pNtQuerySystemInformation@@3P6GJKPAXKPAK@ZA 1004f98c     Proclist.obj
 0003:00000990       ?pNtQueryInformationProcess@@3P6GJPAXW4_PROCESSINFOCLASS@@0KPAK@ZA 1004f990     Proclist.obj
 0003:00000994       ?pNtQueryObject@@3P6GJPAXK0K0@ZA 1004f994     Proclist.obj
 0003:00000998       ?pNtQueryInformationThread@@3P6GJPAXK0KPAK@ZA 1004f998     Proclist.obj
 0003:0000099c       ?pNtQueryInformationFile@@3P6GJPAX00KK@ZA 1004f99c     Proclist.obj
 0003:000009a0       ?pGetGuiResources@@3P6GKPAXK@ZA 1004f9a0     Proclist.obj
 0003:000009a4       ?pNtWow64ReadVirtualMemory64@@3P6GJPAX_K01PA_K@ZA 1004f9a4     Proclist.obj
 0003:000009a8       ?pNtWow64QueryInformationProcess64@@3P6GJPAXW4_PROCESSINFOCLASS@@0KPAK@ZA 1004f9a8     Proclist.obj
 0003:000009ac       ?pEnumProcessModulesEx@@3P6GHPAXPAPAUHINSTANCE__@@KPAKK@ZA 1004f9ac     Proclist.obj
 0003:000009b0       ?pCoSetProxyBlanket@@3P6GJPAUIUnknown@@KKPA_WKKPAXK@ZA 1004f9b0     Proclist.obj
 0003:000009b4       ?pIsWow64Process@@3P6GHPAXPAH@ZA 1004f9b4     Proclist.obj
 0003:000009b8       ?m_PanelModesDataRemote@Plist@@0V?$vector@Umode@@V?$allocator@Umode@@@std@@@std@@A 1004f9b8     fileio.obj
 0003:000009c4       ?m_PanelModesDataLocal@Plist@@0V?$vector@Umode@@V?$allocator@Umode@@@std@@@std@@A 1004f9c4     fileio.obj
 0003:000009d0       ??_R0?AVlogic_error@std@@@8 1004f9d0     libcpmt:xthrow.obj
 0003:000009f0       ??_R0?AVlength_error@std@@@8 1004f9f0     libcpmt:xthrow.obj
 0003:00000a10       ??_R0?AVout_of_range@std@@@8 1004fa10     libcpmt:xthrow.obj
 0003:00000a30       ??_R0?AVbad_function_call@std@@@8 1004fa30     libcpmt:xthrow.obj
 0003:00000a54       ??_R0?AVbad_exception@std@@@8 1004fa54     libvcruntime:frame.obj
 0003:00000a74       ??_R0?AVruntime_error@std@@@8 1004fa74     format.obj
 0003:00000a94       ??_R0?AVformat_error@v10@fmt@@@8 1004fa94     format.obj
 0003:00000ab8       ??_R0?AVbad_alloc@std@@@8  1004fab8     format.obj
 0003:00000ad4       ??_R0?AVexception@std@@@8  1004fad4     format.obj
 0003:00000af0       ??_R0?AVbad_array_new_length@std@@@8 1004faf0     format.obj
 0003:00000b60       ??_R0?AV<lambda_1>@?6??PrintModules@?$ipc_functions@$00@@SAXPAX0AAUoptions@@@Z@@8 1004fb60     Plist.obj
 0003:00000bb8       ??_R0?AV<lambda_1>@?6??PrintModules@?$ipc_functions@$0A@@@SAXPAX0AAUoptions@@@Z@@8 1004fbb8     Plist.obj
 0003:00000ce8       ??_R0?AV_Locimp@locale@std@@@8 1004fce8     libcpmt:locale0.obj
 0003:00000d0c       ??_R0?AVtype_info@@@8      1004fd0c     LIBCMT:std_type_info_static.obj
 0003:00000d28       ??_R0?AV?$basic_memory_buffer@D$0BPE@V?$allocator@D@std@@@v10@fmt@@@8 1004fd28     format.obj
 0003:00000d70       ??_R0?AV?$buffer@_W@detail@v10@fmt@@@8 1004fd70     format.obj
 0003:00000d9c       ??_R0?AV_Facet_base@std@@@8 1004fd9c     format.obj
 0003:00000dbc       ??_R0?AU_Crt_new_delete@std@@@8 1004fdbc     format.obj
 0003:00000de0       ??_R0?AV?$buffer@D@detail@v10@fmt@@@8 1004fde0     format.obj
 0003:00000e08       ??_R0?AV?$numpunct@_W@std@@@8 1004fe08     format.obj
 0003:00000e28       ??_R0?AV?$basic_memory_buffer@H$0BPE@V?$allocator@H@std@@@v10@fmt@@@8 1004fe28     format.obj
 0003:00000e70       ??_R0?AVfacet@locale@std@@@8 1004fe70     format.obj
 0003:00000e90       ??_R0?AV?$basic_memory_buffer@I$0CA@V?$allocator@I@std@@@v10@fmt@@@8 1004fe90     format.obj
 0003:00000ed8       ??_R0?AV?$basic_memory_buffer@_W$0BPE@V?$allocator@_W@std@@@v10@fmt@@@8 1004fed8     format.obj
 0003:00000f24       ??_R0?AV?$buffer@I@detail@v10@fmt@@@8 1004ff24     format.obj
 0003:00000f4c       ??_R0?AV?$buffer@H@detail@v10@fmt@@@8 1004ff4c     format.obj
 0003:00000f74       ??_R0?AVDialogAPIBinding@@@8 1004ff74     Pcfg.obj
 0003:00000f94       ??_R0?AVPluginCheckBoxBinding@@@8 1004ff94     Pcfg.obj
 0003:00000fb8       ??_R0?AVPluginEditFieldBinding@@@8 1004ffb8     Pclass.obj
 0003:00000fe0       ??_R0?AV?$_Func_impl_no_alloc@V<lambda_1>@?6??PrintModules@?$ipc_functions@$00@@SAXPAX0AAUoptions@@@Z@_NPA_WI@std@@@8 1004ffe0     Plist.obj
 0003:00001058       ??_R0?AV?$_Func_impl_no_alloc@V<lambda_1>@?6??PrintModules@?$ipc_functions@$0A@@@SAXPAX0AAUoptions@@@Z@_NPA_WI@std@@@8 10050058     Plist.obj
 0003:000010d4       ??_R0?AV?$_Func_base@_NPA_WI@std@@@8 100500d4     Plist.obj
 0003:00001298       ??_R0?AV?$_Func_base@XABUtagVARIANT@@@std@@@8 10050298     wmi.obj
 0003:00001398       ?_Id_cnt@id@locale@std@@0HA 10050398     libcpmt:locale0.obj
 0003:0000139c       ?_Clocptr@_Locimp@locale@std@@0PAV123@A 1005039c     libcpmt:locale0.obj
 0003:000013a0       ?id@?$ctype@G@std@@2V0locale@2@A 100503a0     libcpmt:locale0.obj
 0003:000013a4       ?id@?$codecvt@_WDU_Mbstatet@@@std@@2V0locale@2@A 100503a4     libcpmt:locale0.obj
 0003:000013a8       ?id@?$codecvt@GDU_Mbstatet@@@std@@2V0locale@2@A 100503a8     libcpmt:locale0.obj
 0003:000013ac       ?id@?$ctype@_W@std@@2V0locale@2@A 100503ac     libcpmt:locale0.obj
 0003:000013b0       ?id@?$ctype@D@std@@2V0locale@2@A 100503b0     libcpmt:locale0.obj
 0003:000013cc       ?id@?$num_get@DV?$istreambuf_iterator@DU?$char_traits@D@std@@@std@@@std@@2V0locale@2@A 100503cc     libcpmt:locale.obj
 0003:000013d0       ?id@?$num_put@DV?$ostreambuf_iterator@DU?$char_traits@D@std@@@std@@@std@@2V0locale@2@A 100503d0     libcpmt:locale.obj
 0003:000013d4       ?id@?$codecvt@DDU_Mbstatet@@@std@@2V0locale@2@A 100503d4     libcpmt:locale.obj
 0003:000013d8       ?_Ptr_cin@std@@3PAV?$basic_istream@DU?$char_traits@D@std@@@1@A 100503d8     libcpmt:iosptrs.obj
 0003:000013dc       ?_Ptr_cout@std@@3PAV?$basic_ostream@DU?$char_traits@D@std@@@1@A 100503dc     libcpmt:iosptrs.obj
 0003:000013e0       ?_Ptr_cerr@std@@3PAV?$basic_ostream@DU?$char_traits@D@std@@@1@A 100503e0     libcpmt:iosptrs.obj
 0003:000013e4       ?_Ptr_clog@std@@3PAV?$basic_ostream@DU?$char_traits@D@std@@@1@A 100503e4     libcpmt:iosptrs.obj
 0003:000013e8       ?_Ptr_wcin@std@@3PAV?$basic_istream@_WU?$char_traits@_W@std@@@1@A 100503e8     libcpmt:iosptrs.obj
 0003:000013ec       ?_Ptr_wcout@std@@3PAV?$basic_ostream@_WU?$char_traits@_W@std@@@1@A 100503ec     libcpmt:iosptrs.obj
 0003:000013f0       ?_Ptr_wcerr@std@@3PAV?$basic_ostream@_WU?$char_traits@_W@std@@@1@A 100503f0     libcpmt:iosptrs.obj
 0003:000013f4       ?_Ptr_wclog@std@@3PAV?$basic_ostream@_WU?$char_traits@_W@std@@@1@A 100503f4     libcpmt:iosptrs.obj
 0003:00001424       ?id@?$time_put@_WV?$ostreambuf_iterator@_WU?$char_traits@_W@std@@@std@@@std@@2V0locale@2@A 10050424     libcpmt:wlocale.obj
 0003:00001428       ?id@?$num_get@_WV?$istreambuf_iterator@_WU?$char_traits@_W@std@@@std@@@std@@2V0locale@2@A 10050428     libcpmt:wlocale.obj
 0003:0000142c       ?id@?$num_put@_WV?$ostreambuf_iterator@_WU?$char_traits@_W@std@@@std@@@std@@2V0locale@2@A 1005042c     libcpmt:wlocale.obj
 0003:00001430       ?id@?$collate@_W@std@@2V0locale@2@A 10050430     libcpmt:wlocale.obj
 0003:00001434       ?id@?$messages@_W@std@@2V0locale@2@A 10050434     libcpmt:wlocale.obj
 0003:00001438       ?id@?$money_get@_WV?$istreambuf_iterator@_WU?$char_traits@_W@std@@@std@@@std@@2V0locale@2@A 10050438     libcpmt:wlocale.obj
 0003:0000143c       ?id@?$money_put@_WV?$ostreambuf_iterator@_WU?$char_traits@_W@std@@@std@@@std@@2V0locale@2@A 1005043c     libcpmt:wlocale.obj
 0003:00001440       ?id@?$moneypunct@_W$0A@@std@@2V0locale@2@A 10050440     libcpmt:wlocale.obj
 0003:00001444       ?id@?$moneypunct@_W$00@std@@2V0locale@2@A 10050444     libcpmt:wlocale.obj
 0003:00001448       ?id@?$time_get@_WV?$istreambuf_iterator@_WU?$char_traits@_W@std@@@std@@@std@@2V0locale@2@A 10050448     libcpmt:wlocale.obj
 0003:0000144c       ?id@?$num_get@GV?$istreambuf_iterator@GU?$char_traits@G@std@@@std@@@std@@2V0locale@2@A 1005044c     libcpmt:wlocale.obj
 0003:00001450       ?id@?$num_put@GV?$ostreambuf_iterator@GU?$char_traits@G@std@@@std@@@std@@2V0locale@2@A 10050450     libcpmt:wlocale.obj
 0003:00001454       ?id@?$numpunct@G@std@@2V0locale@2@A 10050454     libcpmt:wlocale.obj
 0003:00001458       ?id@?$collate@G@std@@2V0locale@2@A 10050458     libcpmt:wlocale.obj
 0003:0000145c       ?id@?$messages@G@std@@2V0locale@2@A 1005045c     libcpmt:wlocale.obj
 0003:00001460       ?id@?$money_get@GV?$istreambuf_iterator@GU?$char_traits@G@std@@@std@@@std@@2V0locale@2@A 10050460     libcpmt:wlocale.obj
 0003:00001464       ?id@?$money_put@GV?$ostreambuf_iterator@GU?$char_traits@G@std@@@std@@@std@@2V0locale@2@A 10050464     libcpmt:wlocale.obj
 0003:00001468       ?id@?$moneypunct@G$0A@@std@@2V0locale@2@A 10050468     libcpmt:wlocale.obj
 0003:0000146c       ?id@?$moneypunct@G$00@std@@2V0locale@2@A 1005046c     libcpmt:wlocale.obj
 0003:00001470       ?id@?$time_get@GV?$istreambuf_iterator@GU?$char_traits@G@std@@@std@@@std@@2V0locale@2@A 10050470     libcpmt:wlocale.obj
 0003:00001474       ?id@?$time_put@GV?$ostreambuf_iterator@GU?$char_traits@G@std@@@std@@@std@@2V0locale@2@A 10050474     libcpmt:wlocale.obj
 0003:00001478       ?id@?$collate@D@std@@2V0locale@2@A 10050478     libcpmt:xlocale.obj
 0003:0000147c       ?id@?$messages@D@std@@2V0locale@2@A 1005047c     libcpmt:xlocale.obj
 0003:00001480       ?id@?$money_get@DV?$istreambuf_iterator@DU?$char_traits@D@std@@@std@@@std@@2V0locale@2@A 10050480     libcpmt:xlocale.obj
 0003:00001484       ?id@?$money_put@DV?$ostreambuf_iterator@DU?$char_traits@D@std@@@std@@@std@@2V0locale@2@A 10050484     libcpmt:xlocale.obj
 0003:00001488       ?id@?$moneypunct@D$0A@@std@@2V0locale@2@A 10050488     libcpmt:xlocale.obj
 0003:0000148c       ?id@?$moneypunct@D$00@std@@2V0locale@2@A 1005048c     libcpmt:xlocale.obj
 0003:00001490       ?id@?$time_get@DV?$istreambuf_iterator@DU?$char_traits@D@std@@@std@@@std@@2V0locale@2@A 10050490     libcpmt:xlocale.obj
 0003:00001494       ?id@?$time_put@DV?$ostreambuf_iterator@DU?$char_traits@D@std@@@std@@@std@@2V0locale@2@A 10050494     libcpmt:xlocale.obj
 0003:00001498       ___scrt_current_native_startup_state 10050498     LIBCMT:utility.obj
 0003:0000149c       ___scrt_native_startup_lock 1005049c     LIBCMT:utility.obj
 0003:000017e0       ___castguard_check_failure_os_handled_fptr 100507e0     LIBCMT:guard_support.obj
 0003:000017e4       ___isa_available           100507e4     LIBCMT:cpu_disp.obj
 0003:000017e8       ___favor                   100507e8     LIBCMT:cpu_disp.obj
 0003:000017ec       ___scrt_debugger_hook_flag 100507ec     LIBCMT:utility_desktop.obj
 0003:000017f0       ?__type_info_root_node@@3U__type_info_node@@A 100507f0     LIBCMT:tncleanup.obj
 0003:000017f8       ?_OptionsStorage@?1??__local_stdio_scanf_options@@9@4_KA 100507f8     LIBCMT:default_local_stdio_options.obj
 0003:00001800       ?__WinRTOutOfMemoryExceptionCallback@@3P6GPAXXZA 10050800     libvcruntime:ehhelpers.obj
 0003:0000182c       ___pPurecall               1005082c     libvcruntime:purevirt_data.obj
 0003:0000184c       ?pArgList@UnDecorator@@0PAVReplicator@@A 1005084c     libvcruntime:undname.obj
 0003:00001850       ?pZNameList@UnDecorator@@0PAVReplicator@@A 10050850     libvcruntime:undname.obj
 0003:00001854       ?pTemplateArgList@UnDecorator@@0PAVReplicator@@A 10050854     libvcruntime:undname.obj
 0003:00001858       ?gName@UnDecorator@@0PBDB  10050858     libvcruntime:undname.obj
 0003:0000185c       ?name@UnDecorator@@0PBDB   1005085c     libvcruntime:undname.obj
 0003:00001860       ?disableFlags@UnDecorator@@0KA 10050860     libvcruntime:undname.obj
 0003:00001864       ?fExplicitTemplateParams@UnDecorator@@0_NA 10050864     libvcruntime:undname.obj
 0003:00001865       ?fGetTemplateArgumentList@UnDecorator@@0_NA 10050865     libvcruntime:undname.obj
 0003:00001868       ?m_pGetParameter@UnDecorator@@0P6APADJ@ZA 10050868     libvcruntime:undname.obj
 0003:0000186c       ?m_CHPENameOffset@UnDecorator@@0KA 1005086c     libvcruntime:undname.obj
 0003:00001870       ?m_recursionLevel@UnDecorator@@0KA 10050870     libvcruntime:undname.obj
 0003:000018ac       __nstream                  100508ac     libucrt:_file.obj
 0003:000018b0       ___piob                    100508b0     libucrt:_file.obj
 0003:000018b4       ___acrt_lconv_static_null  100508b4     libucrt:localeconv.obj
 0003:000018b8       ___acrt_lconv_static_W_null 100508b8     libucrt:localeconv.obj
 0003:00001a1c       ?c_exit_complete@?1???R<lambda_6e4b09c48022b2350581041d5f6b0c4c>@@QBE@XZ@4_NA 10050a1c     libucrt:exit.obj
 0003:00001b28       __environ_table            10050b28     libucrt:environment_initialization.obj
 0003:00001b2c       __wenviron_table           10050b2c     libucrt:environment_initialization.obj
 0003:00001b30       ___dcrt_initial_wide_environment 10050b30     libucrt:environment_initialization.obj
 0003:00001b34       ___dcrt_initial_narrow_environment 10050b34     libucrt:environment_initialization.obj
 0003:00001b38       ___acrt_atexit_table       10050b38     libucrt:onexit.obj
 0003:00001b44       ___acrt_at_quick_exit_table 10050b44     libucrt:onexit.obj
 0003:00001b58       ___pioinfo                 10050b58     libucrt:ioinit.obj
 0003:00001d58       __nhandle                  10050d58     libucrt:ioinit.obj
 0003:00001e44       ___acrt_stdout_buffer      10050e44     libucrt:_sftbuf.obj
 0003:00001e48       ___acrt_stderr_buffer      10050e48     libucrt:_sftbuf.obj
 0003:00001e4c       ___acrt_locale_changed_data 10050e4c     libucrt:wsetlocale.obj
 0003:00001e50       ___acrt_current_locale_data 10050e50     libucrt:nlsdata.obj
 0003:00001e58       ___fastflag                10050e58     libucrt:fp_flags.obj
 0003:00001e6c       ?_timezone@@3V?$dual_state_global@J@__crt_state_management@@A 10050e6c     libucrt:timeset.obj
 0003:00001e70       ?_daylight@@3V?$dual_state_global@H@__crt_state_management@@A 10050e70     libucrt:timeset.obj
 0003:00001e74       ?_dstbias@@3V?$dual_state_global@J@__crt_state_management@@A 10050e74     libucrt:timeset.obj
 0003:00001f34       __mbctype                  10050f34     libucrt:mbctype.obj
 0003:00001f38       __mbcasemap                10050f38     libucrt:mbctype.obj
 0003:00001f3c       ___acrt_current_multibyte_data 10050f3c     libucrt:mbctype.obj
 0003:00001f48       __pgmptr                   10050f48     libucrt:argv_data.obj
 0003:00001f4c       ___argc                    10050f4c     libucrt:argv_data.obj
 0003:00001f50       ___argv                    10050f50     libucrt:argv_data.obj
 0003:00001f54       ___wargv                   10050f54     libucrt:argv_data.obj
 0003:00001f58       __acmdln                   10050f58     libucrt:argv_data.obj
 0003:00001f5c       __wcmdln                   10050f5c     libucrt:argv_data.obj
 0003:00001f60       ___acrt_heap               10050f60     libucrt:heap_handle.obj
 0003:00001f80       ?_OptionsStorage@?1??__local_stdio_printf_options@@9@4_KA 10050f80     format.obj
 0003:00001f88       ?_Psave@?$_Facetptr@V?$numpunct@_W@std@@@std@@2PBVfacet@locale@2@B 10050f88     format.obj
 0003:00002050       ?FSF@@3UFarStandardFunctions@@A 10051050     Proclist.obj
 0003:00002120       ?Opt@@3Uoptions@@A         10051120     Proclist.obj
 0003:00002148       ?PsInfo@@3UPluginStartupInfo@@A 10051148     Proclist.obj
 0003:000021d8       ?id@?$numpunct@_W@std@@2V0locale@2@A 100511d8     fileio.obj
 0003:000021dc       ?id@?$format_facet@Vlocale@std@@@v10@fmt@@2V0locale@std@@A 100511dc     format.obj
 0003:000021e0       ?id@?$numpunct@D@std@@2V0locale@2@A 100511e0     format.obj
 0003:00002cec       ___dyn_tls_init_callback   10051cec     <common>
 0003:00002cf0       ___scrt_ucrt_dll_is_in_use 10051cf0     <common>
 0003:00002cf4       __pmatherr                 10051cf4     <common>
 0003:00002cf8       ___use_sse2_mathfcns       10051cf8     <common>

 entry point at        0001:00026733

 Static symbols

 0000:fffa9000       .debug$S                   10000000     ProcList.exp
 0000:fffa9000       .debug$S                   10000000     advapi32:ADVAPI32.dll
 0000:fffa9000       .debug$S                   10000000     advapi32:ADVAPI32.dll
 0000:fffa9000       .debug$S                   10000000     advapi32:ADVAPI32.dll
 0000:fffa9000       .debug$S                   10000000     advapi32:ADVAPI32.dll
 0000:fffa9000       .debug$S                   10000000     advapi32:ADVAPI32.dll
 0000:fffa9000       .debug$S                   10000000     advapi32:ADVAPI32.dll
 0000:fffa9000       .debug$S                   10000000     advapi32:ADVAPI32.dll
 0000:fffa9000       .debug$S                   10000000     advapi32:ADVAPI32.dll
 0000:fffa9000       .debug$S                   10000000     advapi32:ADVAPI32.dll
 0000:fffa9000       .debug$S                   10000000     advapi32:ADVAPI32.dll
 0000:fffa9000       .debug$S                   10000000     advapi32:ADVAPI32.dll
 0000:fffa9000       .debug$S                   10000000     advapi32:ADVAPI32.dll
 0000:fffa9000       .debug$S                   10000000     kernel32:KERNEL32.dll
 0000:fffa9000       .debug$S                   10000000     kernel32:KERNEL32.dll
 0000:fffa9000       .debug$S                   10000000     kernel32:KERNEL32.dll
 0000:fffa9000       .debug$S                   10000000     kernel32:KERNEL32.dll
 0000:fffa9000       .debug$S                   10000000     kernel32:KERNEL32.dll
 0000:fffa9000       .debug$S                   10000000     kernel32:KERNEL32.dll
 0000:fffa9000       .debug$S                   10000000     kernel32:KERNEL32.dll
 0000:fffa9000       .debug$S                   10000000     kernel32:KERNEL32.dll
 0000:fffa9000       .debug$S                   10000000     kernel32:KERNEL32.dll
 0000:fffa9000       .debug$S                   10000000     kernel32:KERNEL32.dll
 0000:fffa9000       .debug$S                   10000000     kernel32:KERNEL32.dll
 0000:fffa9000       .debug$S                   10000000     kernel32:KERNEL32.dll
 0000:fffa9000       .debug$S                   10000000     kernel32:KERNEL32.dll
 0000:fffa9000       .debug$S                   10000000     kernel32:KERNEL32.dll
 0000:fffa9000       .debug$S                   10000000     kernel32:KERNEL32.dll
 0000:fffa9000       .debug$S                   10000000     kernel32:KERNEL32.dll
 0000:fffa9000       .debug$S                   10000000     kernel32:KERNEL32.dll
 0000:fffa9000       .debug$S                   10000000     kernel32:KERNEL32.dll
 0000:fffa9000       .debug$S                   10000000     kernel32:KERNEL32.dll
 0000:fffa9000       .debug$S                   10000000     kernel32:KERNEL32.dll
 0000:fffa9000       .debug$S                   10000000     kernel32:KERNEL32.dll
 0000:fffa9000       .debug$S                   10000000     kernel32:KERNEL32.dll
 0000:fffa9000       .debug$S                   10000000     kernel32:KERNEL32.dll
 0000:fffa9000       .debug$S                   10000000     kernel32:KERNEL32.dll
 0000:fffa9000       .debug$S                   10000000     kernel32:KERNEL32.dll
 0000:fffa9000       .debug$S                   10000000     kernel32:KERNEL32.dll
 0000:fffa9000       .debug$S                   10000000     kernel32:KERNEL32.dll
 0000:fffa9000       .debug$S                   10000000     kernel32:KERNEL32.dll
 0000:fffa9000       .debug$S                   10000000     kernel32:KERNEL32.dll
 0000:fffa9000       .debug$S                   10000000     kernel32:KERNEL32.dll
 0000:fffa9000       .debug$S                   10000000     kernel32:KERNEL32.dll
 0000:fffa9000       .debug$S                   10000000     kernel32:KERNEL32.dll
 0000:fffa9000       .debug$S                   10000000     kernel32:KERNEL32.dll
 0000:fffa9000       .debug$S                   10000000     kernel32:KERNEL32.dll
 0000:fffa9000       .debug$S                   10000000     kernel32:KERNEL32.dll
 0000:fffa9000       .debug$S                   10000000     kernel32:KERNEL32.dll
 0000:fffa9000       .debug$S                   10000000     kernel32:KERNEL32.dll
 0000:fffa9000       .debug$S                   10000000     kernel32:KERNEL32.dll
 0000:fffa9000       .debug$S                   10000000     kernel32:KERNEL32.dll
 0000:fffa9000       .debug$S                   10000000     kernel32:KERNEL32.dll
 0000:fffa9000       .debug$S                   10000000     kernel32:KERNEL32.dll
 0000:fffa9000       .debug$S                   10000000     kernel32:KERNEL32.dll
 0000:fffa9000       .debug$S                   10000000     kernel32:KERNEL32.dll
 0000:fffa9000       .debug$S                   10000000     kernel32:KERNEL32.dll
 0000:fffa9000       .debug$S                   10000000     kernel32:KERNEL32.dll
 0000:fffa9000       .debug$S                   10000000     kernel32:KERNEL32.dll
 0000:fffa9000       .debug$S                   10000000     kernel32:KERNEL32.dll
 0000:fffa9000       .debug$S                   10000000     kernel32:KERNEL32.dll
 0000:fffa9000       .debug$S                   10000000     kernel32:KERNEL32.dll
 0000:fffa9000       .debug$S                   10000000     kernel32:KERNEL32.dll
 0000:fffa9000       .debug$S                   10000000     kernel32:KERNEL32.dll
 0000:fffa9000       .debug$S                   10000000     kernel32:KERNEL32.dll
 0000:fffa9000       .debug$S                   10000000     kernel32:KERNEL32.dll
 0000:fffa9000       .debug$S                   10000000     kernel32:KERNEL32.dll
 0000:fffa9000       .debug$S                   10000000     kernel32:KERNEL32.dll
 0000:fffa9000       .debug$S                   10000000     kernel32:KERNEL32.dll
 0000:fffa9000       .debug$S                   10000000     kernel32:KERNEL32.dll
 0000:fffa9000       .debug$S                   10000000     kernel32:KERNEL32.dll
 0000:fffa9000       .debug$S                   10000000     kernel32:KERNEL32.dll
 0000:fffa9000       .debug$S                   10000000     kernel32:KERNEL32.dll
 0000:fffa9000       .debug$S                   10000000     kernel32:KERNEL32.dll
 0000:fffa9000       .debug$S                   10000000     kernel32:KERNEL32.dll
 0000:fffa9000       .debug$S                   10000000     kernel32:KERNEL32.dll
 0000:fffa9000       .debug$S                   10000000     kernel32:KERNEL32.dll
 0000:fffa9000       .debug$S                   10000000     kernel32:KERNEL32.dll
 0000:fffa9000       .debug$S                   10000000     kernel32:KERNEL32.dll
 0000:fffa9000       .debug$S                   10000000     kernel32:KERNEL32.dll
 0000:fffa9000       .debug$S                   10000000     kernel32:KERNEL32.dll
 0000:fffa9000       .debug$S                   10000000     kernel32:KERNEL32.dll
 0000:fffa9000       .debug$S                   10000000     kernel32:KERNEL32.dll
 0000:fffa9000       .debug$S                   10000000     kernel32:KERNEL32.dll
 0000:fffa9000       .debug$S                   10000000     kernel32:KERNEL32.dll
 0000:fffa9000       .debug$S                   10000000     kernel32:KERNEL32.dll
 0000:fffa9000       .debug$S                   10000000     kernel32:KERNEL32.dll
 0000:fffa9000       .debug$S                   10000000     kernel32:KERNEL32.dll
 0000:fffa9000       .debug$S                   10000000     kernel32:KERNEL32.dll
 0000:fffa9000       .debug$S                   10000000     kernel32:KERNEL32.dll
 0000:fffa9000       .debug$S                   10000000     kernel32:KERNEL32.dll
 0000:fffa9000       .debug$S                   10000000     kernel32:KERNEL32.dll
 0000:fffa9000       .debug$S                   10000000     kernel32:KERNEL32.dll
 0000:fffa9000       .debug$S                   10000000     kernel32:KERNEL32.dll
 0000:fffa9000       .debug$S                   10000000     kernel32:KERNEL32.dll
 0000:fffa9000       .debug$S                   10000000     kernel32:KERNEL32.dll
 0000:fffa9000       .debug$S                   10000000     kernel32:KERNEL32.dll
 0000:fffa9000       .debug$S                   10000000     kernel32:KERNEL32.dll
 0000:fffa9000       .debug$S                   10000000     kernel32:KERNEL32.dll
 0000:fffa9000       .debug$S                   10000000     kernel32:KERNEL32.dll
 0000:fffa9000       .debug$S                   10000000     kernel32:KERNEL32.dll
 0000:fffa9000       .debug$S                   10000000     kernel32:KERNEL32.dll
 0000:fffa9000       .debug$S                   10000000     kernel32:KERNEL32.dll
 0000:fffa9000       .debug$S                   10000000     kernel32:KERNEL32.dll
 0000:fffa9000       .debug$S                   10000000     kernel32:KERNEL32.dll
 0000:fffa9000       .debug$S                   10000000     kernel32:KERNEL32.dll
 0000:fffa9000       .debug$S                   10000000     kernel32:KERNEL32.dll
 0000:fffa9000       .debug$S                   10000000     kernel32:KERNEL32.dll
 0000:fffa9000       .debug$S                   10000000     kernel32:KERNEL32.dll
 0000:fffa9000       .debug$S                   10000000     kernel32:KERNEL32.dll
 0000:fffa9000       .debug$S                   10000000     kernel32:KERNEL32.dll
 0000:fffa9000       .debug$S                   10000000     kernel32:KERNEL32.dll
 0000:fffa9000       .debug$S                   10000000     kernel32:KERNEL32.dll
 0000:fffa9000       .debug$S                   10000000     kernel32:KERNEL32.dll
 0000:fffa9000       .debug$S                   10000000     kernel32:KERNEL32.dll
 0000:fffa9000       .debug$S                   10000000     kernel32:KERNEL32.dll
 0000:fffa9000       .debug$S                   10000000     kernel32:KERNEL32.dll
 0000:fffa9000       .debug$S                   10000000     kernel32:KERNEL32.dll
 0000:fffa9000       .debug$S                   10000000     kernel32:KERNEL32.dll
 0000:fffa9000       .debug$S                   10000000     kernel32:KERNEL32.dll
 0000:fffa9000       .debug$S                   10000000     kernel32:KERNEL32.dll
 0000:fffa9000       .debug$S                   10000000     mpr:MPR.dll
 0000:fffa9000       .debug$S                   10000000     mpr:MPR.dll
 0000:fffa9000       .debug$S                   10000000     ole32:ole32.dll
 0000:fffa9000       .debug$S                   10000000     ole32:ole32.dll
 0000:fffa9000       .debug$S                   10000000     ole32:ole32.dll
 0000:fffa9000       .debug$S                   10000000     oleaut32:OLEAUT32.dll
 0000:fffa9000       .debug$S                   10000000     oleaut32:OLEAUT32.dll
 0000:fffa9000       .debug$S                   10000000     oleaut32:OLEAUT32.dll
 0000:fffa9000       .debug$S                   10000000     psapi:PSAPI.DLL
 0000:fffa9000       .debug$S                   10000000     psapi:PSAPI.DLL
 0000:fffa9000       .debug$S                   10000000     user32:USER32.dll
 0000:fffa9000       .debug$S                   10000000     user32:USER32.dll
 0000:fffa9000       .debug$S                   10000000     user32:USER32.dll
 0000:fffa9000       .debug$S                   10000000     user32:USER32.dll
 0000:fffa9000       .debug$S                   10000000     user32:USER32.dll
 0000:fffa9000       .debug$S                   10000000     user32:USER32.dll
 0000:fffa9000       .debug$S                   10000000     user32:USER32.dll
 0000:fffa9000       .debug$S                   10000000     user32:USER32.dll
 0000:fffa9000       .debug$S                   10000000     user32:USER32.dll
 0000:fffa9000       .debug$S                   10000000     user32:USER32.dll
 0000:fffa9000       .debug$S                   10000000     user32:USER32.dll
 0000:fffa9000       .debug$S                   10000000     user32:USER32.dll
 0000:fffa9000       .debug$S                   10000000     version:VERSION.dll
 0000:fffa9000       .debug$S                   10000000     version:VERSION.dll
 0000:fffa9000       .debug$S                   10000000     version:VERSION.dll
 0001:00000000       ??__F?m_PanelModesDataLocal@Plist@@0V?$vector@Umode@@V?$allocator@Umode@@@std@@@std@@A@@YAXXZ 10001000 f   fileio.obj
 0001:00000010       ??__F?m_PanelModesDataRemote@Plist@@0V?$vector@Umode@@V?$allocator@Umode@@@std@@@std@@A@@YAXXZ 10001010 f   fileio.obj
 0001:00000020       ??__FhDebugToken@@YAXXZ    10001020 f   Plist.obj
 0001:0000002c       ??__Einitlocks@std@@YAXXZ  1000102c f   libcpmt:xlock.obj
 0001:00000042       ??__Eclassic_locale@std@@YAXXZ 10001042 f   libcpmt:locale0.obj
 0001:0000004e       ??__F_Fac_tidy_reg@std@@YAXXZ 1000104e f   libcpmt:locale0.obj
 0001:0000005a       ??__Einitlocks@std@@YAXXZ  1000105a f   libcpmt:iosptrs.obj
 0001:00000070       ??__Finit_atexit@@YAXXZ    10001070 f   libcpmt:iosptrs.obj
 0001:00005a10       $LN264                     10006a10     handles.obj
 0001:00005a7c       $LN263                     10006a7c     handles.obj
 0001:00005d50       ?query_object@@YA?AV?$unique_ptr@$$BY0A@DU?$default_delete@$$BY0A@D@std@@@std@@PAXW4_OBJECT_INFORMATION_CLASS@@@Z 10006d50 f   handles.obj
 0001:00005e20       ?GetFileName@@YA?AV?$basic_string@_WU?$char_traits@_W@std@@V?$allocator@_W@2@@std@@PAX@Z 10006e20 f   handles.obj
 0001:00005fe0       ?GetFileNameThread@test@?4??GetFileName@@YA?AV?$basic_string@_WU?$char_traits@_W@std@@V?$allocator@_W@2@@std@@PAX@Z@SGK0@Z 10006fe0 f   handles.obj
 0001:000060b0       ??R<lambda_1>@?1??GetUserAccountID@@YA@XZ@QBE?AV?$basic_string@_WU?$char_traits@_W@std@@V?$allocator@_W@2@@std@@XZ 100070b0 f   handles.obj
 0001:000062d0       ?GetNameByType@@YA?AV?$basic_string@_WU?$char_traits@_W@std@@V?$allocator@_W@2@@std@@PAXGPAVPerfThread@@@Z 100072d0 f   handles.obj
 0001:00006868       $LN836                     10007868     handles.obj
 0001:00006910       ?duplicate_handle@@YA?AV?$unique_ptr@XUhandle_closer@@@std@@PAXK@Z 10007910 f   handles.obj
 0001:000080d8       $LN873                     100090d8     handles.obj
 0001:000080ec       $LN872                     100090ec     handles.obj
 0001:000087e0       $LN402                     100097e0     handles.obj
 0001:00008bf0       $LN134                     10009bf0     handles.obj
 0001:00009408       $LN102                     1000a408     handles.obj
 0001:00009548       $LN102                     1000a548     handles.obj
 0001:0000a5a4       $LN313                     1000b5a4     handles.obj
 0001:0000a5ac       $LN312                     1000b5ac     handles.obj
 0001:0000ba18       $LN93                      1000ca18     handles.obj
 0001:0000ba30       $LN92                      1000ca30     handles.obj
 0001:0000d85c       $LN56                      1000e85c     handles.obj
 0001:0000d874       $LN55                      1000e874     handles.obj
 0001:0000dbc4       $LN18                      1000ebc4     handles.obj
 0001:0000dbe8       $LN17                      1000ebe8     handles.obj
 0001:0000e368       $LN133                     1000f368     handles.obj
 0001:0000e37c       $LN132                     1000f37c     handles.obj
 0001:00010a6c       $LN40                      10011a6c     Pcfg.obj
 0001:00010a7c       $LN39                      10011a7c     Pcfg.obj
 0001:00010d54       $LN51                      10011d54     Pcfg.obj
 0001:00010d64       $LN50                      10011d64     Pcfg.obj
 0001:00010fb0       $LN76                      10011fb0     Pcfg.obj
 0001:00010fc0       $LN75                      10011fc0     Pcfg.obj
 0001:00011ad0       ?ui64toa_width@@YA?AV?$basic_string@_WU?$char_traits@_W@std@@V?$allocator@_W@2@@std@@_KI_N@Z 10012ad0 f   Pclass.obj
 0001:00012090       ?PrintTitle@@YA?AV?$basic_string@_WU?$char_traits@_W@std@@V?$allocator@_W@2@@std@@V?$basic_string_view@_WU?$char_traits@_W@std@@@2@@Z 10013090 f   Pclass.obj
 0001:00012260       ?PrintTitle@@YA?AV?$basic_string@_WU?$char_traits@_W@std@@V?$allocator@_W@2@@std@@H@Z 10013260 f   Pclass.obj
 0001:000124d0       ?TranslateMode@@YA_NABV?$basic_string@_WU?$char_traits@_W@std@@V?$allocator@_W@2@@std@@AAV12@@Z 100134d0 f   Pclass.obj
 0001:00012c84       $LN826                     10013c84     Pclass.obj
 0001:00012c8c       $LN825                     10013c8c     Pclass.obj
 0001:00012ca4       $LN828                     10013ca4     Pclass.obj
 0001:00012cac       $LN827                     10013cac     Pclass.obj
 0001:00013ea0       ?generate_titles@@YAXABV?$basic_string@_WU?$char_traits@_W@std@@V?$allocator@_W@2@@std@@AAUPanelMode@@@Z 10014ea0 f   Pclass.obj
 0001:000140a4       $LN89                      100150a4     Pclass.obj
 0001:000140b8       $LN88                      100150b8     Pclass.obj
 0001:000140d0       $LN91                      100150d0     Pclass.obj
 0001:000140f0       $LN90                      100150f0     Pclass.obj
 0001:00014120       ?convert_panel_modes@@YAXABV?$vector@Umode@@V?$allocator@Umode@@@std@@@std@@AAV?$array@UPanelMode@@$09@2@@Z 10015120 f   Pclass.obj
 0001:00014650       ?EnumWndProc@@YGHPAUHWND__@@J@Z 10015650 f   Pclass.obj
 0001:00015620       $LN1463                    10016620     Pclass.obj
 0001:00015634       $LN1462                    10016634     Pclass.obj
 0001:0001564c       $LN1466                    1001664c     Pclass.obj
 0001:0001566c       $LN1465                    1001666c     Pclass.obj
 0001:000157e0       ?window_style@@YA@PAUHWND__@@@Z 100167e0 f   Pclass.obj
 0001:00015ab0       ?window_ex_style@@YA@PAUHWND__@@@Z 10016ab0 f   Pclass.obj
 0001:00015d20       ?DumpNTCounters@@YAXPAXAAVPerfThread@@KK@Z 10016d20 f   Pclass.obj
 0001:000186f8       $LN784                     100196f8     Pclass.obj
 0001:0001a124       $LN2618                    1001b124     Pclass.obj
 0001:0001a134       $LN2617                    1001b134     Pclass.obj
 0001:0001de60       ??R<lambda_1>@?1??RefreshImpl@PerfThread@@AAE_NXZ@QBE@PBU_PERF_COUNTER_BLOCK@@V?$basic_string_view@_WU?$char_traits@_W@std@@@std@@@Z 1001ee60 f   perfthread.obj
 0001:0001f960       ??$transform@V?$_List_const_iterator@V?$_List_val@U?$_List_simple_types@U?$pair@$$CBKUProcessPerfData@@@std@@@std@@@std@@@std@@V?$back_insert_iterator@V?$vector@UProcessPerfData@@V?$allocator@UProcessPerfData@@@std@@@std@@@2@V<lambda_1>@?2??RefreshWMIData@PerfThread@@AAEXXZ@@std@@YA?AV?$back_insert_iterator@V?$vector@UProcessPerfData@@V?$allocator@UProcessPerfData@@@std@@@std@@@0@V?$_List_const_iterator@V?$_List_val@U?$_List_simple_types@U?$pair@$$CBKUProcessPerfData@@@std@@@std@@@std@@@0@0V10@V<lambda_1>@?2??RefreshWMIData@PerfThread@@AAEXXZ@@Z 10020960 f   perfthread.obj
 0001:00020330       ?is_wow64_itself@@YA_NXZ   10021330 f   Plist.obj
 0001:00020600       ?FreeUserData@@YGXQAXQBUFarPanelItemFreeInfo@@@Z 10021600 f   Plist.obj
 0001:00020f60       ?PrintModuleVersion@@YAXPAXPB_W1I@Z 10021f60 f   Plist.obj
 0001:00021050       ?print_module_impl@@YAXQAXABV?$basic_string@_WU?$char_traits@_W@std@@V?$allocator@_W@2@@std@@KABUoptions@@ABV?$function@$$A6A_NPA_WI@Z@2@@Z 10022050 f   Plist.obj
 0001:000216f0       ??R<lambda_2>@?1??PrintModules@@YAXPAXKAAUoptions@@@Z@QBE@XZ 100226f0 f   Plist.obj
 0001:00022540       ??$print_module@PAX@@YAXQAXPAXKAAUoptions@@ABV?$function@$$A6A_NPA_WI@Z@std@@@Z 10023540 f   Plist.obj
 0001:00022700       ??$print_module@_K@@YAXQAX_KKAAUoptions@@ABV?$function@$$A6A_NPA_WI@Z@std@@@Z 10023700 f   Plist.obj
 0001:00022bd0       ?_Delete_this@?$_Func_impl_no_alloc@V<lambda_3>@?N@??PrintModules@@YAXPAXKAAUoptions@@@Z@_NPA_WI@std@@EAEX_N@Z 10023bd0 f i Plist.obj
 0001:00022bf0       ?_Get@?$_Func_impl_no_alloc@V<lambda_3>@?N@??PrintModules@@YAXPAXKAAUoptions@@@Z@_NPA_WI@std@@EBEPBXXZ 10023bf0 f i Plist.obj
 0001:00022bf0       ?_Get@?$_Func_impl_no_alloc@V<lambda_1>@?1??GetProcessInt@WMIConnection@@AAEKKPB_W@Z@XABUtagVARIANT@@@std@@EBEPBXXZ 10023bf0 f i wmi.obj
 0001:00022bf0       ?_Get@?$_Func_impl_no_alloc@V<lambda_1>@?1??GetProcessString@WMIConnection@@AAE?AV?$basic_string@_WU?$char_traits@_W@std@@V?$allocator@_W@2@@std@@KPB_W@Z@XABUtagVARIANT@@@std@@EBEPBXXZ 10023bf0 f i wmi.obj
 0001:00022cf0       ?_Target_type@?$_Func_impl_no_alloc@V<lambda_3>@?N@??PrintModules@@YAXPAXKAAUoptions@@@Z@_NPA_WI@std@@EBEABVtype_info@@XZ 10023cf0 f   Plist.obj
 0001:00022d00       ?_Do_call@?$_Func_impl_no_alloc@V<lambda_3>@?N@??PrintModules@@YAXPAXKAAUoptions@@@Z@_NPA_WI@std@@EAE_N$$QAPA_W$$QAI@Z 10023d00 f   Plist.obj
 0001:00022d30       ?_Copy@?$_Func_impl_no_alloc@V<lambda_3>@?N@??PrintModules@@YAXPAXKAAUoptions@@@Z@_NPA_WI@std@@EBEPAV?$_Func_base@_NPA_WI@2@PAX@Z 10023d30 f   Plist.obj
 0001:00022d30       ?_Move@?$_Func_impl_no_alloc@V<lambda_3>@?N@??PrintModules@@YAXPAXKAAUoptions@@@Z@_NPA_WI@std@@EAEPAV?$_Func_base@_NPA_WI@2@PAX@Z 10023d30 f   Plist.obj
 0001:000232b0       ?ProcessPath@@YA@K@Z       100242b0 f   wmi.obj
 0001:00024120       ?_Delete_this@?$_Func_impl_no_alloc@V<lambda_1>@?1??GetProcessInt@WMIConnection@@AAEKKPB_W@Z@XABUtagVARIANT@@@std@@EAEX_N@Z 10025120 f   wmi.obj
 0001:00024120       ?_Delete_this@?$_Func_impl_no_alloc@V<lambda_1>@?1??GetProcessString@WMIConnection@@AAE?AV?$basic_string@_WU?$char_traits@_W@std@@V?$allocator@_W@2@@std@@KPB_W@Z@XABUtagVARIANT@@@std@@EAEX_N@Z 10025120 f   wmi.obj
 0001:00024140       ?_Target_type@?$_Func_impl_no_alloc@V<lambda_1>@?1??GetProcessString@WMIConnection@@AAE?AV?$basic_string@_WU?$char_traits@_W@std@@V?$allocator@_W@2@@std@@KPB_W@Z@XABUtagVARIANT@@@std@@EBEABVtype_info@@XZ 10025140 f   wmi.obj
 0001:00024150       ?_Do_call@?$_Func_impl_no_alloc@V<lambda_1>@?1??GetProcessString@WMIConnection@@AAE?AV?$basic_string@_WU?$char_traits@_W@std@@V?$allocator@_W@2@@std@@KPB_W@Z@XABUtagVARIANT@@@std@@EAEXABUtagVARIANT@@@Z 10025150 f   wmi.obj
 0001:00024190       ?_Copy@?$_Func_impl_no_alloc@V<lambda_1>@?1??GetProcessString@WMIConnection@@AAE?AV?$basic_string@_WU?$char_traits@_W@std@@V?$allocator@_W@2@@std@@KPB_W@Z@XABUtagVARIANT@@@std@@EBEPAV?$_Func_base@XABUtagVARIANT@@@2@PAX@Z 10025190 f   wmi.obj
 0001:00024190       ?_Move@?$_Func_impl_no_alloc@V<lambda_1>@?1??GetProcessString@WMIConnection@@AAE?AV?$basic_string@_WU?$char_traits@_W@std@@V?$allocator@_W@2@@std@@KPB_W@Z@XABUtagVARIANT@@@std@@EAEPAV?$_Func_base@XABUtagVARIANT@@@2@PAX@Z 10025190 f   wmi.obj
 0001:000241b0       ?_Target_type@?$_Func_impl_no_alloc@V<lambda_1>@?1??GetProcessInt@WMIConnection@@AAEKKPB_W@Z@XABUtagVARIANT@@@std@@EBEABVtype_info@@XZ 100251b0 f   wmi.obj
 0001:000241c0       ?_Do_call@?$_Func_impl_no_alloc@V<lambda_1>@?1??GetProcessInt@WMIConnection@@AAEKKPB_W@Z@XABUtagVARIANT@@@std@@EAEXABUtagVARIANT@@@Z 100251c0 f   wmi.obj
 0001:000241e0       ?_Copy@?$_Func_impl_no_alloc@V<lambda_1>@?1??GetProcessInt@WMIConnection@@AAEKKPB_W@Z@XABUtagVARIANT@@@std@@EBEPAV?$_Func_base@XABUtagVARIANT@@@2@PAX@Z 100251e0 f   wmi.obj
 0001:000241e0       ?_Move@?$_Func_impl_no_alloc@V<lambda_1>@?1??GetProcessInt@WMIConnection@@AAEKKPB_W@Z@XABUtagVARIANT@@@std@@EAEPAV?$_Func_base@XABUtagVARIANT@@@2@PAX@Z 100251e0 f   wmi.obj
 0001:00024200       ?fNtQueryInformationFile@@YGJPAX00KK@Z 10025200 f   Proclist.obj
 0001:00024200       ?fNtQueryInformationProcess@@YGJPAXW4_PROCESSINFOCLASS@@0KPAK@Z 10025200 f   Proclist.obj
 0001:00024200       ?fNtQueryInformationThread@@YGJPAXK0KPAK@Z 10025200 f   Proclist.obj
 0001:00024200       ?fNtQueryObject@@YGJPAXK0K0@Z 10025200 f   Proclist.obj
 0001:00024200       ?fNtWow64QueryInformationProcess64@@YGJPAXW4_PROCESSINFOCLASS@@0KPAK@Z 10025200 f   Proclist.obj
 0001:00024210       ?fNtQuerySystemInformation@@YGJKPAXKPAK@Z 10025210 f   Proclist.obj
 0001:00024220       ?fNtWow64ReadVirtualMemory64@@YGJPAX_K01PA_K@Z 10025220 f   Proclist.obj
 0001:00024230       ?fGetGuiResources@@YGKPAXK@Z 10025230 f   Proclist.obj
 0001:00024230       ?fIsWow64Process@@YGHPAXPAH@Z 10025230 f   Proclist.obj
 0001:00024240       ?fCoSetProxyBlanket@@YGJPAUIUnknown@@KKPA_WKKPAXK@Z 10025240 f   Proclist.obj
 0001:00024250       ?fEnumProcessModulesEx@@YGHPAXPAPAUHINSTANCE__@@KPAKK@Z 10025250 f   Proclist.obj
 0001:00024260       ?dynamic_bind@@YAXXZ       10025260 f   Proclist.obj
 0001:00024bb0       ?DecodePointer@implementation@?1??DecodePointerWrapper@@YGPAXPAX@Z@SGPAX0@Z 10025bb0 f   vc_crt_fix_impl.obj
 0001:00024bb0       ?EncodePointer@implementation@?1??EncodePointerWrapper@@YGPAXPAX@Z@SGPAX0@Z 10025bb0 f   vc_crt_fix_impl.obj
 0001:00024cc0       ?GetModuleHandleExW@implementation@?1??GetModuleHandleExWWrapper@@YGHKPB_WPAPAUHINSTANCE__@@@Z@SGHK01@Z 10025cc0 f   vc_crt_fix_impl.obj
 0001:00024d90       ?InitializeSListHead@implementation@slist@@YGXPAT_SLIST_HEADER@@@Z 10025d90 f   vc_crt_fix_impl.obj
 0001:00024e50       ?InterlockedFlushSList@implementation@slist@@YGPAU_SINGLE_LIST_ENTRY@@PAT_SLIST_HEADER@@@Z 10025e50 f   vc_crt_fix_impl.obj
 0001:00024e80       ?InterlockedPopEntrySList@implementation@slist@@YGPAU_SINGLE_LIST_ENTRY@@PAT_SLIST_HEADER@@@Z 10025e80 f   vc_crt_fix_impl.obj
 0001:00024ed0       ?InterlockedPushEntrySList@implementation@slist@@YGPAU_SINGLE_LIST_ENTRY@@PAT_SLIST_HEADER@@PAU3@@Z 10025ed0 f   vc_crt_fix_impl.obj
 0001:00024f10       ?InterlockedPushListSListEx@implementation@slist@@YGPAU_SINGLE_LIST_ENTRY@@PAT_SLIST_HEADER@@PAU3@1K@Z 10025f10 f   vc_crt_fix_impl.obj
 0001:00024f50       ?RtlFirstEntrySList@implementation@slist@@YGPAU_SINGLE_LIST_ENTRY@@PAT_SLIST_HEADER@@@Z 10025f50 f   vc_crt_fix_impl.obj
 0001:00024f80       ?QueryDepthSList@implementation@slist@@YGGPAT_SLIST_HEADER@@@Z 10025f80 f   vc_crt_fix_impl.obj
 0001:00025230       ?GetNumaHighestNodeNumber@implementation@?1??GetNumaHighestNodeNumberWrapper@@YGHPAK@Z@SGH0@Z 10026230 f   vc_crt_fix_impl.obj
 0001:000252a0       ?GetLogicalProcessorInformation@implementation@?1??GetLogicalProcessorInformationWrapper@@YGHPAU_SYSTEM_LOGICAL_PROCESSOR_INFORMATION@@PAK@Z@SGH01@Z 100262a0 f   vc_crt_fix_impl.obj
 0001:00025300       ?SetThreadStackGuarantee@implementation@?1??SetThreadStackGuaranteeWrapper@@YGHPAK@Z@SGH0@Z 10026300 f   vc_crt_fix_impl.obj
 0001:00025360       ?InitializeCriticalSectionEx@implementation@?1??InitializeCriticalSectionExWrapper@@YGHPAU_RTL_CRITICAL_SECTION@@KK@Z@SGH0KK@Z 10026360 f   vc_crt_fix_impl.obj
 0001:000253e0       ?CompareStringEx@implementation@?1??CompareStringExWrapper@@YGHPB_WK0H0HPAU_nlsversioninfo@@PAXJ@Z@SGH0K0H0H12J@Z 100263e0 f   vc_crt_fix_impl.obj
 0001:00025460       ?CompareStringEx@implementation@?1??LCMapStringExWrapper@@YGHPB_WK0HPA_WHPAU_nlsversioninfo@@PAXJ@Z@SGH0K0H1H23J@Z 10026460 f   vc_crt_fix_impl.obj
 0001:000255c2       __Utf8_trailing_byte_count 100265c2 f   libcpmt:xmbtowc.obj
 0001:00025bb4       _tidy_global               10026bb4 f   libcpmt:locale0.obj
 0001:00025d53       ?find_pe_section@@YAPAU_IMAGE_SECTION_HEADER@@QAEI@Z 10026d53 f   LIBCMT:utility.obj
 0001:000263f3       ?dllmain_crt_dispatch@@YGHQAUHINSTANCE__@@KQAX@Z 100273f3 f   LIBCMT:dll_dllmain.obj
 0001:00026446       ?dllmain_crt_process_attach@@YAHQAUHINSTANCE__@@QAX@Z 10027446 f   LIBCMT:dll_dllmain.obj
 0001:0002654d       ?dllmain_crt_process_detach@@YAH_N@Z 1002754d f   LIBCMT:dll_dllmain.obj
 0001:000265fd       ?dllmain_dispatch@@YAHQAUHINSTANCE__@@KQAX@Z 100275fd f   LIBCMT:dll_dllmain.obj
 0001:00026708       ?dllmain_raw@@YGHQAUHINSTANCE__@@KQAX@Z 10027708 f   LIBCMT:dll_dllmain.obj
 0001:00026820       $$000000                   10027820     LIBCMT:llmul.obj
 0001:00026839       hard                       10027839     LIBCMT:llmul.obj
 0001:00026860       $$000000                   10027860     LIBCMT:alloca16.obj
 0001:00026876       alloca_8                   10027876     LIBCMT:alloca16.obj
 0001:00026b90       $$000000                   10027b90     LIBCMT:sehprolg4.obj
 0001:00026bd5       ___get_entropy             10027bd5 f   LIBCMT:gs_support.obj
 0001:00026d10       $$000000                   10027d10     LIBCMT:chkstk.obj
 0001:00026d24       cs10                       10027d24     LIBCMT:chkstk.obj
 0001:00026d32       cs20                       10027d32     LIBCMT:chkstk.obj
 0001:0002719f       ?_FilterSetCurrentException@@YAKPAU_EXCEPTION_POINTERS@@E@Z 1002819f f   libvcruntime:ehhelpers.obj
 0001:00027490       $$000000                   10028490     libvcruntime:memcpy.obj
 0001:00027490       $$000000                   10028490     libvcruntime:memmove.obj
 0001:000274b0       CopyUp                     100284b0     libvcruntime:memcpy.obj
 0001:000274b0       CopyUp                     100284b0     libvcruntime:memmove.obj
 0001:000274d4       CopyUpLargeMov             100284d4     libvcruntime:memcpy.obj
 0001:000274d4       CopyUpLargeMov             100284d4     libvcruntime:memmove.obj
 0001:000274e7       CopyUpSSE2Check            100284e7     libvcruntime:memcpy.obj
 0001:000274e7       CopyUpSSE2Check            100284e7     libvcruntime:memmove.obj
 0001:00027500       AtomChk                    10028500     libvcruntime:memcpy.obj
 0001:00027500       AtomChk                    10028500     libvcruntime:memmove.obj
 0001:00027526       PalignHead4                10028526     libvcruntime:memcpy.obj
 0001:00027526       PalignHead4                10028526     libvcruntime:memmove.obj
 0001:00027539       PalignHead8                10028539     libvcruntime:memcpy.obj
 0001:00027539       PalignHead8                10028539     libvcruntime:memmove.obj
 0001:00027550       PalignLoop                 10028550     libvcruntime:memcpy.obj
 0001:00027550       PalignLoop                 10028550     libvcruntime:memmove.obj
 0001:00027562       MovPalign12                10028562     libvcruntime:memcpy.obj
 0001:00027562       MovPalign12                10028562     libvcruntime:memmove.obj
 0001:0002756c       PalignLoop12               1002856c     libvcruntime:memcpy.obj
 0001:0002756c       PalignLoop12               1002856c     libvcruntime:memmove.obj
 0001:000275bd       MovPalign8                 100285bd     libvcruntime:memcpy.obj
 0001:000275bd       MovPalign8                 100285bd     libvcruntime:memmove.obj
 0001:000275c8       PalignLoop8                100285c8     libvcruntime:memcpy.obj
 0001:000275c8       PalignLoop8                100285c8     libvcruntime:memmove.obj
 0001:00027616       MovPalign4                 10028616     libvcruntime:memcpy.obj
 0001:00027616       MovPalign4                 10028616     libvcruntime:memmove.obj
 0001:00027620       PalignLoop4                10028620     libvcruntime:memcpy.obj
 0001:00027620       PalignLoop4                10028620     libvcruntime:memmove.obj
 0001:0002766c       PalignTail                 1002866c     libvcruntime:memcpy.obj
 0001:0002766c       PalignTail                 1002866c     libvcruntime:memmove.obj
 0001:00027684       PalignTail4                10028684     libvcruntime:memcpy.obj
 0001:00027684       PalignTail4                10028684     libvcruntime:memmove.obj
 0001:00027697       PalignTail8                10028697     libvcruntime:memcpy.obj
 0001:00027697       PalignTail8                10028697     libvcruntime:memmove.obj
 0001:000276ae       PalignTailLE3              100286ae     libvcruntime:memcpy.obj
 0001:000276ae       PalignTailLE3              100286ae     libvcruntime:memmove.obj
 0001:000276b7       Dword_align                100286b7     libvcruntime:memcpy.obj
 0001:000276b7       Dword_align                100286b7     libvcruntime:memmove.obj
 0001:000276bf       Dword_up_align_loop        100286bf     libvcruntime:memcpy.obj
 0001:000276bf       Dword_up_align_loop        100286bf     libvcruntime:memmove.obj
 0001:000276d2       Dword_align_Ok             100286d2     libvcruntime:memcpy.obj
 0001:000276d2       Dword_align_Ok             100286d2     libvcruntime:memmove.obj
 0001:000276ec       ByteCopyUp                 100286ec     libvcruntime:memcpy.obj
 0001:000276ec       ByteCopyUp                 100286ec     libvcruntime:memmove.obj
 0001:000276f4       TrailingUpVec              100286f4     libvcruntime:memcpy.obj
 0001:000276f4       TrailingUpVec              100286f4     libvcruntime:memmove.obj
 0001:00027704       TrailingUp0                10028704     libvcruntime:memcpy.obj
 0001:00027704       TrailingUp0                10028704     libvcruntime:memmove.obj
 0001:0002770c       TrailingUp1                1002870c     libvcruntime:memcpy.obj
 0001:0002770c       TrailingUp1                1002870c     libvcruntime:memmove.obj
 0001:00027718       TrailingUp2                10028718     libvcruntime:memcpy.obj
 0001:00027718       TrailingUp2                10028718     libvcruntime:memmove.obj
 0001:0002772c       TrailingUp3                1002872c     libvcruntime:memcpy.obj
 0001:0002772c       TrailingUp3                1002872c     libvcruntime:memmove.obj
 0001:00027744       CopyDown                   10028744     libvcruntime:memcpy.obj
 0001:00027744       CopyDown                   10028744     libvcruntime:memmove.obj
 0001:00027769       CopyDownNotAligned         10028769     libvcruntime:memcpy.obj
 0001:00027769       CopyDownNotAligned         10028769     libvcruntime:memmove.obj
 0001:00027770       CopyDownAlignLoop          10028770     libvcruntime:memcpy.obj
 0001:00027770       CopyDownAlignLoop          10028770     libvcruntime:memmove.obj
 0001:0002777d       CopyDownAligned            1002877d     libvcruntime:memcpy.obj
 0001:0002777d       CopyDownAligned            1002877d     libvcruntime:memmove.obj
 0001:000277a0       TrailingDownVec            100287a0     libvcruntime:memcpy.obj
 0001:000277a0       TrailingDownVec            100287a0     libvcruntime:memmove.obj
 0001:000277b0       TrailingDown0              100287b0     libvcruntime:memcpy.obj
 0001:000277b0       TrailingDown0              100287b0     libvcruntime:memmove.obj
 0001:000277b8       TrailingDown1              100287b8     libvcruntime:memcpy.obj
 0001:000277b8       TrailingDown1              100287b8     libvcruntime:memmove.obj
 0001:000277c8       TrailingDown2              100287c8     libvcruntime:memcpy.obj
 0001:000277c8       TrailingDown2              100287c8     libvcruntime:memmove.obj
 0001:000277dc       TrailingDown3              100287dc     libvcruntime:memcpy.obj
 0001:000277dc       TrailingDown3              100287dc     libvcruntime:memmove.obj
 0001:000277f5       XmmMovLargeAlignTest       100287f5     libvcruntime:memcpy.obj
 0001:000277f5       XmmMovLargeAlignTest       100287f5     libvcruntime:memmove.obj
 0001:000277fd       XmmMovAlignLoop            100287fd     libvcruntime:memcpy.obj
 0001:000277fd       XmmMovAlignLoop            100287fd     libvcruntime:memmove.obj
 0001:0002780c       XmmMovLargeLoop            1002880c     libvcruntime:memcpy.obj
 0001:0002780c       XmmMovLargeLoop            1002880c     libvcruntime:memmove.obj
 0001:0002787c       XmmMovSmallTest            1002887c     libvcruntime:memcpy.obj
 0001:0002787c       XmmMovSmallTest            1002887c     libvcruntime:memmove.obj
 0001:00027881       XmmMovSmallLoop            10028881     libvcruntime:memcpy.obj
 0001:00027881       XmmMovSmallLoop            10028881     libvcruntime:memmove.obj
 0001:000278a4       CopyDownSmall              100288a4     libvcruntime:memcpy.obj
 0001:000278a4       CopyDownSmall              100288a4     libvcruntime:memmove.obj
 0001:000278ac       CopyDownDwordLoop          100288ac     libvcruntime:memcpy.obj
 0001:000278ac       CopyDownDwordLoop          100288ac     libvcruntime:memmove.obj
 0001:000278c1       CopyDownByteTest           100288c1     libvcruntime:memcpy.obj
 0001:000278c1       CopyDownByteTest           100288c1     libvcruntime:memmove.obj
 0001:000278c5       CopyDownByteLoop           100288c5     libvcruntime:memcpy.obj
 0001:000278c5       CopyDownByteLoop           100288c5     libvcruntime:memmove.obj
 0001:000278d4       CopyDownReturn             100288d4     libvcruntime:memcpy.obj
 0001:000278d4       CopyDownReturn             100288d4     libvcruntime:memmove.obj
 0001:000278e0       XmmCopy                    100288e0     libvcruntime:memcpy.obj
 0001:000278e0       XmmCopy                    100288e0     libvcruntime:memmove.obj
 0001:000278ed       XmmCopyAligned             100288ed     libvcruntime:memcpy.obj
 0001:000278ed       XmmCopyAligned             100288ed     libvcruntime:memmove.obj
 0001:00027900       XmmCopyLargeLoop           10028900     libvcruntime:memcpy.obj
 0001:00027900       XmmCopyLargeLoop           10028900     libvcruntime:memmove.obj
 0001:0002795d       XmmCopySmallTest           1002895d     libvcruntime:memcpy.obj
 0001:0002795d       XmmCopySmallTest           1002895d     libvcruntime:memmove.obj
 0001:00027970       XmmCopySmallLoop           10028970     libvcruntime:memcpy.obj
 0001:00027970       XmmCopySmallLoop           10028970     libvcruntime:memmove.obj
 0001:0002798b       CopyUpDwordMov             1002898b     libvcruntime:memcpy.obj
 0001:0002798b       CopyUpDwordMov             1002898b     libvcruntime:memmove.obj
 0001:00027990       CopyUpDwordTest            10028990     libvcruntime:memcpy.obj
 0001:00027990       CopyUpDwordTest            10028990     libvcruntime:memmove.obj
 0001:00027997       CopyUpDwordLoop            10028997     libvcruntime:memcpy.obj
 0001:00027997       CopyUpDwordLoop            10028997     libvcruntime:memmove.obj
 0001:000279a6       CopyUpByteTest             100289a6     libvcruntime:memcpy.obj
 0001:000279a6       CopyUpByteTest             100289a6     libvcruntime:memmove.obj
 0001:000279ad       CopyUpByteLoop             100289ad     libvcruntime:memcpy.obj
 0001:000279ad       CopyUpByteLoop             100289ad     libvcruntime:memmove.obj
 0001:000279c0       CopyUpReturn               100289c0     libvcruntime:memcpy.obj
 0001:000279c0       CopyUpReturn               100289c0     libvcruntime:memmove.obj
 0001:000279d0       XmmCopyUnaligned           100289d0     libvcruntime:memcpy.obj
 0001:000279d0       XmmCopyUnaligned           100289d0     libvcruntime:memmove.obj
 0001:000279e3       XmmAlignByte               100289e3     libvcruntime:memcpy.obj
 0001:000279e3       XmmAlignByte               100289e3     libvcruntime:memmove.obj
 0001:000279ec       XmmAlignDwordTest          100289ec     libvcruntime:memcpy.obj
 0001:000279ec       XmmAlignDwordTest          100289ec     libvcruntime:memmove.obj
 0001:000279f1       XmmAlignDwordLoop          100289f1     libvcruntime:memcpy.obj
 0001:000279f1       XmmAlignDwordLoop          100289f1     libvcruntime:memmove.obj
 0001:000279fe       XmmAlignAdjustCnt          100289fe     libvcruntime:memcpy.obj
 0001:000279fe       XmmAlignAdjustCnt          100289fe     libvcruntime:memmove.obj
 0001:00027a10       $$000000                   10028a10     libvcruntime:memset.obj
 0001:00027a55       XMMMov                     10028a55     libvcruntime:memset.obj
 0001:00027a90       LargeRangeBytes            10028a90     libvcruntime:memset.obj
 0001:00027acd       XmmMovSmall                10028acd     libvcruntime:memset.obj
 0001:00027ae0       XmmSmallLoop               10028ae0     libvcruntime:memset.obj
 0001:00027ae5       MidRangeBytes              10028ae5     libvcruntime:memset.obj
 0001:00027b01       XMMTrailingBytes           10028b01     libvcruntime:memset.obj
 0001:00027b15       SmallMov                   10028b15     libvcruntime:memset.obj
 0001:00027b1d       ByteLoop                   10028b1d     libvcruntime:memset.obj
 0001:00027b2b       DwordTest                  10028b2b     libvcruntime:memset.obj
 0001:00027b3b       QwordTest                  10028b3b     libvcruntime:memset.obj
 0001:00027b50       QwordLoop                  10028b50     libvcruntime:memset.obj
 0001:00027b63       toend                      10028b63     libvcruntime:memset.obj
 0001:000289fc       $LN1250                    100299fc     libvcruntime:memcmp.obj
 0001:00028ad0       _ValidateLocalCookies      10029ad0 f   libvcruntime:chandler4.obj
 0001:00028e0d       ??$BuildCatchObjectHelperInternal@V__FrameHandler3@@@@YAHPAUEHExceptionRecord@@PAXPBU_s_HandlerType@@PBU_s_CatchableType@@@Z 10029e0d f   libvcruntime:frame.obj
 0001:00028f4b       ??$BuildCatchObjectInternal@V__FrameHandler3@@@@YAXPAUEHExceptionRecord@@PAXPBU_s_HandlerType@@PBU_s_CatchableType@@@Z 10029f4b f   libvcruntime:frame.obj
 0001:00028fe4       ??$CatchIt@V__FrameHandler3@@@@YAXPAUEHExceptionRecord@@PAUEHRegistrationNode@@PAU_CONTEXT@@PAXPBU_s_FuncInfo@@PBU_s_HandlerType@@PBU_s_CatchableType@@PBU_s_TryBlockMapEntry@@H1EE@Z 10029fe4 f   libvcruntime:frame.obj
 0001:00029064       ??$FindHandler@V__FrameHandler3@@@@YAXPAUEHExceptionRecord@@PAUEHRegistrationNode@@PAU_CONTEXT@@PAXPBU_s_FuncInfo@@EH1@Z 1002a064 f   libvcruntime:frame.obj
 0001:0002940e       ??$FindHandlerForForeignException@V__FrameHandler3@@@@YAXPAUEHExceptionRecord@@PAUEHRegistrationNode@@PAU_CONTEXT@@PAXPBU_s_FuncInfo@@HH1@Z 1002a40e f   libvcruntime:frame.obj
 0001:00029726       ?CallCatchBlock@@YAPAXPAUEHExceptionRecord@@PAUEHRegistrationNode@@PAU_CONTEXT@@PBU_s_FuncInfo@@PAXHK@Z 1002a726 f   libvcruntime:frame.obj
 0001:000298ea       ?CallUnexpected@@YAXPBU_s_ESTypeList@@@Z 1002a8ea f   libvcruntime:frame.obj
 0001:0002990a       __catch$?CallUnexpected@@YAXPBU_s_ESTypeList@@@Z$0 1002a90a f   libvcruntime:frame.obj
 0001:00029929       ?ExFilterRethrow@@YAHPAU_EXCEPTION_POINTERS@@@Z 1002a929 f   libvcruntime:frame.obj
 0001:00029a73       ?IsInExceptionSpec@@YAEPAUEHExceptionRecord@@PBU_s_ESTypeList@@@Z 1002aa73 f   libvcruntime:frame.obj
 0001:00029b40       $$000000                   1002ab40     libvcruntime:lowhelpr.obj
 0001:00029b7f       _NLG_Continue              1002ab7f     libvcruntime:lowhelpr.obj
 0001:00029c30       $$000000                   1002ac30     libvcruntime:exsup4.obj
 0001:00029c62       _lu_top                    1002ac62     libvcruntime:exsup4.obj
 0001:00029cc1       _lu_done                   1002acc1     libvcruntime:exsup4.obj
 0001:00029cd0       $$000000                   1002acd0     libvcruntime:exsup4.obj
 0001:00029cd0       __unwind_handler4          1002acd0 f   libvcruntime:exsup4.obj
 0001:00029d20       $$000000                   1002ad20     libvcruntime:exsup4.obj
 0001:00029d40       $$000000                   1002ad40     libvcruntime:exsup4.obj
 0001:00029d60       $$000000                   1002ad60     libvcruntime:exsup4.obj
 0001:00029d75       ReturnPoint                1002ad75     libvcruntime:exsup4.obj
 0001:00029d80       $$000000                   1002ad80     libvcruntime:exsup4.obj
 0001:00029d97       ?try_get_first_available_module@@YAPAUHINSTANCE__@@QBW4module_id@?A0x26f6bd02@@0@Z 1002ad97 f   libvcruntime:winapi_downlevel.obj
 0001:00029e31       ?try_get_function@@YAPAXW4function_id@?A0x26f6bd02@@QBDQBW4module_id@2@2@Z 1002ae31 f   libvcruntime:winapi_downlevel.obj
 0001:0002a000       $$000000                   1002b000     libvcruntime:exsup.obj
 0001:0002a010       $$000000                   1002b010     libvcruntime:exsup.obj
 0001:0002a01b       __NLG_Go                   1002b01b     libvcruntime:exsup.obj
 0001:0002a030       $$000000                   1002b030     libvcruntime:exsup.obj
 0001:0002a880       $$000000                   1002b880     libucrt:modf_pentium4.obj
 0001:0002ac39       ??$common_tcsncpy_s@_W@@YAHQA_WIQB_WI@Z 1002bc39 f   libucrt:wcsncpy_s.obj
 0001:0002ae1f       ??$?RV<lambda_646e26742ed01d5bc03234f44bb6d3d3>@@AAV<lambda_b37934c380d97b75fd242ea49540127a>@@V<lambda_bbd9d45274666fbb50f81a29ad795c13>@@@?$__crt_seh_guarded_call@PAD@@QAEPAD$$QAV<lambda_646e26742ed01d5bc03234f44bb6d3d3>@@AAV<lambda_b37934c380d97b75fd242ea49540127a>@@$$QAV<lambda_bbd9d45274666fbb50f81a29ad795c13>@@@Z 1002be1f f   libucrt:setlocale.obj
 0001:0002ae7a       ??R<lambda_b37934c380d97b75fd242ea49540127a>@@QBEPADXZ 1002be7a f   libucrt:setlocale.obj
 0001:0002afde       _call_wsetlocale           1002bfde f   libucrt:setlocale.obj
 0001:0002b5f0       $$000000                   1002c5f0     libucrt:strcspn.obj
 0001:0002b640       $$000000                   1002c640     libucrt:pow_impl.obj
 0001:0002b92c       ??$__acrt_convert_wcs_mbs_cp@D_WV<lambda_62f6974d9771e494a5ea317cc32e971c>@@U__crt_win32_buffer_internal_dynamic_resizing@@@@YAHQBDAAV?$__crt_win32_buffer@_WU__crt_win32_buffer_internal_dynamic_resizing@@@@ABV<lambda_62f6974d9771e494a5ea317cc32e971c>@@I@Z 1002c92c f   libucrt:strftime.obj
 0001:0002be20       ??$?RV<lambda_03b1d95aef87969028cfba75ccab2455>@@AAV<lambda_6e4b09c48022b2350581041d5f6b0c4c>@@V<lambda_22bdf7517842c4b3e53723af5aa32b9e>@@@?$__crt_seh_guarded_call@X@@QAEX$$QAV<lambda_03b1d95aef87969028cfba75ccab2455>@@AAV<lambda_6e4b09c48022b2350581041d5f6b0c4c>@@$$QAV<lambda_22bdf7517842c4b3e53723af5aa32b9e>@@@Z 1002ce20 f   libucrt:exit.obj
 0001:0002be6d       ??R<lambda_6e4b09c48022b2350581041d5f6b0c4c>@@QBE@XZ 1002ce6d f   libucrt:exit.obj
 0001:0002bf47       ?atexit_exception_filter@@YAHK@Z 1002cf47 f   libucrt:exit.obj
 0001:0002bf5a       ?common_exit@@YAXHW4_crt_exit_cleanup_mode@@W4_crt_exit_return_mode@@@Z 1002cf5a f   libucrt:exit.obj
 0001:0002bfbe       ?exit_or_terminate_process@@YAXI@Z 1002cfbe f   libucrt:exit.obj
 0001:0002c000       ?is_managed_app@@YA_NXZ    1002d000 f   libucrt:exit.obj
 0001:0002c043       ?try_cor_exit_process@@YAXI@Z 1002d043 f   libucrt:exit.obj
 0001:0002c0d1       ??$common_configure_argv@D@@YAHW4_crt_argv_mode@@@Z 1002d0d1 f   libucrt:argv_parsing.obj
 0001:0002c207       ??$parse_command_line@D@@YAXPADPAPAD0PAI2@Z 1002d207 f   libucrt:argv_parsing.obj
 0001:0002c3d8       ??$common_initialize_environment_nolock@D@@YAHXZ 1002d3d8 f   libucrt:environment_initialization.obj
 0001:0002c42b       ??$create_environment@D@@YAQAPADQAD@Z 1002d42b f   libucrt:environment_initialization.obj
 0001:0002c4fb       ??$free_environment@D@@YAXQAPAD@Z 1002d4fb f   libucrt:environment_initialization.obj
 0001:0002c4fb       ??$free_environment@_W@@YAXQAPA_W@Z 1002d4fb f   libucrt:environment_initialization.obj
 0001:0002c553       ??$uninitialize_environment_internal@D@@YAXAAPAPAD@Z 1002d553 f   libucrt:environment_initialization.obj
 0001:0002c56e       ??$uninitialize_environment_internal@_W@@YAXAAPAPA_W@Z 1002d56e f   libucrt:environment_initialization.obj
 0001:0002c5c5       ??$?RV<lambda_69a2805e680e0e292e8ba93315fe43a8>@@AAV<lambda_f03950bc5685219e0bcd2087efbe011e>@@V<lambda_03fcd07e894ec930e3f35da366ca99d6>@@@?$__crt_seh_guarded_call@H@@QAEH$$QAV<lambda_69a2805e680e0e292e8ba93315fe43a8>@@AAV<lambda_f03950bc5685219e0bcd2087efbe011e>@@$$QAV<lambda_03fcd07e894ec930e3f35da366ca99d6>@@@Z 1002d5c5 f   libucrt:onexit.obj
 0001:0002c620       ??$?RV<lambda_8e746cf0007f6ed984d6f78af1fec997>@@AAV<lambda_22ebabd17bc4fa466a2aca6d8deb888d>@@V<lambda_18ed0c0b38a6dc0daf1e7ac6d6adf05e>@@@?$__crt_seh_guarded_call@H@@QAEH$$QAV<lambda_8e746cf0007f6ed984d6f78af1fec997>@@AAV<lambda_22ebabd17bc4fa466a2aca6d8deb888d>@@$$QAV<lambda_18ed0c0b38a6dc0daf1e7ac6d6adf05e>@@@Z 1002d620 f   libucrt:onexit.obj
 0001:0002c69a       ??R<lambda_22ebabd17bc4fa466a2aca6d8deb888d>@@QBEHXZ 1002d69a f   libucrt:onexit.obj
 0001:0002c7c3       ??R<lambda_f03950bc5685219e0bcd2087efbe011e>@@QBEHXZ 1002d7c3 f   libucrt:onexit.obj
 0001:0002c93c       _initialize_environment    1002d93c f   libucrt:initialization.obj
 0001:0002c93c       _initialize_global_state_isolation 1002d93c f   libucrt:initialization.obj
 0001:0002c93c       _report_memory_leaks       1002d93c f   libucrt:initialization.obj
 0001:0002c93c       _uninitialize_c            1002d93c f   libucrt:initialization.obj
 0001:0002c93c       _uninitialize_global_state_isolation 1002d93c f   libucrt:initialization.obj
 0001:0002c93f       _initialize_global_variables 1002d93f f   libucrt:initialization.obj
 0001:0002c94c       _initialize_c              1002d94c f   libucrt:initialization.obj
 0001:0002c966       _uninitialize_environment  1002d966 f   libucrt:initialization.obj
 0001:0002c96e       _initialize_pointers       1002d96e f   libucrt:initialization.obj
 0001:0002c99c       _uninitialize_vcruntime    1002d99c f   libucrt:initialization.obj
 0001:0002c9a5       _uninitialize_allocated_memory 1002d9a5 f   libucrt:initialization.obj
 0001:0002c9bc       _uninitialize_allocated_io_buffers 1002d9bc f   libucrt:initialization.obj
 0001:0002ca0c       ??R<lambda_af42a3ee9806e9a7305d451646e05244>@@QBEXAAPAU__crt_multibyte_data@@@Z 1002da0c f   libucrt:initialization.obj
 0001:0002d270       $$000000                   1002e270     libucrt:strncmp.obj
 0001:0002d322       ??$?RV<lambda_15ade71b0218206bbe3333a0c9b79046>@@AAV<lambda_da44e0f8b0f19ba52fefafb335991732>@@V<lambda_207f2d024fc103971653565357d6cd41>@@@?$__crt_seh_guarded_call@X@@QAEX$$QAV<lambda_15ade71b0218206bbe3333a0c9b79046>@@AAV<lambda_da44e0f8b0f19ba52fefafb335991732>@@$$QAV<lambda_207f2d024fc103971653565357d6cd41>@@@Z 1002e322 f   libucrt:per_thread_data.obj
 0001:0002d374       ??$?RV<lambda_38edbb1296d33220d7e4dd0ed76b244a>@@AAV<lambda_5ce1d447e08cb34b2473517608e21441>@@V<lambda_fb385d3da700c9147fc39e65dd577a8c>@@@?$__crt_seh_guarded_call@X@@QAEX$$QAV<lambda_38edbb1296d33220d7e4dd0ed76b244a>@@AAV<lambda_5ce1d447e08cb34b2473517608e21441>@@$$QAV<lambda_fb385d3da700c9147fc39e65dd577a8c>@@@Z 1002e374 f   libucrt:per_thread_data.obj
 0001:0002d3df       ??$?RV<lambda_6affb1475c98b40b75cdec977db92e3c>@@AAV<lambda_b8d4b9c228a6ecc3f80208dbb4b4a104>@@V<lambda_608742c3c92a14382c1684fc64f96c88>@@@?$__crt_seh_guarded_call@X@@QAEX$$QAV<lambda_6affb1475c98b40b75cdec977db92e3c>@@AAV<lambda_b8d4b9c228a6ecc3f80208dbb4b4a104>@@$$QAV<lambda_608742c3c92a14382c1684fc64f96c88>@@@Z 1002e3df f   libucrt:per_thread_data.obj
 0001:0002d434       ??$?RV<lambda_a7e850c220f1c8d1e6efeecdedd162c6>@@AAV<lambda_46720907175c18b6c9d2717bc0d2d362>@@V<lambda_9048902d66e8d99359bc9897bbb930a8>@@@?$__crt_seh_guarded_call@X@@QAEX$$QAV<lambda_a7e850c220f1c8d1e6efeecdedd162c6>@@AAV<lambda_46720907175c18b6c9d2717bc0d2d362>@@$$QAV<lambda_9048902d66e8d99359bc9897bbb930a8>@@@Z 1002e434 f   libucrt:per_thread_data.obj
 0001:0002d48e       ?construct_ptd@@YAXQAU__acrt_ptd@@QAPAU__crt_locale_data@@@Z 1002e48e f   libucrt:per_thread_data.obj
 0001:0002d527       ?destroy_fls@@YGXPAX@Z     1002e527 f   libucrt:per_thread_data.obj
 0001:0002d548       ?destroy_ptd@@YAXQAU__acrt_ptd@@@Z 1002e548 f   libucrt:per_thread_data.obj
 0001:0002d615       ?replace_current_thread_locale_nolock@@YAXQAU__acrt_ptd@@QAU__crt_locale_data@@@Z 1002e615 f   libucrt:per_thread_data.obj
 0001:0002d8de       ?initialize_inherited_file_handles_nolock@@YAXXZ 1002e8de f   libucrt:ioinit.obj
 0001:0002d994       ?initialize_stdio_handles_nolock@@YAXXZ 1002e994 f   libucrt:ioinit.obj
 0001:0002db71       ?<lambda_invoker_stdcall>@<lambda_29d3c280b90b41c2ae070ffca879996a>@@CGHPA_W@Z 1002eb71 f   libucrt:winapi_thunks.obj
 0001:0002db7e       ??$?RV<lambda_6b4b7855443974f2b4b77000ea21c99c>@@AAV<lambda_8f7d3b162ab39427f4fa9995c67a7986>@@V<lambda_cc9a5ba8a5d8428b9634eab82665e5dc>@@@?$__crt_seh_guarded_call@H@@QAEH$$QAV<lambda_6b4b7855443974f2b4b77000ea21c99c>@@AAV<lambda_8f7d3b162ab39427f4fa9995c67a7986>@@$$QAV<lambda_cc9a5ba8a5d8428b9634eab82665e5dc>@@@Z 1002eb7e f   libucrt:winapi_thunks.obj
 0001:0002dbfa       ??R<lambda_29d3c280b90b41c2ae070ffca879996a>@@QBEHPA_W@Z 1002ebfa f   libucrt:winapi_thunks.obj
 0001:0002dc29       ?try_get_AreFileApisANSI@@YAP6GHXZXZ 1002ec29 f   libucrt:winapi_thunks.obj
 0001:0002dc43       ?try_get_CompareStringEx@@YAP6GHPB_WK0H0HPAU_nlsversioninfo@@PAXJ@ZXZ 1002ec43 f   libucrt:winapi_thunks.obj
 0001:0002dc5d       ?try_get_EnumSystemLocalesEx@@YAP6GHP6GHPA_WKJ@ZKJPAX@ZXZ 1002ec5d f   libucrt:winapi_thunks.obj
 0001:0002dc77       ?try_get_GetDateFormatEx@@YAP6GHPB_WKPBU_SYSTEMTIME@@0PA_WH0@ZXZ 1002ec77 f   libucrt:winapi_thunks.obj
 0001:0002dc91       ?try_get_GetLocaleInfoEx@@YAP6GHPB_WKPA_WH@ZXZ 1002ec91 f   libucrt:winapi_thunks.obj
 0001:0002dcab       ?try_get_GetTimeFormatEx@@YAP6GHPB_WKPBU_SYSTEMTIME@@0PA_WH@ZXZ 1002ecab f   libucrt:winapi_thunks.obj
 0001:0002dcc5       ?try_get_GetUserDefaultLocaleName@@YAP6GHPA_WH@ZXZ 1002ecc5 f   libucrt:winapi_thunks.obj
 0001:0002dcdf       ?try_get_IsValidLocaleName@@YAP6GHPB_W@ZXZ 1002ecdf f   libucrt:winapi_thunks.obj
 0001:0002dcf9       ?try_get_LCIDToLocaleName@@YAP6GHKPA_WHK@ZXZ 1002ecf9 f   libucrt:winapi_thunks.obj
 0001:0002dd13       ?try_get_LCMapStringEx@@YAP6GHPB_WK0HPA_WHPAU_nlsversioninfo@@PAXJ@ZXZ 1002ed13 f   libucrt:winapi_thunks.obj
 0001:0002dd2d       ?try_get_LocaleNameToLCID@@YAP6GKPB_WK@ZXZ 1002ed2d f   libucrt:winapi_thunks.obj
 0001:0002dd47       ?try_get_first_available_module@@YAPAUHINSTANCE__@@QBW4module_id@?A0x391cf84c@@0@Z 1002ed47 f   libucrt:winapi_thunks.obj
 0001:0002de0e       ?try_get_function@@YAPAXW4function_id@?A0x391cf84c@@QBDQBW4module_id@2@2@Z 1002ee0e f   libucrt:winapi_thunks.obj
 0001:0002e35f       ??$?RV<lambda_2866be3712abc81a800a822484c830d8>@@AAV<lambda_39ca0ed439415581b5b15c265174cece>@@V<lambda_2b24c74d71094a6cd0cb82e44167d71b>@@@?$__crt_seh_guarded_call@X@@QAEX$$QAV<lambda_2866be3712abc81a800a822484c830d8>@@AAV<lambda_39ca0ed439415581b5b15c265174cece>@@$$QAV<lambda_2b24c74d71094a6cd0cb82e44167d71b>@@@Z 1002f35f f   libucrt:fflush.obj
 0001:0002e3eb       ??$?RV<lambda_2cc53f568c5a2bb6f192f930a45d44ea>@@AAV<lambda_ab61a845afdef5b7c387490eaf3616ee>@@V<lambda_c2ffc0b7726aa6be21d5f0026187e748>@@@?$__crt_seh_guarded_call@X@@QAEX$$QAV<lambda_2cc53f568c5a2bb6f192f930a45d44ea>@@AAV<lambda_ab61a845afdef5b7c387490eaf3616ee>@@$$QAV<lambda_c2ffc0b7726aa6be21d5f0026187e748>@@@Z 1002f3eb f   libucrt:fflush.obj
 0001:0002e497       ?common_flush_all@@YAH_N@Z 1002f497 f   libucrt:fflush.obj
 0001:0002e4e4       ?common_flush_all_should_try_to_flush_stream@@YA_NV__crt_stdio_stream@@QAH@Z 1002f4e4 f   libucrt:fflush.obj
 0001:0002e517       ?is_stream_flushable_or_commitable@@YA_NJ@Z 1002f517 f   libucrt:fflush.obj
 0001:0002e632       ?fperrraise_with@@YAXHK@Z  1002f632 f   libucrt:_test.obj
 0001:0002ea92       _no_op_initialize          1002fa92 f   libucrt:wsetlocale.obj
 0001:0002ea95       ??$?RV<lambda_135d2772fca65dc1248eeaa1b56e886a>@@AAV<lambda_2a444430fde8c29194d880d93eed5e8f>@@AAV<lambda_8dff2cf36a5417162780cd64fa2883ef>@@@?$__crt_seh_guarded_call@X@@QAEX$$QAV<lambda_135d2772fca65dc1248eeaa1b56e886a>@@AAV<lambda_2a444430fde8c29194d880d93eed5e8f>@@AAV<lambda_8dff2cf36a5417162780cd64fa2883ef>@@@Z 1002fa95 f   libucrt:wsetlocale.obj
 0001:0002eada       ??$?RV<lambda_4fdada1b837b2abbf20876fac97688ad>@@AAV<lambda_b57350f2640456a0859d250846f69caf>@@V<lambda_eed5e4f92b5b7d55fa22c48c484aaa54>@@@?$__crt_seh_guarded_call@X@@QAEX$$QAV<lambda_4fdada1b837b2abbf20876fac97688ad>@@AAV<lambda_b57350f2640456a0859d250846f69caf>@@$$QAV<lambda_eed5e4f92b5b7d55fa22c48c484aaa54>@@@Z 1002fada f   libucrt:wsetlocale.obj
 0001:0002eb27       ??$?RV<lambda_e5124f882df8998aaf41531e079ba474>@@AAV<lambda_3e16ef9562a7dcce91392c22ab16ea36>@@V<lambda_e25ca0880e6ef98be67edffd8c599615>@@@?$__crt_seh_guarded_call@X@@QAEX$$QAV<lambda_e5124f882df8998aaf41531e079ba474>@@AAV<lambda_3e16ef9562a7dcce91392c22ab16ea36>@@$$QAV<lambda_e25ca0880e6ef98be67edffd8c599615>@@@Z 1002fb27 f   libucrt:wsetlocale.obj
 0001:0002ec0f       ??R<lambda_2a444430fde8c29194d880d93eed5e8f>@@QBE@XZ 1002fc0f f   libucrt:wsetlocale.obj
 0001:0002ec79       ??R<lambda_b57350f2640456a0859d250846f69caf>@@QBEXXZ 1002fc79 f   libucrt:wsetlocale.obj
 0001:0002f042       __copytlocinfo_nolock      10030042 f   libucrt:wsetlocale.obj
 0001:0002f071       __expandlocale             10030071 f   libucrt:wsetlocale.obj
 0001:0002f4fb       __wsetlocale_get_all       100304fb f   libucrt:wsetlocale.obj
 0001:0002f696       __wsetlocale_nolock        10030696 f   libucrt:wsetlocale.obj
 0001:0002f986       __wsetlocale_set_cat       10030986 f   libucrt:wsetlocale.obj
 0001:0002fd4d       _get_default_code_page     10030d4d f   libucrt:wsetlocale.obj
 0001:0002fd7c       _parse_bcp47               10030d7c f   libucrt:wsetlocale.obj
 0001:0002ff66       _parse_bcp47_code_page     10030f66 f   libucrt:wsetlocale.obj
 0001:0002ffa5       _parse_bcp47_language      10030fa5 f   libucrt:wsetlocale.obj
 0001:00030017       _parse_bcp47_region        10031017 f   libucrt:wsetlocale.obj
 0001:000300d0       _parse_bcp47_script        100310d0 f   libucrt:wsetlocale.obj
 0001:00030140       _string_is_alpha           10031140 f   libucrt:wsetlocale.obj
 0001:0003017d       ?write_double_translated_ansi_nolock@@YA?AUwrite_result@?A0x17268360@@HQBDI@Z 1003117d f   libucrt:write.obj
 0001:00030527       ?write_double_translated_unicode_nolock@@YA?AUwrite_result@?A0x17268360@@QBDI@Z 10031527 f   libucrt:write.obj
 0001:0003058f       ?write_requires_double_translation_nolock@@YA_NH@Z 1003158f f   libucrt:write.obj
 0001:00030600       ?write_text_ansi_nolock@@YA?AUwrite_result@?A0x17268360@@HQBDI@Z 10031600 f   libucrt:write.obj
 0001:000306db       ?write_text_utf16le_nolock@@YA?AUwrite_result@?A0x17268360@@HQBDI@Z 100316db f   libucrt:write.obj
 0001:000307c4       ?write_text_utf8_nolock@@YA?AUwrite_result@?A0x17268360@@HQBDI@Z 100317c4 f   libucrt:write.obj
 0001:000310ac       ?_mbstowcs_l_helper@@YAIPA_WPBDIPAU__crt_locale_pointers@@@Z 100320ac f   libucrt:mbstowcs.obj
 0001:0003134f       ?_wcstombs_l_helper@@YAIPADPB_WIPAU__crt_locale_pointers@@@Z 1003234f f   libucrt:wcstombs.obj
 0001:000316c3       ?InternalGetLocaleInfoA@@YAHQAU__crt_locale_pointers@@QB_WKQADH@Z 100326c3 f   libucrt:getlocaleinfoa.obj
 0001:00031a55       ?__acrt_LCMapStringA_stat@@YAHPAU__crt_locale_pointers@@PB_WKPBDHPADHHH@Z 10032a55 f   libucrt:lcmapstringa.obj
 0001:00032690       $$000000                   10033690     libucrt:pow_pentium4.obj
 0001:000331b0       $$000000                   100341b0     libucrt:87tran.obj
 0001:000333c0       $$000000                   100343c0     libucrt:87disp.obj
 0001:00033620       $$000000                   10034620     libucrt:genexcep.obj
 0001:00033680       $$000000                   10034680     libucrt:common.obj
 0001:0003399f       ??$?RV<lambda_cbab9ec6f41b0180b23cc171c22676b0>@@AAV<lambda_44731a7d0e6d81c3e6aa82d741081786>@@V<lambda_4b292cb8dd18144e164572427af410ab>@@@?$__crt_seh_guarded_call@P6AXH@Z@@QAEP6AXH@Z$$QAV<lambda_cbab9ec6f41b0180b23cc171c22676b0>@@AAV<lambda_44731a7d0e6d81c3e6aa82d741081786>@@$$QAV<lambda_4b292cb8dd18144e164572427af410ab>@@@Z 1003499f f   libucrt:signal.obj
 0001:00033a03       ?get_global_action_nolock@@YAPAP6AXH@ZH@Z 10034a03 f   libucrt:signal.obj
 0001:00033a45       ?siglookup@@YAPAU__crt_signal_action_t@@HQAU1@@Z 10034a45 f   libucrt:signal.obj
 0001:0003401c       ?<lambda_invoker_cdecl>@<lambda_838c7f62c73c983481e27c09e84b0b5d>@@CAHPBX0@Z 1003501c f   libucrt:argv_wildcards.obj
 0001:00034034       ??$__acrt_convert_wcs_mbs_cp@_WDV<lambda_28bda7af82a03b66c1cb3803a755f95d>@@U__crt_win32_buffer_internal_dynamic_resizing@@@@YAHQB_WAAV?$__crt_win32_buffer@DU__crt_win32_buffer_internal_dynamic_resizing@@@@ABV<lambda_28bda7af82a03b66c1cb3803a755f95d>@@I@Z 10035034 f   libucrt:argv_wildcards.obj
 0001:00034103       ??$common_expand_argv_wildcards@D@@YAHQAPADQAPAPAD@Z 10035103 f   libucrt:argv_wildcards.obj
 0001:000342f2       ??$copy_and_add_argument_to_buffer@D@@YAHQBD0IAAV?$argument_list@D@?A0x5f5c8891@@@Z 100352f2 f   libucrt:argv_wildcards.obj
 0001:000343a3       ??$expand_argument_wildcards@D@@YAHQAD0AAV?$argument_list@D@?A0x5f5c8891@@@Z 100353a3 f   libucrt:argv_wildcards.obj
 0001:00034675       ?expand_if_necessary@?$argument_list@D@?A0x5f5c8891@@AAEHXZ 10035675 f   libucrt:argv_wildcards.obj
 0001:00034707       ??$__acrt_convert_wcs_mbs_cp@_WDV<lambda_0fec1a7b3f42a53036604e18c2d5e07e>@@U__crt_win32_buffer_no_resizing@@@@YAHQB_WAAV?$__crt_win32_buffer@DU__crt_win32_buffer_no_resizing@@@@ABV<lambda_0fec1a7b3f42a53036604e18c2d5e07e>@@I@Z 10035707 f   libucrt:getmodulefilenamea.obj
 0001:0003486f       ??$?RV<lambda_ceb1ee4838e85a9d631eb091e2fbe199>@@AAV<lambda_ae742caa10f662c28703da3d2ea5e57e>@@V<lambda_cd08b5d6af4937fe54fc07d0c9bf6b37>@@@?$__crt_seh_guarded_call@X@@QAEX$$QAV<lambda_ceb1ee4838e85a9d631eb091e2fbe199>@@AAV<lambda_ae742caa10f662c28703da3d2ea5e57e>@@$$QAV<lambda_cd08b5d6af4937fe54fc07d0c9bf6b37>@@@Z 1003586f f   libucrt:mbctype.obj
 0001:000348bc       ??R<lambda_ae742caa10f662c28703da3d2ea5e57e>@@QBEXXZ 100358bc f   libucrt:mbctype.obj
 0001:0003493f       ?CPtoLocaleName@@YAPB_WH@Z 1003593f f   libucrt:mbctype.obj
 0001:0003497d       ?getSystemCP@@YAHH@Z       1003597d f   libucrt:mbctype.obj
 0001:000349ee       ?setSBCS@@YAXPAU__crt_multibyte_data@@@Z 100359ee f   libucrt:mbctype.obj
 0001:00034a53       ?setSBUpLow@@YAXPAU__crt_multibyte_data@@@Z 10035a53 f   libucrt:mbctype.obj
 0001:00034bd4       ?setmbcp_internal@@YAHH_NQAU__acrt_ptd@@QAPAU__crt_multibyte_data@@@Z 10035bd4 f   libucrt:mbctype.obj
 0001:00034ced       ?update_thread_multibyte_data_internal@@YAPAU__crt_multibyte_data@@QAU__acrt_ptd@@QAPAU1@@Z 10035ced f   libucrt:mbctype.obj
 0001:00034fdb       _memcpy_s                  10035fdb f   libucrt:mbctype.obj
 0001:0003505c       ?x_ismbbtype_l@@YAHPAU__crt_locale_pointers@@IHH@Z 1003605c f   libucrt:ismbbyte.obj
 0001:000350e4       ?find_end_of_double_null_terminated_sequence@@YAPB_WQB_W@Z 100360e4 f   libucrt:get_environment_from_os.obj
 0001:000356b3       ??$common_lseek_nolock@_J@@YA_JH_JH@Z 100366b3 f   libucrt:lseek.obj
 0001:000357c6       ?GetTableIndexFromLocaleName@@YAHPB_W@Z 100367c6 f   libucrt:lcidtoname_downlevel.obj
 0001:000359e7       ??$?RV<lambda_9e9de3de5fa147e2223d7db92bc10aa6>@@AAV<lambda_38ce7e780aa69e748d6df282ebc68efe>@@V<lambda_8ca6da459f0f6780f1cff60fdc3d00e5>@@@?$__crt_seh_guarded_call@H@@QAEH$$QAV<lambda_9e9de3de5fa147e2223d7db92bc10aa6>@@AAV<lambda_38ce7e780aa69e748d6df282ebc68efe>@@$$QAV<lambda_8ca6da459f0f6780f1cff60fdc3d00e5>@@@Z 100369e7 f   libucrt:commit.obj
 0001:00035d59       ??R<lambda_3d301b9e52f5099be73030e1f0bf487e>@@QBEIPBD@Z 10036d59 f   libucrt:mbrtowc.obj
 0001:000366c2       ?free_crt_array_internal@@YAXQAPBXI@Z 100376c2 f   libucrt:inittime.obj
 0001:000366fa       ?initialize_lc_time@@YA_NQAU__crt_lc_time_data@@QAU__crt_locale_data@@@Z 100376fa f   libucrt:inittime.obj
 0001:00036ad5       ??$common_tcsncat_s@_W@@YAHQA_WIQB_WI@Z 10037ad5 f   libucrt:wcsncat_s.obj
 0001:00036bc7       _GetLocaleNameFromDefault  10037bc7 f   libucrt:get_qualified_locale.obj
 0001:00036c4e       _GetLocaleNameFromLangCountry 10037c4e f   libucrt:get_qualified_locale.obj
 0001:00036ce7       _GetLocaleNameFromLanguage 10037ce7 f   libucrt:get_qualified_locale.obj
 0001:00036d40       _GetPrimaryLen             10037d40 f   libucrt:get_qualified_locale.obj
 0001:00036d74       _LangCountryEnumProcEx@12  10037d74 f   libucrt:get_qualified_locale.obj
 0001:00037054       _LanguageEnumProcEx@12     10038054 f   libucrt:get_qualified_locale.obj
 0001:00037113       _ProcessCodePage           10038113 f   libucrt:get_qualified_locale.obj
 0001:00037209       _TestDefaultCountry        10038209 f   libucrt:get_qualified_locale.obj
 0001:00037256       _TranslateName             10038256 f   libucrt:get_qualified_locale.obj
 0001:000374be       _CountryEnumProc@4         100384be f   libucrt:getqloc_downlevel.obj
 0001:00037565       _GetLcidFromCountry        10038565 f   libucrt:getqloc_downlevel.obj
 0001:000375b0       _GetLcidFromLangCountry    100385b0 f   libucrt:getqloc_downlevel.obj
 0001:0003764b       _GetLcidFromLanguage       1003864b f   libucrt:getqloc_downlevel.obj
 0001:000376aa       _GetPrimaryLen             100386aa f   libucrt:getqloc_downlevel.obj
 0001:000376d6       _LangCountryEnumProc@4     100386d6 f   libucrt:getqloc_downlevel.obj
 0001:00037929       _LanguageEnumProc@4        10038929 f   libucrt:getqloc_downlevel.obj
 0001:000379fe       _LcidFromHexString         100389fe f   libucrt:getqloc_downlevel.obj
 0001:00037a4f       _ProcessCodePage           10038a4f f   libucrt:getqloc_downlevel.obj
 0001:00037b30       _TestDefaultCountry        10038b30 f   libucrt:getqloc_downlevel.obj
 0001:00037b55       _TestDefaultLanguage       10038b55 f   libucrt:getqloc_downlevel.obj
 0001:00037bc3       _TranslateName             10038bc3 f   libucrt:getqloc_downlevel.obj
 0001:0003810b       ??$common_tcsncpy_s@D@@YAHQADIQBDI@Z 1003910b f   libucrt:strncpy_s.obj
 0001:00038380       ?swap@@YAXPAD0I@Z          10039380 f   libucrt:qsort.obj
 0001:00038810       $$000000                   10039810     libucrt:strpbrk.obj
 0001:000388f4       ?initialize_multibyte@@YAHXZ 100398f4 f   libucrt:multibyte_initializer.obj
 0001:00038aa4       ??$?RV<lambda_218ce3db14220d0be481dae8ef3383b6>@@AAV<lambda_628dfdc04ba53c8bfc02c9951375f3f5>@@V<lambda_57dc472bd5c9d5f3b2cbca59b8a843ae>@@@?$__crt_seh_guarded_call@H@@QAEH$$QAV<lambda_218ce3db14220d0be481dae8ef3383b6>@@AAV<lambda_628dfdc04ba53c8bfc02c9951375f3f5>@@$$QAV<lambda_57dc472bd5c9d5f3b2cbca59b8a843ae>@@@Z 10039aa4 f   libucrt:close.obj
 0001:00038e60       $$000000                   10039e60     libucrt:log10_impl.obj
 0001:00038f70       $$000000                   10039f70     libucrt:ceil_pentium4.obj
 0001:0003908d       ??$common_xtox@K_W@@YAHKQA_WII_N@Z 1003a08d f   libucrt:xtoa.obj
 0001:00039140       ??$common_xtox_s@K_W@@YAHKQA_WII_N@Z 1003a140 f   libucrt:xtoa.obj
 0001:000391e5       ?__dcrt_lowio_initialize_console_output@@YAXXZ 1003a1e5 f   libucrt:initcon.obj
 0001:00039370       $$000000                   1003a370     libucrt:log10_pentium4.obj
 0001:000396c0       $$000000                   1003a6c0     libucrt:_strnicm.obj
 0001:00039880       $$000000                   1003a880     LIBCMT:ulldvrm.obj
 0001:000398b1       L1                         1003a8b1     LIBCMT:ulldvrm.obj
 0001:000398bf       L3                         1003a8bf     LIBCMT:ulldvrm.obj
 0001:000398ed       L4                         1003a8ed     LIBCMT:ulldvrm.obj
 0001:000398f6       L5                         1003a8f6     LIBCMT:ulldvrm.obj
 0001:000398f8       L2                         1003a8f8     LIBCMT:ulldvrm.obj
 0001:00039920       $$000000                   1003a920     LIBCMT:llshl.obj
 0001:00039930       MORE32                     1003a930     LIBCMT:llshl.obj
 0001:0003993a       RETZERO                    1003a93a     LIBCMT:llshl.obj
 0001:00039940       $$000000                   1003a940     LIBCMT:ullshr.obj
 0001:00039950       MORE32                     1003a950     LIBCMT:ullshr.obj
 0001:0003995a       RETZERO                    1003a95a     LIBCMT:ullshr.obj
 0001:00039960       $$000000                   1003a960     LIBCMT:ftol2.obj
 0001:00039970       $$000000                   1003a970     LIBCMT:ftol2.obj
 0001:00039981       L3B                        1003a981     LIBCMT:ftol2.obj
 0001:000399c4       L3F                        1003a9c4     LIBCMT:ftol2.obj
 0001:000399cc       L40                        1003a9cc     LIBCMT:ftol2.obj
 0001:000399df       L41                        1003a9df     LIBCMT:ftol2.obj
 0001:000399f0       $$000000                   1003a9f0     LIBCMT:ftol2.obj
 0001:00039a0e       L51                        1003aa0e     LIBCMT:ftol2.obj
 0001:00039a53       L52                        1003aa53     LIBCMT:ftol2.obj
 0001:00039a67       L53                        1003aa67     LIBCMT:ftol2.obj
 0001:00039a69       L55                        1003aa69     LIBCMT:ftol2.obj
 0001:00039a73       L56                        1003aa73     LIBCMT:ftol2.obj
 0001:00039a8c       L57                        1003aa8c     LIBCMT:ftol2.obj
 0001:00039b20       $$000000                   1003ab20     LIBCMT:lldiv.obj
 0001:00039b41       L1                         1003ab41     LIBCMT:lldiv.obj
 0001:00039b5d       L2                         1003ab5d     LIBCMT:lldiv.obj
 0001:00039b79       L3                         1003ab79     LIBCMT:lldiv.obj
 0001:00039b87       L5                         1003ab87     LIBCMT:lldiv.obj
 0001:00039bb5       L6                         1003abb5     LIBCMT:lldiv.obj
 0001:00039bb6       L7                         1003abb6     LIBCMT:lldiv.obj
 0001:00039bba       L4                         1003abba     LIBCMT:lldiv.obj
 0001:00039bc4       L8                         1003abc4     LIBCMT:lldiv.obj
 0001:00039bf0       __unwindfunclet$?adjust_precision@detail@v10@fmt@@YAXAAHH@Z$0 1003abf0 f   format.obj
 0001:00039bfd       __ehhandler$?adjust_precision@detail@v10@fmt@@YAXAAHH@Z 1003abfd f   format.obj
 0001:00039c20       __unwindfunclet$?square@bigint@detail@v10@fmt@@QAEXXZ$0 1003ac20 f   format.obj
 0001:00039c30       __ehhandler$?square@bigint@detail@v10@fmt@@QAEXXZ 1003ac30 f   format.obj
 0001:00039c60       __unwindfunclet$?format_dragon@detail@v10@fmt@@YAXU?$basic_fp@Vuint128_fallback@detail@v10@fmt@@@123@IHAAV?$buffer@D@123@AAH@Z$0 1003ac60 f   format.obj
 0001:00039c6b       __unwindfunclet$?format_dragon@detail@v10@fmt@@YAXU?$basic_fp@Vuint128_fallback@detail@v10@fmt@@@123@IHAAV?$buffer@D@123@AAH@Z$1 1003ac6b f   format.obj
 0001:00039c76       __unwindfunclet$?format_dragon@detail@v10@fmt@@YAXU?$basic_fp@Vuint128_fallback@detail@v10@fmt@@@123@IHAAV?$buffer@D@123@AAH@Z$2 1003ac76 f   format.obj
 0001:00039c81       __unwindfunclet$?format_dragon@detail@v10@fmt@@YAXU?$basic_fp@Vuint128_fallback@detail@v10@fmt@@@123@IHAAV?$buffer@D@123@AAH@Z$3 1003ac81 f   format.obj
 0001:00039c91       __ehhandler$?format_dragon@detail@v10@fmt@@YAXU?$basic_fp@Vuint128_fallback@detail@v10@fmt@@@123@IHAAV?$buffer@D@123@AAH@Z 1003ac91 f   format.obj
 0001:00039cc0       __unwindfunclet$??0_Locinfo@std@@QAE@PBD@Z$0 1003acc0 f   format.obj
 0001:00039cc8       __unwindfunclet$??0_Locinfo@std@@QAE@PBD@Z$1 1003acc8 f   format.obj
 0001:00039cd3       __unwindfunclet$??0_Locinfo@std@@QAE@PBD@Z$2 1003acd3 f   format.obj
 0001:00039cde       __unwindfunclet$??0_Locinfo@std@@QAE@PBD@Z$3 1003acde f   format.obj
 0001:00039ce9       __unwindfunclet$??0_Locinfo@std@@QAE@PBD@Z$4 1003ace9 f   format.obj
 0001:00039cf4       __unwindfunclet$??0_Locinfo@std@@QAE@PBD@Z$5 1003acf4 f   format.obj
 0001:00039cff       __unwindfunclet$??0_Locinfo@std@@QAE@PBD@Z$6 1003acff f   format.obj
 0001:00039d0f       __ehhandler$??0_Locinfo@std@@QAE@PBD@Z 1003ad0f f   format.obj
 0001:00039d30       __ehhandler$??1_Locinfo@std@@QAE@XZ 1003ad30 f   format.obj
 0001:00039d30       __ehhandler$??1WMIConnection@@QAE@XZ 1003ad30 f   wmi.obj
 0001:00039d30       __ehhandler$??1_Init_atexit@@QAE@XZ 1003ad30 f   libcpmt:iosptrs.obj
 0001:00039d50       __unwindfunclet$?throw_format_error@detail@v10@fmt@@YAXPBD@Z$0 1003ad50 f   format.obj
 0001:00039d5d       __ehhandler$?throw_format_error@detail@v10@fmt@@YAXPBD@Z 1003ad5d f   format.obj
 0001:00039d80       __ehhandler$??0?$basic_string@_WU?$char_traits@_W@std@@V?$allocator@_W@2@@std@@QAE@QB_W@Z 1003ad80 f   format.obj
 0001:00039d80       __ehhandler$?do_falsename@?$numpunct@_W@std@@MBE?AV?$basic_string@_WU?$char_traits@_W@std@@V?$allocator@_W@2@@2@XZ 1003ad80 f   format.obj
 0001:00039d80       __ehhandler$?do_grouping@?$numpunct@_W@std@@MBE?AV?$basic_string@DU?$char_traits@D@std@@V?$allocator@D@2@@2@XZ 1003ad80 f   format.obj
 0001:00039d80       __ehhandler$?do_truename@?$numpunct@_W@std@@MBE?AV?$basic_string@_WU?$char_traits@_W@std@@V?$allocator@_W@2@@2@XZ 1003ad80 f   format.obj
 0001:00039d80       __ehhandler$??$?0V?$basic_string_view@_WU?$char_traits@_W@std@@@std@@$0A@@?$basic_string@_WU?$char_traits@_W@std@@V?$allocator@_W@2@@std@@QAE@ABV?$basic_string_view@_WU?$char_traits@_W@std@@@1@ABV?$allocator@_W@1@@Z 1003ad80 f   handles.obj
 0001:00039d80       __ehhandler$??__Ks@string_literals@literals@std@@YA?AV?$basic_string@_WU?$char_traits@_W@std@@V?$allocator@_W@2@@3@PB_WI@Z 1003ad80 f   handles.obj
 0001:00039da0       __unwindfunclet$??$use_facet@V?$numpunct@_W@std@@@std@@YAABV?$numpunct@_W@0@ABVlocale@0@@Z$0 1003ada0 f   format.obj
 0001:00039da8       __unwindfunclet$??$use_facet@V?$numpunct@_W@std@@@std@@YAABV?$numpunct@_W@0@ABVlocale@0@@Z$2 1003ada8 f   format.obj
 0001:00039db7       __unwindfunclet$??$use_facet@V?$numpunct@_W@std@@@std@@YAABV?$numpunct@_W@0@ABVlocale@0@@Z$3 1003adb7 f   format.obj
 0001:00039dd3       __unwindfunclet$??$use_facet@V?$numpunct@_W@std@@@std@@YAABV?$numpunct@_W@0@ABVlocale@0@@Z$4 1003add3 f   format.obj
 0001:00039ddb       __unwindfunclet$??$use_facet@V?$numpunct@_W@std@@@std@@YAABV?$numpunct@_W@0@ABVlocale@0@@Z$5 1003addb f   format.obj
 0001:00039de3       __unwindfunclet$??$use_facet@V?$numpunct@_W@std@@@std@@YAABV?$numpunct@_W@0@ABVlocale@0@@Z$1 1003ade3 f   format.obj
 0001:00039df0       __ehhandler$??$use_facet@V?$numpunct@_W@std@@@std@@YAABV?$numpunct@_W@0@ABVlocale@0@@Z 1003adf0 f   format.obj
 0001:00039e20       __unwindfunclet$??$decimal_point@_W@detail@v10@fmt@@YA_WVlocale_ref@012@@Z$0 1003ae20 f   handles.obj
 0001:00039e2d       __ehhandler$??$decimal_point@_W@detail@v10@fmt@@YA_WVlocale_ref@012@@Z 1003ae2d f   handles.obj
 0001:00039e50       __unwindfunclet$?write_loc@detail@v10@fmt@@YA_NV?$back_insert_iterator@V?$buffer@_W@detail@v10@fmt@@@std@@Vloc_value@23@ABU?$format_specs@_W@23@Vlocale_ref@123@@Z$0 1003ae50 f   handles.obj
 0001:00039e5b       __unwindfunclet$?write_loc@detail@v10@fmt@@YA_NV?$back_insert_iterator@V?$buffer@_W@detail@v10@fmt@@@std@@Vloc_value@23@ABU?$format_specs@_W@23@Vlocale_ref@123@@Z$1 1003ae5b f   handles.obj
 0001:00039e63       __unwindfunclet$?write_loc@detail@v10@fmt@@YA_NV?$back_insert_iterator@V?$buffer@_W@detail@v10@fmt@@@std@@Vloc_value@23@ABU?$format_specs@_W@23@Vlocale_ref@123@@Z$2 1003ae63 f   handles.obj
 0001:00039e6b       __unwindfunclet$?write_loc@detail@v10@fmt@@YA_NV?$back_insert_iterator@V?$buffer@_W@detail@v10@fmt@@@std@@Vloc_value@23@ABU?$format_specs@_W@23@Vlocale_ref@123@@Z$4 1003ae6b f   handles.obj
 0001:00039e76       __unwindfunclet$?write_loc@detail@v10@fmt@@YA_NV?$back_insert_iterator@V?$buffer@_W@detail@v10@fmt@@@std@@Vloc_value@23@ABU?$format_specs@_W@23@Vlocale_ref@123@@Z$7 1003ae76 f   handles.obj
 0001:00039e86       __ehhandler$?write_loc@detail@v10@fmt@@YA_NV?$back_insert_iterator@V?$buffer@_W@detail@v10@fmt@@@std@@Vloc_value@23@ABU?$format_specs@_W@23@Vlocale_ref@123@@Z 1003ae86 f   handles.obj
 0001:00039eb0       __unwindfunclet$?query_object@@YA?AV?$unique_ptr@$$BY0A@DU?$default_delete@$$BY0A@D@std@@@std@@PAXW4_OBJECT_INFORMATION_CLASS@@@Z$0 1003aeb0 f   handles.obj
 0001:00039ebd       __ehhandler$?query_object@@YA?AV?$unique_ptr@$$BY0A@DU?$default_delete@$$BY0A@D@std@@@std@@PAXW4_OBJECT_INFORMATION_CLASS@@@Z 1003aebd f   handles.obj
 0001:00039ee0       __unwindfunclet$?GetFileName@@YA?AV?$basic_string@_WU?$char_traits@_W@std@@V?$allocator@_W@2@@std@@PAX@Z$0 1003aee0 f   handles.obj
 0001:00039ee8       __unwindfunclet$?GetFileName@@YA?AV?$basic_string@_WU?$char_traits@_W@std@@V?$allocator@_W@2@@std@@PAX@Z$2 1003aee8 f   handles.obj
 0001:00039ef5       __ehhandler$?GetFileName@@YA?AV?$basic_string@_WU?$char_traits@_W@std@@V?$allocator@_W@2@@std@@PAX@Z 1003aef5 f   handles.obj
 0001:00039f20       __unwindfunclet$??R<lambda_1>@?1??GetUserAccountID@@YA@XZ@QBE?AV?$basic_string@_WU?$char_traits@_W@std@@V?$allocator@_W@2@@std@@XZ$1 1003af20 f   handles.obj
 0001:00039f2b       __unwindfunclet$??R<lambda_1>@?1??GetUserAccountID@@YA@XZ@QBE?AV?$basic_string@_WU?$char_traits@_W@std@@V?$allocator@_W@2@@std@@XZ$2 1003af2b f   handles.obj
 0001:00039f36       __unwindfunclet$??R<lambda_1>@?1??GetUserAccountID@@YA@XZ@QBE?AV?$basic_string@_WU?$char_traits@_W@std@@V?$allocator@_W@2@@std@@XZ$3 1003af36 f   handles.obj
 0001:00039f46       __ehhandler$??R<lambda_1>@?1??GetUserAccountID@@YA@XZ@QBE?AV?$basic_string@_WU?$char_traits@_W@std@@V?$allocator@_W@2@@std@@XZ 1003af46 f   handles.obj
 0001:00039f70       __unwindfunclet$?GetNameByType@@YA?AV?$basic_string@_WU?$char_traits@_W@std@@V?$allocator@_W@2@@std@@PAXGPAVPerfThread@@@Z$1 1003af70 f   handles.obj
 0001:00039f7b       __unwindfunclet$?GetNameByType@@YA?AV?$basic_string@_WU?$char_traits@_W@std@@V?$allocator@_W@2@@std@@PAXGPAVPerfThread@@@Z$2 1003af7b f   handles.obj
 0001:00039f86       __unwindfunclet$?GetNameByType@@YA?AV?$basic_string@_WU?$char_traits@_W@std@@V?$allocator@_W@2@@std@@PAXGPAVPerfThread@@@Z$25 1003af86 f   handles.obj
 0001:00039f94       __unwindfunclet$?GetNameByType@@YA?AV?$basic_string@_WU?$char_traits@_W@std@@V?$allocator@_W@2@@std@@PAXGPAVPerfThread@@@Z$3 1003af94 f   handles.obj
 0001:00039fa1       __ehhandler$?GetNameByType@@YA?AV?$basic_string@_WU?$char_traits@_W@std@@V?$allocator@_W@2@@std@@PAXGPAVPerfThread@@@Z 1003afa1 f   handles.obj
 0001:00039fd0       __unwindfunclet$?PrintHandleInfo@@YA_NKPAX_NPAVPerfThread@@@Z$0 1003afd0 f   handles.obj
 0001:00039fd8       __unwindfunclet$?PrintHandleInfo@@YA_NKPAX_NPAVPerfThread@@@Z$3 1003afd8 f   handles.obj
 0001:00039fe0       __unwindfunclet$?PrintHandleInfo@@YA_NKPAX_NPAVPerfThread@@@Z$10 1003afe0 f   handles.obj
 0001:00039feb       __unwindfunclet$?PrintHandleInfo@@YA_NKPAX_NPAVPerfThread@@@Z$5 1003afeb f   handles.obj
 0001:00039ff3       __unwindfunclet$?PrintHandleInfo@@YA_NKPAX_NPAVPerfThread@@@Z$6 1003aff3 f   handles.obj
 0001:0003a000       __ehhandler$?PrintHandleInfo@@YA_NKPAX_NPAVPerfThread@@@Z 1003b000 f   handles.obj
 0001:0003a030       __ehhandler$??4?$basic_string@_WU?$char_traits@_W@std@@V?$allocator@_W@2@@std@@QAEAAV01@$$QAV01@@Z 1003b030 f   handles.obj
 0001:0003a050       __ehhandler$??0?$basic_string@_WU?$char_traits@_W@std@@V?$allocator@_W@2@@std@@QAE@$$QAV01@@Z 1003b050 f   handles.obj
 0001:0003a070       __ehhandler$??0?$basic_string@_WU?$char_traits@_W@std@@V?$allocator@_W@2@@std@@QAE@XZ 1003b070 f   handles.obj
 0001:0003a070       __ehhandler$??1?$ptr_setter@V?$unique_ptr@UIWbemClassObject@@Ucom_closer@@@std@@@@QAE@XZ 1003b070 f   wmi.obj
 0001:0003a090       __unwindfunclet$??$vformat@_W$0A@@v10@fmt@@YA?AV?$basic_string@_WU?$char_traits@_W@std@@V?$allocator@_W@2@@std@@V?$basic_string_view@_W@01@V?$basic_format_args@V?$basic_format_context@V?$back_insert_iterator@V?$buffer@_W@detail@v10@fmt@@@std@@_W@v10@fmt@@@01@@Z$0 1003b090 f   handles.obj
 0001:0003a0a0       __ehhandler$??$vformat@_W$0A@@v10@fmt@@YA?AV?$basic_string@_WU?$char_traits@_W@std@@V?$allocator@_W@2@@std@@V?$basic_string_view@_W@01@V?$basic_format_args@V?$basic_format_context@V?$back_insert_iterator@V?$buffer@_W@detail@v10@fmt@@@std@@_W@v10@fmt@@@01@@Z 1003b0a0 f   handles.obj
 0001:0003a0d0       __unwindfunclet$??$visit_format_arg@AAU?$loc_writer@_W@detail@v10@fmt@@V?$basic_format_context@Vappender@v10@fmt@@D@34@@v10@fmt@@YA_NAAU?$loc_writer@_W@detail@01@ABV?$basic_format_arg@V?$basic_format_context@Vappender@v10@fmt@@D@v10@fmt@@@01@@Z$0 1003b0d0 f   handles.obj
 0001:0003a0d8       __unwindfunclet$??$visit_format_arg@AAU?$loc_writer@_W@detail@v10@fmt@@V?$basic_format_context@Vappender@v10@fmt@@D@34@@v10@fmt@@YA_NAAU?$loc_writer@_W@detail@01@ABV?$basic_format_arg@V?$basic_format_context@Vappender@v10@fmt@@D@v10@fmt@@@01@@Z$2 1003b0d8 f   handles.obj
 0001:0003a0e0       __unwindfunclet$??$visit_format_arg@AAU?$loc_writer@_W@detail@v10@fmt@@V?$basic_format_context@Vappender@v10@fmt@@D@34@@v10@fmt@@YA_NAAU?$loc_writer@_W@detail@01@ABV?$basic_format_arg@V?$basic_format_context@Vappender@v10@fmt@@D@v10@fmt@@@01@@Z$18 1003b0e0 f   handles.obj
 0001:0003a0e8       __unwindfunclet$??$visit_format_arg@AAU?$loc_writer@_W@detail@v10@fmt@@V?$basic_format_context@Vappender@v10@fmt@@D@34@@v10@fmt@@YA_NAAU?$loc_writer@_W@detail@01@ABV?$basic_format_arg@V?$basic_format_context@Vappender@v10@fmt@@D@v10@fmt@@@01@@Z$20 1003b0e8 f   handles.obj
 0001:0003a0f0       __unwindfunclet$??$visit_format_arg@AAU?$loc_writer@_W@detail@v10@fmt@@V?$basic_format_context@Vappender@v10@fmt@@D@34@@v10@fmt@@YA_NAAU?$loc_writer@_W@detail@01@ABV?$basic_format_arg@V?$basic_format_context@Vappender@v10@fmt@@D@v10@fmt@@@01@@Z$33 1003b0f0 f   handles.obj
 0001:0003a0fb       __unwindfunclet$??$visit_format_arg@AAU?$loc_writer@_W@detail@v10@fmt@@V?$basic_format_context@Vappender@v10@fmt@@D@34@@v10@fmt@@YA_NAAU?$loc_writer@_W@detail@01@ABV?$basic_format_arg@V?$basic_format_context@Vappender@v10@fmt@@D@v10@fmt@@@01@@Z$35 1003b0fb f   handles.obj
 0001:0003a103       __unwindfunclet$??$visit_format_arg@AAU?$loc_writer@_W@detail@v10@fmt@@V?$basic_format_context@Vappender@v10@fmt@@D@34@@v10@fmt@@YA_NAAU?$loc_writer@_W@detail@01@ABV?$basic_format_arg@V?$basic_format_context@Vappender@v10@fmt@@D@v10@fmt@@@01@@Z$36 1003b103 f   handles.obj
 0001:0003a10e       __unwindfunclet$??$visit_format_arg@AAU?$loc_writer@_W@detail@v10@fmt@@V?$basic_format_context@Vappender@v10@fmt@@D@34@@v10@fmt@@YA_NAAU?$loc_writer@_W@detail@01@ABV?$basic_format_arg@V?$basic_format_context@Vappender@v10@fmt@@D@v10@fmt@@@01@@Z$38 1003b10e f   handles.obj
 0001:0003a11e       __ehhandler$??$visit_format_arg@AAU?$loc_writer@_W@detail@v10@fmt@@V?$basic_format_context@Vappender@v10@fmt@@D@34@@v10@fmt@@YA_NAAU?$loc_writer@_W@detail@01@ABV?$basic_format_arg@V?$basic_format_context@Vappender@v10@fmt@@D@v10@fmt@@@01@@Z 1003b11e f   handles.obj
 0001:0003a150       __unwindfunclet$??$parse_format_string@$0A@_WUformat_handler@?1???$vformat_to@_W@detail@v10@fmt@@YAXAAV?$buffer@_W@234@V?$basic_string_view@_W@34@V?$basic_format_args@V?$basic_format_context@V?$back_insert_iterator@V?$buffer@_W@detail@v10@fmt@@@std@@_W@v10@fmt@@@34@Vlocale_ref@234@@Z@@detail@v10@fmt@@YAXV?$basic_string_view@_W@12@$$QAUformat_handler@?1???$vformat_to@_W@012@YAXAAV?$buffer@_W@012@0V?$basic_format_args@V?$basic_format_context@V?$back_insert_iterator@V?$buffer@_W@detail@v10@fmt@@@std@@_W@v10@fmt@@@12@Vlocale_ref@012@@Z@@Z$0 1003b150 f   handles.obj
 0001:0003a15d       __ehhandler$??$parse_format_string@$0A@_WUformat_handler@?1???$vformat_to@_W@detail@v10@fmt@@YAXAAV?$buffer@_W@234@V?$basic_string_view@_W@34@V?$basic_format_args@V?$basic_format_context@V?$back_insert_iterator@V?$buffer@_W@detail@v10@fmt@@@std@@_W@v10@fmt@@@34@Vlocale_ref@234@@Z@@detail@v10@fmt@@YAXV?$basic_string_view@_W@12@$$QAUformat_handler@?1???$vformat_to@_W@012@YAXAAV?$buffer@_W@012@0V?$basic_format_args@V?$basic_format_context@V?$back_insert_iterator@V?$buffer@_W@detail@v10@fmt@@@std@@_W@v10@fmt@@@12@Vlocale_ref@012@@Z@@Z 1003b15d f   handles.obj
 0001:0003a180       __ehhandler$??0?$digit_grouping@_W@detail@v10@fmt@@QAE@V?$basic_string@DU?$char_traits@D@std@@V?$allocator@D@2@@std@@V?$basic_string@_WU?$char_traits@_W@std@@V?$allocator@_W@2@@5@@Z 1003b180 f   handles.obj
 0001:0003a1a0       __unwindfunclet$??$apply@V?$back_insert_iterator@V?$buffer@_W@detail@v10@fmt@@@std@@D@?$digit_grouping@_W@detail@v10@fmt@@QBE?AV?$back_insert_iterator@V?$buffer@_W@detail@v10@fmt@@@std@@V45@V?$basic_string_view@D@23@@Z$0 1003b1a0 f   handles.obj
 0001:0003a1a0       __unwindfunclet$??$apply@V?$back_insert_iterator@V?$buffer@_W@detail@v10@fmt@@@std@@_W@?$digit_grouping@_W@detail@v10@fmt@@QBE?AV?$back_insert_iterator@V?$buffer@_W@detail@v10@fmt@@@std@@V45@V?$basic_string_view@_W@23@@Z$0 1003b1a0 f   handles.obj
 0001:0003a1b0       __ehhandler$??$apply@V?$back_insert_iterator@V?$buffer@_W@detail@v10@fmt@@@std@@D@?$digit_grouping@_W@detail@v10@fmt@@QBE?AV?$back_insert_iterator@V?$buffer@_W@detail@v10@fmt@@@std@@V45@V?$basic_string_view@D@23@@Z 1003b1b0 f   handles.obj
 0001:0003a1b0       __ehhandler$??$apply@V?$back_insert_iterator@V?$buffer@_W@detail@v10@fmt@@@std@@_W@?$digit_grouping@_W@detail@v10@fmt@@QBE?AV?$back_insert_iterator@V?$buffer@_W@detail@v10@fmt@@@std@@V45@V?$basic_string_view@_W@23@@Z 1003b1b0 f   handles.obj
 0001:0003a1e0       __unwindfunclet$??$write_float@_WV?$back_insert_iterator@V?$buffer@_W@detail@v10@fmt@@@std@@M@detail@v10@fmt@@YA?AV?$back_insert_iterator@V?$buffer@_W@detail@v10@fmt@@@std@@V34@MU?$format_specs@_W@12@Vlocale_ref@012@@Z$0 1003b1e0 f   handles.obj
 0001:0003a1f0       __ehhandler$??$write_float@_WV?$back_insert_iterator@V?$buffer@_W@detail@v10@fmt@@@std@@M@detail@v10@fmt@@YA?AV?$back_insert_iterator@V?$buffer@_W@detail@v10@fmt@@@std@@V34@MU?$format_specs@_W@12@Vlocale_ref@012@@Z 1003b1f0 f   handles.obj
 0001:0003a220       __unwindfunclet$??$write_float@_WV?$back_insert_iterator@V?$buffer@_W@detail@v10@fmt@@@std@@N@detail@v10@fmt@@YA?AV?$back_insert_iterator@V?$buffer@_W@detail@v10@fmt@@@std@@V34@NU?$format_specs@_W@12@Vlocale_ref@012@@Z$0 1003b220 f   handles.obj
 0001:0003a220       __unwindfunclet$??$write_float@_WV?$back_insert_iterator@V?$buffer@_W@detail@v10@fmt@@@std@@O@detail@v10@fmt@@YA?AV?$back_insert_iterator@V?$buffer@_W@detail@v10@fmt@@@std@@V34@OU?$format_specs@_W@12@Vlocale_ref@012@@Z$0 1003b220 f   handles.obj
 0001:0003a230       __ehhandler$??$write_float@_WV?$back_insert_iterator@V?$buffer@_W@detail@v10@fmt@@@std@@N@detail@v10@fmt@@YA?AV?$back_insert_iterator@V?$buffer@_W@detail@v10@fmt@@@std@@V34@NU?$format_specs@_W@12@Vlocale_ref@012@@Z 1003b230 f   handles.obj
 0001:0003a230       __ehhandler$??$write_float@_WV?$back_insert_iterator@V?$buffer@_W@detail@v10@fmt@@@std@@O@detail@v10@fmt@@YA?AV?$back_insert_iterator@V?$buffer@_W@detail@v10@fmt@@@std@@V34@OU?$format_specs@_W@12@Vlocale_ref@012@@Z 1003b230 f   handles.obj
 0001:0003a260       __unwindfunclet$??$do_write_float@V?$back_insert_iterator@V?$buffer@_W@detail@v10@fmt@@@std@@U?$decimal_fp@M@dragonbox@detail@v10@fmt@@_WV?$digit_grouping@_W@567@@detail@v10@fmt@@YA?AV?$back_insert_iterator@V?$buffer@_W@detail@v10@fmt@@@std@@V34@ABU?$decimal_fp@M@dragonbox@012@ABU?$format_specs@_W@12@Ufloat_specs@012@Vlocale_ref@012@@Z$0 1003b260 f   handles.obj
 0001:0003a260       __unwindfunclet$??$do_write_float@V?$back_insert_iterator@V?$buffer@_W@detail@v10@fmt@@@std@@Ubig_decimal_fp@detail@v10@fmt@@_WV?$digit_grouping@_W@456@@detail@v10@fmt@@YA?AV?$back_insert_iterator@V?$buffer@_W@detail@v10@fmt@@@std@@V34@ABUbig_decimal_fp@012@ABU?$format_specs@_W@12@Ufloat_specs@012@Vlocale_ref@012@@Z$0 1003b260 f   handles.obj
 0001:0003a268       __unwindfunclet$??$do_write_float@V?$back_insert_iterator@V?$buffer@_W@detail@v10@fmt@@@std@@U?$decimal_fp@M@dragonbox@detail@v10@fmt@@_WV?$digit_grouping@_W@567@@detail@v10@fmt@@YA?AV?$back_insert_iterator@V?$buffer@_W@detail@v10@fmt@@@std@@V34@ABU?$decimal_fp@M@dragonbox@012@ABU?$format_specs@_W@12@Ufloat_specs@012@Vlocale_ref@012@@Z$1 1003b268 f   handles.obj
 0001:0003a268       __unwindfunclet$??$do_write_float@V?$back_insert_iterator@V?$buffer@_W@detail@v10@fmt@@@std@@Ubig_decimal_fp@detail@v10@fmt@@_WV?$digit_grouping@_W@456@@detail@v10@fmt@@YA?AV?$back_insert_iterator@V?$buffer@_W@detail@v10@fmt@@@std@@V34@ABUbig_decimal_fp@012@ABU?$format_specs@_W@12@Ufloat_specs@012@Vlocale_ref@012@@Z$1 1003b268 f   handles.obj
 0001:0003a275       __ehhandler$??$do_write_float@V?$back_insert_iterator@V?$buffer@_W@detail@v10@fmt@@@std@@U?$decimal_fp@M@dragonbox@detail@v10@fmt@@_WV?$digit_grouping@_W@567@@detail@v10@fmt@@YA?AV?$back_insert_iterator@V?$buffer@_W@detail@v10@fmt@@@std@@V34@ABU?$decimal_fp@M@dragonbox@012@ABU?$format_specs@_W@12@Ufloat_specs@012@Vlocale_ref@012@@Z 1003b275 f   handles.obj
 0001:0003a275       __ehhandler$??$do_write_float@V?$back_insert_iterator@V?$buffer@_W@detail@v10@fmt@@@std@@Ubig_decimal_fp@detail@v10@fmt@@_WV?$digit_grouping@_W@456@@detail@v10@fmt@@YA?AV?$back_insert_iterator@V?$buffer@_W@detail@v10@fmt@@@std@@V34@ABUbig_decimal_fp@012@ABU?$format_specs@_W@12@Ufloat_specs@012@Vlocale_ref@012@@Z 1003b275 f   handles.obj
 0001:0003a2a0       __unwindfunclet$??R<lambda_3>@?BD@???$do_write_float@V?$back_insert_iterator@V?$buffer@_W@detail@v10@fmt@@@std@@U?$decimal_fp@M@dragonbox@detail@v10@fmt@@_WV?$digit_grouping@_W@567@@detail@v10@fmt@@YA?AV?$back_insert_iterator@V?$buffer@_W@detail@v10@fmt@@@std@@V45@ABU?$decimal_fp@M@dragonbox@123@ABU?$format_specs@_W@23@Ufloat_specs@123@Vlocale_ref@123@@Z@QBE@0@Z$0 1003b2a0 f   handles.obj
 0001:0003a2b0       __ehhandler$??R<lambda_3>@?BD@???$do_write_float@V?$back_insert_iterator@V?$buffer@_W@detail@v10@fmt@@@std@@U?$decimal_fp@M@dragonbox@detail@v10@fmt@@_WV?$digit_grouping@_W@567@@detail@v10@fmt@@YA?AV?$back_insert_iterator@V?$buffer@_W@detail@v10@fmt@@@std@@V45@ABU?$decimal_fp@M@dragonbox@123@ABU?$format_specs@_W@23@Ufloat_specs@123@Vlocale_ref@123@@Z@QBE@0@Z 1003b2b0 f   handles.obj
 0001:0003a2e0       __unwindfunclet$??R<lambda_4>@?BO@???$do_write_float@V?$back_insert_iterator@V?$buffer@_W@detail@v10@fmt@@@std@@U?$decimal_fp@M@dragonbox@detail@v10@fmt@@_WV?$digit_grouping@_W@567@@detail@v10@fmt@@YA?AV?$back_insert_iterator@V?$buffer@_W@detail@v10@fmt@@@std@@V45@ABU?$decimal_fp@M@dragonbox@123@ABU?$format_specs@_W@23@Ufloat_specs@123@Vlocale_ref@123@@Z@QBE@0@Z$0 1003b2e0 f   handles.obj
 0001:0003a2e0       __unwindfunclet$??R<lambda_4>@?BO@???$do_write_float@V?$back_insert_iterator@V?$buffer@_W@detail@v10@fmt@@@std@@Ubig_decimal_fp@detail@v10@fmt@@_WV?$digit_grouping@_W@456@@detail@v10@fmt@@YA?AV?$back_insert_iterator@V?$buffer@_W@detail@v10@fmt@@@std@@V45@ABUbig_decimal_fp@123@ABU?$format_specs@_W@23@Ufloat_specs@123@Vlocale_ref@123@@Z@QBE@0@Z$0 1003b2e0 f   handles.obj
 0001:0003a2f0       __ehhandler$??R<lambda_4>@?BO@???$do_write_float@V?$back_insert_iterator@V?$buffer@_W@detail@v10@fmt@@@std@@U?$decimal_fp@M@dragonbox@detail@v10@fmt@@_WV?$digit_grouping@_W@567@@detail@v10@fmt@@YA?AV?$back_insert_iterator@V?$buffer@_W@detail@v10@fmt@@@std@@V45@ABU?$decimal_fp@M@dragonbox@123@ABU?$format_specs@_W@23@Ufloat_specs@123@Vlocale_ref@123@@Z@QBE@0@Z 1003b2f0 f   handles.obj
 0001:0003a2f0       __ehhandler$??R<lambda_4>@?BO@???$do_write_float@V?$back_insert_iterator@V?$buffer@_W@detail@v10@fmt@@@std@@Ubig_decimal_fp@detail@v10@fmt@@_WV?$digit_grouping@_W@456@@detail@v10@fmt@@YA?AV?$back_insert_iterator@V?$buffer@_W@detail@v10@fmt@@@std@@V45@ABUbig_decimal_fp@123@ABU?$format_specs@_W@23@Ufloat_specs@123@Vlocale_ref@123@@Z@QBE@0@Z 1003b2f0 f   handles.obj
 0001:0003a320       __unwindfunclet$??$do_write_float@V?$back_insert_iterator@V?$buffer@_W@detail@v10@fmt@@@std@@U?$decimal_fp@N@dragonbox@detail@v10@fmt@@_WV?$digit_grouping@_W@567@@detail@v10@fmt@@YA?AV?$back_insert_iterator@V?$buffer@_W@detail@v10@fmt@@@std@@V34@ABU?$decimal_fp@N@dragonbox@012@ABU?$format_specs@_W@12@Ufloat_specs@012@Vlocale_ref@012@@Z$0 1003b320 f   handles.obj
 0001:0003a328       __unwindfunclet$??$do_write_float@V?$back_insert_iterator@V?$buffer@_W@detail@v10@fmt@@@std@@U?$decimal_fp@N@dragonbox@detail@v10@fmt@@_WV?$digit_grouping@_W@567@@detail@v10@fmt@@YA?AV?$back_insert_iterator@V?$buffer@_W@detail@v10@fmt@@@std@@V34@ABU?$decimal_fp@N@dragonbox@012@ABU?$format_specs@_W@12@Ufloat_specs@012@Vlocale_ref@012@@Z$1 1003b328 f   handles.obj
 0001:0003a335       __ehhandler$??$do_write_float@V?$back_insert_iterator@V?$buffer@_W@detail@v10@fmt@@@std@@U?$decimal_fp@N@dragonbox@detail@v10@fmt@@_WV?$digit_grouping@_W@567@@detail@v10@fmt@@YA?AV?$back_insert_iterator@V?$buffer@_W@detail@v10@fmt@@@std@@V34@ABU?$decimal_fp@N@dragonbox@012@ABU?$format_specs@_W@12@Ufloat_specs@012@Vlocale_ref@012@@Z 1003b335 f   handles.obj
 0001:0003a360       __unwindfunclet$??R<lambda_3>@?BD@???$do_write_float@V?$back_insert_iterator@V?$buffer@_W@detail@v10@fmt@@@std@@U?$decimal_fp@N@dragonbox@detail@v10@fmt@@_WV?$digit_grouping@_W@567@@detail@v10@fmt@@YA?AV?$back_insert_iterator@V?$buffer@_W@detail@v10@fmt@@@std@@V45@ABU?$decimal_fp@N@dragonbox@123@ABU?$format_specs@_W@23@Ufloat_specs@123@Vlocale_ref@123@@Z@QBE@0@Z$0 1003b360 f   handles.obj
 0001:0003a370       __ehhandler$??R<lambda_3>@?BD@???$do_write_float@V?$back_insert_iterator@V?$buffer@_W@detail@v10@fmt@@@std@@U?$decimal_fp@N@dragonbox@detail@v10@fmt@@_WV?$digit_grouping@_W@567@@detail@v10@fmt@@YA?AV?$back_insert_iterator@V?$buffer@_W@detail@v10@fmt@@@std@@V45@ABU?$decimal_fp@N@dragonbox@123@ABU?$format_specs@_W@23@Ufloat_specs@123@Vlocale_ref@123@@Z@QBE@0@Z 1003b370 f   handles.obj
 0001:0003a3a0       __unwindfunclet$??R<lambda_4>@?BO@???$do_write_float@V?$back_insert_iterator@V?$buffer@_W@detail@v10@fmt@@@std@@U?$decimal_fp@N@dragonbox@detail@v10@fmt@@_WV?$digit_grouping@_W@567@@detail@v10@fmt@@YA?AV?$back_insert_iterator@V?$buffer@_W@detail@v10@fmt@@@std@@V45@ABU?$decimal_fp@N@dragonbox@123@ABU?$format_specs@_W@23@Ufloat_specs@123@Vlocale_ref@123@@Z@QBE@0@Z$0 1003b3a0 f   handles.obj
 0001:0003a3b0       __ehhandler$??R<lambda_4>@?BO@???$do_write_float@V?$back_insert_iterator@V?$buffer@_W@detail@v10@fmt@@@std@@U?$decimal_fp@N@dragonbox@detail@v10@fmt@@_WV?$digit_grouping@_W@567@@detail@v10@fmt@@YA?AV?$back_insert_iterator@V?$buffer@_W@detail@v10@fmt@@@std@@V45@ABU?$decimal_fp@N@dragonbox@123@ABU?$format_specs@_W@23@Ufloat_specs@123@Vlocale_ref@123@@Z@QBE@0@Z 1003b3b0 f   handles.obj
 0001:0003a3e0       __unwindfunclet$??0?$digit_grouping@_W@detail@v10@fmt@@QAE@Vlocale_ref@123@_N@Z$0 1003b3e0 f   handles.obj
 0001:0003a3e8       __unwindfunclet$??0?$digit_grouping@_W@detail@v10@fmt@@QAE@Vlocale_ref@123@_N@Z$1 1003b3e8 f   handles.obj
 0001:0003a3f3       __unwindfunclet$??0?$digit_grouping@_W@detail@v10@fmt@@QAE@Vlocale_ref@123@_N@Z$12 1003b3f3 f   handles.obj
 0001:0003a3fb       __unwindfunclet$??0?$digit_grouping@_W@detail@v10@fmt@@QAE@Vlocale_ref@123@_N@Z$13 1003b3fb f   handles.obj
 0001:0003a403       __unwindfunclet$??0?$digit_grouping@_W@detail@v10@fmt@@QAE@Vlocale_ref@123@_N@Z$2 1003b403 f   handles.obj
 0001:0003a410       __ehhandler$??0?$digit_grouping@_W@detail@v10@fmt@@QAE@Vlocale_ref@123@_N@Z 1003b410 f   handles.obj
 0001:0003a440       __unwindfunclet$??R<lambda_3>@?BD@???$do_write_float@V?$back_insert_iterator@V?$buffer@_W@detail@v10@fmt@@@std@@Ubig_decimal_fp@detail@v10@fmt@@_WV?$digit_grouping@_W@456@@detail@v10@fmt@@YA?AV?$back_insert_iterator@V?$buffer@_W@detail@v10@fmt@@@std@@V45@ABUbig_decimal_fp@123@ABU?$format_specs@_W@23@Ufloat_specs@123@Vlocale_ref@123@@Z@QBE@0@Z$0 1003b440 f   handles.obj
 0001:0003a450       __ehhandler$??R<lambda_3>@?BD@???$do_write_float@V?$back_insert_iterator@V?$buffer@_W@detail@v10@fmt@@@std@@Ubig_decimal_fp@detail@v10@fmt@@_WV?$digit_grouping@_W@456@@detail@v10@fmt@@YA?AV?$back_insert_iterator@V?$buffer@_W@detail@v10@fmt@@@std@@V45@ABUbig_decimal_fp@123@ABU?$format_specs@_W@23@Ufloat_specs@123@Vlocale_ref@123@@Z@QBE@0@Z 1003b450 f   handles.obj
 0001:0003a480       __ehhandler$??1PluginSettings@@QAE@XZ 1003b480 f   Pcfg.obj
 0001:0003a480       __ehhandler$??1?$unique_ptr@UIWbemClassObject@@Ucom_closer@@@std@@QAE@XZ 1003b480 f   wmi.obj
 0001:0003a480       __ehhandler$??1?$unique_ptr@UIWbemLocator@@Ucom_closer@@@std@@QAE@XZ 1003b480 f   wmi.obj
 0001:0003a4a0       __ehhandler$??1PluginDialogBuilder@@QAE@XZ 1003b4a0 f   Pcfg.obj
 0001:0003a4c0       __unwindfunclet$?Config@@YAHXZ$0 1003b4c0 f   Pcfg.obj
 0001:0003a4cb       __unwindfunclet$?Config@@YAHXZ$1 1003b4cb f   Pcfg.obj
 0001:0003a4d8       __ehhandler$?Config@@YAHXZ 1003b4d8 f   Pcfg.obj
 0001:0003a510       __unwindfunclet$?Read@options@@QAEXXZ$0 1003b510 f   Pcfg.obj
 0001:0003a51d       __ehhandler$?Read@options@@QAEXXZ 1003b51d f   Pcfg.obj
 0001:0003a550       __unwindfunclet$?ui64toa_width@@YA?AV?$basic_string@_WU?$char_traits@_W@std@@V?$allocator@_W@2@@std@@_KI_N@Z$0 1003b550 f   Pclass.obj
 0001:0003a55d       __ehhandler$?ui64toa_width@@YA?AV?$basic_string@_WU?$char_traits@_W@std@@V?$allocator@_W@2@@std@@_KI_N@Z 1003b55d f   Pclass.obj
 0001:0003a590       __unwindfunclet$?PrintTitle@@YA?AV?$basic_string@_WU?$char_traits@_W@std@@V?$allocator@_W@2@@std@@V?$basic_string_view@_WU?$char_traits@_W@std@@@2@@Z$0 1003b590 f   Pclass.obj
 0001:0003a59d       __ehhandler$?PrintTitle@@YA?AV?$basic_string@_WU?$char_traits@_W@std@@V?$allocator@_W@2@@std@@V?$basic_string_view@_WU?$char_traits@_W@std@@@2@@Z 1003b59d f   Pclass.obj
 0001:0003a5d0       __unwindfunclet$??0Plist@@QAE@XZ$0 1003b5d0 f   Pclass.obj
 0001:0003a5db       __unwindfunclet$??0Plist@@QAE@XZ$1 1003b5db f   Pclass.obj
 0001:0003a5e6       __unwindfunclet$??0Plist@@QAE@XZ$2 1003b5e6 f   Pclass.obj
 0001:0003a5f1       __unwindfunclet$??0Plist@@QAE@XZ$3 1003b5f1 f   Pclass.obj
 0001:0003a5f9       __unwindfunclet$??0Plist@@QAE@XZ$10 1003b5f9 f   Pclass.obj
 0001:0003a610       __ehhandler$??0Plist@@QAE@XZ 1003b610 f   Pclass.obj
 0001:0003a640       __unwindfunclet$?TranslateMode@@YA_NABV?$basic_string@_WU?$char_traits@_W@std@@V?$allocator@_W@2@@std@@AAV12@@Z$0 1003b640 f   Pclass.obj
 0001:0003a64d       __ehhandler$?TranslateMode@@YA_NABV?$basic_string@_WU?$char_traits@_W@std@@V?$allocator@_W@2@@std@@AAV12@@Z 1003b64d f   Pclass.obj
 0001:0003a680       __unwindfunclet$?InitializePanelModes@Plist@@SAXXZ$0 1003b680 f   Pclass.obj
 0001:0003a68b       __unwindfunclet$?InitializePanelModes@Plist@@SAXXZ$8 1003b68b f   Pclass.obj
 0001:0003a696       __unwindfunclet$?InitializePanelModes@Plist@@SAXXZ$9 1003b696 f   Pclass.obj
 0001:0003a6a1       __unwindfunclet$?InitializePanelModes@Plist@@SAXXZ$17 1003b6a1 f   Pclass.obj
 0001:0003a6ac       __unwindfunclet$?InitializePanelModes@Plist@@SAXXZ$18 1003b6ac f   Pclass.obj
 0001:0003a6b7       __unwindfunclet$?InitializePanelModes@Plist@@SAXXZ$26 1003b6b7 f   Pclass.obj
 0001:0003a6c2       __unwindfunclet$?InitializePanelModes@Plist@@SAXXZ$27 1003b6c2 f   Pclass.obj
 0001:0003a6cd       __unwindfunclet$?InitializePanelModes@Plist@@SAXXZ$35 1003b6cd f   Pclass.obj
 0001:0003a6d8       __unwindfunclet$?InitializePanelModes@Plist@@SAXXZ$36 1003b6d8 f   Pclass.obj
 0001:0003a6e3       __unwindfunclet$?InitializePanelModes@Plist@@SAXXZ$44 1003b6e3 f   Pclass.obj
 0001:0003a6ee       __unwindfunclet$?InitializePanelModes@Plist@@SAXXZ$45 1003b6ee f   Pclass.obj
 0001:0003a6f9       __unwindfunclet$?InitializePanelModes@Plist@@SAXXZ$53 1003b6f9 f   Pclass.obj
 0001:0003a704       __unwindfunclet$?InitializePanelModes@Plist@@SAXXZ$54 1003b704 f   Pclass.obj
 0001:0003a70f       __unwindfunclet$?InitializePanelModes@Plist@@SAXXZ$62 1003b70f f   Pclass.obj
 0001:0003a71a       __unwindfunclet$?InitializePanelModes@Plist@@SAXXZ$63 1003b71a f   Pclass.obj
 0001:0003a725       __unwindfunclet$?InitializePanelModes@Plist@@SAXXZ$71 1003b725 f   Pclass.obj
 0001:0003a730       __unwindfunclet$?InitializePanelModes@Plist@@SAXXZ$72 1003b730 f   Pclass.obj
 0001:0003a73b       __unwindfunclet$?InitializePanelModes@Plist@@SAXXZ$80 1003b73b f   Pclass.obj
 0001:0003a746       __unwindfunclet$?InitializePanelModes@Plist@@SAXXZ$81 1003b746 f   Pclass.obj
 0001:0003a751       __unwindfunclet$?InitializePanelModes@Plist@@SAXXZ$90 1003b751 f   Pclass.obj
 0001:0003a76a       __unwindfunclet$?InitializePanelModes@Plist@@SAXXZ$91 1003b76a f   Pclass.obj
 0001:0003a775       __unwindfunclet$?InitializePanelModes@Plist@@SAXXZ$99 1003b775 f   Pclass.obj
 0001:0003a780       __unwindfunclet$?InitializePanelModes@Plist@@SAXXZ$100 1003b780 f   Pclass.obj
 0001:0003a78b       __unwindfunclet$?InitializePanelModes@Plist@@SAXXZ$108 1003b78b f   Pclass.obj
 0001:0003a796       __unwindfunclet$?InitializePanelModes@Plist@@SAXXZ$109 1003b796 f   Pclass.obj
 0001:0003a7a1       __unwindfunclet$?InitializePanelModes@Plist@@SAXXZ$117 1003b7a1 f   Pclass.obj
 0001:0003a7ac       __unwindfunclet$?InitializePanelModes@Plist@@SAXXZ$118 1003b7ac f   Pclass.obj
 0001:0003a7b7       __unwindfunclet$?InitializePanelModes@Plist@@SAXXZ$126 1003b7b7 f   Pclass.obj
 0001:0003a7c2       __unwindfunclet$?InitializePanelModes@Plist@@SAXXZ$127 1003b7c2 f   Pclass.obj
 0001:0003a7cd       __unwindfunclet$?InitializePanelModes@Plist@@SAXXZ$135 1003b7cd f   Pclass.obj
 0001:0003a7d8       __unwindfunclet$?InitializePanelModes@Plist@@SAXXZ$136 1003b7d8 f   Pclass.obj
 0001:0003a7e3       __unwindfunclet$?InitializePanelModes@Plist@@SAXXZ$144 1003b7e3 f   Pclass.obj
 0001:0003a7ee       __unwindfunclet$?InitializePanelModes@Plist@@SAXXZ$145 1003b7ee f   Pclass.obj
 0001:0003a7f9       __unwindfunclet$?InitializePanelModes@Plist@@SAXXZ$153 1003b7f9 f   Pclass.obj
 0001:0003a804       __unwindfunclet$?InitializePanelModes@Plist@@SAXXZ$154 1003b804 f   Pclass.obj
 0001:0003a80f       __unwindfunclet$?InitializePanelModes@Plist@@SAXXZ$162 1003b80f f   Pclass.obj
 0001:0003a81a       __unwindfunclet$?InitializePanelModes@Plist@@SAXXZ$163 1003b81a f   Pclass.obj
 0001:0003a825       __unwindfunclet$?InitializePanelModes@Plist@@SAXXZ$171 1003b825 f   Pclass.obj
 0001:0003a830       __unwindfunclet$?InitializePanelModes@Plist@@SAXXZ$172 1003b830 f   Pclass.obj
 0001:0003a83b       __unwindfunclet$?InitializePanelModes@Plist@@SAXXZ$181 1003b83b f   Pclass.obj
 0001:0003a854       __unwindfunclet$?InitializePanelModes@Plist@@SAXXZ$182 1003b854 f   Pclass.obj
 0001:0003a85f       __unwindfunclet$?InitializePanelModes@Plist@@SAXXZ$183 1003b85f f   Pclass.obj
 0001:0003a86f       __ehhandler$?InitializePanelModes@Plist@@SAXXZ 1003b86f f   Pclass.obj
 0001:0003a8a0       __unwindfunclet$?SavePanelModes@Plist@@SAXXZ$0 1003b8a0 f   Pclass.obj
 0001:0003a8a8       __unwindfunclet$?SavePanelModes@Plist@@SAXXZ$1 1003b8a8 f   Pclass.obj
 0001:0003a8b5       __ehhandler$?SavePanelModes@Plist@@SAXXZ 1003b8b5 f   Pclass.obj
 0001:0003a8e0       __unwindfunclet$?generate_titles@@YAXABV?$basic_string@_WU?$char_traits@_W@std@@V?$allocator@_W@2@@std@@AAUPanelMode@@@Z$0 1003b8e0 f   Pclass.obj
 0001:0003a8ed       __ehhandler$?generate_titles@@YAXABV?$basic_string@_WU?$char_traits@_W@std@@V?$allocator@_W@2@@std@@AAUPanelMode@@@Z 1003b8ed f   Pclass.obj
 0001:0003a910       __unwindfunclet$?GetOpenPanelInfo@Plist@@QAEXPAUOpenPanelInfo@@@Z$0 1003b910 f   Pclass.obj
 0001:0003a91d       __ehhandler$?GetOpenPanelInfo@Plist@@QAEXPAUOpenPanelInfo@@@Z 1003b91d f   Pclass.obj
 0001:0003a950       __unwindfunclet$?GetFindData@Plist@@QAEHAAPAUPluginPanelItem@@AAI_K@Z$0 1003b950 f   Pclass.obj
 0001:0003a95b       __unwindfunclet$?GetFindData@Plist@@QAEHAAPAUPluginPanelItem@@AAI_K@Z$1 1003b95b f   Pclass.obj
 0001:0003a966       __unwindfunclet$?GetFindData@Plist@@QAEHAAPAUPluginPanelItem@@AAI_K@Z$13 1003b966 f   Pclass.obj
 0001:0003a971       __unwindfunclet$?GetFindData@Plist@@QAEHAAPAUPluginPanelItem@@AAI_K@Z$14 1003b971 f   Pclass.obj
 0001:0003a97c       __unwindfunclet$?GetFindData@Plist@@QAEHAAPAUPluginPanelItem@@AAI_K@Z$2 1003b97c f   Pclass.obj
 0001:0003a987       __unwindfunclet$?GetFindData@Plist@@QAEHAAPAUPluginPanelItem@@AAI_K@Z$3 1003b987 f   Pclass.obj
 0001:0003a992       __unwindfunclet$?GetFindData@Plist@@QAEHAAPAUPluginPanelItem@@AAI_K@Z$4 1003b992 f   Pclass.obj
 0001:0003a99d       __unwindfunclet$?GetFindData@Plist@@QAEHAAPAUPluginPanelItem@@AAI_K@Z$5 1003b99d f   Pclass.obj
 0001:0003a9a8       __unwindfunclet$?GetFindData@Plist@@QAEHAAPAUPluginPanelItem@@AAI_K@Z$6 1003b9a8 f   Pclass.obj
 0001:0003a9b3       __unwindfunclet$?GetFindData@Plist@@QAEHAAPAUPluginPanelItem@@AAI_K@Z$7 1003b9b3 f   Pclass.obj
 0001:0003a9be       __unwindfunclet$?GetFindData@Plist@@QAEHAAPAUPluginPanelItem@@AAI_K@Z$8 1003b9be f   Pclass.obj
 0001:0003a9ce       __ehhandler$?GetFindData@Plist@@QAEHAAPAUPluginPanelItem@@AAI_K@Z 1003b9ce f   Pclass.obj
 0001:0003aa00       __ehhandler$??$emplace_back@V?$basic_string@_WU?$char_traits@_W@std@@V?$allocator@_W@2@@std@@@?$vector@V?$basic_string@_WU?$char_traits@_W@std@@V?$allocator@_W@2@@std@@V?$allocator@V?$basic_string@_WU?$char_traits@_W@std@@V?$allocator@_W@2@@std@@@2@@std@@QAE?A_T$$QAV?$basic_string@_WU?$char_traits@_W@std@@V?$allocator@_W@2@@1@@Z 1003ba00 f   Pclass.obj
 0001:0003aa20       __unwindfunclet$?window_ex_style@@YA@PAUHWND__@@@Z$0 1003ba20 f   Pclass.obj
 0001:0003aa20       __unwindfunclet$?window_style@@YA@PAUHWND__@@@Z$0 1003ba20 f   Pclass.obj
 0001:0003aa2d       __ehhandler$?window_ex_style@@YA@PAUHWND__@@@Z 1003ba2d f   Pclass.obj
 0001:0003aa2d       __ehhandler$?window_style@@YA@PAUHWND__@@@Z 1003ba2d f   Pclass.obj
 0001:0003aa60       __unwindfunclet$?DumpNTCounters@@YAXPAXAAVPerfThread@@KK@Z$0 1003ba60 f   Pclass.obj
 0001:0003aa68       __unwindfunclet$?DumpNTCounters@@YAXPAXAAVPerfThread@@KK@Z$3 1003ba68 f   Pclass.obj
 0001:0003aa75       __ehhandler$?DumpNTCounters@@YAXPAXAAVPerfThread@@KK@Z 1003ba75 f   Pclass.obj
 0001:0003aaa0       __unwindfunclet$?GetFiles@Plist@@QAEHPAUPluginPanelItem@@IHPAPB_W_KAAUoptions@@@Z$0 1003baa0 f   Pclass.obj
 0001:0003aaab       __unwindfunclet$?GetFiles@Plist@@QAEHPAUPluginPanelItem@@IHPAPB_W_KAAUoptions@@@Z$1 1003baab f   Pclass.obj
 0001:0003aab6       __unwindfunclet$?GetFiles@Plist@@QAEHPAUPluginPanelItem@@IHPAPB_W_KAAUoptions@@@Z$2 1003bab6 f   Pclass.obj
 0001:0003aac1       __unwindfunclet$?GetFiles@Plist@@QAEHPAUPluginPanelItem@@IHPAPB_W_KAAUoptions@@@Z$3 1003bac1 f   Pclass.obj
 0001:0003aacc       __unwindfunclet$?GetFiles@Plist@@QAEHPAUPluginPanelItem@@IHPAPB_W_KAAUoptions@@@Z$4 1003bacc f   Pclass.obj
 0001:0003aad7       __unwindfunclet$?GetFiles@Plist@@QAEHPAUPluginPanelItem@@IHPAPB_W_KAAUoptions@@@Z$6 1003bad7 f   Pclass.obj
 0001:0003aae2       __unwindfunclet$?GetFiles@Plist@@QAEHPAUPluginPanelItem@@IHPAPB_W_KAAUoptions@@@Z$65 1003bae2 f   Pclass.obj
 0001:0003aaed       __unwindfunclet$?GetFiles@Plist@@QAEHPAUPluginPanelItem@@IHPAPB_W_KAAUoptions@@@Z$8 1003baed f   Pclass.obj
 0001:0003aaf8       __unwindfunclet$?GetFiles@Plist@@QAEHPAUPluginPanelItem@@IHPAPB_W_KAAUoptions@@@Z$11 1003baf8 f   Pclass.obj
 0001:0003ab03       __unwindfunclet$?GetFiles@Plist@@QAEHPAUPluginPanelItem@@IHPAPB_W_KAAUoptions@@@Z$66 1003bb03 f   Pclass.obj
 0001:0003ab0e       __unwindfunclet$?GetFiles@Plist@@QAEHPAUPluginPanelItem@@IHPAPB_W_KAAUoptions@@@Z$68 1003bb0e f   Pclass.obj
 0001:0003ab19       __unwindfunclet$?GetFiles@Plist@@QAEHPAUPluginPanelItem@@IHPAPB_W_KAAUoptions@@@Z$14 1003bb19 f   Pclass.obj
 0001:0003ab24       __unwindfunclet$?GetFiles@Plist@@QAEHPAUPluginPanelItem@@IHPAPB_W_KAAUoptions@@@Z$16 1003bb24 f   Pclass.obj
 0001:0003ab2f       __unwindfunclet$?GetFiles@Plist@@QAEHPAUPluginPanelItem@@IHPAPB_W_KAAUoptions@@@Z$20 1003bb2f f   Pclass.obj
 0001:0003ab3a       __unwindfunclet$?GetFiles@Plist@@QAEHPAUPluginPanelItem@@IHPAPB_W_KAAUoptions@@@Z$18 1003bb3a f   Pclass.obj
 0001:0003ab45       __unwindfunclet$?GetFiles@Plist@@QAEHPAUPluginPanelItem@@IHPAPB_W_KAAUoptions@@@Z$22 1003bb45 f   Pclass.obj
 0001:0003ab50       __unwindfunclet$?GetFiles@Plist@@QAEHPAUPluginPanelItem@@IHPAPB_W_KAAUoptions@@@Z$23 1003bb50 f   Pclass.obj
 0001:0003ab5b       __unwindfunclet$?GetFiles@Plist@@QAEHPAUPluginPanelItem@@IHPAPB_W_KAAUoptions@@@Z$26 1003bb5b f   Pclass.obj
 0001:0003ab66       __unwindfunclet$?GetFiles@Plist@@QAEHPAUPluginPanelItem@@IHPAPB_W_KAAUoptions@@@Z$27 1003bb66 f   Pclass.obj
 0001:0003ab71       __unwindfunclet$?GetFiles@Plist@@QAEHPAUPluginPanelItem@@IHPAPB_W_KAAUoptions@@@Z$28 1003bb71 f   Pclass.obj
 0001:0003ab7c       __unwindfunclet$?GetFiles@Plist@@QAEHPAUPluginPanelItem@@IHPAPB_W_KAAUoptions@@@Z$29 1003bb7c f   Pclass.obj
 0001:0003ab87       __unwindfunclet$?GetFiles@Plist@@QAEHPAUPluginPanelItem@@IHPAPB_W_KAAUoptions@@@Z$31 1003bb87 f   Pclass.obj
 0001:0003ab92       __unwindfunclet$?GetFiles@Plist@@QAEHPAUPluginPanelItem@@IHPAPB_W_KAAUoptions@@@Z$33 1003bb92 f   Pclass.obj
 0001:0003ab9d       __unwindfunclet$?GetFiles@Plist@@QAEHPAUPluginPanelItem@@IHPAPB_W_KAAUoptions@@@Z$35 1003bb9d f   Pclass.obj
 0001:0003aba8       __unwindfunclet$?GetFiles@Plist@@QAEHPAUPluginPanelItem@@IHPAPB_W_KAAUoptions@@@Z$37 1003bba8 f   Pclass.obj
 0001:0003abb3       __unwindfunclet$?GetFiles@Plist@@QAEHPAUPluginPanelItem@@IHPAPB_W_KAAUoptions@@@Z$38 1003bbb3 f   Pclass.obj
 0001:0003abbe       __unwindfunclet$?GetFiles@Plist@@QAEHPAUPluginPanelItem@@IHPAPB_W_KAAUoptions@@@Z$40 1003bbbe f   Pclass.obj
 0001:0003abc9       __unwindfunclet$?GetFiles@Plist@@QAEHPAUPluginPanelItem@@IHPAPB_W_KAAUoptions@@@Z$41 1003bbc9 f   Pclass.obj
 0001:0003abd9       __ehhandler$?GetFiles@Plist@@QAEHPAUPluginPanelItem@@IHPAPB_W_KAAUoptions@@@Z 1003bbd9 f   Pclass.obj
 0001:0003ac10       __ehhandler$??0ProcessData@@QAE@XZ 1003bc10 f   Pclass.obj
 0001:0003ac30       __unwindfunclet$?DeleteFiles@Plist@@QAEHPAUPluginPanelItem@@I_K@Z$0 1003bc30 f   Pclass.obj
 0001:0003ac3b       __unwindfunclet$?DeleteFiles@Plist@@QAEHPAUPluginPanelItem@@I_K@Z$1 1003bc3b f   Pclass.obj
 0001:0003ac43       __unwindfunclet$?DeleteFiles@Plist@@QAEHPAUPluginPanelItem@@I_K@Z$4 1003bc43 f   Pclass.obj
 0001:0003ac50       __ehhandler$?DeleteFiles@Plist@@QAEHPAUPluginPanelItem@@I_K@Z 1003bc50 f   Pclass.obj
 0001:0003ac80       __unwindfunclet$?Connect@Plist@@QAE_NPB_W00@Z$0 1003bc80 f   Pclass.obj
 0001:0003ac88       __unwindfunclet$?Connect@Plist@@QAE_NPB_W00@Z$6 1003bc88 f   Pclass.obj
 0001:0003ac9a       __unwindfunclet$?Connect@Plist@@QAE_NPB_W00@Z$1 1003bc9a f   Pclass.obj
 0001:0003aca7       __ehhandler$?Connect@Plist@@QAE_NPB_W00@Z 1003bca7 f   Pclass.obj
 0001:0003acd0       __unwindfunclet$?ProcessKey@Plist@@QAEHPBU_INPUT_RECORD@@@Z$0 1003bcd0 f   Pclass.obj
 0001:0003acdb       __unwindfunclet$?ProcessKey@Plist@@QAEHPBU_INPUT_RECORD@@@Z$1 1003bcdb f   Pclass.obj
 0001:0003ace6       __unwindfunclet$?ProcessKey@Plist@@QAEHPBU_INPUT_RECORD@@@Z$2 1003bce6 f   Pclass.obj
 0001:0003acf1       __unwindfunclet$?ProcessKey@Plist@@QAEHPBU_INPUT_RECORD@@@Z$3 1003bcf1 f   Pclass.obj
 0001:0003acfc       __unwindfunclet$?ProcessKey@Plist@@QAEHPBU_INPUT_RECORD@@@Z$4 1003bcfc f   Pclass.obj
 0001:0003ad07       __unwindfunclet$?ProcessKey@Plist@@QAEHPBU_INPUT_RECORD@@@Z$5 1003bd07 f   Pclass.obj
 0001:0003ad12       __unwindfunclet$?ProcessKey@Plist@@QAEHPBU_INPUT_RECORD@@@Z$213 1003bd12 f   Pclass.obj
 0001:0003ad27       __unwindfunclet$?ProcessKey@Plist@@QAEHPBU_INPUT_RECORD@@@Z$8 1003bd27 f   Pclass.obj
 0001:0003ad32       __unwindfunclet$?ProcessKey@Plist@@QAEHPBU_INPUT_RECORD@@@Z$9 1003bd32 f   Pclass.obj
 0001:0003ad3d       __unwindfunclet$?ProcessKey@Plist@@QAEHPBU_INPUT_RECORD@@@Z$10 1003bd3d f   Pclass.obj
 0001:0003ad48       __unwindfunclet$?ProcessKey@Plist@@QAEHPBU_INPUT_RECORD@@@Z$11 1003bd48 f   Pclass.obj
 0001:0003ad53       __unwindfunclet$?ProcessKey@Plist@@QAEHPBU_INPUT_RECORD@@@Z$217 1003bd53 f   Pclass.obj
 0001:0003ad5e       __unwindfunclet$?ProcessKey@Plist@@QAEHPBU_INPUT_RECORD@@@Z$12 1003bd5e f   Pclass.obj
 0001:0003ad69       __unwindfunclet$?ProcessKey@Plist@@QAEHPBU_INPUT_RECORD@@@Z$13 1003bd69 f   Pclass.obj
 0001:0003ad74       __unwindfunclet$?ProcessKey@Plist@@QAEHPBU_INPUT_RECORD@@@Z$14 1003bd74 f   Pclass.obj
 0001:0003ad7f       __unwindfunclet$?ProcessKey@Plist@@QAEHPBU_INPUT_RECORD@@@Z$15 1003bd7f f   Pclass.obj
 0001:0003ada1       __unwindfunclet$?ProcessKey@Plist@@QAEHPBU_INPUT_RECORD@@@Z$16 1003bda1 f   Pclass.obj
 0001:0003adc8       __ehhandler$?ProcessKey@Plist@@QAEHPBU_INPUT_RECORD@@@Z 1003bdc8 f   Pclass.obj
 0001:0003ae00       __unwindfunclet$?GetVersionInfo@Plist@@SA_NPB_WAAV?$unique_ptr@$$BY0A@DU?$default_delete@$$BY0A@D@std@@@std@@AAPB_W2@Z$1 1003be00 f   Pclass.obj
 0001:0003ae08       __unwindfunclet$?GetVersionInfo@Plist@@SA_NPB_WAAV?$unique_ptr@$$BY0A@DU?$default_delete@$$BY0A@D@std@@@std@@AAPB_W2@Z$2 1003be08 f   Pclass.obj
 0001:0003ae10       __unwindfunclet$?GetVersionInfo@Plist@@SA_NPB_WAAV?$unique_ptr@$$BY0A@DU?$default_delete@$$BY0A@D@std@@@std@@AAPB_W2@Z$4 1003be10 f   Pclass.obj
 0001:0003ae1d       __ehhandler$?GetVersionInfo@Plist@@SA_NPB_WAAV?$unique_ptr@$$BY0A@DU?$default_delete@$$BY0A@D@std@@@std@@AAPB_W2@Z 1003be1d f   Pclass.obj
 0001:0003ae50       __unwindfunclet$?PrintOwnerInfo@Plist@@AAEXPAXK@Z$0 1003be50 f   Pclass.obj
 0001:0003ae58       __unwindfunclet$?PrintOwnerInfo@Plist@@AAEXPAXK@Z$1 1003be58 f   Pclass.obj
 0001:0003ae60       __unwindfunclet$?PrintOwnerInfo@Plist@@AAEXPAXK@Z$2 1003be60 f   Pclass.obj
 0001:0003ae68       __unwindfunclet$?PrintOwnerInfo@Plist@@AAEXPAXK@Z$6 1003be68 f   Pclass.obj
 0001:0003ae78       __ehhandler$?PrintOwnerInfo@Plist@@AAEXPAXK@Z 1003be78 f   Pclass.obj
 0001:0003aeb0       __unwindfunclet$?Compare@Plist@@QBEHPBUPluginPanelItem@@0I@Z$0 1003beb0 f   Pclass.obj
 0001:0003aeb8       __unwindfunclet$?Compare@Plist@@QBEHPBUPluginPanelItem@@0I@Z$1 1003beb8 f   Pclass.obj
 0001:0003aec5       __ehhandler$?Compare@Plist@@QBEHPBUPluginPanelItem@@0I@Z 1003bec5 f   Pclass.obj
 0001:0003aef0       __unwindfunclet$??4?$vector@Umode@@V?$allocator@Umode@@@std@@@std@@QAEAAV01@V?$initializer_list@Umode@@@1@@Z$0 1003bef0 f   Pclass.obj
 0001:0003aefd       __ehhandler$??4?$vector@Umode@@V?$allocator@Umode@@@std@@@std@@QAEAAV01@V?$initializer_list@Umode@@@1@@Z 1003befd f   Pclass.obj
 0001:0003af20       __ehhandler$??1?$unique_ptr@VWMIConnection@@U?$default_delete@VWMIConnection@@@std@@@std@@QAE@XZ 1003bf20 f   Pclass.obj
 0001:0003af20       __ehhandler$?reset@?$unique_ptr@VWMIConnection@@U?$default_delete@VWMIConnection@@@std@@@std@@QAEXPAVWMIConnection@@@Z 1003bf20 f   Pclass.obj
 0001:0003af40       __unwindfunclet$??$make_unique@VPerfThread@@PAVPlist@@$0A@@std@@YA?AV?$unique_ptr@VPerfThread@@U?$default_delete@VPerfThread@@@std@@@0@$$QAPAVPlist@@@Z$0 1003bf40 f   Pclass.obj
 0001:0003af57       __ehhandler$??$make_unique@VPerfThread@@PAVPlist@@$0A@@std@@YA?AV?$unique_ptr@VPerfThread@@U?$default_delete@VPerfThread@@@std@@@0@$$QAPAVPlist@@@Z 1003bf57 f   Pclass.obj
 0001:0003af80       __ehhandler$??$construct@V?$basic_string@_WU?$char_traits@_W@std@@V?$allocator@_W@2@@std@@V12@@?$_Default_allocator_traits@V?$allocator@V?$basic_string@_WU?$char_traits@_W@std@@V?$allocator@_W@2@@std@@@std@@@std@@SAXAAV?$allocator@V?$basic_string@_WU?$char_traits@_W@std@@V?$allocator@_W@2@@std@@@1@QAV?$basic_string@_WU?$char_traits@_W@std@@V?$allocator@_W@2@@1@$$QAV31@@Z 1003bf80 f   Pclass.obj
 0001:0003afa0       __ehhandler$??$_Emplace_reallocate@V?$basic_string@_WU?$char_traits@_W@std@@V?$allocator@_W@2@@std@@@?$vector@V?$basic_string@_WU?$char_traits@_W@std@@V?$allocator@_W@2@@std@@V?$allocator@V?$basic_string@_WU?$char_traits@_W@std@@V?$allocator@_W@2@@std@@@2@@std@@QAEPAV?$basic_string@_WU?$char_traits@_W@std@@V?$allocator@_W@2@@1@QAV21@$$QAV21@@Z 1003bfa0 f   Pclass.obj
 0001:0003afc0       __ehhandler$??$?H_WU?$char_traits@_W@std@@V?$allocator@_W@1@@std@@YA?AV?$basic_string@_WU?$char_traits@_W@std@@V?$allocator@_W@2@@0@ABV10@$$QAV10@@Z 1003bfc0 f   Pclass.obj
 0001:0003afe0       __unwindfunclet$??$_Try_emplace@ABK$$V@?$_Hash@V?$_Umap_traits@KPAUHWND__@@V?$_Uhash_compare@KU?$hash@K@std@@U?$equal_to@K@2@@std@@V?$allocator@U?$pair@$$CBKPAUHWND__@@@std@@@3@$0A@@std@@@std@@IAE?AU?$pair@PAU?$_List_node@U?$pair@$$CBKPAUHWND__@@@std@@PAX@std@@_N@1@ABK@Z$1 1003bfe0 f   Pclass.obj
 0001:0003afe8       __unwindfunclet$??$_Try_emplace@ABK$$V@?$_Hash@V?$_Umap_traits@KPAUHWND__@@V?$_Uhash_compare@KU?$hash@K@std@@U?$equal_to@K@2@@std@@V?$allocator@U?$pair@$$CBKPAUHWND__@@@std@@@3@$0A@@std@@@std@@IAE?AU?$pair@PAU?$_List_node@U?$pair@$$CBKPAUHWND__@@@std@@PAX@std@@_N@1@ABK@Z$0 1003bfe8 f   Pclass.obj
 0001:0003aff5       __ehhandler$??$_Try_emplace@ABK$$V@?$_Hash@V?$_Umap_traits@KPAUHWND__@@V?$_Uhash_compare@KU?$hash@K@std@@U?$equal_to@K@2@@std@@V?$allocator@U?$pair@$$CBKPAUHWND__@@@std@@@3@$0A@@std@@@std@@IAE?AU?$pair@PAU?$_List_node@U?$pair@$$CBKPAUHWND__@@@std@@PAX@std@@_N@1@ABK@Z 1003bff5 f   Pclass.obj
 0001:0003b020       __ehhandler$??$_Uninitialized_move@PAV?$basic_string@_WU?$char_traits@_W@std@@V?$allocator@_W@2@@std@@V?$allocator@V?$basic_string@_WU?$char_traits@_W@std@@V?$allocator@_W@2@@std@@@2@@std@@YAPAV?$basic_string@_WU?$char_traits@_W@std@@V?$allocator@_W@2@@0@QAV10@0PAV10@AAV?$allocator@V?$basic_string@_WU?$char_traits@_W@std@@V?$allocator@_W@2@@std@@@0@@Z 1003c020 f   Pclass.obj
 0001:0003b040       __unwindfunclet$??0mode@@QAE@ABU0@@Z$2 1003c040 f   Pclass.obj
 0001:0003b048       __unwindfunclet$??0mode@@QAE@ABU0@@Z$3 1003c048 f   Pclass.obj
 0001:0003b053       __unwindfunclet$??0mode@@QAE@ABU0@@Z$0 1003c053 f   Pclass.obj
 0001:0003b05b       __unwindfunclet$??0mode@@QAE@ABU0@@Z$5 1003c05b f   Pclass.obj
 0001:0003b063       __unwindfunclet$??0mode@@QAE@ABU0@@Z$6 1003c063 f   Pclass.obj
 0001:0003b073       __ehhandler$??0mode@@QAE@ABU0@@Z 1003c073 f   Pclass.obj
 0001:0003b090       __unwindfunclet$??0PerfThread@@QAE@PAVPlist@@PB_W11@Z$15 1003c090 f   perfthread.obj
 0001:0003b09e       __unwindfunclet$??0PerfThread@@QAE@PAVPlist@@PB_W11@Z$0 1003c09e f   perfthread.obj
 0001:0003b0a9       __unwindfunclet$??0PerfThread@@QAE@PAVPlist@@PB_W11@Z$1 1003c0a9 f   perfthread.obj
 0001:0003b0b4       __unwindfunclet$??0PerfThread@@QAE@PAVPlist@@PB_W11@Z$2 1003c0b4 f   perfthread.obj
 0001:0003b0bf       __unwindfunclet$??0PerfThread@@QAE@PAVPlist@@PB_W11@Z$3 1003c0bf f   perfthread.obj
 0001:0003b0ca       __unwindfunclet$??0PerfThread@@QAE@PAVPlist@@PB_W11@Z$4 1003c0ca f   perfthread.obj
 0001:0003b0d5       __unwindfunclet$??0PerfThread@@QAE@PAVPlist@@PB_W11@Z$5 1003c0d5 f   perfthread.obj
 0001:0003b0e0       __unwindfunclet$??0PerfThread@@QAE@PAVPlist@@PB_W11@Z$6 1003c0e0 f   perfthread.obj
 0001:0003b0eb       __unwindfunclet$??0PerfThread@@QAE@PAVPlist@@PB_W11@Z$7 1003c0eb f   perfthread.obj
 0001:0003b0f6       __unwindfunclet$??0PerfThread@@QAE@PAVPlist@@PB_W11@Z$8 1003c0f6 f   perfthread.obj
 0001:0003b101       __unwindfunclet$??0PerfThread@@QAE@PAVPlist@@PB_W11@Z$9 1003c101 f   perfthread.obj
 0001:0003b10f       __unwindfunclet$??0PerfThread@@QAE@PAVPlist@@PB_W11@Z$10 1003c10f f   perfthread.obj
 0001:0003b11d       __unwindfunclet$??0PerfThread@@QAE@PAVPlist@@PB_W11@Z$11 1003c11d f   perfthread.obj
 0001:0003b12b       __unwindfunclet$??0PerfThread@@QAE@PAVPlist@@PB_W11@Z$12 1003c12b f   perfthread.obj
 0001:0003b133       __unwindfunclet$??0PerfThread@@QAE@PAVPlist@@PB_W11@Z$13 1003c133 f   perfthread.obj
 0001:0003b140       __ehhandler$??0PerfThread@@QAE@PAVPlist@@PB_W11@Z 1003c140 f   perfthread.obj
 0001:0003b170       __ehhandler$??1PerfThread@@QAE@XZ 1003c170 f   perfthread.obj
 0001:0003b190       __unwindfunclet$?RefreshImpl@PerfThread@@AAE_NXZ$0 1003c190 f   perfthread.obj
 0001:0003b19b       __unwindfunclet$?RefreshImpl@PerfThread@@AAE_NXZ$1 1003c19b f   perfthread.obj
 0001:0003b1a6       __unwindfunclet$?RefreshImpl@PerfThread@@AAE_NXZ$2 1003c1a6 f   perfthread.obj
 0001:0003b1b6       __ehhandler$?RefreshImpl@PerfThread@@AAE_NXZ 1003c1b6 f   perfthread.obj
 0001:0003b1e0       __unwindfunclet$??R<lambda_1>@?1??RefreshImpl@PerfThread@@AAE_NXZ@QBE@PBU_PERF_COUNTER_BLOCK@@V?$basic_string_view@_WU?$char_traits@_W@std@@@std@@@Z$4 1003c1e0 f   perfthread.obj
 0001:0003b1eb       __unwindfunclet$??R<lambda_1>@?1??RefreshImpl@PerfThread@@AAE_NXZ@QBE@PBU_PERF_COUNTER_BLOCK@@V?$basic_string_view@_WU?$char_traits@_W@std@@@std@@@Z$26 1003c1eb f   perfthread.obj
 0001:0003b1f6       __unwindfunclet$??R<lambda_1>@?1??RefreshImpl@PerfThread@@AAE_NXZ@QBE@PBU_PERF_COUNTER_BLOCK@@V?$basic_string_view@_WU?$char_traits@_W@std@@@std@@@Z$25 1003c1f6 f   perfthread.obj
 0001:0003b201       __unwindfunclet$??R<lambda_1>@?1??RefreshImpl@PerfThread@@AAE_NXZ@QBE@PBU_PERF_COUNTER_BLOCK@@V?$basic_string_view@_WU?$char_traits@_W@std@@@std@@@Z$8 1003c201 f   perfthread.obj
 0001:0003b211       __ehhandler$??R<lambda_1>@?1??RefreshImpl@PerfThread@@AAE_NXZ@QBE@PBU_PERF_COUNTER_BLOCK@@V?$basic_string_view@_WU?$char_traits@_W@std@@@std@@@Z 1003c211 f   perfthread.obj
 0001:0003b240       __unwindfunclet$?RefreshWMIData@PerfThread@@AAEXXZ$0 1003c240 f   perfthread.obj
 0001:0003b248       __unwindfunclet$?RefreshWMIData@PerfThread@@AAEXXZ$1 1003c248 f   perfthread.obj
 0001:0003b250       __unwindfunclet$?RefreshWMIData@PerfThread@@AAEXXZ$12 1003c250 f   perfthread.obj
 0001:0003b258       __unwindfunclet$?RefreshWMIData@PerfThread@@AAEXXZ$4 1003c258 f   perfthread.obj
 0001:0003b260       __unwindfunclet$?RefreshWMIData@PerfThread@@AAEXXZ$6 1003c260 f   perfthread.obj
 0001:0003b26d       __ehhandler$?RefreshWMIData@PerfThread@@AAEXXZ 1003c26d f   perfthread.obj
 0001:0003b2a0       __unwindfunclet$??0?$unordered_multimap@KUProcessPerfData@@U?$hash@K@std@@U?$equal_to@K@3@V?$allocator@U?$pair@$$CBKUProcessPerfData@@@std@@@3@@std@@QAE@XZ$1 1003c2a0 f   perfthread.obj
 0001:0003b2ab       __unwindfunclet$??0?$unordered_multimap@KUProcessPerfData@@U?$hash@K@std@@U?$equal_to@K@3@V?$allocator@U?$pair@$$CBKUProcessPerfData@@@std@@@3@@std@@QAE@XZ$2 1003c2ab f   perfthread.obj
 0001:0003b2bb       __ehhandler$??0?$unordered_multimap@KUProcessPerfData@@U?$hash@K@std@@U?$equal_to@K@3@V?$allocator@U?$pair@$$CBKUProcessPerfData@@@std@@@3@@std@@QAE@XZ 1003c2bb f   perfthread.obj
 0001:0003b2e0       __unwindfunclet$??$transform@V?$_List_const_iterator@V?$_List_val@U?$_List_simple_types@U?$pair@$$CBKUProcessPerfData@@@std@@@std@@@std@@@std@@V?$back_insert_iterator@V?$vector@UProcessPerfData@@V?$allocator@UProcessPerfData@@@std@@@std@@@2@V<lambda_1>@?2??RefreshWMIData@PerfThread@@AAEXXZ@@std@@YA?AV?$back_insert_iterator@V?$vector@UProcessPerfData@@V?$allocator@UProcessPerfData@@@std@@@std@@@0@V?$_List_const_iterator@V?$_List_val@U?$_List_simple_types@U?$pair@$$CBKUProcessPerfData@@@std@@@std@@@std@@@0@0V10@V<lambda_1>@?2??RefreshWMIData@PerfThread@@AAEXXZ@@Z$0 1003c2e0 f   perfthread.obj
 0001:0003b2f0       __ehhandler$??$transform@V?$_List_const_iterator@V?$_List_val@U?$_List_simple_types@U?$pair@$$CBKUProcessPerfData@@@std@@@std@@@std@@@std@@V?$back_insert_iterator@V?$vector@UProcessPerfData@@V?$allocator@UProcessPerfData@@@std@@@std@@@2@V<lambda_1>@?2??RefreshWMIData@PerfThread@@AAEXXZ@@std@@YA?AV?$back_insert_iterator@V?$vector@UProcessPerfData@@V?$allocator@UProcessPerfData@@@std@@@std@@@0@V?$_List_const_iterator@V?$_List_val@U?$_List_simple_types@U?$pair@$$CBKUProcessPerfData@@@std@@@std@@@std@@@0@0V10@V<lambda_1>@?2??RefreshWMIData@PerfThread@@AAEXXZ@@Z 1003c2f0 f   perfthread.obj
 0001:0003b320       __unwindfunclet$??0ProcessPerfData@@QAE@ABU0@@Z$0 1003c320 f   perfthread.obj
 0001:0003b32e       __unwindfunclet$??0ProcessPerfData@@QAE@ABU0@@Z$1 1003c32e f   perfthread.obj
 0001:0003b33c       __unwindfunclet$??0ProcessPerfData@@QAE@ABU0@@Z$2 1003c33c f   perfthread.obj
 0001:0003b34f       __ehhandler$??0ProcessPerfData@@QAE@ABU0@@Z 1003c34f f   perfthread.obj
 0001:0003b370       __ehhandler$??0ProcessPerfData@@QAE@$$QAU0@@Z 1003c370 f   perfthread.obj
 0001:0003b390       __unwindfunclet$?is_wow64_itself@@YA_NXZ$0 1003c390 f   Plist.obj
 0001:0003b3a3       __ehhandler$?is_wow64_itself@@YA_NXZ 1003c3a3 f   Plist.obj
 0001:0003b3c0       __unwindfunclet$?GetList@@YA_NAAPAUPluginPanelItem@@AAIAAVPerfThread@@@Z$2 1003c3c0 f   Plist.obj
 0001:0003b3c8       __unwindfunclet$?GetList@@YA_NAAPAUPluginPanelItem@@AAIAAVPerfThread@@@Z$3 1003c3c8 f   Plist.obj
 0001:0003b3d0       __unwindfunclet$?GetList@@YA_NAAPAUPluginPanelItem@@AAIAAVPerfThread@@@Z$0 1003c3d0 f   Plist.obj
 0001:0003b3dd       __ehhandler$?GetList@@YA_NAAPAUPluginPanelItem@@AAIAAVPerfThread@@@Z 1003c3dd f   Plist.obj
 0001:0003b400       __unwindfunclet$?KillProcess@@YA_NKPAUHWND__@@@Z$0 1003c400 f   Plist.obj
 0001:0003b408       __unwindfunclet$?KillProcess@@YA_NKPAUHWND__@@@Z$1 1003c408 f   Plist.obj
 0001:0003b415       __ehhandler$?KillProcess@@YA_NKPAUHWND__@@@Z 1003c415 f   Plist.obj
 0001:0003b440       __unwindfunclet$?PrintNTCurDirAndEnv@@YAXPAX0H@Z$0 1003c440 f   Plist.obj
 0001:0003b448       __unwindfunclet$?PrintNTCurDirAndEnv@@YAXPAX0H@Z$1 1003c448 f   Plist.obj
 0001:0003b455       __ehhandler$?PrintNTCurDirAndEnv@@YAXPAX0H@Z 1003c455 f   Plist.obj
 0001:0003b480       __unwindfunclet$?print_module_impl@@YAXQAXABV?$basic_string@_WU?$char_traits@_W@std@@V?$allocator@_W@2@@std@@KABUoptions@@ABV?$function@$$A6A_NPA_WI@Z@2@@Z$2 1003c480 f   Plist.obj
 0001:0003b490       __ehhandler$?print_module_impl@@YAXQAXABV?$basic_string@_WU?$char_traits@_W@std@@V?$allocator@_W@2@@std@@KABUoptions@@ABV?$function@$$A6A_NPA_WI@Z@2@@Z 1003c490 f   Plist.obj
 0001:0003b4c0       __unwindfunclet$?PrintModules@@YAXPAXKAAUoptions@@@Z$0 1003c4c0 f   Plist.obj
 0001:0003b4c8       __unwindfunclet$?PrintModules@@YAXPAXKAAUoptions@@@Z$1 1003c4c8 f   Plist.obj
 0001:0003b4d0       __unwindfunclet$?PrintModules@@YAXPAXKAAUoptions@@@Z$2 1003c4d0 f   Plist.obj
 0001:0003b4d8       __unwindfunclet$?PrintModules@@YAXPAXKAAUoptions@@@Z$3 1003c4d8 f   Plist.obj
 0001:0003b4e5       __ehhandler$?PrintModules@@YAXPAXKAAUoptions@@@Z 1003c4e5 f   Plist.obj
 0001:0003b510       __unwindfunclet$?PrintModules@?$ipc_functions@$0A@@@SAXPAX0AAUoptions@@@Z$0 1003c510 f   Plist.obj
 0001:0003b51d       __ehhandler$?PrintModules@?$ipc_functions@$0A@@@SAXPAX0AAUoptions@@@Z 1003c51d f   Plist.obj
 0001:0003b550       __unwindfunclet$?PrintModules@?$ipc_functions@$00@@SAXPAX0AAUoptions@@@Z$0 1003c550 f   Plist.obj
 0001:0003b55d       __ehhandler$?PrintModules@?$ipc_functions@$00@@SAXPAX0AAUoptions@@@Z 1003c55d f   Plist.obj
 0001:0003b590       __ehhandler$?read_string@?$ipc_functions@$0A@@@SA?AV?$basic_string@_WU?$char_traits@_W@std@@V?$allocator@_W@2@@std@@PAXQBX@Z 1003c590 f   Plist.obj
 0001:0003b5b0       __ehhandler$?read_string@?$ipc_functions@$0A@@@SA?AV?$basic_string@_WU?$char_traits@_W@std@@V?$allocator@_W@2@@std@@PAXABUUNICODE_STRING_SAME@detail@@@Z 1003c5b0 f   Plist.obj
 0001:0003b5e0       __ehhandler$?read_string@?$ipc_functions@$00@@SA?AV?$basic_string@_WU?$char_traits@_W@std@@V?$allocator@_W@2@@std@@PAX_K@Z 1003c5e0 f   Plist.obj
 0001:0003b610       __unwindfunclet$?read_string@?$ipc_functions@$00@@SA?AV?$basic_string@_WU?$char_traits@_W@std@@V?$allocator@_W@2@@std@@PAXABUUNICODE_STRING_64@detail@@@Z$0 1003c610 f   Plist.obj
 0001:0003b61d       __ehhandler$?read_string@?$ipc_functions@$00@@SA?AV?$basic_string@_WU?$char_traits@_W@std@@V?$allocator@_W@2@@std@@PAXABUUNICODE_STRING_64@detail@@@Z 1003c61d f   Plist.obj
 0001:0003b650       __unwindfunclet$??$print_module@PAX@@YAXQAXPAXKAAUoptions@@ABV?$function@$$A6A_NPA_WI@Z@std@@@Z$0 1003c650 f   Plist.obj
 0001:0003b65d       __ehhandler$??$print_module@PAX@@YAXQAXPAXKAAUoptions@@ABV?$function@$$A6A_NPA_WI@Z@std@@@Z 1003c65d f   Plist.obj
 0001:0003b690       __unwindfunclet$??$print_module@_K@@YAXQAX_KKAAUoptions@@ABV?$function@$$A6A_NPA_WI@Z@std@@@Z$0 1003c690 f   Plist.obj
 0001:0003b69d       __ehhandler$??$print_module@_K@@YAXQAX_KKAAUoptions@@ABV?$function@$$A6A_NPA_WI@Z@std@@@Z 1003c69d f   Plist.obj
 0001:0003b6d0       __unwindfunclet$??$insert@V?$_List_unchecked_const_iterator@V?$_List_val@U?$_List_simple_types@U?$pair@$$CBKUProcessPerfData@@@std@@@std@@@std@@U_Iterator_base0@2@@std@@@?$_Hash@V?$_Umap_traits@KUProcessPerfData@@V?$_Uhash_compare@KU?$hash@K@std@@U?$equal_to@K@2@@std@@V?$allocator@U?$pair@$$CBKUProcessPerfData@@@std@@@3@$00@std@@@std@@QAEXV?$_List_unchecked_const_iterator@V?$_List_val@U?$_List_simple_types@U?$pair@$$CBKUProcessPerfData@@@std@@@std@@@std@@U_Iterator_base0@2@@1@0@Z$1 1003c6d0 f   Plist.obj
 0001:0003b6d8       __unwindfunclet$??$insert@V?$_List_unchecked_const_iterator@V?$_List_val@U?$_List_simple_types@U?$pair@$$CBKUProcessPerfData@@@std@@@std@@@std@@U_Iterator_base0@2@@std@@@?$_Hash@V?$_Umap_traits@KUProcessPerfData@@V?$_Uhash_compare@KU?$hash@K@std@@U?$equal_to@K@2@@std@@V?$allocator@U?$pair@$$CBKUProcessPerfData@@@std@@@3@$00@std@@@std@@QAEXV?$_List_unchecked_const_iterator@V?$_List_val@U?$_List_simple_types@U?$pair@$$CBKUProcessPerfData@@@std@@@std@@@std@@U_Iterator_base0@2@@1@0@Z$0 1003c6d8 f   Plist.obj
 0001:0003b6e5       __ehhandler$??$insert@V?$_List_unchecked_const_iterator@V?$_List_val@U?$_List_simple_types@U?$pair@$$CBKUProcessPerfData@@@std@@@std@@@std@@U_Iterator_base0@2@@std@@@?$_Hash@V?$_Umap_traits@KUProcessPerfData@@V?$_Uhash_compare@KU?$hash@K@std@@U?$equal_to@K@2@@std@@V?$allocator@U?$pair@$$CBKUProcessPerfData@@@std@@@3@$00@std@@@std@@QAEXV?$_List_unchecked_const_iterator@V?$_List_val@U?$_List_simple_types@U?$pair@$$CBKUProcessPerfData@@@std@@@std@@@std@@U_Iterator_base0@2@@1@0@Z 1003c6e5 f   Plist.obj
 0001:0003b710       __unwindfunclet$?WinError@@YAHPB_W@Z$0 1003c710 f   Pmix.obj
 0001:0003b718       __unwindfunclet$?WinError@@YAHPB_W@Z$1 1003c718 f   Pmix.obj
 0001:0003b725       __ehhandler$?WinError@@YAHPB_W@Z 1003c725 f   Pmix.obj
 0001:0003b750       __unwindfunclet$?GetProcessOwner@WMIConnection@@QAE?AV?$basic_string@_WU?$char_traits@_W@std@@V?$allocator@_W@2@@std@@KPAV23@@Z$0 1003c750 f   wmi.obj
 0001:0003b758       __unwindfunclet$?GetProcessOwner@WMIConnection@@QAE?AV?$basic_string@_WU?$char_traits@_W@std@@V?$allocator@_W@2@@std@@KPAV23@@Z$1 1003c758 f   wmi.obj
 0001:0003b760       __unwindfunclet$?GetProcessOwner@WMIConnection@@QAE?AV?$basic_string@_WU?$char_traits@_W@std@@V?$allocator@_W@2@@std@@KPAV23@@Z$2 1003c760 f   wmi.obj
 0001:0003b768       __unwindfunclet$?GetProcessOwner@WMIConnection@@QAE?AV?$basic_string@_WU?$char_traits@_W@std@@V?$allocator@_W@2@@std@@KPAV23@@Z$3 1003c768 f   wmi.obj
 0001:0003b770       __unwindfunclet$?GetProcessOwner@WMIConnection@@QAE?AV?$basic_string@_WU?$char_traits@_W@std@@V?$allocator@_W@2@@std@@KPAV23@@Z$5 1003c770 f   wmi.obj
 0001:0003b77d       __ehhandler$?GetProcessOwner@WMIConnection@@QAE?AV?$basic_string@_WU?$char_traits@_W@std@@V?$allocator@_W@2@@std@@KPAV23@@Z 1003c77d f   wmi.obj
 0001:0003b7b0       __unwindfunclet$?GetProcessUserSid@WMIConnection@@QAE?AV?$basic_string@_WU?$char_traits@_W@std@@V?$allocator@_W@2@@std@@K@Z$0 1003c7b0 f   wmi.obj
 0001:0003b7b8       __unwindfunclet$?GetProcessUserSid@WMIConnection@@QAE?AV?$basic_string@_WU?$char_traits@_W@std@@V?$allocator@_W@2@@std@@K@Z$1 1003c7b8 f   wmi.obj
 0001:0003b7c0       __unwindfunclet$?GetProcessUserSid@WMIConnection@@QAE?AV?$basic_string@_WU?$char_traits@_W@std@@V?$allocator@_W@2@@std@@K@Z$2 1003c7c0 f   wmi.obj
 0001:0003b7c8       __unwindfunclet$?GetProcessUserSid@WMIConnection@@QAE?AV?$basic_string@_WU?$char_traits@_W@std@@V?$allocator@_W@2@@std@@K@Z$3 1003c7c8 f   wmi.obj
 0001:0003b7d0       __unwindfunclet$?GetProcessUserSid@WMIConnection@@QAE?AV?$basic_string@_WU?$char_traits@_W@std@@V?$allocator@_W@2@@std@@K@Z$5 1003c7d0 f   wmi.obj
 0001:0003b7dd       __ehhandler$?GetProcessUserSid@WMIConnection@@QAE?AV?$basic_string@_WU?$char_traits@_W@std@@V?$allocator@_W@2@@std@@K@Z 1003c7dd f   wmi.obj
 0001:0003b810       __unwindfunclet$?GetProcessSessionId@WMIConnection@@QAEKK@Z$0 1003c810 f   wmi.obj
 0001:0003b81d       __ehhandler$?GetProcessSessionId@WMIConnection@@QAEKK@Z 1003c81d f   wmi.obj
 0001:0003b850       __unwindfunclet$?ExecMethod@WMIConnection@@AAEHKPB_W0K@Z$0 1003c850 f   wmi.obj
 0001:0003b858       __unwindfunclet$?ExecMethod@WMIConnection@@AAEHKPB_W0K@Z$1 1003c858 f   wmi.obj
 0001:0003b860       __unwindfunclet$?ExecMethod@WMIConnection@@AAEHKPB_W0K@Z$2 1003c860 f   wmi.obj
 0001:0003b868       __unwindfunclet$?ExecMethod@WMIConnection@@AAEHKPB_W0K@Z$3 1003c868 f   wmi.obj
 0001:0003b870       __unwindfunclet$?ExecMethod@WMIConnection@@AAEHKPB_W0K@Z$4 1003c870 f   wmi.obj
 0001:0003b878       __unwindfunclet$?ExecMethod@WMIConnection@@AAEHKPB_W0K@Z$5 1003c878 f   wmi.obj
 0001:0003b880       __unwindfunclet$?ExecMethod@WMIConnection@@AAEHKPB_W0K@Z$6 1003c880 f   wmi.obj
 0001:0003b888       __unwindfunclet$?ExecMethod@WMIConnection@@AAEHKPB_W0K@Z$7 1003c888 f   wmi.obj
 0001:0003b890       __unwindfunclet$?ExecMethod@WMIConnection@@AAEHKPB_W0K@Z$8 1003c890 f   wmi.obj
 0001:0003b898       __unwindfunclet$?ExecMethod@WMIConnection@@AAEHKPB_W0K@Z$9 1003c898 f   wmi.obj
 0001:0003b8a0       __unwindfunclet$?ExecMethod@WMIConnection@@AAEHKPB_W0K@Z$10 1003c8a0 f   wmi.obj
 0001:0003b8ad       __ehhandler$?ExecMethod@WMIConnection@@AAEHKPB_W0K@Z 1003c8ad f   wmi.obj
 0001:0003b8d0       __unwindfunclet$?GetProcessProperty@WMIConnection@@AAE_NKPB_WABV?$function@$$A6AXABUtagVARIANT@@@Z@std@@@Z$0 1003c8d0 f   wmi.obj
 0001:0003b8d8       __unwindfunclet$?GetProcessProperty@WMIConnection@@AAE_NKPB_WABV?$function@$$A6AXABUtagVARIANT@@@Z@std@@@Z$1 1003c8d8 f   wmi.obj
 0001:0003b8e0       __unwindfunclet$?GetProcessProperty@WMIConnection@@AAE_NKPB_WABV?$function@$$A6AXABUtagVARIANT@@@Z@std@@@Z$2 1003c8e0 f   wmi.obj
 0001:0003b8ed       __ehhandler$?GetProcessProperty@WMIConnection@@AAE_NKPB_WABV?$function@$$A6AXABUtagVARIANT@@@Z@std@@@Z 1003c8ed f   wmi.obj
 0001:0003b910       __unwindfunclet$?GetProcessInt@WMIConnection@@AAEKKPB_W@Z$0 1003c910 f   wmi.obj
 0001:0003b91d       __ehhandler$?GetProcessInt@WMIConnection@@AAEKKPB_W@Z 1003c91d f   wmi.obj
 0001:0003b950       __unwindfunclet$?GetProcessString@WMIConnection@@AAE?AV?$basic_string@_WU?$char_traits@_W@std@@V?$allocator@_W@2@@std@@KPB_W@Z$0 1003c950 f   wmi.obj
 0001:0003b969       __unwindfunclet$?GetProcessString@WMIConnection@@AAE?AV?$basic_string@_WU?$char_traits@_W@std@@V?$allocator@_W@2@@std@@KPB_W@Z$1 1003c969 f   wmi.obj
 0001:0003b976       __ehhandler$?GetProcessString@WMIConnection@@AAE?AV?$basic_string@_WU?$char_traits@_W@std@@V?$allocator@_W@2@@std@@KPB_W@Z 1003c976 f   wmi.obj
 0001:0003b9a0       __unwindfunclet$?Connect@WMIConnection@@QAE_NPB_W00@Z$0 1003c9a0 f   wmi.obj
 0001:0003b9a8       __unwindfunclet$?Connect@WMIConnection@@QAE_NPB_W00@Z$2 1003c9a8 f   wmi.obj
 0001:0003b9b0       __unwindfunclet$?Connect@WMIConnection@@QAE_NPB_W00@Z$3 1003c9b0 f   wmi.obj
 0001:0003b9b8       __unwindfunclet$?Connect@WMIConnection@@QAE_NPB_W00@Z$4 1003c9b8 f   wmi.obj
 0001:0003b9c0       __unwindfunclet$?Connect@WMIConnection@@QAE_NPB_W00@Z$5 1003c9c0 f   wmi.obj
 0001:0003b9cd       __ehhandler$?Connect@WMIConnection@@QAE_NPB_W00@Z 1003c9cd f   wmi.obj
 0001:0003ba00       __ehhandler$_ProcessPanelEventW@4 1003ca00 f   Proclist.obj
 0001:0003ba27       __unwindfunclet$?_Init@locale@std@@CAPAV_Locimp@12@_N@Z$0 1003ca27 f   libcpmt:locale0.obj
 0001:0003ba34       __ehhandler$?_Init@locale@std@@CAPAV_Locimp@12@_N@Z 1003ca34 f   libcpmt:locale0.obj
 0001:0003ba51       __ehhandler$?CallUnexpected@@YAXPBU_s_ESTypeList@@@Z 1003ca51 f   libvcruntime:frame.obj
 0001:0003ba6e       __unwindfunclet$?_wcstombs_l_helper@@YAIPADPB_WIPAU__crt_locale_pointers@@@Z$0 1003ca6e f   libucrt:wcstombs.obj
 0001:0003ba76       __ehhandler$?_wcstombs_l_helper@@YAIPADPB_WIPAU__crt_locale_pointers@@@Z 1003ca76 f   libucrt:wcstombs.obj
 0001:0003baa0       ??__F?m_PanelModesDataRemote@Plist@@0V?$vector@Umode@@V?$allocator@Umode@@@std@@@std@@A@@YAXXZ 1003caa0 f   fileio.obj
 0001:0003bab0       ??__F?m_PanelModesDataLocal@Plist@@0V?$vector@Umode@@V?$allocator@Umode@@@std@@@std@@A@@YAXXZ 1003cab0 f   fileio.obj
 0001:0003bac0       ??__FUserAccountID@?1??GetUserAccountID@@YA@XZ@YAXXZ 1003cac0 f   handles.obj
 0001:0003bb20       ??__FTitle@?1??GetOpenPanelInfo@Plist@@QAEXPAUOpenPanelInfo@@@Z@YAXXZ 1003cb20 f   Pclass.obj
 0001:0003bb80       ??__FhDebugToken@@YAXXZ    1003cb80 f   Plist.obj
 0001:0003bba0       ??__FDeleter@?1??InitializeSListHead@implementation@slist@@YGXPAT_SLIST_HEADER@@@Z@YAXXZ 1003cba0 f   vc_crt_fix_impl.obj
 0001:0003bbdd       ??__Finitlocks@std@@YAXXZ  1003cbdd f   libcpmt:xlock.obj
 0001:0003bbe7       ??__F_Fac_tidy_reg@std@@YAXXZ 1003cbe7 f   libcpmt:locale0.obj
 0001:0003bbf1       ??__Fclassic_locale@std@@YAXXZ 1003cbf1 f   libcpmt:locale0.obj
 0001:0003bbfb       ??__Finit_atexit@@YAXXZ    1003cbfb f   libcpmt:iosptrs.obj
 0001:0003bc05       ??__Finitlocks@std@@YAXXZ  1003cc05 f   libcpmt:iosptrs.obj
 0002:00000248       ?initlocks$initializer$@std@@3P6AXXZA 1003d248     libcpmt:xlock.obj
 0002:0000024c       ?initlocks$initializer$@std@@3P6AXXZA 1003d24c     libcpmt:iosptrs.obj
 0002:00000250       ?init_atexit$initializer$@@3P6AXXZA 1003d250     libcpmt:iosptrs.obj
 0002:00000254       ?_Fac_tidy_reg$initializer$@std@@3P6AXXZA 1003d254     libcpmt:locale0.obj
 0002:00000258       ?classic_locale$initializer$@std@@3P6AXXZA 1003d258     libcpmt:locale0.obj
 0002:0000025c       ??m_PanelModesDataLocal$initializer$@Plist@@0P6AXXZA@@3P6AXXZA 1003d25c     fileio.obj
 0002:00000260       ??m_PanelModesDataRemote$initializer$@Plist@@0P6AXXZA@@3P6AXXZA 1003d260     fileio.obj
 0002:00000264       ?hDebugToken$initializer$@@3P6AXXZA 1003d264     Plist.obj
 0002:00000270       _pinit                     1003d270     LIBCMT:lconv_unsigned_char.obj
 0002:000003b0       ?_Win_errtab@?A0xa968df57@@3QBU_Win_errtab_t@1@B 1003d3b0     libcpmt:syserror.obj
 0002:00000628       ?_Sys_errtab@?A0xa968df57@@3QBU_Sys_errtab_t@1@B 1003d628     libcpmt:syserror.obj
 0002:00000ec8       ?_Whitespace_bitmap@?A0x3454a962@@3U_Whitespace_bitmap_t@1@B 1003dec8     libcpmt:syserror_import_lib.obj
 0002:00000ff4       _digits                    1003dff4     libcpmt:xstoul.obj
 0002:0000101c       _ndigs                     1003e01c     libcpmt:xstoul.obj
 0002:00001044       _digits                    1003e044     libcpmt:xstoull.obj
 0002:0000106c       _ndigs                     1003e06c     libcpmt:xstoull.obj
 0002:0000109c       _GS_ExceptionPointers      1003e09c     LIBCMT:gs_report.obj
 0002:000010c8       ?tokenTable@@3QBUStringLiteral@@B 1003e0c8     libvcruntime:undname.obj
 0002:00001148       ?nameTable@@3QBUStringLiteral@@B 1003e148     libvcruntime:undname.obj
 0002:000013e0       ?rttiTable@@3QBUStringLiteral@@B 1003e3e0     libvcruntime:undname.obj
 0002:00001408       ?IndirectionName@@3QBUStringLiteral@@B 1003e408     libvcruntime:undname.obj
 0002:00001438       ?PrefixName@@3QBUStringLiteral@@B 1003e438     libvcruntime:undname.obj
 0002:00001a60       ?module_names@?A0x26f6bd02@@3QBQB_WB 1003ea60     libvcruntime:winapi_downlevel.obj
 0002:00001af4       ?candidate_modules@?1??try_get_FlsAlloc@@YAP6GKP6GXPAX@Z@ZXZ@4QBW4module_id@?A0x26f6bd02@@B 1003eaf4     libvcruntime:winapi_downlevel.obj
 0002:00001b08       ?candidate_modules@?1??try_get_FlsFree@@YAP6GHK@ZXZ@4QBW4module_id@?A0x26f6bd02@@B 1003eb08     libvcruntime:winapi_downlevel.obj
 0002:00001b18       ?candidate_modules@?1??try_get_FlsGetValue@@YAP6GPAXK@ZXZ@4QBW4module_id@?A0x26f6bd02@@B 1003eb18     libvcruntime:winapi_downlevel.obj
 0002:00001b2c       ?candidate_modules@?1??try_get_FlsSetValue@@YAP6GHKPAX@ZXZ@4QBW4module_id@?A0x26f6bd02@@B 1003eb2c     libvcruntime:winapi_downlevel.obj
 0002:00001b40       ?candidate_modules@?1??try_get_InitializeCriticalSectionEx@@YAP6GHPAU_RTL_CRITICAL_SECTION@@KK@ZXZ@4QBW4module_id@?A0x26f6bd02@@B 1003eb40     libvcruntime:winapi_downlevel.obj
 0002:00001b48       ?errtable@@3QBUerrentry@?A0x31fdb9ec@@B 1003eb48     libucrt:errno.obj
 0002:00001cb0       _Mantissa                  1003ecb0     libucrt:modf_pentium4.obj
 0002:00001cc0       _Bns                       1003ecc0     libucrt:modf_pentium4.obj
 0002:00001cd0       _Sign                      1003ecd0     libucrt:modf_pentium4.obj
 0002:00001ce0       _Zero                      1003ece0     libucrt:modf_pentium4.obj
 0002:00002590       POW_name                   1003f590     libucrt:pow_impl.obj
 0002:00002668       ___acrt_initializers       1003f668     libucrt:initialization.obj
 0002:000026e8       ?module_names@?A0x391cf84c@@3QBQB_WB 1003f6e8     libucrt:winapi_thunks.obj
 0002:00002b30       ?candidate_modules@?1??try_get_AreFileApisANSI@@YAP6GHXZXZ@4QBW4module_id@?A0x391cf84c@@B 1003fb30     libucrt:winapi_thunks.obj
 0002:00002b44       ?candidate_modules@?1??try_get_CompareStringEx@@YAP6GHPB_WK0H0HPAU_nlsversioninfo@@PAXJ@ZXZ@4QBW4module_id@?A0x391cf84c@@B 1003fb44     libucrt:winapi_thunks.obj
 0002:00002b4c       ?candidate_modules@?1??try_get_EnumSystemLocalesEx@@YAP6GHP6GHPA_WKJ@ZKJPAX@ZXZ@4QBW4module_id@?A0x391cf84c@@B 1003fb4c     libucrt:winapi_thunks.obj
 0002:00002b68       ?candidate_modules@?1??try_get_FlsAlloc@@YAP6GKP6GXPAX@Z@ZXZ@4QBW4module_id@?A0x391cf84c@@B 1003fb68     libucrt:winapi_thunks.obj
 0002:00002b70       ?candidate_modules@?1??try_get_FlsFree@@YAP6GHK@ZXZ@4QBW4module_id@?A0x391cf84c@@B 1003fb70     libucrt:winapi_thunks.obj
 0002:00002b78       ?candidate_modules@?1??try_get_FlsGetValue@@YAP6GPAXK@ZXZ@4QBW4module_id@?A0x391cf84c@@B 1003fb78     libucrt:winapi_thunks.obj
 0002:00002b80       ?candidate_modules@?1??try_get_FlsSetValue@@YAP6GHKPAX@ZXZ@4QBW4module_id@?A0x391cf84c@@B 1003fb80     libucrt:winapi_thunks.obj
 0002:00002b88       ?candidate_modules@?1??try_get_GetDateFormatEx@@YAP6GHPB_WKPBU_SYSTEMTIME@@0PA_WH0@ZXZ@4QBW4module_id@?A0x391cf84c@@B 1003fb88     libucrt:winapi_thunks.obj
 0002:00002ba0       ?candidate_modules@?1??try_get_GetLocaleInfoEx@@YAP6GHPB_WKPA_WH@ZXZ@4QBW4module_id@?A0x391cf84c@@B 1003fba0     libucrt:winapi_thunks.obj
 0002:00002bb8       ?candidate_modules@?1??try_get_GetTimeFormatEx@@YAP6GHPB_WKPBU_SYSTEMTIME@@0PA_WH@ZXZ@4QBW4module_id@?A0x391cf84c@@B 1003fbb8     libucrt:winapi_thunks.obj
 0002:00002bd0       ?candidate_modules@?1??try_get_GetUserDefaultLocaleName@@YAP6GHPA_WH@ZXZ@4QBW4module_id@?A0x391cf84c@@B 1003fbd0     libucrt:winapi_thunks.obj
 0002:00002bf4       ?candidate_modules@?1??try_get_InitializeCriticalSectionEx@@YAP6GHPAU_RTL_CRITICAL_SECTION@@KK@ZXZ@4QBW4module_id@?A0x391cf84c@@B 1003fbf4     libucrt:winapi_thunks.obj
 0002:00002bfc       ?candidate_modules@?1??try_get_IsValidLocaleName@@YAP6GHPB_W@ZXZ@4QBW4module_id@?A0x391cf84c@@B 1003fbfc     libucrt:winapi_thunks.obj
 0002:00002c18       ?candidate_modules@?1??try_get_LCMapStringEx@@YAP6GHPB_WK0HPA_WHPAU_nlsversioninfo@@PAXJ@ZXZ@4QBW4module_id@?A0x391cf84c@@B 1003fc18     libucrt:winapi_thunks.obj
 0002:00002c30       ?candidate_modules@?1??try_get_LCIDToLocaleName@@YAP6GHKPA_WHK@ZXZ@4QBW4module_id@?A0x391cf84c@@B 1003fc30     libucrt:winapi_thunks.obj
 0002:00002c4c       ?candidate_modules@?1??try_get_LocaleNameToLCID@@YAP6GKPB_WK@ZXZ@4QBW4module_id@?A0x391cf84c@@B 1003fc4c     libucrt:winapi_thunks.obj
 0002:00002c68       ?candidate_modules@?1??try_get_AppPolicyGetProcessTerminationMethod@@YAP6GJPAXPAW4AppPolicyProcessTerminationMethod@@@ZXZ@4QBW4module_id@?A0x391cf84c@@B 1003fc68     libucrt:winapi_thunks.obj
 0002:00002c94       ?mask@?P@??_d_int@@9@4QBGB 1003fc94     libucrt:_test.obj
 0002:00002cb4       ?sub@?P@??_d_int@@9@4QBIB  1003fcb4     libucrt:_test.obj
 0002:00002cd8       __first_127char            1003fcd8     libucrt:wsetlocale.obj
 0002:00003338       ?_names@?1??_get_fname@@9@9 10040338     libucrt:fpexcept.obj
 0002:000034e0       _over                      100404e0     libucrt:fpctrl.obj
 0002:000034ec       _under                     100404ec     libucrt:fpctrl.obj
 0002:00003500       Shifter                    10040500     libucrt:pow_pentium4.obj
 0002:00003510       SIGMASK                    10040510     libucrt:pow_pentium4.obj
 0002:00003520       ONEMASK                    10040520     libucrt:pow_pentium4.obj
 0002:00003530       ABSVALMASK                 10040530     libucrt:pow_pentium4.obj
 0002:00003540       cev                        10040540     libucrt:pow_pentium4.obj
 0002:00003568       HALFSIG                    10040568     libucrt:pow_pentium4.obj
 0002:00003570       LHN                        10040570     libucrt:pow_pentium4.obj
 0002:00003578       sNaN                       10040578     libucrt:pow_pentium4.obj
 0002:00003580       INF                        10040580     libucrt:pow_pentium4.obj
 0002:00003588       NEG_INF                    10040588     libucrt:pow_pentium4.obj
 0002:00003590       NEG_ZERO                   10040590     libucrt:pow_pentium4.obj
 0002:00003598       NEG_BIG                    10040598     libucrt:pow_pentium4.obj
 0002:000035a0       POS_BIG                    100405a0     libucrt:pow_pentium4.obj
 0002:000035a8       EMIN                       100405a8     libucrt:pow_pentium4.obj
 0002:000035b0       QIND                       100405b0     libucrt:pow_pentium4.obj
 0002:000035de       _log2max                   100405de     libucrt:87tran.obj
 0002:000035e8       _smallarg                  100405e8     libucrt:87tran.obj
 0002:000035f2       _half                      100405f2     libucrt:87tran.obj
 0002:0000363e       One                        1004063e     libucrt:87disp.obj
 0002:00003646       Three                      10040646     libucrt:87disp.obj
 0002:0000364e       XAMtoTagTab                1004064e     libucrt:87disp.obj
 0002:00003660       One                        10040660     libucrt:common.obj
 0002:00003674       DblMax                     10040674     libucrt:common.obj
 0002:0000367c       DblMin                     1004067c     libucrt:common.obj
 0002:00003684       IeeeAdjO                   10040684     libucrt:common.obj
 0002:0000368c       IeeeAdjU                   1004068c     libucrt:common.obj
 0002:00003694       _infinity                  10040694     libucrt:common.obj
 0002:0000369c       _zero                      1004069c     libucrt:common.obj
 0002:000036a4       ?_mb_locale_names@@3QBQB_WB 100406a4     libucrt:mbctype.obj
 0002:000036e8       ?LcidToLocaleNameTable@?A0x881e4c05@@3QBULcidToLocaleName@1@B 100406e8     libucrt:lcidtoname_downlevel.obj
 0002:00004810       ?LocaleNameToIndexTable@?A0x881e4c05@@3QBULocaleNameIndex@1@B 10041810     libucrt:lcidtoname_downlevel.obj
 0002:00009db0       LOG_name                   10046db0     libucrt:log10_impl.obj
 0002:00009dc0       _One                       10046dc0     libucrt:ceil_pentium4.obj
 0002:00009dd0       _Bns                       10046dd0     libucrt:ceil_pentium4.obj
 0002:00009de0       _Zero                      10046de0     libucrt:ceil_pentium4.obj
 0002:00009df0       _S                         10046df0     libucrt:ceil_pentium4.obj
 0002:00009e00       _NegZero                   10046e00     libucrt:ceil_pentium4.obj
 0002:00009e20       emask                      10046e20     libucrt:log10_pentium4.obj
 0002:00009e30       CC                         10046e30     libucrt:log10_pentium4.obj
 0002:00009e40       Magic                      10046e40     libucrt:log10_pentium4.obj
 0002:00009e50       hi_mask                    10046e50     libucrt:log10_pentium4.obj
 0002:00009e60       LOG10_2                    10046e60     libucrt:log10_pentium4.obj
 0002:00009e70       place_L                    10046e70     libucrt:log10_pentium4.obj
 0002:00009e90       One                        10046e90     libucrt:log10_pentium4.obj
 0002:00009ea0       Zero                       10046ea0     libucrt:log10_pentium4.obj
 0002:00009eb0       Two52                      10046eb0     libucrt:log10_pentium4.obj
 0002:00009ec0       Infs                       10046ec0     libucrt:log10_pentium4.obj
 0002:00009ed0       NaN                        10046ed0     libucrt:log10_pentium4.obj
 0002:00009ee0       coeff                      10046ee0     libucrt:log10_pentium4.obj
 0002:0000a740       two32                      10047740     LIBCMT:ftol2.obj
 0002:0000a744       two63                      10047744     LIBCMT:ftol2.obj
 0002:0000a748       _NaN                       10047748     LIBCMT:ftol2.obj
 0002:0000ab10       ?normal0@?1??is_printable@detail@v10@fmt@@YA_NI@Z@4QBEB 10047b10     format.obj
 0002:0000ae40       ?normal1@?1??is_printable@detail@v10@fmt@@YA_NI@Z@4QBEB 10047e40     format.obj
 0002:0000aff0       ?singletons1_lower@?1??is_printable@detail@v10@fmt@@YA_NI@Z@4QBEB 10047ff0     format.obj
 0002:0000b0a0       ?singletons0@?1??is_printable@detail@v10@fmt@@YA_NI@Z@4QBUsingleton@234@B 100480a0     format.obj
 0002:0000b370       ?singletons0_lower@?1??is_printable@detail@v10@fmt@@YA_NI@Z@4QBEB 10048370     format.obj
 0002:0000b4a0       ?singletons1@?1??is_printable@detail@v10@fmt@@YA_NI@Z@4QBUsingleton@234@B 100484a0     format.obj
 0002:0000b980       ?constStrTypes@@3QBQB_WB   10048980     handles.obj
 0002:0000c6a4       ?StatusCols@?1??InitializePanelModes@Plist@@SAXXZ@4QB_WB 100496a4     Pclass.obj
 0002:0000c6c0       ?ExtStyles@?1??window_ex_style@@YA@PAUHWND__@@@Z@4QBU?$pair@HPB_W@std@@B 100496c0     Pclass.obj
 0002:0000c760       ?PrClasses@?ED@??ProcessKey@Plist@@QAEHPBU_INPUT_RECORD@@@Z@4QBGB 10049760     Pclass.obj
 0002:0000c76c       ?StatusWidths@?1??InitializePanelModes@Plist@@SAXXZ@4QB_WB 1004976c     Pclass.obj
 0002:0000c788       ?Pr@?HB@??ProcessKey@Plist@@QAEHPBU_INPUT_RECORD@@@Z@4QBEB 10049788     Pclass.obj
 0002:0000c790       ?Styles@?1??window_style@@YA@PAUHWND__@@@Z@4QBU?$pair@HPB_W@std@@B 10049790     Pclass.obj
 0002:0000c810       ?invalid_chars@?1??GetFiles@Plist@@QAEHPAUPluginPanelItem@@IHPAPB_W_KAAUoptions@@@Z@4QB_WB 10049810     Pclass.obj
 0002:0000c830       ?StaticItems@?JA@??ProcessKey@Plist@@QAEHPBU_INPUT_RECORD@@@Z@4QBU<unnamed-type-StaticItems>@?JA@??12@QAEH0@Z@B 10049830     Pclass.obj
 0002:0000ce94       ??_7?$_Func_impl_no_alloc@V<lambda_3>@?N@??PrintModules@@YAXPAXKAAUoptions@@@Z@_NPA_WI@std@@6B@ 10049e94     Plist.obj
 0002:0000d054       ??_7?$_Func_impl_no_alloc@V<lambda_1>@?1??GetProcessInt@WMIConnection@@AAEKKPB_W@Z@XABUtagVARIANT@@@std@@6B@ 1004a054     wmi.obj
 0002:0000d070       ??_7?$_Func_impl_no_alloc@V<lambda_1>@?1??GetProcessString@WMIConnection@@AAE?AV?$basic_string@_WU?$char_traits@_W@std@@V?$allocator@_W@2@@std@@KPB_W@Z@XABUtagVARIANT@@@std@@6B@ 1004a070     wmi.obj
 0002:0000d458       ?ntdll@modules@@3QB_WB     1004a458     vc_crt_fix_impl.obj
 0002:0000d464       ?kernel32@modules@@3QB_WB  1004a464     vc_crt_fix_impl.obj
 0002:0000dde4       ??_R4?$_Func_impl_no_alloc@V<lambda_3>@?N@??PrintModules@@YAXPAXKAAUoptions@@@Z@_NPA_WI@std@@6B@ 1004ade4     Plist.obj
 0002:0000ddf8       ??_R3?$_Func_impl_no_alloc@V<lambda_3>@?N@??PrintModules@@YAXPAXKAAUoptions@@@Z@_NPA_WI@std@@8 1004adf8     Plist.obj
 0002:0000de24       ??_R1A@?0A@EA@?$_Func_impl_no_alloc@V<lambda_3>@?N@??PrintModules@@YAXPAXKAAUoptions@@@Z@_NPA_WI@std@@8 1004ae24     Plist.obj
 0002:0000de60       ??_R2?$_Func_impl_no_alloc@V<lambda_3>@?N@??PrintModules@@YAXPAXKAAUoptions@@@Z@_NPA_WI@std@@8 1004ae60     Plist.obj
 0002:0000de6c       ??_R4?$_Func_impl_no_alloc@V<lambda_1>@?1??GetProcessString@WMIConnection@@AAE?AV?$basic_string@_WU?$char_traits@_W@std@@V?$allocator@_W@2@@std@@KPB_W@Z@XABUtagVARIANT@@@std@@6B@ 1004ae6c     wmi.obj
 0002:0000deac       ??_R3?$_Func_impl_no_alloc@V<lambda_1>@?1??GetProcessInt@WMIConnection@@AAEKKPB_W@Z@XABUtagVARIANT@@@std@@8 1004aeac     wmi.obj
 0002:0000debc       ??_R2?$_Func_impl_no_alloc@V<lambda_1>@?1??GetProcessString@WMIConnection@@AAE?AV?$basic_string@_WU?$char_traits@_W@std@@V?$allocator@_W@2@@std@@KPB_W@Z@XABUtagVARIANT@@@std@@8 1004aebc     wmi.obj
 0002:0000dec8       ??_R1A@?0A@EA@?$_Func_impl_no_alloc@V<lambda_1>@?1??GetProcessInt@WMIConnection@@AAEKKPB_W@Z@XABUtagVARIANT@@@std@@8 1004aec8     wmi.obj
 0002:0000dee4       ??_R1A@?0A@EA@?$_Func_impl_no_alloc@V<lambda_1>@?1??GetProcessString@WMIConnection@@AAE?AV?$basic_string@_WU?$char_traits@_W@std@@V?$allocator@_W@2@@std@@KPB_W@Z@XABUtagVARIANT@@@std@@8 1004aee4     wmi.obj
 0002:0000df08       ??_R3?$_Func_impl_no_alloc@V<lambda_1>@?1??GetProcessString@WMIConnection@@AAE?AV?$basic_string@_WU?$char_traits@_W@std@@V?$allocator@_W@2@@std@@KPB_W@Z@XABUtagVARIANT@@@std@@8 1004af08     wmi.obj
 0002:0000df18       ??_R2?$_Func_impl_no_alloc@V<lambda_1>@?1??GetProcessInt@WMIConnection@@AAEKKPB_W@Z@XABUtagVARIANT@@@std@@8 1004af18     wmi.obj
 0002:0000df24       ??_R4?$_Func_impl_no_alloc@V<lambda_1>@?1??GetProcessInt@WMIConnection@@AAEKKPB_W@Z@XABUtagVARIANT@@@std@@6B@ 1004af24     wmi.obj
 0002:0000e4c8       __ehfuncinfo$?adjust_precision@detail@v10@fmt@@YAXAAHH@Z 1004b4c8     format.obj
 0002:0000e4ec       __unwindtable$?adjust_precision@detail@v10@fmt@@YAXAAHH@Z 1004b4ec     format.obj
 0002:0000e4f4       __ehfuncinfo$?square@bigint@detail@v10@fmt@@QAEXXZ 1004b4f4     format.obj
 0002:0000e518       __unwindtable$?square@bigint@detail@v10@fmt@@QAEXXZ 1004b518     format.obj
 0002:0000e528       __ehfuncinfo$?format_dragon@detail@v10@fmt@@YAXU?$basic_fp@Vuint128_fallback@detail@v10@fmt@@@123@IHAAV?$buffer@D@123@AAH@Z 1004b528     format.obj
 0002:0000e54c       __unwindtable$?format_dragon@detail@v10@fmt@@YAXU?$basic_fp@Vuint128_fallback@detail@v10@fmt@@@123@IHAAV?$buffer@D@123@AAH@Z 1004b54c     format.obj
 0002:0000e56c       __ehfuncinfo$??0_Locinfo@std@@QAE@PBD@Z 1004b56c     format.obj
 0002:0000e590       __unwindtable$??0_Locinfo@std@@QAE@PBD@Z 1004b590     format.obj
 0002:0000e5c8       __ehfuncinfo$??1PluginDialogBuilder@@QAE@XZ 1004b5c8     Pcfg.obj
 0002:0000e5c8       __ehfuncinfo$??1PluginSettings@@QAE@XZ 1004b5c8     Pcfg.obj
 0002:0000e5c8       __ehfuncinfo$??1_Locinfo@std@@QAE@XZ 1004b5c8     format.obj
 0002:0000e5c8       __ehfuncinfo$??1?$unique_ptr@UIWbemClassObject@@Ucom_closer@@@std@@QAE@XZ 1004b5c8     wmi.obj
 0002:0000e5c8       __ehfuncinfo$??1?$unique_ptr@UIWbemLocator@@Ucom_closer@@@std@@QAE@XZ 1004b5c8     wmi.obj
 0002:0000e5c8       __ehfuncinfo$??1WMIConnection@@QAE@XZ 1004b5c8     wmi.obj
 0002:0000e5c8       __ehfuncinfo$??1_Init_atexit@@QAE@XZ 1004b5c8     libcpmt:iosptrs.obj
 0002:0000e5ec       __ehfuncinfo$?throw_format_error@detail@v10@fmt@@YAXPBD@Z 1004b5ec     format.obj
 0002:0000e610       __unwindtable$?throw_format_error@detail@v10@fmt@@YAXPBD@Z 1004b610     format.obj
 0002:0000e618       __ehfuncinfo$?read_string@?$ipc_functions@$00@@SA?AV?$basic_string@_WU?$char_traits@_W@std@@V?$allocator@_W@2@@std@@PAX_K@Z 1004b618     Plist.obj
 0002:0000e618       __ehfuncinfo$?read_string@?$ipc_functions@$0A@@@SA?AV?$basic_string@_WU?$char_traits@_W@std@@V?$allocator@_W@2@@std@@PAXQBX@Z 1004b618     Plist.obj
 0002:0000e618       __ehfuncinfo$_ProcessPanelEventW@4 1004b618     Proclist.obj
 0002:0000e618       __ehfuncinfo$??0?$basic_string@_WU?$char_traits@_W@std@@V?$allocator@_W@2@@std@@QAE@QB_W@Z 1004b618     format.obj
 0002:0000e618       __ehfuncinfo$?do_falsename@?$numpunct@_W@std@@MBE?AV?$basic_string@_WU?$char_traits@_W@std@@V?$allocator@_W@2@@2@XZ 1004b618     format.obj
 0002:0000e618       __ehfuncinfo$?do_grouping@?$numpunct@_W@std@@MBE?AV?$basic_string@DU?$char_traits@D@std@@V?$allocator@D@2@@2@XZ 1004b618     format.obj
 0002:0000e618       __ehfuncinfo$?do_truename@?$numpunct@_W@std@@MBE?AV?$basic_string@_WU?$char_traits@_W@std@@V?$allocator@_W@2@@2@XZ 1004b618     format.obj
 0002:0000e618       __ehfuncinfo$??$?0V?$basic_string_view@_WU?$char_traits@_W@std@@@std@@$0A@@?$basic_string@_WU?$char_traits@_W@std@@V?$allocator@_W@2@@std@@QAE@ABV?$basic_string_view@_WU?$char_traits@_W@std@@@1@ABV?$allocator@_W@1@@Z 1004b618     handles.obj
 0002:0000e618       __ehfuncinfo$??__Ks@string_literals@literals@std@@YA?AV?$basic_string@_WU?$char_traits@_W@std@@V?$allocator@_W@2@@3@PB_WI@Z 1004b618     handles.obj
 0002:0000e63c       __unwindtable$?read_string@?$ipc_functions@$00@@SA?AV?$basic_string@_WU?$char_traits@_W@std@@V?$allocator@_W@2@@std@@PAX_K@Z 1004b63c     Plist.obj
 0002:0000e63c       __unwindtable$?read_string@?$ipc_functions@$0A@@@SA?AV?$basic_string@_WU?$char_traits@_W@std@@V?$allocator@_W@2@@std@@PAXQBX@Z 1004b63c     Plist.obj
 0002:0000e63c       __unwindtable$_ProcessPanelEventW@4 1004b63c     Proclist.obj
 0002:0000e63c       __unwindtable$??0?$basic_string@_WU?$char_traits@_W@std@@V?$allocator@_W@2@@std@@QAE@QB_W@Z 1004b63c     format.obj
 0002:0000e63c       __unwindtable$?do_falsename@?$numpunct@_W@std@@MBE?AV?$basic_string@_WU?$char_traits@_W@std@@V?$allocator@_W@2@@2@XZ 1004b63c     format.obj
 0002:0000e63c       __unwindtable$?do_grouping@?$numpunct@_W@std@@MBE?AV?$basic_string@DU?$char_traits@D@std@@V?$allocator@D@2@@2@XZ 1004b63c     format.obj
 0002:0000e63c       __unwindtable$?do_truename@?$numpunct@_W@std@@MBE?AV?$basic_string@_WU?$char_traits@_W@std@@V?$allocator@_W@2@@2@XZ 1004b63c     format.obj
 0002:0000e63c       __unwindtable$??$?0V?$basic_string_view@_WU?$char_traits@_W@std@@@std@@$0A@@?$basic_string@_WU?$char_traits@_W@std@@V?$allocator@_W@2@@std@@QAE@ABV?$basic_string_view@_WU?$char_traits@_W@std@@@1@ABV?$allocator@_W@1@@Z 1004b63c     handles.obj
 0002:0000e63c       __unwindtable$??__Ks@string_literals@literals@std@@YA?AV?$basic_string@_WU?$char_traits@_W@std@@V?$allocator@_W@2@@3@PB_WI@Z 1004b63c     handles.obj
 0002:0000e644       __ehfuncinfo$??$use_facet@V?$numpunct@_W@std@@@std@@YAABV?$numpunct@_W@0@ABVlocale@0@@Z 1004b644     format.obj
 0002:0000e668       __unwindtable$??$use_facet@V?$numpunct@_W@std@@@std@@YAABV?$numpunct@_W@0@ABVlocale@0@@Z 1004b668     format.obj
 0002:0000e6a0       __ehfuncinfo$??$decimal_point@_W@detail@v10@fmt@@YA_WVlocale_ref@012@@Z 1004b6a0     handles.obj
 0002:0000e6c4       __unwindtable$??$decimal_point@_W@detail@v10@fmt@@YA_WVlocale_ref@012@@Z 1004b6c4     handles.obj
 0002:0000e6d8       __ehfuncinfo$?write_loc@detail@v10@fmt@@YA_NV?$back_insert_iterator@V?$buffer@_W@detail@v10@fmt@@@std@@Vloc_value@23@ABU?$format_specs@_W@23@Vlocale_ref@123@@Z 1004b6d8     handles.obj
 0002:0000e700       __unwindtable$?write_loc@detail@v10@fmt@@YA_NV?$back_insert_iterator@V?$buffer@_W@detail@v10@fmt@@@std@@Vloc_value@23@ABU?$format_specs@_W@23@Vlocale_ref@123@@Z 1004b700     handles.obj
 0002:0000e758       __ehfuncinfo$?query_object@@YA?AV?$unique_ptr@$$BY0A@DU?$default_delete@$$BY0A@D@std@@@std@@PAXW4_OBJECT_INFORMATION_CLASS@@@Z 1004b758     handles.obj
 0002:0000e77c       __unwindtable$?query_object@@YA?AV?$unique_ptr@$$BY0A@DU?$default_delete@$$BY0A@D@std@@@std@@PAXW4_OBJECT_INFORMATION_CLASS@@@Z 1004b77c     handles.obj
 0002:0000e784       __ehfuncinfo$?GetFileName@@YA?AV?$basic_string@_WU?$char_traits@_W@std@@V?$allocator@_W@2@@std@@PAX@Z 1004b784     handles.obj
 0002:0000e7a8       __unwindtable$?GetFileName@@YA?AV?$basic_string@_WU?$char_traits@_W@std@@V?$allocator@_W@2@@std@@PAX@Z 1004b7a8     handles.obj
 0002:0000e7c8       __ehfuncinfo$??R<lambda_1>@?1??GetUserAccountID@@YA@XZ@QBE?AV?$basic_string@_WU?$char_traits@_W@std@@V?$allocator@_W@2@@std@@XZ 1004b7c8     handles.obj
 0002:0000e7ec       __unwindtable$??R<lambda_1>@?1??GetUserAccountID@@YA@XZ@QBE?AV?$basic_string@_WU?$char_traits@_W@std@@V?$allocator@_W@2@@std@@XZ 1004b7ec     handles.obj
 0002:0000e828       __ehfuncinfo$?GetNameByType@@YA?AV?$basic_string@_WU?$char_traits@_W@std@@V?$allocator@_W@2@@std@@PAXGPAVPerfThread@@@Z 1004b828     handles.obj
 0002:0000e850       __unwindtable$?GetNameByType@@YA?AV?$basic_string@_WU?$char_traits@_W@std@@V?$allocator@_W@2@@std@@PAXGPAVPerfThread@@@Z 1004b850     handles.obj
 0002:0000e8a0       __ehfuncinfo$?PrintHandleInfo@@YA_NKPAX_NPAVPerfThread@@@Z 1004b8a0     handles.obj
 0002:0000e8c4       __unwindtable$?PrintHandleInfo@@YA_NKPAX_NPAVPerfThread@@@Z 1004b8c4     handles.obj
 0002:0000e8fc       __ehfuncinfo$??0?$basic_string@_WU?$char_traits@_W@std@@V?$allocator@_W@2@@std@@QAE@$$QAV01@@Z 1004b8fc     handles.obj
 0002:0000e8fc       __ehfuncinfo$??4?$basic_string@_WU?$char_traits@_W@std@@V?$allocator@_W@2@@std@@QAEAAV01@$$QAV01@@Z 1004b8fc     handles.obj
 0002:0000e920       __unwindtable$??0?$basic_string@_WU?$char_traits@_W@std@@V?$allocator@_W@2@@std@@QAE@$$QAV01@@Z 1004b920     handles.obj
 0002:0000e920       __unwindtable$??4?$basic_string@_WU?$char_traits@_W@std@@V?$allocator@_W@2@@std@@QAEAAV01@$$QAV01@@Z 1004b920     handles.obj
 0002:0000e930       __ehfuncinfo$??1?$unique_ptr@VWMIConnection@@U?$default_delete@VWMIConnection@@@std@@@std@@QAE@XZ 1004b930     Pclass.obj
 0002:0000e930       __ehfuncinfo$?reset@?$unique_ptr@VWMIConnection@@U?$default_delete@VWMIConnection@@@std@@@std@@QAEXPAVWMIConnection@@@Z 1004b930     Pclass.obj
 0002:0000e930       __ehfuncinfo$??0?$basic_string@_WU?$char_traits@_W@std@@V?$allocator@_W@2@@std@@QAE@XZ 1004b930     handles.obj
 0002:0000e930       __ehfuncinfo$??1PerfThread@@QAE@XZ 1004b930     perfthread.obj
 0002:0000e930       __ehfuncinfo$??1?$ptr_setter@V?$unique_ptr@UIWbemClassObject@@Ucom_closer@@@std@@@@QAE@XZ 1004b930     wmi.obj
 0002:0000e954       __unwindtable$??1?$unique_ptr@VWMIConnection@@U?$default_delete@VWMIConnection@@@std@@@std@@QAE@XZ 1004b954     Pclass.obj
 0002:0000e954       __unwindtable$?reset@?$unique_ptr@VWMIConnection@@U?$default_delete@VWMIConnection@@@std@@@std@@QAEXPAVWMIConnection@@@Z 1004b954     Pclass.obj
 0002:0000e954       __unwindtable$??0?$basic_string@_WU?$char_traits@_W@std@@V?$allocator@_W@2@@std@@QAE@XZ 1004b954     handles.obj
 0002:0000e954       __unwindtable$??1PerfThread@@QAE@XZ 1004b954     perfthread.obj
 0002:0000e954       __unwindtable$??1?$ptr_setter@V?$unique_ptr@UIWbemClassObject@@Ucom_closer@@@std@@@@QAE@XZ 1004b954     wmi.obj
 0002:0000e95c       __ehfuncinfo$??$vformat@_W$0A@@v10@fmt@@YA?AV?$basic_string@_WU?$char_traits@_W@std@@V?$allocator@_W@2@@std@@V?$basic_string_view@_W@01@V?$basic_format_args@V?$basic_format_context@V?$back_insert_iterator@V?$buffer@_W@detail@v10@fmt@@@std@@_W@v10@fmt@@@01@@Z 1004b95c     handles.obj
 0002:0000e980       __unwindtable$??$vformat@_W$0A@@v10@fmt@@YA?AV?$basic_string@_WU?$char_traits@_W@std@@V?$allocator@_W@2@@std@@V?$basic_string_view@_W@01@V?$basic_format_args@V?$basic_format_context@V?$back_insert_iterator@V?$buffer@_W@detail@v10@fmt@@@std@@_W@v10@fmt@@@01@@Z 1004b980     handles.obj
 0002:0000e998       __ehfuncinfo$??$visit_format_arg@AAU?$loc_writer@_W@detail@v10@fmt@@V?$basic_format_context@Vappender@v10@fmt@@D@34@@v10@fmt@@YA_NAAU?$loc_writer@_W@detail@01@ABV?$basic_format_arg@V?$basic_format_context@Vappender@v10@fmt@@D@v10@fmt@@@01@@Z 1004b998     handles.obj
 0002:0000e9c0       __unwindtable$??$visit_format_arg@AAU?$loc_writer@_W@detail@v10@fmt@@V?$basic_format_context@Vappender@v10@fmt@@D@34@@v10@fmt@@YA_NAAU?$loc_writer@_W@detail@01@ABV?$basic_format_arg@V?$basic_format_context@Vappender@v10@fmt@@D@v10@fmt@@@01@@Z 1004b9c0     handles.obj
 0002:0000ea40       __ehfuncinfo$??$parse_format_string@$0A@_WUformat_handler@?1???$vformat_to@_W@detail@v10@fmt@@YAXAAV?$buffer@_W@234@V?$basic_string_view@_W@34@V?$basic_format_args@V?$basic_format_context@V?$back_insert_iterator@V?$buffer@_W@detail@v10@fmt@@@std@@_W@v10@fmt@@@34@Vlocale_ref@234@@Z@@detail@v10@fmt@@YAXV?$basic_string_view@_W@12@$$QAUformat_handler@?1???$vformat_to@_W@012@YAXAAV?$buffer@_W@012@0V?$basic_format_args@V?$basic_format_context@V?$back_insert_iterator@V?$buffer@_W@detail@v10@fmt@@@std@@_W@v10@fmt@@@12@Vlocale_ref@012@@Z@@Z 1004ba40     handles.obj
 0002:0000ea64       __unwindtable$??$parse_format_string@$0A@_WUformat_handler@?1???$vformat_to@_W@detail@v10@fmt@@YAXAAV?$buffer@_W@234@V?$basic_string_view@_W@34@V?$basic_format_args@V?$basic_format_context@V?$back_insert_iterator@V?$buffer@_W@detail@v10@fmt@@@std@@_W@v10@fmt@@@34@Vlocale_ref@234@@Z@@detail@v10@fmt@@YAXV?$basic_string_view@_W@12@$$QAUformat_handler@?1???$vformat_to@_W@012@YAXAAV?$buffer@_W@012@0V?$basic_format_args@V?$basic_format_context@V?$back_insert_iterator@V?$buffer@_W@detail@v10@fmt@@@std@@_W@v10@fmt@@@12@Vlocale_ref@012@@Z@@Z 1004ba64     handles.obj
 0002:0000ea6c       __ehfuncinfo$??0?$digit_grouping@_W@detail@v10@fmt@@QAE@V?$basic_string@DU?$char_traits@D@std@@V?$allocator@D@2@@std@@V?$basic_string@_WU?$char_traits@_W@std@@V?$allocator@_W@2@@5@@Z 1004ba6c     handles.obj
 0002:0000ea90       __unwindtable$??0?$digit_grouping@_W@detail@v10@fmt@@QAE@V?$basic_string@DU?$char_traits@D@std@@V?$allocator@D@2@@std@@V?$basic_string@_WU?$char_traits@_W@std@@V?$allocator@_W@2@@5@@Z 1004ba90     handles.obj
 0002:0000eab0       __ehfuncinfo$??$apply@V?$back_insert_iterator@V?$buffer@_W@detail@v10@fmt@@@std@@D@?$digit_grouping@_W@detail@v10@fmt@@QBE?AV?$back_insert_iterator@V?$buffer@_W@detail@v10@fmt@@@std@@V45@V?$basic_string_view@D@23@@Z 1004bab0     handles.obj
 0002:0000eab0       __ehfuncinfo$??$apply@V?$back_insert_iterator@V?$buffer@_W@detail@v10@fmt@@@std@@_W@?$digit_grouping@_W@detail@v10@fmt@@QBE?AV?$back_insert_iterator@V?$buffer@_W@detail@v10@fmt@@@std@@V45@V?$basic_string_view@_W@23@@Z 1004bab0     handles.obj
 0002:0000ead4       __unwindtable$??$apply@V?$back_insert_iterator@V?$buffer@_W@detail@v10@fmt@@@std@@D@?$digit_grouping@_W@detail@v10@fmt@@QBE?AV?$back_insert_iterator@V?$buffer@_W@detail@v10@fmt@@@std@@V45@V?$basic_string_view@D@23@@Z 1004bad4     handles.obj
 0002:0000ead4       __unwindtable$??$apply@V?$back_insert_iterator@V?$buffer@_W@detail@v10@fmt@@@std@@_W@?$digit_grouping@_W@detail@v10@fmt@@QBE?AV?$back_insert_iterator@V?$buffer@_W@detail@v10@fmt@@@std@@V45@V?$basic_string_view@_W@23@@Z 1004bad4     handles.obj
 0002:0000eadc       __ehfuncinfo$??$write_float@_WV?$back_insert_iterator@V?$buffer@_W@detail@v10@fmt@@@std@@M@detail@v10@fmt@@YA?AV?$back_insert_iterator@V?$buffer@_W@detail@v10@fmt@@@std@@V34@MU?$format_specs@_W@12@Vlocale_ref@012@@Z 1004badc     handles.obj
 0002:0000eb00       __unwindtable$??$write_float@_WV?$back_insert_iterator@V?$buffer@_W@detail@v10@fmt@@@std@@M@detail@v10@fmt@@YA?AV?$back_insert_iterator@V?$buffer@_W@detail@v10@fmt@@@std@@V34@MU?$format_specs@_W@12@Vlocale_ref@012@@Z 1004bb00     handles.obj
 0002:0000eb08       __ehfuncinfo$??$write_float@_WV?$back_insert_iterator@V?$buffer@_W@detail@v10@fmt@@@std@@N@detail@v10@fmt@@YA?AV?$back_insert_iterator@V?$buffer@_W@detail@v10@fmt@@@std@@V34@NU?$format_specs@_W@12@Vlocale_ref@012@@Z 1004bb08     handles.obj
 0002:0000eb08       __ehfuncinfo$??$write_float@_WV?$back_insert_iterator@V?$buffer@_W@detail@v10@fmt@@@std@@O@detail@v10@fmt@@YA?AV?$back_insert_iterator@V?$buffer@_W@detail@v10@fmt@@@std@@V34@OU?$format_specs@_W@12@Vlocale_ref@012@@Z 1004bb08     handles.obj
 0002:0000eb2c       __unwindtable$??$write_float@_WV?$back_insert_iterator@V?$buffer@_W@detail@v10@fmt@@@std@@N@detail@v10@fmt@@YA?AV?$back_insert_iterator@V?$buffer@_W@detail@v10@fmt@@@std@@V34@NU?$format_specs@_W@12@Vlocale_ref@012@@Z 1004bb2c     handles.obj
 0002:0000eb2c       __unwindtable$??$write_float@_WV?$back_insert_iterator@V?$buffer@_W@detail@v10@fmt@@@std@@O@detail@v10@fmt@@YA?AV?$back_insert_iterator@V?$buffer@_W@detail@v10@fmt@@@std@@V34@OU?$format_specs@_W@12@Vlocale_ref@012@@Z 1004bb2c     handles.obj
 0002:0000eb34       __ehfuncinfo$??$do_write_float@V?$back_insert_iterator@V?$buffer@_W@detail@v10@fmt@@@std@@U?$decimal_fp@M@dragonbox@detail@v10@fmt@@_WV?$digit_grouping@_W@567@@detail@v10@fmt@@YA?AV?$back_insert_iterator@V?$buffer@_W@detail@v10@fmt@@@std@@V34@ABU?$decimal_fp@M@dragonbox@012@ABU?$format_specs@_W@12@Ufloat_specs@012@Vlocale_ref@012@@Z 1004bb34     handles.obj
 0002:0000eb34       __ehfuncinfo$??$do_write_float@V?$back_insert_iterator@V?$buffer@_W@detail@v10@fmt@@@std@@Ubig_decimal_fp@detail@v10@fmt@@_WV?$digit_grouping@_W@456@@detail@v10@fmt@@YA?AV?$back_insert_iterator@V?$buffer@_W@detail@v10@fmt@@@std@@V34@ABUbig_decimal_fp@012@ABU?$format_specs@_W@12@Ufloat_specs@012@Vlocale_ref@012@@Z 1004bb34     handles.obj
 0002:0000eb58       __unwindtable$??$do_write_float@V?$back_insert_iterator@V?$buffer@_W@detail@v10@fmt@@@std@@U?$decimal_fp@M@dragonbox@detail@v10@fmt@@_WV?$digit_grouping@_W@567@@detail@v10@fmt@@YA?AV?$back_insert_iterator@V?$buffer@_W@detail@v10@fmt@@@std@@V34@ABU?$decimal_fp@M@dragonbox@012@ABU?$format_specs@_W@12@Ufloat_specs@012@Vlocale_ref@012@@Z 1004bb58     handles.obj
 0002:0000eb58       __unwindtable$??$do_write_float@V?$back_insert_iterator@V?$buffer@_W@detail@v10@fmt@@@std@@Ubig_decimal_fp@detail@v10@fmt@@_WV?$digit_grouping@_W@456@@detail@v10@fmt@@YA?AV?$back_insert_iterator@V?$buffer@_W@detail@v10@fmt@@@std@@V34@ABUbig_decimal_fp@012@ABU?$format_specs@_W@12@Ufloat_specs@012@Vlocale_ref@012@@Z 1004bb58     handles.obj
 0002:0000eb68       __ehfuncinfo$??R<lambda_3>@?BD@???$do_write_float@V?$back_insert_iterator@V?$buffer@_W@detail@v10@fmt@@@std@@U?$decimal_fp@M@dragonbox@detail@v10@fmt@@_WV?$digit_grouping@_W@567@@detail@v10@fmt@@YA?AV?$back_insert_iterator@V?$buffer@_W@detail@v10@fmt@@@std@@V45@ABU?$decimal_fp@M@dragonbox@123@ABU?$format_specs@_W@23@Ufloat_specs@123@Vlocale_ref@123@@Z@QBE@0@Z 1004bb68     handles.obj
 0002:0000eb8c       __unwindtable$??R<lambda_3>@?BD@???$do_write_float@V?$back_insert_iterator@V?$buffer@_W@detail@v10@fmt@@@std@@U?$decimal_fp@M@dragonbox@detail@v10@fmt@@_WV?$digit_grouping@_W@567@@detail@v10@fmt@@YA?AV?$back_insert_iterator@V?$buffer@_W@detail@v10@fmt@@@std@@V45@ABU?$decimal_fp@M@dragonbox@123@ABU?$format_specs@_W@23@Ufloat_specs@123@Vlocale_ref@123@@Z@QBE@0@Z 1004bb8c     handles.obj
 0002:0000eb94       __ehfuncinfo$??R<lambda_4>@?BO@???$do_write_float@V?$back_insert_iterator@V?$buffer@_W@detail@v10@fmt@@@std@@U?$decimal_fp@M@dragonbox@detail@v10@fmt@@_WV?$digit_grouping@_W@567@@detail@v10@fmt@@YA?AV?$back_insert_iterator@V?$buffer@_W@detail@v10@fmt@@@std@@V45@ABU?$decimal_fp@M@dragonbox@123@ABU?$format_specs@_W@23@Ufloat_specs@123@Vlocale_ref@123@@Z@QBE@0@Z 1004bb94     handles.obj
 0002:0000eb94       __ehfuncinfo$??R<lambda_4>@?BO@???$do_write_float@V?$back_insert_iterator@V?$buffer@_W@detail@v10@fmt@@@std@@Ubig_decimal_fp@detail@v10@fmt@@_WV?$digit_grouping@_W@456@@detail@v10@fmt@@YA?AV?$back_insert_iterator@V?$buffer@_W@detail@v10@fmt@@@std@@V45@ABUbig_decimal_fp@123@ABU?$format_specs@_W@23@Ufloat_specs@123@Vlocale_ref@123@@Z@QBE@0@Z 1004bb94     handles.obj
 0002:0000ebb8       __unwindtable$??R<lambda_4>@?BO@???$do_write_float@V?$back_insert_iterator@V?$buffer@_W@detail@v10@fmt@@@std@@U?$decimal_fp@M@dragonbox@detail@v10@fmt@@_WV?$digit_grouping@_W@567@@detail@v10@fmt@@YA?AV?$back_insert_iterator@V?$buffer@_W@detail@v10@fmt@@@std@@V45@ABU?$decimal_fp@M@dragonbox@123@ABU?$format_specs@_W@23@Ufloat_specs@123@Vlocale_ref@123@@Z@QBE@0@Z 1004bbb8     handles.obj
 0002:0000ebb8       __unwindtable$??R<lambda_4>@?BO@???$do_write_float@V?$back_insert_iterator@V?$buffer@_W@detail@v10@fmt@@@std@@Ubig_decimal_fp@detail@v10@fmt@@_WV?$digit_grouping@_W@456@@detail@v10@fmt@@YA?AV?$back_insert_iterator@V?$buffer@_W@detail@v10@fmt@@@std@@V45@ABUbig_decimal_fp@123@ABU?$format_specs@_W@23@Ufloat_specs@123@Vlocale_ref@123@@Z@QBE@0@Z 1004bbb8     handles.obj
 0002:0000ebc0       __ehfuncinfo$??$do_write_float@V?$back_insert_iterator@V?$buffer@_W@detail@v10@fmt@@@std@@U?$decimal_fp@N@dragonbox@detail@v10@fmt@@_WV?$digit_grouping@_W@567@@detail@v10@fmt@@YA?AV?$back_insert_iterator@V?$buffer@_W@detail@v10@fmt@@@std@@V34@ABU?$decimal_fp@N@dragonbox@012@ABU?$format_specs@_W@12@Ufloat_specs@012@Vlocale_ref@012@@Z 1004bbc0     handles.obj
 0002:0000ebe4       __unwindtable$??$do_write_float@V?$back_insert_iterator@V?$buffer@_W@detail@v10@fmt@@@std@@U?$decimal_fp@N@dragonbox@detail@v10@fmt@@_WV?$digit_grouping@_W@567@@detail@v10@fmt@@YA?AV?$back_insert_iterator@V?$buffer@_W@detail@v10@fmt@@@std@@V34@ABU?$decimal_fp@N@dragonbox@012@ABU?$format_specs@_W@12@Ufloat_specs@012@Vlocale_ref@012@@Z 1004bbe4     handles.obj
 0002:0000ebf4       __ehfuncinfo$??R<lambda_3>@?BD@???$do_write_float@V?$back_insert_iterator@V?$buffer@_W@detail@v10@fmt@@@std@@U?$decimal_fp@N@dragonbox@detail@v10@fmt@@_WV?$digit_grouping@_W@567@@detail@v10@fmt@@YA?AV?$back_insert_iterator@V?$buffer@_W@detail@v10@fmt@@@std@@V45@ABU?$decimal_fp@N@dragonbox@123@ABU?$format_specs@_W@23@Ufloat_specs@123@Vlocale_ref@123@@Z@QBE@0@Z 1004bbf4     handles.obj
 0002:0000ec18       __unwindtable$??R<lambda_3>@?BD@???$do_write_float@V?$back_insert_iterator@V?$buffer@_W@detail@v10@fmt@@@std@@U?$decimal_fp@N@dragonbox@detail@v10@fmt@@_WV?$digit_grouping@_W@567@@detail@v10@fmt@@YA?AV?$back_insert_iterator@V?$buffer@_W@detail@v10@fmt@@@std@@V45@ABU?$decimal_fp@N@dragonbox@123@ABU?$format_specs@_W@23@Ufloat_specs@123@Vlocale_ref@123@@Z@QBE@0@Z 1004bc18     handles.obj
 0002:0000ec20       __ehfuncinfo$??R<lambda_4>@?BO@???$do_write_float@V?$back_insert_iterator@V?$buffer@_W@detail@v10@fmt@@@std@@U?$decimal_fp@N@dragonbox@detail@v10@fmt@@_WV?$digit_grouping@_W@567@@detail@v10@fmt@@YA?AV?$back_insert_iterator@V?$buffer@_W@detail@v10@fmt@@@std@@V45@ABU?$decimal_fp@N@dragonbox@123@ABU?$format_specs@_W@23@Ufloat_specs@123@Vlocale_ref@123@@Z@QBE@0@Z 1004bc20     handles.obj
 0002:0000ec44       __unwindtable$??R<lambda_4>@?BO@???$do_write_float@V?$back_insert_iterator@V?$buffer@_W@detail@v10@fmt@@@std@@U?$decimal_fp@N@dragonbox@detail@v10@fmt@@_WV?$digit_grouping@_W@567@@detail@v10@fmt@@YA?AV?$back_insert_iterator@V?$buffer@_W@detail@v10@fmt@@@std@@V45@ABU?$decimal_fp@N@dragonbox@123@ABU?$format_specs@_W@23@Ufloat_specs@123@Vlocale_ref@123@@Z@QBE@0@Z 1004bc44     handles.obj
 0002:0000ec50       __ehfuncinfo$??0?$digit_grouping@_W@detail@v10@fmt@@QAE@Vlocale_ref@123@_N@Z 1004bc50     handles.obj
 0002:0000ec78       __unwindtable$??0?$digit_grouping@_W@detail@v10@fmt@@QAE@Vlocale_ref@123@_N@Z 1004bc78     handles.obj
 0002:0000ecc8       __ehfuncinfo$??R<lambda_3>@?BD@???$do_write_float@V?$back_insert_iterator@V?$buffer@_W@detail@v10@fmt@@@std@@Ubig_decimal_fp@detail@v10@fmt@@_WV?$digit_grouping@_W@456@@detail@v10@fmt@@YA?AV?$back_insert_iterator@V?$buffer@_W@detail@v10@fmt@@@std@@V45@ABUbig_decimal_fp@123@ABU?$format_specs@_W@23@Ufloat_specs@123@Vlocale_ref@123@@Z@QBE@0@Z 1004bcc8     handles.obj
 0002:0000ecec       __unwindtable$??R<lambda_3>@?BD@???$do_write_float@V?$back_insert_iterator@V?$buffer@_W@detail@v10@fmt@@@std@@Ubig_decimal_fp@detail@v10@fmt@@_WV?$digit_grouping@_W@456@@detail@v10@fmt@@YA?AV?$back_insert_iterator@V?$buffer@_W@detail@v10@fmt@@@std@@V45@ABUbig_decimal_fp@123@ABU?$format_specs@_W@23@Ufloat_specs@123@Vlocale_ref@123@@Z@QBE@0@Z 1004bcec     handles.obj
 0002:0000ecf4       __ehfuncinfo$?Config@@YAHXZ 1004bcf4     Pcfg.obj
 0002:0000ed18       __unwindtable$?Config@@YAHXZ 1004bd18     Pcfg.obj
 0002:0000ed38       __ehfuncinfo$?Read@options@@QAEXXZ 1004bd38     Pcfg.obj
 0002:0000ed5c       __unwindtable$?Read@options@@QAEXXZ 1004bd5c     Pcfg.obj
 0002:0000ed6c       __ehfuncinfo$?ui64toa_width@@YA?AV?$basic_string@_WU?$char_traits@_W@std@@V?$allocator@_W@2@@std@@_KI_N@Z 1004bd6c     Pclass.obj
 0002:0000ed90       __unwindtable$?ui64toa_width@@YA?AV?$basic_string@_WU?$char_traits@_W@std@@V?$allocator@_W@2@@std@@_KI_N@Z 1004bd90     Pclass.obj
 0002:0000edc8       __ehfuncinfo$?PrintTitle@@YA?AV?$basic_string@_WU?$char_traits@_W@std@@V?$allocator@_W@2@@std@@V?$basic_string_view@_WU?$char_traits@_W@std@@@2@@Z 1004bdc8     Pclass.obj
 0002:0000edec       __unwindtable$?PrintTitle@@YA?AV?$basic_string@_WU?$char_traits@_W@std@@V?$allocator@_W@2@@std@@V?$basic_string_view@_WU?$char_traits@_W@std@@@2@@Z 1004bdec     Pclass.obj
 0002:0000edf4       __ehfuncinfo$??0Plist@@QAE@XZ 1004bdf4     Pclass.obj
 0002:0000ee18       __unwindtable$??0Plist@@QAE@XZ 1004be18     Pclass.obj
 0002:0000ee50       __ehfuncinfo$?TranslateMode@@YA_NABV?$basic_string@_WU?$char_traits@_W@std@@V?$allocator@_W@2@@std@@AAV12@@Z 1004be50     Pclass.obj
 0002:0000ee74       __unwindtable$?TranslateMode@@YA_NABV?$basic_string@_WU?$char_traits@_W@std@@V?$allocator@_W@2@@std@@AAV12@@Z 1004be74     Pclass.obj
 0002:0000ee88       __ehfuncinfo$?InitializePanelModes@Plist@@SAXXZ 1004be88     Pclass.obj
 0002:0000eeb0       __unwindtable$?InitializePanelModes@Plist@@SAXXZ 1004beb0     Pclass.obj
 0002:0000f1b0       __ehfuncinfo$?SavePanelModes@Plist@@SAXXZ 1004c1b0     Pclass.obj
 0002:0000f1d4       __unwindtable$?SavePanelModes@Plist@@SAXXZ 1004c1d4     Pclass.obj
 0002:0000f1ec       __ehfuncinfo$?generate_titles@@YAXABV?$basic_string@_WU?$char_traits@_W@std@@V?$allocator@_W@2@@std@@AAUPanelMode@@@Z 1004c1ec     Pclass.obj
 0002:0000f210       __unwindtable$?generate_titles@@YAXABV?$basic_string@_WU?$char_traits@_W@std@@V?$allocator@_W@2@@std@@AAUPanelMode@@@Z 1004c210     Pclass.obj
 0002:0000f218       __ehfuncinfo$?GetOpenPanelInfo@Plist@@QAEXPAUOpenPanelInfo@@@Z 1004c218     Pclass.obj
 0002:0000f23c       __unwindtable$?GetOpenPanelInfo@Plist@@QAEXPAUOpenPanelInfo@@@Z 1004c23c     Pclass.obj
 0002:0000f270       __ehfuncinfo$?GetFindData@Plist@@QAEHAAPAUPluginPanelItem@@AAI_K@Z 1004c270     Pclass.obj
 0002:0000f298       __unwindtable$?GetFindData@Plist@@QAEHAAPAUPluginPanelItem@@AAI_K@Z 1004c298     Pclass.obj
 0002:0000f328       __ehfuncinfo$??$_Uninitialized_move@PAV?$basic_string@_WU?$char_traits@_W@std@@V?$allocator@_W@2@@std@@V?$allocator@V?$basic_string@_WU?$char_traits@_W@std@@V?$allocator@_W@2@@std@@@2@@std@@YAPAV?$basic_string@_WU?$char_traits@_W@std@@V?$allocator@_W@2@@0@QAV10@0PAV10@AAV?$allocator@V?$basic_string@_WU?$char_traits@_W@std@@V?$allocator@_W@2@@std@@@0@@Z 1004c328     Pclass.obj
 0002:0000f328       __ehfuncinfo$??$construct@V?$basic_string@_WU?$char_traits@_W@std@@V?$allocator@_W@2@@std@@V12@@?$_Default_allocator_traits@V?$allocator@V?$basic_string@_WU?$char_traits@_W@std@@V?$allocator@_W@2@@std@@@std@@@std@@SAXAAV?$allocator@V?$basic_string@_WU?$char_traits@_W@std@@V?$allocator@_W@2@@std@@@1@QAV?$basic_string@_WU?$char_traits@_W@std@@V?$allocator@_W@2@@1@$$QAV31@@Z 1004c328     Pclass.obj
 0002:0000f328       __ehfuncinfo$??$emplace_back@V?$basic_string@_WU?$char_traits@_W@std@@V?$allocator@_W@2@@std@@@?$vector@V?$basic_string@_WU?$char_traits@_W@std@@V?$allocator@_W@2@@std@@V?$allocator@V?$basic_string@_WU?$char_traits@_W@std@@V?$allocator@_W@2@@std@@@2@@std@@QAE?A_T$$QAV?$basic_string@_WU?$char_traits@_W@std@@V?$allocator@_W@2@@1@@Z 1004c328     Pclass.obj
 0002:0000f34c       __unwindtable$??$_Uninitialized_move@PAV?$basic_string@_WU?$char_traits@_W@std@@V?$allocator@_W@2@@std@@V?$allocator@V?$basic_string@_WU?$char_traits@_W@std@@V?$allocator@_W@2@@std@@@2@@std@@YAPAV?$basic_string@_WU?$char_traits@_W@std@@V?$allocator@_W@2@@0@QAV10@0PAV10@AAV?$allocator@V?$basic_string@_WU?$char_traits@_W@std@@V?$allocator@_W@2@@std@@@0@@Z 1004c34c     Pclass.obj
 0002:0000f34c       __unwindtable$??$construct@V?$basic_string@_WU?$char_traits@_W@std@@V?$allocator@_W@2@@std@@V12@@?$_Default_allocator_traits@V?$allocator@V?$basic_string@_WU?$char_traits@_W@std@@V?$allocator@_W@2@@std@@@std@@@std@@SAXAAV?$allocator@V?$basic_string@_WU?$char_traits@_W@std@@V?$allocator@_W@2@@std@@@1@QAV?$basic_string@_WU?$char_traits@_W@std@@V?$allocator@_W@2@@1@$$QAV31@@Z 1004c34c     Pclass.obj
 0002:0000f34c       __unwindtable$??$emplace_back@V?$basic_string@_WU?$char_traits@_W@std@@V?$allocator@_W@2@@std@@@?$vector@V?$basic_string@_WU?$char_traits@_W@std@@V?$allocator@_W@2@@std@@V?$allocator@V?$basic_string@_WU?$char_traits@_W@std@@V?$allocator@_W@2@@std@@@2@@std@@QAE?A_T$$QAV?$basic_string@_WU?$char_traits@_W@std@@V?$allocator@_W@2@@1@@Z 1004c34c     Pclass.obj
 0002:0000f36c       __ehfuncinfo$?window_ex_style@@YA@PAUHWND__@@@Z 1004c36c     Pclass.obj
 0002:0000f36c       __ehfuncinfo$?window_style@@YA@PAUHWND__@@@Z 1004c36c     Pclass.obj
 0002:0000f390       __unwindtable$?window_ex_style@@YA@PAUHWND__@@@Z 1004c390     Pclass.obj
 0002:0000f390       __unwindtable$?window_style@@YA@PAUHWND__@@@Z 1004c390     Pclass.obj
 0002:0000f3a0       __ehfuncinfo$?DumpNTCounters@@YAXPAXAAVPerfThread@@KK@Z 1004c3a0     Pclass.obj
 0002:0000f3c4       __unwindtable$?DumpNTCounters@@YAXPAXAAVPerfThread@@KK@Z 1004c3c4     Pclass.obj
 0002:0000f3d8       __ehfuncinfo$?GetFiles@Plist@@QAEHPAUPluginPanelItem@@IHPAPB_W_KAAUoptions@@@Z 1004c3d8     Pclass.obj
 0002:0000f400       __unwindtable$?GetFiles@Plist@@QAEHPAUPluginPanelItem@@IHPAPB_W_KAAUoptions@@@Z 1004c400     Pclass.obj
 0002:0000f4f8       __ehfuncinfo$??0ProcessData@@QAE@XZ 1004c4f8     Pclass.obj
 0002:0000f51c       __unwindtable$??0ProcessData@@QAE@XZ 1004c51c     Pclass.obj
 0002:0000f530       __ehfuncinfo$?DeleteFiles@Plist@@QAEHPAUPluginPanelItem@@I_K@Z 1004c530     Pclass.obj
 0002:0000f558       __unwindtable$?DeleteFiles@Plist@@QAEHPAUPluginPanelItem@@I_K@Z 1004c558     Pclass.obj
 0002:0000f598       __ehfuncinfo$?Connect@Plist@@QAE_NPB_W00@Z 1004c598     Pclass.obj
 0002:0000f5bc       __unwindtable$?Connect@Plist@@QAE_NPB_W00@Z 1004c5bc     Pclass.obj
 0002:0000f5e0       __ehfuncinfo$?ProcessKey@Plist@@QAEHPBU_INPUT_RECORD@@@Z 1004c5e0     Pclass.obj
 0002:0000f608       __unwindtable$?ProcessKey@Plist@@QAEHPBU_INPUT_RECORD@@@Z 1004c608     Pclass.obj
 0002:0000f690       __ehfuncinfo$?GetVersionInfo@Plist@@SA_NPB_WAAV?$unique_ptr@$$BY0A@DU?$default_delete@$$BY0A@D@std@@@std@@AAPB_W2@Z 1004c690     Pclass.obj
 0002:0000f6b4       __unwindtable$?GetVersionInfo@Plist@@SA_NPB_WAAV?$unique_ptr@$$BY0A@DU?$default_delete@$$BY0A@D@std@@@std@@AAPB_W2@Z 1004c6b4     Pclass.obj
 0002:0000f6dc       __ehfuncinfo$?PrintOwnerInfo@Plist@@AAEXPAXK@Z 1004c6dc     Pclass.obj
 0002:0000f700       __unwindtable$?PrintOwnerInfo@Plist@@AAEXPAXK@Z 1004c700     Pclass.obj
 0002:0000f728       __ehfuncinfo$?Compare@Plist@@QBEHPBUPluginPanelItem@@0I@Z 1004c728     Pclass.obj
 0002:0000f74c       __unwindtable$?Compare@Plist@@QBEHPBUPluginPanelItem@@0I@Z 1004c74c     Pclass.obj
 0002:0000f75c       __ehfuncinfo$??4?$vector@Umode@@V?$allocator@Umode@@@std@@@std@@QAEAAV01@V?$initializer_list@Umode@@@1@@Z 1004c75c     Pclass.obj
 0002:0000f780       __unwindtable$??4?$vector@Umode@@V?$allocator@Umode@@@std@@@std@@QAEAAV01@V?$initializer_list@Umode@@@1@@Z 1004c780     Pclass.obj
 0002:0000f788       __ehfuncinfo$??$make_unique@VPerfThread@@PAVPlist@@$0A@@std@@YA?AV?$unique_ptr@VPerfThread@@U?$default_delete@VPerfThread@@@std@@@0@$$QAPAVPlist@@@Z 1004c788     Pclass.obj
 0002:0000f7ac       __unwindtable$??$make_unique@VPerfThread@@PAVPlist@@$0A@@std@@YA?AV?$unique_ptr@VPerfThread@@U?$default_delete@VPerfThread@@@std@@@0@$$QAPAVPlist@@@Z 1004c7ac     Pclass.obj
 0002:0000f7b4       __ehfuncinfo$??$_Emplace_reallocate@V?$basic_string@_WU?$char_traits@_W@std@@V?$allocator@_W@2@@std@@@?$vector@V?$basic_string@_WU?$char_traits@_W@std@@V?$allocator@_W@2@@std@@V?$allocator@V?$basic_string@_WU?$char_traits@_W@std@@V?$allocator@_W@2@@std@@@2@@std@@QAEPAV?$basic_string@_WU?$char_traits@_W@std@@V?$allocator@_W@2@@1@QAV21@$$QAV21@@Z 1004c7b4     Pclass.obj
 0002:0000f7d8       __unwindtable$??$_Emplace_reallocate@V?$basic_string@_WU?$char_traits@_W@std@@V?$allocator@_W@2@@std@@@?$vector@V?$basic_string@_WU?$char_traits@_W@std@@V?$allocator@_W@2@@std@@V?$allocator@V?$basic_string@_WU?$char_traits@_W@std@@V?$allocator@_W@2@@std@@@2@@std@@QAEPAV?$basic_string@_WU?$char_traits@_W@std@@V?$allocator@_W@2@@1@QAV21@$$QAV21@@Z 1004c7d8     Pclass.obj
 0002:0000f808       __ehfuncinfo$??$?H_WU?$char_traits@_W@std@@V?$allocator@_W@1@@std@@YA?AV?$basic_string@_WU?$char_traits@_W@std@@V?$allocator@_W@2@@0@ABV10@$$QAV10@@Z 1004c808     Pclass.obj
 0002:0000f82c       __unwindtable$??$?H_WU?$char_traits@_W@std@@V?$allocator@_W@1@@std@@YA?AV?$basic_string@_WU?$char_traits@_W@std@@V?$allocator@_W@2@@0@ABV10@$$QAV10@@Z 1004c82c     Pclass.obj
 0002:0000f83c       __ehfuncinfo$??$_Try_emplace@ABK$$V@?$_Hash@V?$_Umap_traits@KPAUHWND__@@V?$_Uhash_compare@KU?$hash@K@std@@U?$equal_to@K@2@@std@@V?$allocator@U?$pair@$$CBKPAUHWND__@@@std@@@3@$0A@@std@@@std@@IAE?AU?$pair@PAU?$_List_node@U?$pair@$$CBKPAUHWND__@@@std@@PAX@std@@_N@1@ABK@Z 1004c83c     Pclass.obj
 0002:0000f860       __unwindtable$??$_Try_emplace@ABK$$V@?$_Hash@V?$_Umap_traits@KPAUHWND__@@V?$_Uhash_compare@KU?$hash@K@std@@U?$equal_to@K@2@@std@@V?$allocator@U?$pair@$$CBKPAUHWND__@@@std@@@3@$0A@@std@@@std@@IAE?AU?$pair@PAU?$_List_node@U?$pair@$$CBKPAUHWND__@@@std@@PAX@std@@_N@1@ABK@Z 1004c860     Pclass.obj
 0002:0000f870       __ehfuncinfo$??0mode@@QAE@ABU0@@Z 1004c870     Pclass.obj
 0002:0000f894       __unwindtable$??0mode@@QAE@ABU0@@Z 1004c894     Pclass.obj
 0002:0000f8c0       __ehfuncinfo$??0PerfThread@@QAE@PAVPlist@@PB_W11@Z 1004c8c0     perfthread.obj
 0002:0000f8e8       __unwindtable$??0PerfThread@@QAE@PAVPlist@@PB_W11@Z 1004c8e8     perfthread.obj
 0002:0000f990       __ehfuncinfo$?RefreshImpl@PerfThread@@AAE_NXZ 1004c990     perfthread.obj
 0002:0000f9b4       __unwindtable$?RefreshImpl@PerfThread@@AAE_NXZ 1004c9b4     perfthread.obj
 0002:0000f9d0       __ehfuncinfo$??R<lambda_1>@?1??RefreshImpl@PerfThread@@AAE_NXZ@QBE@PBU_PERF_COUNTER_BLOCK@@V?$basic_string_view@_WU?$char_traits@_W@std@@@std@@@Z 1004c9d0     perfthread.obj
 0002:0000f9f8       __unwindtable$??R<lambda_1>@?1??RefreshImpl@PerfThread@@AAE_NXZ@QBE@PBU_PERF_COUNTER_BLOCK@@V?$basic_string_view@_WU?$char_traits@_W@std@@@std@@@Z 1004c9f8     perfthread.obj
 0002:0000fa38       __ehfuncinfo$?RefreshWMIData@PerfThread@@AAEXXZ 1004ca38     perfthread.obj
 0002:0000fa60       __unwindtable$?RefreshWMIData@PerfThread@@AAEXXZ 1004ca60     perfthread.obj
 0002:0000faa8       __ehfuncinfo$??0?$unordered_multimap@KUProcessPerfData@@U?$hash@K@std@@U?$equal_to@K@3@V?$allocator@U?$pair@$$CBKUProcessPerfData@@@std@@@3@@std@@QAE@XZ 1004caa8     perfthread.obj
 0002:0000facc       __unwindtable$??0?$unordered_multimap@KUProcessPerfData@@U?$hash@K@std@@U?$equal_to@K@3@V?$allocator@U?$pair@$$CBKUProcessPerfData@@@std@@@3@@std@@QAE@XZ 1004cacc     perfthread.obj
 0002:0000fadc       __ehfuncinfo$??$transform@V?$_List_const_iterator@V?$_List_val@U?$_List_simple_types@U?$pair@$$CBKUProcessPerfData@@@std@@@std@@@std@@@std@@V?$back_insert_iterator@V?$vector@UProcessPerfData@@V?$allocator@UProcessPerfData@@@std@@@std@@@2@V<lambda_1>@?2??RefreshWMIData@PerfThread@@AAEXXZ@@std@@YA?AV?$back_insert_iterator@V?$vector@UProcessPerfData@@V?$allocator@UProcessPerfData@@@std@@@std@@@0@V?$_List_const_iterator@V?$_List_val@U?$_List_simple_types@U?$pair@$$CBKUProcessPerfData@@@std@@@std@@@std@@@0@0V10@V<lambda_1>@?2??RefreshWMIData@PerfThread@@AAEXXZ@@Z 1004cadc     perfthread.obj
 0002:0000fb00       __unwindtable$??$transform@V?$_List_const_iterator@V?$_List_val@U?$_List_simple_types@U?$pair@$$CBKUProcessPerfData@@@std@@@std@@@std@@@std@@V?$back_insert_iterator@V?$vector@UProcessPerfData@@V?$allocator@UProcessPerfData@@@std@@@std@@@2@V<lambda_1>@?2??RefreshWMIData@PerfThread@@AAEXXZ@@std@@YA?AV?$back_insert_iterator@V?$vector@UProcessPerfData@@V?$allocator@UProcessPerfData@@@std@@@std@@@0@V?$_List_const_iterator@V?$_List_val@U?$_List_simple_types@U?$pair@$$CBKUProcessPerfData@@@std@@@std@@@std@@@0@0V10@V<lambda_1>@?2??RefreshWMIData@PerfThread@@AAEXXZ@@Z 1004cb00     perfthread.obj
 0002:0000fb08       __ehfuncinfo$??0ProcessPerfData@@QAE@ABU0@@Z 1004cb08     perfthread.obj
 0002:0000fb2c       __unwindtable$??0ProcessPerfData@@QAE@ABU0@@Z 1004cb2c     perfthread.obj
 0002:0000fb48       __ehfuncinfo$??0ProcessPerfData@@QAE@$$QAU0@@Z 1004cb48     perfthread.obj
 0002:0000fb70       __unwindtable$??0ProcessPerfData@@QAE@$$QAU0@@Z 1004cb70     perfthread.obj
 0002:0000fbb0       __ehfuncinfo$?is_wow64_itself@@YA_NXZ 1004cbb0     Plist.obj
 0002:0000fbd4       __unwindtable$?is_wow64_itself@@YA_NXZ 1004cbd4     Plist.obj
 0002:0000fbdc       __ehfuncinfo$?GetList@@YA_NAAPAUPluginPanelItem@@AAIAAVPerfThread@@@Z 1004cbdc     Plist.obj
 0002:0000fc00       __unwindtable$?GetList@@YA_NAAPAUPluginPanelItem@@AAIAAVPerfThread@@@Z 1004cc00     Plist.obj
 0002:0000fc18       __ehfuncinfo$?KillProcess@@YA_NKPAUHWND__@@@Z 1004cc18     Plist.obj
 0002:0000fc3c       __unwindtable$?KillProcess@@YA_NKPAUHWND__@@@Z 1004cc3c     Plist.obj
 0002:0000fc4c       __ehfuncinfo$?PrintNTCurDirAndEnv@@YAXPAX0H@Z 1004cc4c     Plist.obj
 0002:0000fc70       __unwindtable$?PrintNTCurDirAndEnv@@YAXPAX0H@Z 1004cc70     Plist.obj
 0002:0000fc90       __ehfuncinfo$?print_module_impl@@YAXQAXABV?$basic_string@_WU?$char_traits@_W@std@@V?$allocator@_W@2@@std@@KABUoptions@@ABV?$function@$$A6A_NPA_WI@Z@2@@Z 1004cc90     Plist.obj
 0002:0000fcb4       __unwindtable$?print_module_impl@@YAXQAXABV?$basic_string@_WU?$char_traits@_W@std@@V?$allocator@_W@2@@std@@KABUoptions@@ABV?$function@$$A6A_NPA_WI@Z@2@@Z 1004ccb4     Plist.obj
 0002:0000fcbc       __ehfuncinfo$?PrintModules@@YAXPAXKAAUoptions@@@Z 1004ccbc     Plist.obj
 0002:0000fce0       __unwindtable$?PrintModules@@YAXPAXKAAUoptions@@@Z 1004cce0     Plist.obj
 0002:0000fd00       __ehfuncinfo$?PrintModules@?$ipc_functions@$0A@@@SAXPAX0AAUoptions@@@Z 1004cd00     Plist.obj
 0002:0000fd24       __unwindtable$?PrintModules@?$ipc_functions@$0A@@@SAXPAX0AAUoptions@@@Z 1004cd24     Plist.obj
 0002:0000fd2c       __ehfuncinfo$?PrintModules@?$ipc_functions@$00@@SAXPAX0AAUoptions@@@Z 1004cd2c     Plist.obj
 0002:0000fd50       __unwindtable$?PrintModules@?$ipc_functions@$00@@SAXPAX0AAUoptions@@@Z 1004cd50     Plist.obj
 0002:0000fd58       __ehfuncinfo$?read_string@?$ipc_functions@$0A@@@SA?AV?$basic_string@_WU?$char_traits@_W@std@@V?$allocator@_W@2@@std@@PAXABUUNICODE_STRING_SAME@detail@@@Z 1004cd58     Plist.obj
 0002:0000fd7c       __unwindtable$?read_string@?$ipc_functions@$0A@@@SA?AV?$basic_string@_WU?$char_traits@_W@std@@V?$allocator@_W@2@@std@@PAXABUUNICODE_STRING_SAME@detail@@@Z 1004cd7c     Plist.obj
 0002:0000fd9c       __ehfuncinfo$?read_string@?$ipc_functions@$00@@SA?AV?$basic_string@_WU?$char_traits@_W@std@@V?$allocator@_W@2@@std@@PAXABUUNICODE_STRING_64@detail@@@Z 1004cd9c     Plist.obj
 0002:0000fdc0       __unwindtable$?read_string@?$ipc_functions@$00@@SA?AV?$basic_string@_WU?$char_traits@_W@std@@V?$allocator@_W@2@@std@@PAXABUUNICODE_STRING_64@detail@@@Z 1004cdc0     Plist.obj
 0002:0000fde8       __ehfuncinfo$??$print_module@PAX@@YAXQAXPAXKAAUoptions@@ABV?$function@$$A6A_NPA_WI@Z@std@@@Z 1004cde8     Plist.obj
 0002:0000fe0c       __unwindtable$??$print_module@PAX@@YAXQAXPAXKAAUoptions@@ABV?$function@$$A6A_NPA_WI@Z@std@@@Z 1004ce0c     Plist.obj
 0002:0000fe2c       __ehfuncinfo$??$print_module@_K@@YAXQAX_KKAAUoptions@@ABV?$function@$$A6A_NPA_WI@Z@std@@@Z 1004ce2c     Plist.obj
 0002:0000fe50       __unwindtable$??$print_module@_K@@YAXQAX_KKAAUoptions@@ABV?$function@$$A6A_NPA_WI@Z@std@@@Z 1004ce50     Plist.obj
 0002:0000fe70       __ehfuncinfo$??$insert@V?$_List_unchecked_const_iterator@V?$_List_val@U?$_List_simple_types@U?$pair@$$CBKUProcessPerfData@@@std@@@std@@@std@@U_Iterator_base0@2@@std@@@?$_Hash@V?$_Umap_traits@KUProcessPerfData@@V?$_Uhash_compare@KU?$hash@K@std@@U?$equal_to@K@2@@std@@V?$allocator@U?$pair@$$CBKUProcessPerfData@@@std@@@3@$00@std@@@std@@QAEXV?$_List_unchecked_const_iterator@V?$_List_val@U?$_List_simple_types@U?$pair@$$CBKUProcessPerfData@@@std@@@std@@@std@@U_Iterator_base0@2@@1@0@Z 1004ce70     Plist.obj
 0002:0000fe94       __unwindtable$??$insert@V?$_List_unchecked_const_iterator@V?$_List_val@U?$_List_simple_types@U?$pair@$$CBKUProcessPerfData@@@std@@@std@@@std@@U_Iterator_base0@2@@std@@@?$_Hash@V?$_Umap_traits@KUProcessPerfData@@V?$_Uhash_compare@KU?$hash@K@std@@U?$equal_to@K@2@@std@@V?$allocator@U?$pair@$$CBKUProcessPerfData@@@std@@@3@$00@std@@@std@@QAEXV?$_List_unchecked_const_iterator@V?$_List_val@U?$_List_simple_types@U?$pair@$$CBKUProcessPerfData@@@std@@@std@@@std@@U_Iterator_base0@2@@1@0@Z 1004ce94     Plist.obj
 0002:0000fea8       __ehfuncinfo$?WinError@@YAHPB_W@Z 1004cea8     Pmix.obj
 0002:0000fed0       __unwindtable$?WinError@@YAHPB_W@Z 1004ced0     Pmix.obj
 0002:0000ff10       __ehfuncinfo$?GetProcessOwner@WMIConnection@@QAE?AV?$basic_string@_WU?$char_traits@_W@std@@V?$allocator@_W@2@@std@@KPAV23@@Z 1004cf10     wmi.obj
 0002:0000ff38       __unwindtable$?GetProcessOwner@WMIConnection@@QAE?AV?$basic_string@_WU?$char_traits@_W@std@@V?$allocator@_W@2@@std@@KPAV23@@Z 1004cf38     wmi.obj
 0002:0000ff88       __ehfuncinfo$?GetProcessUserSid@WMIConnection@@QAE?AV?$basic_string@_WU?$char_traits@_W@std@@V?$allocator@_W@2@@std@@K@Z 1004cf88     wmi.obj
 0002:0000ffb0       __unwindtable$?GetProcessUserSid@WMIConnection@@QAE?AV?$basic_string@_WU?$char_traits@_W@std@@V?$allocator@_W@2@@std@@K@Z 1004cfb0     wmi.obj
 0002:00010000       __ehfuncinfo$?GetProcessSessionId@WMIConnection@@QAEKK@Z 1004d000     wmi.obj
 0002:00010024       __unwindtable$?GetProcessSessionId@WMIConnection@@QAEKK@Z 1004d024     wmi.obj
 0002:00010030       __ehfuncinfo$?ExecMethod@WMIConnection@@AAEHKPB_W0K@Z 1004d030     wmi.obj
 0002:00010058       __unwindtable$?ExecMethod@WMIConnection@@AAEHKPB_W0K@Z 1004d058     wmi.obj
 0002:000100f8       __ehfuncinfo$?GetProcessProperty@WMIConnection@@AAE_NKPB_WABV?$function@$$A6AXABUtagVARIANT@@@Z@std@@@Z 1004d0f8     wmi.obj
 0002:0001011c       __unwindtable$?GetProcessProperty@WMIConnection@@AAE_NKPB_WABV?$function@$$A6AXABUtagVARIANT@@@Z@std@@@Z 1004d11c     wmi.obj
 0002:00010154       __ehfuncinfo$?GetProcessInt@WMIConnection@@AAEKKPB_W@Z 1004d154     wmi.obj
 0002:00010178       __unwindtable$?GetProcessInt@WMIConnection@@AAEKKPB_W@Z 1004d178     wmi.obj
 0002:00010180       __ehfuncinfo$?GetProcessString@WMIConnection@@AAE?AV?$basic_string@_WU?$char_traits@_W@std@@V?$allocator@_W@2@@std@@KPB_W@Z 1004d180     wmi.obj
 0002:000101a4       __unwindtable$?GetProcessString@WMIConnection@@AAE?AV?$basic_string@_WU?$char_traits@_W@std@@V?$allocator@_W@2@@std@@KPB_W@Z 1004d1a4     wmi.obj
 0002:000101bc       __ehfuncinfo$?Connect@WMIConnection@@QAE_NPB_W00@Z 1004d1bc     wmi.obj
 0002:000101e0       __unwindtable$?Connect@WMIConnection@@QAE_NPB_W00@Z 1004d1e0     wmi.obj
 0002:00010300       __unwindtable$?_Init@locale@std@@CAPAV_Locimp@12@_N@Z 1004d300     libcpmt:locale0.obj
 0002:00010308       __ehfuncinfo$?_Init@locale@std@@CAPAV_Locimp@12@_N@Z 1004d308     libcpmt:locale0.obj
 0002:00010330       __sehtable$___scrt_is_nonwritable_in_current_image 1004d330     LIBCMT:utility.obj
 0002:00010350       __sehtable$??_M@YGXPAXIIP6EX0@Z@Z 1004d350     LIBCMT:ehvecdtr.obj
 0002:00010370       __sehtable$?__ArrayUnwind@@YGXPAXIIP6EX0@Z@Z 1004d370     LIBCMT:ehvecdtr.obj
 0002:00010390       __sehtable$?dllmain_crt_process_attach@@YAHQAUHINSTANCE__@@QAX@Z 1004d390     LIBCMT:dll_dllmain.obj
 0002:000103b0       __sehtable$?dllmain_crt_process_detach@@YAH_N@Z 1004d3b0     LIBCMT:dll_dllmain.obj
 0002:000103d8       __sehtable$?dllmain_dispatch@@YAHQAUHINSTANCE__@@KQAX@Z 1004d3d8     LIBCMT:dll_dllmain.obj
 0002:000103f8       __sehtable$___DestructExceptionObject 1004d3f8     libvcruntime:ehhelpers.obj
 0002:00010418       __sehtable$?FrameUnwindToState@__FrameHandler3@@SAXPAUEHRegistrationNode@@PAXPBU_s_FuncInfo@@H@Z 1004d418     libvcruntime:frame.obj
 0002:00010440       __sehtable$?CallCatchBlock@@YAPAXPAUEHExceptionRecord@@PAUEHRegistrationNode@@PAU_CONTEXT@@PBU_s_FuncInfo@@PAXHK@Z 1004d440     libvcruntime:frame.obj
 0002:00010468       __catchsym$?CallUnexpected@@YAXPBU_s_ESTypeList@@@Z$2 1004d468     libvcruntime:frame.obj
 0002:00010478       __unwindtable$?CallUnexpected@@YAXPBU_s_ESTypeList@@@Z 1004d478     libvcruntime:frame.obj
 0002:00010488       __tryblocktable$?CallUnexpected@@YAXPBU_s_ESTypeList@@@Z 1004d488     libvcruntime:frame.obj
 0002:0001049c       __ehfuncinfo$?CallUnexpected@@YAXPBU_s_ESTypeList@@@Z 1004d49c     libvcruntime:frame.obj
 0002:000104c0       __sehtable$??$BuildCatchObjectHelperInternal@V__FrameHandler3@@@@YAHPAUEHExceptionRecord@@PAXPBU_s_HandlerType@@PBU_s_CatchableType@@@Z 1004d4c0     libvcruntime:frame.obj
 0002:000104e0       __sehtable$??$BuildCatchObjectInternal@V__FrameHandler3@@@@YAXPAUEHExceptionRecord@@PAXPBU_s_HandlerType@@PBU_s_CatchableType@@@Z 1004d4e0     libvcruntime:frame.obj
 0002:00010538       __sehtable$___acrt_lowio_ensure_fh_exists 1004d538     libucrt:osfinfo.obj
 0002:00010558       __sehtable$_terminate      1004d558     libucrt:terminate.obj
 0002:00010578       __sehtable$??$?RV<lambda_646e26742ed01d5bc03234f44bb6d3d3>@@AAV<lambda_b37934c380d97b75fd242ea49540127a>@@V<lambda_bbd9d45274666fbb50f81a29ad795c13>@@@?$__crt_seh_guarded_call@PAD@@QAEPAD$$QAV<lambda_646e26742ed01d5bc03234f44bb6d3d3>@@AAV<lambda_b37934c380d97b75fd242ea49540127a>@@$$QAV<lambda_bbd9d45274666fbb50f81a29ad795c13>@@@Z 1004d578     libucrt:setlocale.obj
 0002:00010598       __sehtable$??R<lambda_6e4b09c48022b2350581041d5f6b0c4c>@@QBE@XZ 1004d598     libucrt:exit.obj
 0002:000105b8       __sehtable$??$?RV<lambda_03b1d95aef87969028cfba75ccab2455>@@AAV<lambda_6e4b09c48022b2350581041d5f6b0c4c>@@V<lambda_22bdf7517842c4b3e53723af5aa32b9e>@@@?$__crt_seh_guarded_call@X@@QAEX$$QAV<lambda_03b1d95aef87969028cfba75ccab2455>@@AAV<lambda_6e4b09c48022b2350581041d5f6b0c4c>@@$$QAV<lambda_22bdf7517842c4b3e53723af5aa32b9e>@@@Z 1004d5b8     libucrt:exit.obj
 0002:000105d8       __sehtable$??$?RV<lambda_8e746cf0007f6ed984d6f78af1fec997>@@AAV<lambda_22ebabd17bc4fa466a2aca6d8deb888d>@@V<lambda_18ed0c0b38a6dc0daf1e7ac6d6adf05e>@@@?$__crt_seh_guarded_call@H@@QAEH$$QAV<lambda_8e746cf0007f6ed984d6f78af1fec997>@@AAV<lambda_22ebabd17bc4fa466a2aca6d8deb888d>@@$$QAV<lambda_18ed0c0b38a6dc0daf1e7ac6d6adf05e>@@@Z 1004d5d8     libucrt:onexit.obj
 0002:000105f8       __sehtable$??$?RV<lambda_69a2805e680e0e292e8ba93315fe43a8>@@AAV<lambda_f03950bc5685219e0bcd2087efbe011e>@@V<lambda_03fcd07e894ec930e3f35da366ca99d6>@@@?$__crt_seh_guarded_call@H@@QAEH$$QAV<lambda_69a2805e680e0e292e8ba93315fe43a8>@@AAV<lambda_f03950bc5685219e0bcd2087efbe011e>@@$$QAV<lambda_03fcd07e894ec930e3f35da366ca99d6>@@@Z 1004d5f8     libucrt:onexit.obj
 0002:00010618       __sehtable$__query_new_handler 1004d618     libucrt:new_handler.obj
 0002:00010638       __sehtable$??$?RV<lambda_15ade71b0218206bbe3333a0c9b79046>@@AAV<lambda_da44e0f8b0f19ba52fefafb335991732>@@V<lambda_207f2d024fc103971653565357d6cd41>@@@?$__crt_seh_guarded_call@X@@QAEX$$QAV<lambda_15ade71b0218206bbe3333a0c9b79046>@@AAV<lambda_da44e0f8b0f19ba52fefafb335991732>@@$$QAV<lambda_207f2d024fc103971653565357d6cd41>@@@Z 1004d638     libucrt:per_thread_data.obj
 0002:00010658       __sehtable$??$?RV<lambda_a7e850c220f1c8d1e6efeecdedd162c6>@@AAV<lambda_46720907175c18b6c9d2717bc0d2d362>@@V<lambda_9048902d66e8d99359bc9897bbb930a8>@@@?$__crt_seh_guarded_call@X@@QAEX$$QAV<lambda_a7e850c220f1c8d1e6efeecdedd162c6>@@AAV<lambda_46720907175c18b6c9d2717bc0d2d362>@@$$QAV<lambda_9048902d66e8d99359bc9897bbb930a8>@@@Z 1004d658     libucrt:per_thread_data.obj
 0002:00010678       __sehtable$??$?RV<lambda_38edbb1296d33220d7e4dd0ed76b244a>@@AAV<lambda_5ce1d447e08cb34b2473517608e21441>@@V<lambda_fb385d3da700c9147fc39e65dd577a8c>@@@?$__crt_seh_guarded_call@X@@QAEX$$QAV<lambda_38edbb1296d33220d7e4dd0ed76b244a>@@AAV<lambda_5ce1d447e08cb34b2473517608e21441>@@$$QAV<lambda_fb385d3da700c9147fc39e65dd577a8c>@@@Z 1004d678     libucrt:per_thread_data.obj
 0002:00010698       __sehtable$??$?RV<lambda_6affb1475c98b40b75cdec977db92e3c>@@AAV<lambda_b8d4b9c228a6ecc3f80208dbb4b4a104>@@V<lambda_608742c3c92a14382c1684fc64f96c88>@@@?$__crt_seh_guarded_call@X@@QAEX$$QAV<lambda_6affb1475c98b40b75cdec977db92e3c>@@AAV<lambda_b8d4b9c228a6ecc3f80208dbb4b4a104>@@$$QAV<lambda_608742c3c92a14382c1684fc64f96c88>@@@Z 1004d698     libucrt:per_thread_data.obj
 0002:000106b8       __sehtable$___acrt_initialize_lowio 1004d6b8     libucrt:ioinit.obj
 0002:000106d8       __sehtable$??$?RV<lambda_6b4b7855443974f2b4b77000ea21c99c>@@AAV<lambda_8f7d3b162ab39427f4fa9995c67a7986>@@V<lambda_cc9a5ba8a5d8428b9634eab82665e5dc>@@@?$__crt_seh_guarded_call@H@@QAEH$$QAV<lambda_6b4b7855443974f2b4b77000ea21c99c>@@AAV<lambda_8f7d3b162ab39427f4fa9995c67a7986>@@$$QAV<lambda_cc9a5ba8a5d8428b9634eab82665e5dc>@@@Z 1004d6d8     libucrt:winapi_thunks.obj
 0002:000106f8       __sehtable$__fcloseall     1004d6f8     libucrt:closeall.obj
 0002:00010718       __sehtable$??$?RV<lambda_2866be3712abc81a800a822484c830d8>@@AAV<lambda_39ca0ed439415581b5b15c265174cece>@@V<lambda_2b24c74d71094a6cd0cb82e44167d71b>@@@?$__crt_seh_guarded_call@X@@QAEX$$QAV<lambda_2866be3712abc81a800a822484c830d8>@@AAV<lambda_39ca0ed439415581b5b15c265174cece>@@$$QAV<lambda_2b24c74d71094a6cd0cb82e44167d71b>@@@Z 1004d718     libucrt:fflush.obj
 0002:00010738       __sehtable$??$?RV<lambda_2cc53f568c5a2bb6f192f930a45d44ea>@@AAV<lambda_ab61a845afdef5b7c387490eaf3616ee>@@V<lambda_c2ffc0b7726aa6be21d5f0026187e748>@@@?$__crt_seh_guarded_call@X@@QAEX$$QAV<lambda_2cc53f568c5a2bb6f192f930a45d44ea>@@AAV<lambda_ab61a845afdef5b7c387490eaf3616ee>@@$$QAV<lambda_c2ffc0b7726aa6be21d5f0026187e748>@@@Z 1004d738     libucrt:fflush.obj
 0002:00010758       __sehtable$??$?RV<lambda_e5124f882df8998aaf41531e079ba474>@@AAV<lambda_3e16ef9562a7dcce91392c22ab16ea36>@@V<lambda_e25ca0880e6ef98be67edffd8c599615>@@@?$__crt_seh_guarded_call@X@@QAEX$$QAV<lambda_e5124f882df8998aaf41531e079ba474>@@AAV<lambda_3e16ef9562a7dcce91392c22ab16ea36>@@$$QAV<lambda_e25ca0880e6ef98be67edffd8c599615>@@@Z 1004d758     libucrt:wsetlocale.obj
 0002:00010778       __sehtable$??$?RV<lambda_4fdada1b837b2abbf20876fac97688ad>@@AAV<lambda_b57350f2640456a0859d250846f69caf>@@V<lambda_eed5e4f92b5b7d55fa22c48c484aaa54>@@@?$__crt_seh_guarded_call@X@@QAEX$$QAV<lambda_4fdada1b837b2abbf20876fac97688ad>@@AAV<lambda_b57350f2640456a0859d250846f69caf>@@$$QAV<lambda_eed5e4f92b5b7d55fa22c48c484aaa54>@@@Z 1004d778     libucrt:wsetlocale.obj
 0002:00010798       __sehtable$??$?RV<lambda_135d2772fca65dc1248eeaa1b56e886a>@@AAV<lambda_2a444430fde8c29194d880d93eed5e8f>@@AAV<lambda_8dff2cf36a5417162780cd64fa2883ef>@@@?$__crt_seh_guarded_call@X@@QAEX$$QAV<lambda_135d2772fca65dc1248eeaa1b56e886a>@@AAV<lambda_2a444430fde8c29194d880d93eed5e8f>@@AAV<lambda_8dff2cf36a5417162780cd64fa2883ef>@@@Z 1004d798     libucrt:wsetlocale.obj
 0002:000107b8       __sehtable$__write         1004d7b8     libucrt:write.obj
 0002:000107d4       __unwindtable$?_wcstombs_l_helper@@YAIPADPB_WIPAU__crt_locale_pointers@@@Z 1004d7d4     libucrt:wcstombs.obj
 0002:000107dc       __ehfuncinfo$?_wcstombs_l_helper@@YAIPADPB_WIPAU__crt_locale_pointers@@@Z 1004d7dc     libucrt:wcstombs.obj
 0002:00010800       __sehtable$_raise          1004d800     libucrt:signal.obj
 0002:00010820       __sehtable$??$?RV<lambda_cbab9ec6f41b0180b23cc171c22676b0>@@AAV<lambda_44731a7d0e6d81c3e6aa82d741081786>@@V<lambda_4b292cb8dd18144e164572427af410ab>@@@?$__crt_seh_guarded_call@P6AXH@Z@@QAEP6AXH@Z$$QAV<lambda_cbab9ec6f41b0180b23cc171c22676b0>@@AAV<lambda_44731a7d0e6d81c3e6aa82d741081786>@@$$QAV<lambda_4b292cb8dd18144e164572427af410ab>@@@Z 1004d820     libucrt:signal.obj
 0002:00010840       __sehtable$?update_thread_multibyte_data_internal@@YAPAU__crt_multibyte_data@@QAU__acrt_ptd@@QAPAU1@@Z 1004d840     libucrt:mbctype.obj
 0002:00010860       __sehtable$??$?RV<lambda_ceb1ee4838e85a9d631eb091e2fbe199>@@AAV<lambda_ae742caa10f662c28703da3d2ea5e57e>@@V<lambda_cd08b5d6af4937fe54fc07d0c9bf6b37>@@@?$__crt_seh_guarded_call@X@@QAEX$$QAV<lambda_ceb1ee4838e85a9d631eb091e2fbe199>@@AAV<lambda_ae742caa10f662c28703da3d2ea5e57e>@@$$QAV<lambda_cd08b5d6af4937fe54fc07d0c9bf6b37>@@@Z 1004d860     libucrt:mbctype.obj
 0002:00010880       __sehtable$___acrt_update_thread_locale_data 1004d880     libucrt:locale_refcounting.obj
 0002:000108a0       __sehtable$_fclose         1004d8a0     libucrt:fclose.obj
 0002:000108c0       __sehtable$??$?RV<lambda_9e9de3de5fa147e2223d7db92bc10aa6>@@AAV<lambda_38ce7e780aa69e748d6df282ebc68efe>@@V<lambda_8ca6da459f0f6780f1cff60fdc3d00e5>@@@?$__crt_seh_guarded_call@H@@QAEH$$QAV<lambda_9e9de3de5fa147e2223d7db92bc10aa6>@@AAV<lambda_38ce7e780aa69e748d6df282ebc68efe>@@$$QAV<lambda_8ca6da459f0f6780f1cff60fdc3d00e5>@@@Z 1004d8c0     libucrt:commit.obj
 0002:000108e0       __sehtable$??$?RV<lambda_218ce3db14220d0be481dae8ef3383b6>@@AAV<lambda_628dfdc04ba53c8bfc02c9951375f3f5>@@V<lambda_57dc472bd5c9d5f3b2cbca59b8a843ae>@@@?$__crt_seh_guarded_call@H@@QAEH$$QAV<lambda_218ce3db14220d0be481dae8ef3383b6>@@AAV<lambda_628dfdc04ba53c8bfc02c9951375f3f5>@@$$QAV<lambda_57dc472bd5c9d5f3b2cbca59b8a843ae>@@@Z 1004d8e0     libucrt:close.obj
 0002:00010900       __sehtable$__IsNonwritableInCurrentImage 1004d900     LIBCMT:pesect.obj
 0002:00010a10       .edata                     1004da10     ProcList.exp
 0002:00010a38       rgpv                       1004da38     ProcList.exp
 0002:00010a74       rgszName                   1004da74     ProcList.exp
 0002:00010ab0       rgwOrd                     1004dab0     ProcList.exp
 0002:00010ace       szName                     1004dace     ProcList.exp
 0002:00010adb       $N00001                    1004dadb     ProcList.exp
 0002:00010ae7       $N00002                    1004dae7     ProcList.exp
 0002:00010af0       $N00003                    1004daf0     ProcList.exp
 0002:00010afb       $N00004                    1004dafb     ProcList.exp
 0002:00010b08       $N00005                    1004db08     ProcList.exp
 0002:00010b16       $N00006                    1004db16     ProcList.exp
 0002:00010b20       $N00007                    1004db20     ProcList.exp
 0002:00010b2d       $N00008                    1004db2d     ProcList.exp
 0002:00010b3c       $N00009                    1004db3c     ProcList.exp
 0002:00010b4e       $N00010                    1004db4e     ProcList.exp
 0002:00010b5d       $N00011                    1004db5d     ProcList.exp
 0002:00010b63       $N00012                    1004db63     ProcList.exp
 0002:00010b76       $N00013                    1004db76     ProcList.exp
 0002:00010b89       $N00014                    1004db89     ProcList.exp
 0002:00010b9e       $N00015                    1004db9e     ProcList.exp
 0002:00011282       .idata$6                   1004e282     kernel32:KERNEL32.dll
 0002:00011384       .idata$6                   1004e384     advapi32:ADVAPI32.dll
 0002:00011468       .idata$6                   1004e468     user32:USER32.dll
 0002:000114a4       .idata$6                   1004e4a4     mpr:MPR.dll
 0002:000114e2       .idata$6                   1004e4e2     ole32:ole32.dll
 0002:000114ec       .idata$6                   1004e4ec     oleaut32:OLEAUT32.dll
 0002:0001152a       .idata$6                   1004e52a     psapi:PSAPI.DLL
 0002:00011576       .idata$6                   1004e576     version:VERSION.dll
 0003:00000000       ?init@std@@3JA             1004f000     libcpmt:xlock.obj
 0003:00000004       ?atcount_cdecl@@3IA        1004f004     libcpmt:iosptrs.obj
 0003:00000030       ?__vcrt_flsindex@@3KA      1004f030     libvcruntime:per_thread_data.obj
 0003:00000154       ?errno_no_memory@@3HA      1004f154     libucrt:errno.obj
 0003:00000158       ?doserrno_no_memory@@3KA   1004f158     libucrt:errno.obj
 0003:00000180       ?__acrt_flsindex@@3KA      1004f180     libucrt:per_thread_data.obj
 0003:00000184       __ctype_loc_style          1004f184     libucrt:wsetlocale.obj
 0003:00000250       _newcw                     1004f250     libucrt:modf.obj
 0003:00000260       ?tzstd_program@@3PADA      1004f260     libucrt:timeset.obj
 0003:000002a0       ?tzdst_program@@3PADA      1004f2a0     libucrt:timeset.obj
 0003:000002e0       ?tzname_states@@3PAY01PADA 1004f2e0     libucrt:timeset.obj
 0003:00000508       __mbctypes                 1004f508     libucrt:mbctype.obj
 0003:00000610       __mbcasemaps               1004f610     libucrt:mbctype.obj
 0003:00000710       ?__rgctypeflag@@3PADA      1004f710     libucrt:mbctype.obj
 0003:00000718       ?__rgcode_page_info@@3PAUcode_page_info@@A 1004f718     libucrt:mbctype.obj
 0003:00000910       ?__dcrt_lowio_console_output_handle@@3PAXA 1004f910     libucrt:initcon.obj
 0003:00000920       ?FKeys@?1??GetOpenPanelInfo@Plist@@QAEXPAUOpenPanelInfo@@@Z@4PAGA 1004f920     Pclass.obj
 0003:00000964       ?kbt@?1??GetOpenPanelInfo@Plist@@QAEXPAUOpenPanelInfo@@@Z@4UKeyBarTitles@@A 1004f964     Pclass.obj
 0003:0000096c       ?nr@?7??Connect@Plist@@QAE_NPB_W00@Z@4U_NETRESOURCEW@@A 1004f96c     Pclass.obj
 0003:00000b18       ??_R0?AV<lambda_3>@?N@??PrintModules@@YAXPAXKAAUoptions@@@Z@@8 1004fb18     Plist.obj
 0003:00000c10       ??_R0?AV<lambda_1>@?1??GetProcessString@WMIConnection@@AAE?AV?$basic_string@_WU?$char_traits@_W@std@@V?$allocator@_W@2@@std@@KPB_W@Z@@8 1004fc10     wmi.obj
 0003:00000ca0       ??_R0?AV<lambda_1>@?1??GetProcessInt@WMIConnection@@AAEKKPB_W@Z@@8 1004fca0     wmi.obj
 0003:00001100       ??_R0?AV?$_Func_impl_no_alloc@V<lambda_3>@?N@??PrintModules@@YAXPAXKAAUoptions@@@Z@_NPA_WI@std@@@8 10050100     Plist.obj
 0003:00001168       ??_R0?AV?$_Func_impl_no_alloc@V<lambda_1>@?1??GetProcessInt@WMIConnection@@AAEKKPB_W@Z@XABUtagVARIANT@@@std@@@8 10050168     wmi.obj
 0003:000011e0       ??_R0?AV?$_Func_impl_no_alloc@V<lambda_1>@?1??GetProcessString@WMIConnection@@AAE?AV?$basic_string@_WU?$char_traits@_W@std@@V?$allocator@_W@2@@std@@KPB_W@Z@XABUtagVARIANT@@@std@@@8 100501e0     wmi.obj
 0003:000012d0       ?initlocks@std@@3V_Init_locks@1@A 100502d0     libcpmt:xlock.obj
 0003:000012d8       ?mtx@std@@3PAU_RTL_CRITICAL_SECTION@@A 100502d8     libcpmt:xlock.obj
 0003:000013b4       ?classic_locale@std@@3Vlocale@1@A 100503b4     libcpmt:locale0.obj
 0003:000013bc       ?_Fac_head@std@@3PAU_Fac_node@1@A 100503bc     libcpmt:locale0.obj
 0003:000013c0       ?_Fac_tidy_reg@std@@3U_Fac_tidy_reg_t@1@B 100503c0     libcpmt:locale0.obj
 0003:000013c4       _global_locale             100503c4     libcpmt:locale0.obj
 0003:000013c8       ?registered@?1??_Setgloballocale@locale@std@@CAXPAX@Z@4_NA 100503c8     libcpmt:locale0.obj
 0003:000013f8       ?initlocks@std@@3V_Init_locks@1@A 100503f8     libcpmt:iosptrs.obj
 0003:000013f9       ?init_atexit@@3U_Init_atexit@@A 100503f9     libcpmt:iosptrs.obj
 0003:000013fc       ?atfuns_cdecl@@3PAP6AXXZA  100503fc     libcpmt:iosptrs.obj
 0003:000014a0       ?is_initialized_as_dll@@3_NA 100504a0     LIBCMT:utility.obj
 0003:000014a1       ?module_local_atexit_table_initialized@@3_NA 100504a1     LIBCMT:utility.obj
 0003:000014a4       ?module_local_atexit_table@@3U_onexit_table_t@@A 100504a4     LIBCMT:utility.obj
 0003:000014b0       ?module_local_at_quick_exit_table@@3U_onexit_table_t@@A 100504b0     LIBCMT:utility.obj
 0003:000014c0       _GS_ExceptionRecord        100504c0     LIBCMT:gs_report.obj
 0003:00001510       _GS_ContextRecord          10050510     LIBCMT:gs_report.obj
 0003:000017dc       ?__proc_attached@@3HA      100507dc     LIBCMT:dll_dllmain.obj
 0003:00001804       ?__vcrt_startup_thread_ptd@@3U__vcrt_ptd@@A 10050804     libvcruntime:per_thread_data.obj
 0003:00001830       ___vcrt_lock_table         10050830     libvcruntime:locks.obj
 0003:00001848       ___vcrt_locks_initialized  10050848     libvcruntime:locks.obj
 0003:00001874       ?heap@@3V_HeapManager@@A   10050874     libvcruntime:undname.obj
 0003:00001888       ?module_handles@@3PAPAUHINSTANCE__@@A 10050888     libvcruntime:winapi_downlevel.obj
 0003:00001894       ?function_pointers@@3PAPAXA 10050894     libvcruntime:winapi_downlevel.obj
 0003:000018a8       ?__acrt_invalid_parameter_handler@@3V?$dual_state_global@P6AXPB_W00II@Z@__crt_state_management@@A 100508a8     libucrt:invalid_parameter.obj
 0003:000018c0       ?__acrt_lock_table@@3PAU_RTL_CRITICAL_SECTION@@A 100508c0     libucrt:locks.obj
 0003:00001a10       ?__acrt_locks_initialized@@3IA 10050a10     libucrt:locks.obj
 0003:00001a14       ?c_termination_complete@@3JA 10050a14     libucrt:exit.obj
 0003:00001a18       ?thread_local_exit_callback_func@@3P6GXPAXK0@ZA 10050a18     libucrt:exit.obj
 0003:00001a20       ?program_name@?1???$common_configure_argv@D@@YAHW4_crt_argv_mode@@@Z@4PADA 10050a20     libucrt:argv_parsing.obj
 0003:00001b50       ?__acrt_new_handler@@3V?$dual_state_global@P6AHI@Z@__crt_state_management@@A 10050b50     libucrt:new_handler.obj
 0003:00001d5c       ?__acrt_app_type@@3W4_crt_app_type@@A 10050d5c     libucrt:report_runtime_error.obj
 0003:00001d60       ?module_handles@@3PAPAUHINSTANCE__@@A 10050d60     libucrt:winapi_thunks.obj
 0003:00001db0       ?encoded_function_pointers@@3PAPAXA 10050db0     libucrt:winapi_thunks.obj
 0003:00001e38       ?static_enum_proc@?1??enum_system_locales_ex_nolock@@YAHQ6GHPA_WKJ@Z@Z@4P6GH0KJ@ZA 10050e38     libucrt:winapi_thunks.obj
 0003:00001e3c       ?internal_state@?1??_mbtowc_l@@9@4U_Mbstatet@@A 10050e3c     libucrt:mbtowc.obj
 0003:00001e54       __pmatherr_set             10050e54     libucrt:libm_error.obj
 0003:00001e5c       ?ctrlc_action@@3V?$dual_state_global@P6AXH@Z@__crt_state_management@@A 10050e5c     libucrt:signal.obj
 0003:00001e60       ?ctrlbreak_action@@3V?$dual_state_global@P6AXH@Z@__crt_state_management@@A 10050e60     libucrt:signal.obj
 0003:00001e64       ?abort_action@@3V?$dual_state_global@P6AXH@Z@__crt_state_management@@A 10050e64     libucrt:signal.obj
 0003:00001e68       ?term_action@@3V?$dual_state_global@P6AXH@Z@__crt_state_management@@A 10050e68     libucrt:signal.obj
 0003:00001e78       ?_tzname@@3V?$dual_state_global@PAPAD@__crt_state_management@@A 10050e78     libucrt:timeset.obj
 0003:00001e80       ?tz_api_used@@3HA          10050e80     libucrt:tzset.obj
 0003:00001e88       ?tz_info@@3U_TIME_ZONE_INFORMATION@@A 10050e88     libucrt:tzset.obj
 0003:00001f40       ?fSystemSet@@3HA           10050f40     libucrt:mbctype.obj
 0003:00001f44       ?initialized@?1??__acrt_initialize_multibyte@@9@4_NA 10050f44     libucrt:mbctype.obj
 0003:00001f64       ?user_matherr@@3V?$dual_state_global@P6AHPAU_exception@@@Z@__crt_state_management@@A 10050f64     libucrt:matherr.obj
 0003:00001f68       ?__acrt_global_new_mode@@3V?$dual_state_global@J@__crt_state_management@@A 10050f68     libucrt:new_mode.obj
 0003:00001f6c       ?internal_pst@?1??__mbrtoc32_utf8@__crt_mbstring@@YAIPA_UPBDIPAU_Mbstatet@@@Z@4U3@A 10050f6c     libucrt:mbrtoc32.obj
 0003:00001f74       ?internal_pst@?1??__c16rtomb_utf8@__crt_mbstring@@YAIPAD_SPAU_Mbstatet@@@Z@4U3@A 10050f74     libucrt:c16rtomb.obj
 0003:00001f90       ?kbl@?1??GetOpenPanelInfo@Plist@@QAEXPAUOpenPanelInfo@@@Z@4PAUKeyBarLabel@@A 10050f90     Pclass.obj
 0003:00002040       ?ArraysInited@?2??PanelModes@Plist@@QAEPAUPanelMode@@AAI@Z@4_NA 10051040     Pclass.obj
 0003:000021d4       ?Inited@?1??dynamic_bind@@YAXXZ@4_NA 100511d4     Proclist.obj
 0003:000021e4       ?UserAccountID@?1??GetUserAccountID@@YA@XZ@4V?$basic_string@_WU?$char_traits@_W@std@@V?$allocator@_W@2@@std@@B 100511e4     handles.obj
 0003:000021fc       ?$S1@?1??GetUserAccountID@@YA@XZ@4IA 100511fc     handles.obj
 0003:00002200       ?PanelModesRemote@?1??PanelModes@Plist@@QAEPAUPanelMode@@AAI@Z@4V?$array@UPanelMode@@$09@std@@A 10051200     Pclass.obj
 0003:00002340       ?PanelModesLocal@?1??PanelModes@Plist@@QAEPAUPanelMode@@AAI@Z@4V?$array@UPanelMode@@$09@std@@A 10051340     Pclass.obj
 0003:00002480       ?TitlesLocal@?1??PanelModes@Plist@@QAEPAUPanelMode@@AAI@Z@4V?$array@V?$array@PA_W$0BI@@std@@$09@std@@A 10051480     Pclass.obj
 0003:00002840       ?TitlesRemote@?1??PanelModes@Plist@@QAEPAUPanelMode@@AAI@Z@4V?$array@V?$array@PA_W$0BI@@std@@$09@std@@A 10051840     Pclass.obj
 0003:00002c00       ?$S1@?1??GetOpenPanelInfo@Plist@@QAEXPAUOpenPanelInfo@@@Z@4IA 10051c00     Pclass.obj
 0003:00002c04       ?Title@?1??GetOpenPanelInfo@Plist@@QAEXPAUOpenPanelInfo@@@Z@4V?$basic_string@_WU?$char_traits@_W@std@@V?$allocator@_W@2@@std@@A 10051c04     Pclass.obj
 0003:00002c1c       ?$S1@?1??Is64BitWindows@@YA_NXZ@4IA 10051c1c     perfthread.obj
 0003:00002c20       ?IsWow64@?1??Is64BitWindows@@YA_NXZ@4_NB 10051c20     perfthread.obj
 0003:00002c24       ?$S1@?1??is_wow64_itself@@YA_NXZ@4IA 10051c24     Plist.obj
 0003:00002c28       ?IsWow64@?1??is_wow64_itself@@YA_NXZ@4_NB 10051c28     Plist.obj
 0003:00002c2c       ?hDebugToken@@3V?$unique_ptr@XUhandle_closer@@@std@@A 10051c2c     Plist.obj
 0003:00002c30       ?PluginMenuStrings@?4??GetPluginInfoW@@9@4@4PAPB_WA 10051c30     Proclist.obj
 0003:00002c34       ?PluginCfgStrings@?1??GetPluginInfoW@@9@4@4PAPB_WA 10051c34     Proclist.obj
 0003:00002c38       ?DiskMenuStrings@?7??GetPluginInfoW@@9@4@4PAPB_WA 10051c38     Proclist.obj
 0003:00002c3c       ?Function@?1??RtlFirstEntrySListWrapper@@9@4@4Q6GPAU_SINGLE_LIST_ENTRY@@PAT_SLIST_HEADER@@@ZA 10051c3c     vc_crt_fix_impl.obj
 0003:00002c40       ?$S17@?1??CompareStringExWrapper@@9@36@4IA 10051c40     vc_crt_fix_impl.obj
 0003:00002c44       ?Cookie@?1??XorPointer@@YAPAXPAX@Z@4IB 10051c44     vc_crt_fix_impl.obj
 0003:00002c48       ?$S1@?1??XorPointer@@YAPAXPAX@Z@4IA 10051c48     vc_crt_fix_impl.obj
 0003:00002c4c       ?Function@?1??CompareStringExWrapper@@9@36@4Q6GHPB_WK0H0HPAU_nlsversioninfo@@PAXJ@ZA 10051c4c     vc_crt_fix_impl.obj
 0003:00002c50       ?Function@?1??InterlockedPushEntrySListWrapper@@9@8@4Q6GPAU_SINGLE_LIST_ENTRY@@PAT_SLIST_HEADER@@PAU2@@ZA 10051c50     vc_crt_fix_impl.obj
 0003:00002c54       ?Function@?1??EncodePointerWrapper@@9@4@4Q6GPAXPAX@ZA 10051c54     vc_crt_fix_impl.obj
 0003:00002c58       ?Function@?1??DecodePointerWrapper@@9@4@4Q6GPAXPAX@ZA 10051c58     vc_crt_fix_impl.obj
 0003:00002c5c       ?Function@?1??QueryDepthSListWrapper@@9@4@4Q6GGPAT_SLIST_HEADER@@@ZA 10051c5c     vc_crt_fix_impl.obj
 0003:00002c60       ?$S9@?1??InterlockedPushEntrySListWrapper@@9@8@4IA 10051c60     vc_crt_fix_impl.obj
 0003:00002c64       ?$S11@?1??RtlFirstEntrySListWrapper@@9@4@4IA 10051c64     vc_crt_fix_impl.obj
 0003:00002c68       ?$S12@?1??QueryDepthSListWrapper@@9@4@4IA 10051c68     vc_crt_fix_impl.obj
 0003:00002c6c       ?Deleter@?1??InitializeSListHead@implementation@slist@@YGXPAT_SLIST_HEADER@@@Z@4Vservice_deleter@23@A 10051c6c     vc_crt_fix_impl.obj
 0003:00002c8c       ?$S15@?1??SetThreadStackGuaranteeWrapper@@9@4@4IA 10051c8c     vc_crt_fix_impl.obj
 0003:00002c90       ?Function@?1??SetThreadStackGuaranteeWrapper@@9@4@4Q6GHPAK@ZA 10051c90     vc_crt_fix_impl.obj
 0003:00002c94       ?Function@?1??LCMapStringExWrapper@@9@36@4Q6GHPB_WK0HPA_WHPAU_nlsversioninfo@@PAXJ@ZA 10051c94     vc_crt_fix_impl.obj
 0003:00002c98       ?$S3@?1??DecodePointerWrapper@@9@4@4IA 10051c98     vc_crt_fix_impl.obj
 0003:00002c9c       ?Function@?1??InterlockedPushListSListExWrapper@@9@16@4Q6GPAU_SINGLE_LIST_ENTRY@@PAT_SLIST_HEADER@@PAU2@1K@ZA 10051c9c     vc_crt_fix_impl.obj
 0003:00002ca0       ?Function@?1??GetModuleHandleExWWrapper@@9@12@4Q6GHKPB_WPAPAUHINSTANCE__@@@ZA 10051ca0     vc_crt_fix_impl.obj
 0003:00002ca4       ?$S2@?1??EncodePointerWrapper@@9@4@4IA 10051ca4     vc_crt_fix_impl.obj
 0003:00002ca8       ?Function@?1??GetLogicalProcessorInformationWrapper@@9@8@4Q6GHPAU_SYSTEM_LOGICAL_PROCESSOR_INFORMATION@@PAK@ZA 10051ca8     vc_crt_fix_impl.obj
 0003:00002cac       ?$S18@?1??LCMapStringExWrapper@@9@36@4IA 10051cac     vc_crt_fix_impl.obj
 0003:00002cb0       ?$S6@?1??InitializeSListHeadWrapper@@9@4@4IA 10051cb0     vc_crt_fix_impl.obj
 0003:00002cb4       ?Function@?1??InitializeCriticalSectionExWrapper@@9@12@4Q6GHPAU_RTL_CRITICAL_SECTION@@KK@ZA 10051cb4     vc_crt_fix_impl.obj
 0003:00002cb8       ?Function@?1??InterlockedFlushSListWrapper@@9@4@4Q6GPAU_SINGLE_LIST_ENTRY@@PAT_SLIST_HEADER@@@ZA 10051cb8     vc_crt_fix_impl.obj
 0003:00002cbc       ?$S14@?1??GetLogicalProcessorInformationWrapper@@9@8@4IA 10051cbc     vc_crt_fix_impl.obj
 0003:00002cc0       ?$S13@?1??GetNumaHighestNodeNumberWrapper@@9@4@4IA 10051cc0     vc_crt_fix_impl.obj
 0003:00002cc4       ?Function@?1??InterlockedPopEntrySListWrapper@@9@4@4Q6GPAU_SINGLE_LIST_ENTRY@@PAT_SLIST_HEADER@@@ZA 10051cc4     vc_crt_fix_impl.obj
 0003:00002cc8       ?Function@?1??InitializeSListHeadWrapper@@9@4@4Q6GXPAT_SLIST_HEADER@@@ZA 10051cc8     vc_crt_fix_impl.obj
 0003:00002ccc       ?$S8@?1??InterlockedPopEntrySListWrapper@@9@4@4IA 10051ccc     vc_crt_fix_impl.obj
 0003:00002cd0       ?$S5@?1??InitializeSListHead@implementation@slist@@YGXPAT_SLIST_HEADER@@@Z@4IA 10051cd0     vc_crt_fix_impl.obj
 0003:00002cd4       ?$S7@?1??InterlockedFlushSListWrapper@@9@4@4IA 10051cd4     vc_crt_fix_impl.obj
 0003:00002cd8       ?$S10@?1??InterlockedPushListSListExWrapper@@9@16@4IA 10051cd8     vc_crt_fix_impl.obj
 0003:00002cdc       ?$S16@?1??InitializeCriticalSectionExWrapper@@9@12@4IA 10051cdc     vc_crt_fix_impl.obj
 0003:00002ce0       ?$S4@?1??GetModuleHandleExWWrapper@@9@12@4IA 10051ce0     vc_crt_fix_impl.obj
 0003:00002ce4       ?Ptr@?1???R<lambda_1>@?1??XorPointer@@YAPAXPAX@Z@QBE@XZ@4PAXA 10051ce4     vc_crt_fix_impl.obj
 0003:00002ce8       ?Function@?1??GetNumaHighestNodeNumberWrapper@@9@4@4Q6GHPAK@ZA 10051ce8     vc_crt_fix_impl.obj
 0004:00000060       $R000000                   10052060     ProcList.res
